 wevote_support

 Timestamp is 5c7622c6 (Wed Feb 27 12:40:22 2019)

 Preferred load address is 10000000

 Start         Length     Name                   Class
 0001:00000000 000031d8H .text$di                CODE
 0001:000031e0 0000d33eH .text$mn                CODE
 0001:00010520 00002c34H .text$x                 CODE
 0001:00013160 0000091bH .text$yd                CODE
 0002:00000000 0000072cH .idata$5                DATA
 0002:0000072c 00000004H .CRT$XCA                DATA
 0002:00000730 000001ccH .CRT$XCU                DATA
 0002:000008fc 00000004H .CRT$XCZ                DATA
 0002:00000900 00000004H .CRT$XIA                DATA
 0002:00000904 00000004H .CRT$XIAA               DATA
 0002:00000908 00000004H .CRT$XIC                DATA
 0002:0000090c 00000004H .CRT$XIZ                DATA
 0002:00000910 000015f8H .rdata                  DATA
 0002:00001f08 00000074H .rdata$debug            DATA
 0002:00001f7c 00000e80H .rdata$r                DATA
 0002:00002e00 000002a4H .rdata$sxdata           DATA
 0002:000030a4 00000004H .rtc$IAA                DATA
 0002:000030a8 00000004H .rtc$IZZ                DATA
 0002:000030ac 00000004H .rtc$TAA                DATA
 0002:000030b0 00000004H .rtc$TZZ                DATA
 0002:000030b8 000031ecH .xdata$x                DATA
 0002:000062b0 00000057H .edata                  DATA
 0002:00006308 00000104H .idata$2                DATA
 0002:0000640c 00000014H .idata$3                DATA
 0002:00006420 0000072cH .idata$4                DATA
 0002:00006b4c 00005cd0H .idata$6                DATA
 0003:00000000 00000084H .data                   DATA
 0003:00000088 0000076cH .data$r                 DATA
 0003:000007f8 000006acH .bss                    DATA
 0004:00000000 00000058H .rsrc$01                DATA
 0004:00000060 00000180H .rsrc$02                DATA

  Address         Publics by Value              Rva+Base       Lib:Object

 0000:00000000       __except_list              00000000     <absolute>
 0000:00000000       ___guard_flags             00000000     <absolute>
 0000:00000000       ___guard_fids_table        00000000     <absolute>
 0000:00000000       ___guard_fids_count        00000000     <absolute>
 0000:000000a9       ___safe_se_handler_count   000000a9     <absolute>
 0000:00009876       __fltused                  00009876     <absolute>
 0000:00009876       __ldused                   00009876     <absolute>
 0000:00000000       ___ImageBase               10000000     <linker-defined>
 0001:000031e0       ??$_Allocate@D@std@@YAPADIPAD@Z 100041e0 f i PrepareWevoteTaxonomyDataTask.obj
 0001:00003210       ??$addressof@D@std@@YAPADAAD@Z 10004210 f i PrepareWevoteTaxonomyDataTask.obj
 0001:00003220       ??$construct@PADAAPAD@?$_Wrap_alloc@V?$allocator@D@std@@@std@@QAEXPAPADAAPAD@Z 10004220 f i PrepareWevoteTaxonomyDataTask.obj
 0001:00003240       ??$construct@PADAAPAD@?$allocator@D@std@@QAEXPAPADAAPAD@Z 10004240 f i PrepareWevoteTaxonomyDataTask.obj
 0001:00003260       ??$construct@PADAAPAD@?$allocator_traits@V?$allocator@D@std@@@std@@SAXAAV?$allocator@D@1@PAPADAAPAD@Z 10004260 f i PrepareWevoteTaxonomyDataTask.obj
 0001:00003280       ??$destroy@PAD@?$_Wrap_alloc@V?$allocator@D@std@@@std@@QAEXPAPAD@Z 10004280 f i PrepareWevoteTaxonomyDataTask.obj
 0001:00003290       ??$destroy@PAD@?$allocator@D@std@@QAEXPAPAD@Z 10004290 f i PrepareWevoteTaxonomyDataTask.obj
 0001:000032a0       ??$destroy@PAD@?$allocator_traits@V?$allocator@D@std@@@std@@SAXAAV?$allocator@D@1@PAPAD@Z 100042a0 f i PrepareWevoteTaxonomyDataTask.obj
 0001:000032b0       ??$forward@AAPAD@std@@YAAAPADAAPAD@Z 100042b0 f i PrepareWevoteTaxonomyDataTask.obj
 0001:000032c0       ??0?$QFlags@W4OpenModeFlag@QIODevice@@@@QAE@W4OpenModeFlag@QIODevice@@@Z 100042c0 f i PrepareWevoteTaxonomyDataTask.obj
 0001:000032d0       ??0?$QFlags@W4TaskFlag@U2@@@@QAE@W4TaskFlag@U2@@@Z 100042d0 f i PrepareWevoteTaxonomyDataTask.obj
 0001:000032e0       ??0?$_String_alloc@$0A@U?$_String_base_types@DV?$allocator@D@std@@@std@@@std@@QAE@ABV?$allocator@D@1@@Z 100042e0 f i PrepareWevoteTaxonomyDataTask.obj
 0001:00003300       ??0?$_String_val@U?$_Simple_types@D@std@@@std@@QAE@XZ 10004300 f i PrepareWevoteTaxonomyDataTask.obj
 0001:00003320       ??0?$_Wrap_alloc@V?$allocator@D@std@@@std@@QAE@XZ 10004320 f i PrepareWevoteTaxonomyDataTask.obj
 0001:00003330       ??0?$allocator@D@std@@QAE@XZ 10004330 f i PrepareWevoteTaxonomyDataTask.obj
 0001:00003340       ??0?$basic_string@DU?$char_traits@D@std@@V?$allocator@D@2@@std@@QAE@PBD@Z 10004340 f i PrepareWevoteTaxonomyDataTask.obj
 0001:000033a0       ??0PrepareWevoteTaxonomyDataTask@U2@@QAE@AAVWorkflowProcess@FileStorage@1@@Z 100043a0 f   PrepareWevoteTaxonomyDataTask.obj
 0001:00003700       ??0QLatin1Char@@QAE@D@Z    10004700 f i PrepareWevoteTaxonomyDataTask.obj
 0001:00003710       ??0_Generic_error_category@std@@QAE@XZ 10004710 f i PrepareWevoteTaxonomyDataTask.obj
 0001:00003720       ??0_Ignore@std@@QAE@XZ     10004720 f i PrepareWevoteTaxonomyDataTask.obj
 0001:00003730       ??0_Iostream_error_category@std@@QAE@XZ 10004730 f i PrepareWevoteTaxonomyDataTask.obj
 0001:00003740       ??0_System_error_category@std@@QAE@XZ 10004740 f i PrepareWevoteTaxonomyDataTask.obj
 0001:00003750       ??0error_category@std@@QAE@XZ 10004750 f i PrepareWevoteTaxonomyDataTask.obj
 0001:00003760       ??0error_condition@std@@QAE@HABVerror_category@1@@Z 10004760 f i PrepareWevoteTaxonomyDataTask.obj
 0001:00003780       ??1?$basic_string@DU?$char_traits@D@std@@V?$allocator@D@2@@std@@QAE@XZ 10004780 f i PrepareWevoteTaxonomyDataTask.obj
 0001:000037b0       ??1PrepareWevoteTaxonomyDataTask@U2@@UAE@XZ 100047b0 f i PrepareWevoteTaxonomyDataTask.obj
 0001:00003830       ??1_Generic_error_category@std@@UAE@XZ 10004830 f i PrepareWevoteTaxonomyDataTask.obj
 0001:00003840       ??1_Iostream_error_category@std@@UAE@XZ 10004840 f i PrepareWevoteTaxonomyDataTask.obj
 0001:00003850       ??1_System_error_category@std@@UAE@XZ 10004850 f i PrepareWevoteTaxonomyDataTask.obj
 0001:00003860       ??1error_category@std@@UAE@XZ 10004860 f i PrepareWevoteTaxonomyDataTask.obj
 0001:00003870       ??2@YAPAXIPAX@Z            10004870 f i PrepareWevoteTaxonomyDataTask.obj
 0001:00003880       ??3@YAXPAX0@Z              10004880 f i PrepareWevoteTaxonomyDataTask.obj
 0001:00003890       ??8error_category@std@@QBE_NABV01@@Z 10004890 f i PrepareWevoteTaxonomyDataTask.obj
 0001:000038a0       ??8error_condition@std@@QBE_NABV01@@Z 100048a0 f i PrepareWevoteTaxonomyDataTask.obj
 0001:000038c0       ??H@YA?BVQString@@ABV0@0@Z 100048c0 f i PrepareWevoteTaxonomyDataTask.obj
 0001:00003930       ??H@YA?BVQString@@ABV0@PBD@Z 10004930 f i PrepareWevoteTaxonomyDataTask.obj
 0001:000039d0       ??_EPrepareWevoteTaxonomyDataTask@U2@@UAEPAXI@Z 100049d0 f i PrepareWevoteTaxonomyDataTask.obj
 0001:000039d0       ??_GPrepareWevoteTaxonomyDataTask@U2@@UAEPAXI@Z 100049d0 f i PrepareWevoteTaxonomyDataTask.obj
 0001:00003a60       ??_E_Generic_error_category@std@@UAEPAXI@Z 10004a60 f i PrepareWevoteTaxonomyDataTask.obj
 0001:00003a60       ??_G_Generic_error_category@std@@UAEPAXI@Z 10004a60 f i PrepareWevoteTaxonomyDataTask.obj
 0001:00003a90       ??_G_Iostream_error_category@std@@UAEPAXI@Z 10004a90 f i PrepareWevoteTaxonomyDataTask.obj
 0001:00003a90       ??_E_Iostream_error_category@std@@UAEPAXI@Z 10004a90 f i PrepareWevoteTaxonomyDataTask.obj
 0001:00003ac0       ??_G_System_error_category@std@@UAEPAXI@Z 10004ac0 f i PrepareWevoteTaxonomyDataTask.obj
 0001:00003ac0       ??_E_System_error_category@std@@UAEPAXI@Z 10004ac0 f i PrepareWevoteTaxonomyDataTask.obj
 0001:00003af0       ??_Gerror_category@std@@UAEPAXI@Z 10004af0 f i PrepareWevoteTaxonomyDataTask.obj
 0001:00003af0       ??_Eerror_category@std@@UAEPAXI@Z 10004af0 f i PrepareWevoteTaxonomyDataTask.obj
 0001:00003b20       ?_Copy@?$basic_string@DU?$char_traits@D@std@@V?$allocator@D@2@@std@@QAEXII@Z 10004b20 f i PrepareWevoteTaxonomyDataTask.obj
 0001:00003c70       ?_Eos@?$basic_string@DU?$char_traits@D@std@@V?$allocator@D@2@@std@@QAEXI@Z 10004c70 f i PrepareWevoteTaxonomyDataTask.obj
 0001:00003ca0       ?_Getal@?$_String_alloc@$0A@U?$_String_base_types@DV?$allocator@D@std@@@std@@@std@@QBE?AU?$_Wrap_alloc@V?$allocator@D@std@@@2@XZ 10004ca0 f i PrepareWevoteTaxonomyDataTask.obj
 0001:00003cb0       ?_Grow@?$basic_string@DU?$char_traits@D@std@@V?$allocator@D@2@@std@@QAE_NI_N@Z 10004cb0 f i PrepareWevoteTaxonomyDataTask.obj
 0001:00003d60       ?_Inside@?$basic_string@DU?$char_traits@D@std@@V?$allocator@D@2@@std@@QAE_NPBD@Z 10004d60 f i PrepareWevoteTaxonomyDataTask.obj
 0001:00003da0       ?_Myptr@?$_String_val@U?$_Simple_types@D@std@@@std@@QAEPADXZ 10004da0 f i PrepareWevoteTaxonomyDataTask.obj
 0001:00003db0       ?_Myptr@?$_String_val@U?$_Simple_types@D@std@@@std@@QBEPBDXZ 10004db0 f i PrepareWevoteTaxonomyDataTask.obj
 0001:00003dc0       ?_Tidy@?$basic_string@DU?$char_traits@D@std@@V?$allocator@D@2@@std@@QAEX_NI@Z 10004dc0 f i PrepareWevoteTaxonomyDataTask.obj
 0001:00003e10       ?_Xlen@?$basic_string@DU?$char_traits@D@std@@V?$allocator@D@2@@std@@QBEXXZ 10004e10 f i PrepareWevoteTaxonomyDataTask.obj
 0001:00003e20       ?_Xran@?$basic_string@DU?$char_traits@D@std@@V?$allocator@D@2@@std@@QBEXXZ 10004e20 f i PrepareWevoteTaxonomyDataTask.obj
 0001:00003e30       ?allocate@?$_Wrap_alloc@V?$allocator@D@std@@@std@@QAEPADI@Z 10004e30 f i PrepareWevoteTaxonomyDataTask.obj
 0001:00003e60       ?allocate@?$allocator@D@std@@QAEPADI@Z 10004e60 f i PrepareWevoteTaxonomyDataTask.obj
 0001:00003e90       ?assign@?$basic_string@DU?$char_traits@D@std@@V?$allocator@D@2@@std@@QAEAAV12@ABV12@II@Z 10004e90 f i PrepareWevoteTaxonomyDataTask.obj
 0001:00003fb0       ?assign@?$basic_string@DU?$char_traits@D@std@@V?$allocator@D@2@@std@@QAEAAV12@PBD@Z 10004fb0 f i PrepareWevoteTaxonomyDataTask.obj
 0001:00003ff0       ?assign@?$basic_string@DU?$char_traits@D@std@@V?$allocator@D@2@@std@@QAEAAV12@PBDI@Z 10004ff0 f i PrepareWevoteTaxonomyDataTask.obj
 0001:000040f0       ?assign@?$char_traits@D@std@@SAXAADABD@Z 100050f0 f i PrepareWevoteTaxonomyDataTask.obj
 0001:00004100       ?category@error_code@std@@QBEABVerror_category@2@XZ 10005100 f i PrepareWevoteTaxonomyDataTask.obj
 0001:00004110       ?category@error_condition@std@@QBEABVerror_category@2@XZ 10005110 f i PrepareWevoteTaxonomyDataTask.obj
 0001:00004120       ?copy@?$char_traits@D@std@@SAPADPADPBDI@Z 10005120 f i PrepareWevoteTaxonomyDataTask.obj
 0001:00004140       ?deallocate@?$_Wrap_alloc@V?$allocator@D@std@@@std@@QAEXPADI@Z 10005140 f i PrepareWevoteTaxonomyDataTask.obj
 0001:00004160       ?deallocate@?$allocator@D@std@@QAEXPADI@Z 10005160 f i PrepareWevoteTaxonomyDataTask.obj
 0001:00004180       ?default_error_condition@_System_error_category@std@@UBE?AVerror_condition@2@H@Z 10005180 f i PrepareWevoteTaxonomyDataTask.obj
 0001:000041c0       ?default_error_condition@error_category@std@@UBE?AVerror_condition@2@H@Z 100051c0 f i PrepareWevoteTaxonomyDataTask.obj
 0001:000041e0       ?equivalent@error_category@std@@UBE_NABVerror_code@2@H@Z 100051e0 f i PrepareWevoteTaxonomyDataTask.obj
 0001:00004200       ?equivalent@error_category@std@@UBE_NHABVerror_condition@2@@Z 10005200 f i PrepareWevoteTaxonomyDataTask.obj
 0001:00004240       ?erase@?$basic_string@DU?$char_traits@D@std@@V?$allocator@D@2@@std@@QAEAAV12@I@Z 10005240 f i PrepareWevoteTaxonomyDataTask.obj
 0001:00004280       ?erase@?$basic_string@DU?$char_traits@D@std@@V?$allocator@D@2@@std@@QAEAAV12@II@Z 10005280 f i PrepareWevoteTaxonomyDataTask.obj
 0001:00004320       ?generic_category@std@@YAABVerror_category@1@XZ 10005320 f i PrepareWevoteTaxonomyDataTask.obj
 0001:00004330       ?getWevoteTaxonomyDir@PrepareWevoteTaxonomyDataTask@U2@@QBEABVQString@@XZ 10005330 f   PrepareWevoteTaxonomyDataTask.obj
 0001:00004340       ?isActual@PrepareWevoteTaxonomyDataTask@U2@@ABE_NXZ 10005340 f   PrepareWevoteTaxonomyDataTask.obj
 0001:00004400       ?length@?$char_traits@D@std@@SAIPBD@Z 10005400 f i PrepareWevoteTaxonomyDataTask.obj
 0001:00004420       ?max_size@?$_Wrap_alloc@V?$allocator@D@std@@@std@@QBEIXZ 10005420 f i PrepareWevoteTaxonomyDataTask.obj
 0001:00004430       ?max_size@?$allocator@D@std@@QBEIXZ 10005430 f i PrepareWevoteTaxonomyDataTask.obj
 0001:00004440       ?max_size@?$allocator_traits@V?$allocator@D@std@@@std@@SAIABV?$allocator@D@2@@Z 10005440 f i PrepareWevoteTaxonomyDataTask.obj
 0001:00004450       ?max_size@?$basic_string@DU?$char_traits@D@std@@V?$allocator@D@2@@std@@QBEIXZ 10005450 f i PrepareWevoteTaxonomyDataTask.obj
 0001:00004460       ?message@_Generic_error_category@std@@UBE?AV?$basic_string@DU?$char_traits@D@std@@V?$allocator@D@2@@2@H@Z 10005460 f i PrepareWevoteTaxonomyDataTask.obj
 0001:000044e0       ?message@_Iostream_error_category@std@@UBE?AV?$basic_string@DU?$char_traits@D@std@@V?$allocator@D@2@@2@H@Z 100054e0 f i PrepareWevoteTaxonomyDataTask.obj
 0001:00004530       ?message@_System_error_category@std@@UBE?AV?$basic_string@DU?$char_traits@D@std@@V?$allocator@D@2@@2@H@Z 10005530 f i PrepareWevoteTaxonomyDataTask.obj
 0001:000045b0       ?move@?$char_traits@D@std@@SAPADPADPBDI@Z 100055b0 f i PrepareWevoteTaxonomyDataTask.obj
 0001:000045d0       ?name@_Generic_error_category@std@@UBEPBDXZ 100055d0 f i PrepareWevoteTaxonomyDataTask.obj
 0001:000045e0       ?name@_Iostream_error_category@std@@UBEPBDXZ 100055e0 f i PrepareWevoteTaxonomyDataTask.obj
 0001:000045f0       ?name@_System_error_category@std@@UBEPBDXZ 100055f0 f i PrepareWevoteTaxonomyDataTask.obj
 0001:00004600       ?prepareNamesFile@PrepareWevoteTaxonomyDataTask@U2@@AAEXXZ 10005600 f   PrepareWevoteTaxonomyDataTask.obj
 0001:00004920       ?prepareNodesFile@PrepareWevoteTaxonomyDataTask@U2@@AAEXXZ 10005920 f   PrepareWevoteTaxonomyDataTask.obj
 0001:00004c00       ?report@PrepareWevoteTaxonomyDataTask@U2@@EAE?AW4ReportResult@Task@2@XZ 10005c00 f   PrepareWevoteTaxonomyDataTask.obj
 0001:00004d30       ?run@PrepareWevoteTaxonomyDataTask@U2@@EAEXXZ 10005d30 f   PrepareWevoteTaxonomyDataTask.obj
 0001:00004e30       ?size@?$basic_string@DU?$char_traits@D@std@@V?$allocator@D@2@@std@@QBEIXZ 10005e30 f i PrepareWevoteTaxonomyDataTask.obj
 0001:00004e40       ?system_category@std@@YAABVerror_category@1@XZ 10005e40 f i PrepareWevoteTaxonomyDataTask.obj
 0001:00004e50       ?value@error_code@std@@QBEHXZ 10005e50 f i PrepareWevoteTaxonomyDataTask.obj
 0001:00004e60       ?value@error_condition@std@@QBEHXZ 10005e60 f i PrepareWevoteTaxonomyDataTask.obj
 0001:00004e70       _hypot                     10005e70 f i PrepareWevoteTaxonomyDataTask.obj
 0001:00004ea0       ??$atomic@H@?$QAtomicOpsBySize@$03@@CAPAJPAH@Z 10005ea0 f i WevotePrompter.obj
 0001:00004eb0       ??$deref@H@?$QAtomicOpsBySize@$03@@SA_NAAH@Z 10005eb0 f i WevotePrompter.obj
 0001:00004ed0       ??$load@H@?$QGenericAtomicOps@U?$QAtomicOpsBySize@$03@@@@SAHABH@Z 10005ed0 f i WevotePrompter.obj
 0001:00004ee0       ??$ref@H@?$QAtomicOpsBySize@$03@@SA_NAAH@Z 10005ee0 f i WevotePrompter.obj
 0001:00004f00       ??0?$PrompterBase@VWevotePrompter@LocalWorkflow@U2@@@U2@@QAE@PAVActor@Workflow@1@_N@Z 10005f00 f i WevotePrompter.obj
 0001:00004f30       ??0?$QForeachContainer@V?$QList@PAVPort@Workflow@U2@@@@@@QAE@ABV?$QList@PAVPort@Workflow@U2@@@@@Z 10005f30 f i WevotePrompter.obj
 0001:00004f70       ??0?$QList@PAVPort@Workflow@U2@@@@QAE@ABV0@@Z 10005f70 f i WevotePrompter.obj
 0001:00005030       ??0WevotePrompter@LocalWorkflow@U2@@QAE@PAVActor@Workflow@2@@Z 10006030 f   WevotePrompter.obj
 0001:00005060       ??0const_iterator@?$QList@PAVPort@Workflow@U2@@@@QAE@PAUNode@1@@Z 10006060 f i WevotePrompter.obj
 0001:00005070       ??1?$PrompterBase@VWevotePrompter@LocalWorkflow@U2@@@U2@@UAE@XZ 10006070 f i WevotePrompter.obj
 0001:00005080       ??1?$QForeachContainer@V?$QList@PAVPort@Workflow@U2@@@@@@QAE@XZ 10006080 f i WevotePrompter.obj
 0001:000050b0       ??1?$QList@PAVPort@Workflow@U2@@@@QAE@XZ 100060b0 f i WevotePrompter.obj
 0001:000050e0       ??1WevotePrompter@LocalWorkflow@U2@@UAE@XZ 100060e0 f i WevotePrompter.obj
 0001:000050f0       ??9const_iterator@?$QList@PAVPort@Workflow@U2@@@@QBE_NABV01@@Z 100060f0 f i WevotePrompter.obj
 0001:00005110       ??Dconst_iterator@?$QList@PAVPort@Workflow@U2@@@@QBEABQAVPort@Workflow@U2@@XZ 10006110 f i WevotePrompter.obj
 0001:00005120       ??Econst_iterator@?$QList@PAVPort@Workflow@U2@@@@QAEAAV01@XZ 10006120 f i WevotePrompter.obj
 0001:00005126       ??_E?$PrompterBase@VWevotePrompter@LocalWorkflow@U2@@@U2@@WM@AEPAXI@Z 10006126 f i WevotePrompter.obj
 0001:0000512e       ??_EWevotePrompter@LocalWorkflow@U2@@WM@AEPAXI@Z 1000612e f i WevotePrompter.obj
 0001:00005140       ??_G?$PrompterBase@VWevotePrompter@LocalWorkflow@U2@@@U2@@UAEPAXI@Z 10006140 f i WevotePrompter.obj
 0001:00005140       ??_E?$PrompterBase@VWevotePrompter@LocalWorkflow@U2@@@U2@@UAEPAXI@Z 10006140 f i WevotePrompter.obj
 0001:00005170       ??_EWevotePrompter@LocalWorkflow@U2@@UAEPAXI@Z 10006170 f i WevotePrompter.obj
 0001:00005170       ??_GWevotePrompter@LocalWorkflow@U2@@UAEPAXI@Z 10006170 f i WevotePrompter.obj
 0001:000051a0       ?begin@?$QList@PAVPort@Workflow@U2@@@@QBE?AVconst_iterator@1@XZ 100061a0 f i WevotePrompter.obj
 0001:000051c0       ?composeRichDoc@WevotePrompter@LocalWorkflow@U2@@EAE?AVQString@@XZ 100061c0 f   WevotePrompter.obj
 0001:000051f0       ?createDescription@?$PrompterBase@VWevotePrompter@LocalWorkflow@U2@@@U2@@UAEPAVActorDocument@Workflow@2@PAVActor@42@@Z 100061f0 f i WevotePrompter.obj
 0001:00005490       ?dealloc@?$QList@PAVPort@Workflow@U2@@@@AAEXPAUData@QListData@@@Z 10006490 f i WevotePrompter.obj
 0001:000054b0       ?deref@?$QBasicAtomicInteger@H@@QAE_NXZ 100064b0 f i WevotePrompter.obj
 0001:000054c0       ?deref@RefCount@QtPrivate@@QAE_NXZ 100064c0 f i WevotePrompter.obj
 0001:000054e0       ?end@?$QList@PAVPort@Workflow@U2@@@@QBE?AVconst_iterator@1@XZ 100064e0 f i WevotePrompter.obj
 0001:00005500       ?load@?$QBasicAtomicInteger@H@@QBEHXZ 10006500 f i WevotePrompter.obj
 0001:00005510       ?node_copy@?$QList@PAVPort@Workflow@U2@@@@AAEXPAUNode@1@00@Z 10006510 f i WevotePrompter.obj
 0001:00005540       ?node_destruct@?$QList@PAVPort@Workflow@U2@@@@AAEXPAUNode@1@0@Z 10006540 f i WevotePrompter.obj
 0001:00005550       ?ref@?$QBasicAtomicInteger@H@@QAE_NXZ 10006550 f i WevotePrompter.obj
 0001:00005570       ?ref@RefCount@QtPrivate@@QAE_NXZ 10006570 f i WevotePrompter.obj
 0001:00005590       ?t@Node@?$QList@PAVPort@Workflow@U2@@@@QAEAAPAVPort@Workflow@U2@@XZ 10006590 f i WevotePrompter.obj
 0001:000055a0       ?tr@WevotePrompter@LocalWorkflow@U2@@SA?AVQString@@PBD0H@Z 100065a0 f i WevotePrompter.obj
 0001:000055d0       ??0WevoteSupport@U2@@QAE@XZ 100065d0 f   WevoteSupport.obj
 0001:000056b0       ??1WevoteSupport@U2@@UAE@XZ 100066b0 f i WevoteSupport.obj
 0001:000056c0       ??_GWevoteSupport@U2@@UAEPAXI@Z 100066c0 f i WevoteSupport.obj
 0001:000056c0       ??_EWevoteSupport@U2@@UAEPAXI@Z 100066c0 f i WevoteSupport.obj
 0001:000056f0       ??0WevoteSupportPlugin@U2@@QAE@XZ 100066f0 f   WevoteSupportPlugin.obj
 0001:00005790       ??1WevoteSupportPlugin@U2@@UAE@XZ 10006790 f   WevoteSupportPlugin.obj
 0001:00005800       ??_GWevoteSupportPlugin@U2@@UAEPAXI@Z 10006800 f i WevoteSupportPlugin.obj
 0001:00005800       ??_EWevoteSupportPlugin@U2@@UAEPAXI@Z 10006800 f i WevoteSupportPlugin.obj
 0001:00005880       _ugene_plugin_init         10006880 f   WevoteSupportPlugin.obj
 0001:000058a0       ??$qMapLessThanKey@VQString@@@@YA_NABVQString@@0@Z 100068a0 f i WevoteTask.obj
 0001:000058b0       ??0?$QFlags@W4TaskFlag@U2@@@@QAE@VQFlag@@@Z 100068b0 f i WevoteTask.obj
 0001:000058c0       ??0?$QList@PAVTask@U2@@@@QAE@$$QAV0@@Z 100068c0 f i WevoteTask.obj
 0001:000058e0       ??0?$QList@PAVTask@U2@@@@QAE@XZ 100068e0 f i WevoteTask.obj
 0001:000058f0       ??0?$QList@VQString@@@@QAE@ABV0@@Z 100068f0 f i WevoteTask.obj
 0001:000059b0       ??0?$QList@VQString@@@@QAE@XZ 100069b0 f i WevoteTask.obj
 0001:000059c0       ??0?$QMap@VQString@@I@@QAE@XZ 100069c0 f i WevoteTask.obj
 0001:000059d0       ??0?$QScopedPointer@VIOAdapter@U2@@U?$QScopedPointerDeleter@VIOAdapter@U2@@@@@@QAE@PAVIOAdapter@U2@@@Z 100069d0 f i WevoteTask.obj
 0001:000059e0       ??0QFlag@@QAE@H@Z          100069e0 f i WevoteTask.obj
 0001:000059f0       ??0QStringList@@QAE@ABV0@@Z 100069f0 f i WevoteTask.obj
 0001:00005a10       ??0QStringList@@QAE@XZ     10006a10 f i WevoteTask.obj
 0001:00005a20       ??0WevoteTask@U2@@QAE@ABUWevoteTaskSettings@1@AAVWorkflowProcess@FileStorage@1@@Z 10006a20 f   WevoteTask.obj
 0001:00005ba0       ??0WevoteTaskSettings@U2@@QAE@ABU01@@Z 10006ba0 f i WevoteTask.obj
 0001:00005c30       ??0WevoteTaskSettings@U2@@QAE@XZ 10006c30 f   WevoteTask.obj
 0001:00005cb0       ??0iterator@?$QMap@VQString@@I@@QAE@PAU?$QMapNode@VQString@@I@@@Z 10006cb0 f i WevoteTask.obj
 0001:00005cc0       ??1?$QList@PAVTask@U2@@@@QAE@XZ 10006cc0 f i WevoteTask.obj
 0001:00005cf0       ??1?$QList@VQString@@@@QAE@XZ 10006cf0 f i WevoteTask.obj
 0001:00005d50       ??1?$QMap@VQString@@I@@QAE@XZ 10006d50 f i WevoteTask.obj
 0001:00005dc0       ??1?$QScopedPointer@VIOAdapter@U2@@U?$QScopedPointerDeleter@VIOAdapter@U2@@@@@@QAE@XZ 10006dc0 f i WevoteTask.obj
 0001:00005dd0       ??1QStringList@@QAE@XZ     10006dd0 f i WevoteTask.obj
 0001:00005de0       ??1WevoteTask@U2@@UAE@XZ   10006de0 f i WevoteTask.obj
 0001:00005e80       ??1WevoteTaskSettings@U2@@QAE@XZ 10006e80 f i WevoteTask.obj
 0001:00005ef0       ??6?$QList@PAVTask@U2@@@@QAEAAV0@ABQAVTask@U2@@@Z 10006ef0 f i WevoteTask.obj
 0001:00005f10       ??6QStringList@@QAEAAV0@ABVQString@@@Z 10006f10 f i WevoteTask.obj
 0001:00005f30       ??9@YA_NABVQString@@0@Z    10006f30 f i WevoteTask.obj
 0001:00005f50       ??BQFlag@@QBEHXZ           10006f50 f i WevoteTask.obj
 0001:00005f60       ??U?$QFlags@W4TaskFlag@U2@@@@QBE?AV0@W4TaskFlag@U2@@@Z 10006f60 f i WevoteTask.obj
 0001:00005f80       ??_EExternalToolLogParser@U2@@UAEPAXI@Z 10006f80 f i WevoteTask.obj
 0001:00005f80       ??_GExternalToolLogParser@U2@@UAEPAXI@Z 10006f80 f i WevoteTask.obj
 0001:00005fb0       ??_GExternalToolRunTask@U2@@UAEPAXI@Z 10006fb0 f i WevoteTask.obj
 0001:00005fb0       ??_EExternalToolRunTask@U2@@UAEPAXI@Z 10006fb0 f i WevoteTask.obj
 0001:00005fe0       ??_GQString@@QAEPAXI@Z     10006fe0 f i WevoteTask.obj
 0001:00006010       ??_GWevoteTask@U2@@UAEPAXI@Z 10007010 f i WevoteTask.obj
 0001:00006010       ??_EWevoteTask@U2@@UAEPAXI@Z 10007010 f i WevoteTask.obj
 0001:00006040       ?append@?$QList@PAVTask@U2@@@@QAEXABQAVTask@U2@@@Z 10007040 f i WevoteTask.obj
 0001:000060d0       ?append@?$QList@VQString@@@@QAEXABVQString@@@Z 100070d0 f i WevoteTask.obj
 0001:000061c0       ?at@?$QList@VQString@@@@QBEABVQString@@H@Z 100071c0 f i WevoteTask.obj
 0001:000061e0       ?checkSettings@WevoteTask@U2@@AAEXXZ 100071e0 f   WevoteTask.obj
 0001:00006370       ?cleanup@?$QScopedPointerDeleter@VIOAdapter@U2@@@@SAXPAVIOAdapter@U2@@@Z 10007370 f i WevoteTask.obj
 0001:00006390       ?copy@?$QMapNode@VQString@@I@@QBEPAU1@PAU?$QMapData@VQString@@I@@@Z 10007390 f i WevoteTask.obj
 0001:00006420       ?count@?$QList@VQString@@@@QBEHXZ 10007420 f i WevoteTask.obj
 0001:00006430       ?create@?$QMapData@VQString@@I@@SAPAU1@XZ 10007430 f i WevoteTask.obj
 0001:00006440       ?createNode@?$QMapData@VQString@@I@@QAEPAU?$QMapNode@VQString@@I@@ABVQString@@ABIPAU2@_N@Z 10007440 f i WevoteTask.obj
 0001:000064e0       ?data@?$QScopedPointer@VIOAdapter@U2@@U?$QScopedPointerDeleter@VIOAdapter@U2@@@@@@QBEPAVIOAdapter@U2@@XZ 100074e0 f i WevoteTask.obj
 0001:000064f0       ?dealloc@?$QList@PAVTask@U2@@@@AAEXPAUData@QListData@@@Z 100074f0 f i WevoteTask.obj
 0001:00006510       ?dealloc@?$QList@VQString@@@@AAEXPAUData@QListData@@@Z 10007510 f i WevoteTask.obj
 0001:00006550       ?destroy@?$QMapData@VQString@@I@@QAEXXZ 10007550 f i WevoteTask.obj
 0001:000065a0       ?destroySubTree@?$QMapNode@VQString@@I@@QAEXXZ 100075a0 f i WevoteTask.obj
 0001:000065d0       ?detach@?$QMap@VQString@@I@@QAEXXZ 100075d0 f i WevoteTask.obj
 0001:000065f0       ?detach_helper@?$QMap@VQString@@I@@AAEXXZ 100075f0 f i WevoteTask.obj
 0001:000066a0       ?detach_helper_grow@?$QList@PAVTask@U2@@@@AAEPAUNode@1@HH@Z 100076a0 f i WevoteTask.obj
 0001:000067b0       ?detach_helper_grow@?$QList@VQString@@@@AAEPAUNode@1@HH@Z 100077b0 f i WevoteTask.obj
 0001:00006930       ?end@?$QMapData@VQString@@I@@QAEPAU?$QMapNode@VQString@@I@@XZ 10007930 f i WevoteTask.obj
 0001:00006940       ?first@?$QList@VQString@@@@QBEABVQString@@XZ 10007940 f i WevoteTask.obj
 0001:00006950       ?getArguments@WevoteTask@U2@@AAE?AVQStringList@@XZ 10007950 f   WevoteTask.obj
 0001:00006cc0       ?getClassification@WevoteTask@U2@@QBEABV?$QMap@VQString@@I@@XZ 10007cc0 f   WevoteTask.obj
 0001:00006cd0       ?getClassificationUrl@WevoteTask@U2@@QBEABVQString@@XZ 10007cd0 f   WevoteTask.obj
 0001:00006ce0       ?insert@?$QMap@VQString@@I@@QAE?AViterator@1@ABVQString@@ABI@Z 10007ce0 f i WevoteTask.obj
 0001:00006da0       ?isShared@RefCount@QtPrivate@@QBE_NXZ 10007da0 f i WevoteTask.obj
 0001:00006dc0       ?last@?$QList@VQString@@@@QBEABVQString@@XZ 10007dc0 f i WevoteTask.obj
 0001:00006dd0       ?leftNode@?$QMapNode@VQString@@I@@QBEPAU1@XZ 10007dd0 f i WevoteTask.obj
 0001:00006de0       ?moveFile@WevoteTask@U2@@AAEXXZ 10007de0 f   WevoteTask.obj
 0001:00006f10       ?node_construct@?$QList@PAVTask@U2@@@@AAEXPAUNode@1@ABQAVTask@U2@@@Z 10007f10 f i WevoteTask.obj
 0001:00006f30       ?node_construct@?$QList@VQString@@@@AAEXPAUNode@1@ABVQString@@@Z 10007f30 f i WevoteTask.obj
 0001:00006f80       ?node_copy@?$QList@PAVTask@U2@@@@AAEXPAUNode@1@00@Z 10007f80 f i WevoteTask.obj
 0001:00006fb0       ?node_copy@?$QList@VQString@@@@AAEXPAUNode@1@00@Z 10007fb0 f i WevoteTask.obj
 0001:00007050       ?node_destruct@?$QList@PAVTask@U2@@@@AAEXPAUNode@1@0@Z 10008050 f i WevoteTask.obj
 0001:00007060       ?node_destruct@?$QList@PAVTask@U2@@@@AAEXPAUNode@1@@Z 10008060 f i WevoteTask.obj
 0001:00007070       ?node_destruct@?$QList@VQString@@@@AAEXPAUNode@1@0@Z 10008070 f i WevoteTask.obj
 0001:000070a0       ?node_destruct@?$QList@VQString@@@@AAEXPAUNode@1@@Z 100080a0 f i WevoteTask.obj
 0001:000070b0       ?onSubTaskFinished@WevoteTask@U2@@EAE?AV?$QList@PAVTask@U2@@@@PAVTask@2@@Z 100080b0 f   WevoteTask.obj
 0001:00007300       ?parseClassification@WevoteTask@U2@@AAEXXZ 10008300 f   WevoteTask.obj
 0001:000075d0       ?prepare@WevoteTask@U2@@EAEXXZ 100085d0 f   WevoteTask.obj
 0001:00007650       ?qt_noop@@YAXXZ            10008650 f i WevoteTask.obj
 0001:00007660       ?rightNode@?$QMapNode@VQString@@I@@QBEPAU1@XZ 10008660 f i WevoteTask.obj
 0001:00007670       ?root@?$QMapData@VQString@@I@@QBEPAU?$QMapNode@VQString@@I@@XZ 10008670 f i WevoteTask.obj
 0001:00007680       ?run@WevoteTask@U2@@EAEXXZ 10008680 f   WevoteTask.obj
 0001:00007790       ?size@?$QList@VQString@@@@QBEHXZ 10008790 f i WevoteTask.obj
 0001:000077a0       ?t@Node@?$QList@VQString@@@@QAEAAVQString@@XZ 100087a0 f i WevoteTask.obj
 0001:000077b0       ?tr@WevoteTask@U2@@SA?AVQString@@PBD0H@Z 100087b0 f i WevoteTask.obj
 0001:000077e0       ??6?$QList@VWorkflowNotification@U2@@@@QAEAAV0@ABVWorkflowNotification@U2@@@Z 100087e0 f i WevoteValidator.obj
 0001:00007800       ??_GWorkflowNotification@U2@@QAEPAXI@Z 10008800 f i WevoteValidator.obj
 0001:00007830       ?append@?$QList@VWorkflowNotification@U2@@@@QAEXABVWorkflowNotification@U2@@@Z 10008830 f i WevoteValidator.obj
 0001:00007910       ?dealloc@?$QList@VWorkflowNotification@U2@@@@AAEXPAUData@QListData@@@Z 10008910 f i WevoteValidator.obj
 0001:00007970       ?detach_helper_grow@?$QList@VWorkflowNotification@U2@@@@AAEPAUNode@1@HH@Z 10008970 f i WevoteValidator.obj
 0001:00007ac0       ?node_construct@?$QList@VWorkflowNotification@U2@@@@AAEXPAUNode@1@ABVWorkflowNotification@U2@@@Z 10008ac0 f i WevoteValidator.obj
 0001:00007b40       ?node_copy@?$QList@VWorkflowNotification@U2@@@@AAEXPAUNode@1@00@Z 10008b40 f i WevoteValidator.obj
 0001:00007c10       ?node_destruct@?$QList@VWorkflowNotification@U2@@@@AAEXPAUNode@1@0@Z 10008c10 f i WevoteValidator.obj
 0001:00007c50       ?node_destruct@?$QList@VWorkflowNotification@U2@@@@AAEXPAUNode@1@@Z 10008c50 f i WevoteValidator.obj
 0001:00007c80       ?tr@WevoteValidator@Workflow@U2@@SA?AVQString@@PBD0H@Z 10008c80 f i WevoteValidator.obj
 0001:00007cb0       ?validate@WevoteValidator@Workflow@U2@@UBE_NPBVActor@23@AAV?$QList@VWorkflowNotification@U2@@@@ABV?$QMap@VQString@@V1@@@@Z 10008cb0 f   WevoteValidator.obj
 0001:00007cd0       ?validateTaxonomy@WevoteValidator@Workflow@U2@@ABE_NPBVActor@23@AAV?$QList@VWorkflowNotification@U2@@@@@Z 10008cd0 f   WevoteValidator.obj
 0001:00007fd0       ??$?0V?$QMap@VQString@@I@@@QAssociativeIterableImpl@QtMetaTypePrivate@@QAE@PBV?$QMap@VQString@@I@@@Z 10008fd0 f i WevoteWorker.obj
 0001:00008040       ??$_Advance@Vconst_iterator@?$QMap@VQString@@I@@H@std@@YAXAAVconst_iterator@?$QMap@VQString@@I@@HUbidirectional_iterator_tag@0@@Z 10009040 f i WevoteWorker.obj
 0001:00008080       ??$_Distance2@Vconst_iterator@?$QMap@VQString@@I@@H@std@@YAXVconst_iterator@?$QMap@VQString@@I@@0AAHUbidirectional_iterator_tag@0@@Z 10009080 f i WevoteWorker.obj
 0001:000080b0       ??$_Iter_cat@Vconst_iterator@?$QMap@VQString@@I@@@std@@YA?AUbidirectional_iterator_tag@0@ABVconst_iterator@?$QMap@VQString@@I@@@Z 100090b0 f i WevoteWorker.obj
 0001:000080c0       ??$acquireMemoryFence@H@?$QGenericAtomicOps@U?$QAtomicOpsBySize@$03@@@@SAXABH@Z 100090c0 f i WevoteWorker.obj
 0001:000080d0       ??$advance@Vconst_iterator@?$QMap@VQString@@I@@H@std@@YAXAAVconst_iterator@?$QMap@VQString@@I@@H@Z 100090d0 f i WevoteWorker.obj
 0001:00008110       ??$advanceImpl@V?$QMap@VQString@@I@@@QAssociativeIterableImpl@QtMetaTypePrivate@@SAXPAPAXH@Z 10009110 f i WevoteWorker.obj
 0001:00008150       ??$beginImpl@V?$QMap@VQString@@I@@@QAssociativeIterableImpl@QtMetaTypePrivate@@SAXPBXPAPAX@Z 10009150 f i WevoteWorker.obj
 0001:00008190       ??$distance@Vconst_iterator@?$QMap@VQString@@I@@@std@@YAHVconst_iterator@?$QMap@VQString@@I@@0@Z 10009190 f i WevoteWorker.obj
 0001:000081c0       ??$endImpl@V?$QMap@VQString@@I@@@QAssociativeIterableImpl@QtMetaTypePrivate@@SAXPBXPAPAX@Z 100091c0 f i WevoteWorker.obj
 0001:000081f0       ??$findImpl@V?$QMap@VQString@@I@@@QAssociativeIterableImpl@QtMetaTypePrivate@@SAXPBX0PAPAX@Z 100091f0 f i WevoteWorker.obj
 0001:00008250       ??$fromValue@V?$QMap@VQString@@I@@@QVariant@@SA?AV0@ABV?$QMap@VQString@@I@@@Z 10009250 f i WevoteWorker.obj
 0001:00008270       ??$getAttributeValue@H@Attribute@U2@@QBEHPAVWorkflowContext@Workflow@1@@Z 10009270 f i WevoteWorker.obj
 0001:00008640       ??$getAttributeValue@VQString@@@Attribute@U2@@QBE?AVQString@@PAVWorkflowContext@Workflow@1@@Z 10009640 f i WevoteWorker.obj
 0001:000089d0       ??$getAttributeValueWithoutScript@H@Attribute@U2@@QBEHXZ 100099d0 f i WevoteWorker.obj
 0001:00008a10       ??$getAttributeValueWithoutScript@VQString@@@Attribute@U2@@QBE?AVQString@@XZ 10009a10 f i WevoteWorker.obj
 0001:00008a30       ??$getKeyImpl@V?$QMap@VQString@@I@@@QAssociativeIterableImpl@QtMetaTypePrivate@@SA?AUVariantData@1@PBQAXHI@Z 10009a30 f i WevoteWorker.obj
 0001:00008a50       ??$getValue@H@BaseWorker@LocalWorkflow@U2@@IBEHABVQString@@@Z 10009a50 f i WevoteWorker.obj
 0001:00008a80       ??$getValue@VQString@@@BaseWorker@LocalWorkflow@U2@@IBE?AVQString@@ABV3@@Z 10009a80 f i WevoteWorker.obj
 0001:00008b90       ??$getValueImpl@V?$QMap@VQString@@I@@@QAssociativeIterableImpl@QtMetaTypePrivate@@SA?AUVariantData@1@PBQAXHI@Z 10009b90 f i WevoteWorker.obj
 0001:00008bb0       ??$loadAcquire@H@?$QGenericAtomicOps@U?$QAtomicOpsBySize@$03@@@@SAHABH@Z 10009bb0 f i WevoteWorker.obj
 0001:00008bc0       ??$orderedMemoryFence@H@?$QGenericAtomicOps@U?$QAtomicOpsBySize@$03@@@@SAXABH@Z 10009bc0 f i WevoteWorker.obj
 0001:00008bd0       ??$qMapLessThanKey@VDescriptor@U2@@@@YA_NABVDescriptor@U2@@0@Z 10009bd0 f i WevoteWorker.obj
 0001:00008bf0       ??$qMetaTypeId@H@@YAHXZ    10009bf0 f i WevoteWorker.obj
 0001:00008c00       ??$qMetaTypeId@I@@YAHXZ    10009c00 f i WevoteWorker.obj
 0001:00008c10       ??$qMetaTypeId@V?$QMap@VQString@@I@@@@YAHXZ 10009c10 f i WevoteWorker.obj
 0001:00008c20       ??$qMetaTypeId@VQAssociativeIterableImpl@QtMetaTypePrivate@@@@YAHXZ 10009c20 f i WevoteWorker.obj
 0001:00008c30       ??$qMetaTypeId@VQString@@@@YAHXZ 10009c30 f i WevoteWorker.obj
 0001:00008c40       ??$qRegisterMetaType@V?$QMap@VQString@@I@@@@YAHPBDPAV?$QMap@VQString@@I@@W4DefinedType@?$MetaTypeDefinedHelper@V?$QMap@VQString@@I@@$00@QtPrivate@@@Z 10009c40 f i WevoteWorker.obj
 0001:00008cb0       ??$qRegisterMetaType@VQAssociativeIterableImpl@QtMetaTypePrivate@@@@YAHPBDPAVQAssociativeIterableImpl@QtMetaTypePrivate@@W4DefinedType@?$MetaTypeDefinedHelper@VQAssociativeIterableImpl@QtMetaTypePrivate@@$00@QtPrivate@@@Z 10009cb0 f i WevoteWorker.obj
 0001:00008d70       ??$qRegisterNormalizedMetaType@V?$QMap@VQString@@I@@@@YAHABVQByteArray@@PAV?$QMap@VQString@@I@@W4DefinedType@?$MetaTypeDefinedHelper@V?$QMap@VQString@@I@@$00@QtPrivate@@@Z 10009d70 f i WevoteWorker.obj
 0001:00008de0       ??$qRegisterNormalizedMetaType@VQAssociativeIterableImpl@QtMetaTypePrivate@@@@YAHABVQByteArray@@PAVQAssociativeIterableImpl@QtMetaTypePrivate@@W4DefinedType@?$MetaTypeDefinedHelper@VQAssociativeIterableImpl@QtMetaTypePrivate@@$00@QtPrivate@@@Z 10009de0 f i WevoteWorker.obj
 0001:00008e40       ??$qVariantFromValue@V?$QMap@VQString@@I@@@@YA?AVQVariant@@ABV?$QMap@VQString@@I@@@Z 10009e40 f i WevoteWorker.obj
 0001:00008e70       ??$qobject_cast@PAVWevoteTask@U2@@@@YAPAVWevoteTask@U2@@PAVQObject@@@Z 10009e70 f i WevoteWorker.obj
 0001:00008e90       ??$qvariant_cast@H@@YAHABVQVariant@@@Z 10009e90 f i WevoteWorker.obj
 0001:00008ed0       ??$qvariant_cast@VQString@@@@YA?AVQString@@ABVQVariant@@@Z 10009ed0 f i WevoteWorker.obj
 0001:00008ef0       ??$releaseMemoryFence@H@?$QGenericAtomicOps@U?$QAtomicOpsBySize@$03@@@@SAXABH@Z 10009ef0 f i WevoteWorker.obj
 0001:00008f00       ??$sizeImpl@V?$QMap@VQString@@I@@@QAssociativeIterableImpl@QtMetaTypePrivate@@SAHPBX@Z 10009f00 f i WevoteWorker.obj
 0001:00008f40       ??$storeRelease@HH@?$QGenericAtomicOps@U?$QAtomicOpsBySize@$03@@@@SAXAAHH@Z 10009f40 f i WevoteWorker.obj
 0001:00008f50       ??$value@H@QVariant@@QBEHXZ 10009f50 f i WevoteWorker.obj
 0001:00008f90       ??$value@VQString@@@QVariant@@QBE?AVQString@@XZ 10009f90 f i WevoteWorker.obj
 0001:00008fb0       ??0?$ConverterFunctor@V?$QMap@VQString@@I@@VQAssociativeIterableImpl@QtMetaTypePrivate@@U?$QAssociativeIterableConvertFunctor@V?$QMap@VQString@@I@@@3@@QtPrivate@@QAE@U?$QAssociativeIterableConvertFunctor@V?$QMap@VQString@@I@@@QtMetaTypePrivate@@@Z 10009fb0 f i WevoteWorker.obj
 0001:00008fc0       ??0?$QFlags@W4TypeFlag@QMetaType@@@@QAE@VQFlag@@@Z 10009fc0 f i WevoteWorker.obj
 0001:00008fd0       ??0?$QForeachContainer@V?$QList@VDescriptor@U2@@@@@@QAE@ABV?$QList@VDescriptor@U2@@@@@Z 10009fd0 f i WevoteWorker.obj
 0001:00009010       ??0?$QList@VDescriptor@U2@@@@QAE@$$QAV0@@Z 1000a010 f i WevoteWorker.obj
 0001:00009030       ??0?$QList@VDescriptor@U2@@@@QAE@ABV0@@Z 1000a030 f i WevoteWorker.obj
 0001:000090f0       ??0?$QList@VDescriptor@U2@@@@QAE@XZ 1000a0f0 f i WevoteWorker.obj
 0001:00009100       ??0?$QMap@VQString@@I@@QAE@ABV0@@Z 1000a100 f i WevoteWorker.obj
 0001:00009170       ??0?$QMap@VQString@@VQScriptValue@@@@QAE@XZ 1000a170 f i WevoteWorker.obj
 0001:00009180       ??0?$QMap@VQString@@VQVariant@@@@QAE@XZ 1000a180 f i WevoteWorker.obj
 0001:00009190       ??0AbstractConverterFunction@QtPrivate@@QAE@P6A_NPBU01@PBXPAX@Z@Z 1000a190 f i WevoteWorker.obj
 0001:000091a0       ??0QAssociativeIterableImpl@QtMetaTypePrivate@@QAE@XZ 1000a1a0 f i WevoteWorker.obj
 0001:00009210       ??0VariantData@QtMetaTypePrivate@@QAE@HPBXI@Z 1000a210 f i WevoteWorker.obj
 0001:00009230       ??0WevoteWorker@LocalWorkflow@U2@@QAE@PAVActor@Workflow@2@@Z 1000a230 f   WevoteWorker.obj
 0001:00009270       ??0const_iterator@?$QList@VDescriptor@U2@@@@QAE@PAUNode@1@@Z 1000a270 f i WevoteWorker.obj
 0001:00009280       ??0const_iterator@?$QMap@VDescriptor@U2@@VQVariant@@@@QAE@PBU?$QMapNode@VDescriptor@U2@@VQVariant@@@@@Z 1000a280 f i WevoteWorker.obj
 0001:00009290       ??0const_iterator@?$QMap@VQString@@I@@QAE@PBU?$QMapNode@VQString@@I@@@Z 1000a290 f i WevoteWorker.obj
 0001:000092a0       ??0iterator@?$QMap@VQString@@VQScriptValue@@@@QAE@PAU?$QMapNode@VQString@@VQScriptValue@@@@@Z 1000a2a0 f i WevoteWorker.obj
 0001:000092b0       ??0iterator@?$QMap@VQString@@VQVariant@@@@QAE@PAU?$QMapNode@VQString@@VQVariant@@@@@Z 1000a2b0 f i WevoteWorker.obj
 0001:000092c0       ??1?$ConverterFunctor@V?$QMap@VQString@@I@@VQAssociativeIterableImpl@QtMetaTypePrivate@@U?$QAssociativeIterableConvertFunctor@V?$QMap@VQString@@I@@@3@@QtPrivate@@QAE@XZ 1000a2c0 f i WevoteWorker.obj
 0001:000092e0       ??1?$QExplicitlySharedDataPointer@VDataType@U2@@@@QAE@XZ 1000a2e0 f i WevoteWorker.obj
 0001:00009300       ??1?$QForeachContainer@V?$QList@VDescriptor@U2@@@@@@QAE@XZ 1000a300 f i WevoteWorker.obj
 0001:00009330       ??1?$QList@PAVExternalToolListener@U2@@@@QAE@XZ 1000a330 f i WevoteWorker.obj
 0001:00009360       ??1?$QList@VDescriptor@U2@@@@QAE@XZ 1000a360 f i WevoteWorker.obj
 0001:00009390       ??1?$QMap@VQString@@VQScriptValue@@@@QAE@XZ 1000a390 f i WevoteWorker.obj
 0001:000093e0       ??1?$QMap@VQString@@VQVariant@@@@QAE@XZ 1000a3e0 f i WevoteWorker.obj
 0001:00009430       ??1WevoteWorker@LocalWorkflow@U2@@UAE@XZ 1000a430 f i WevoteWorker.obj
 0001:00009440       ??8const_iterator@?$QMap@VDescriptor@U2@@VQVariant@@@@QBE_NABV01@@Z 1000a440 f i WevoteWorker.obj
 0001:00009460       ??8const_iterator@?$QMap@VQString@@I@@QBE_NABV01@@Z 1000a460 f i WevoteWorker.obj
 0001:00009480       ??9const_iterator@?$QList@VDescriptor@U2@@@@QBE_NABV01@@Z 1000a480 f i WevoteWorker.obj
 0001:000094a0       ??9const_iterator@?$QMap@VDescriptor@U2@@VQVariant@@@@QBE_NABV01@@Z 1000a4a0 f i WevoteWorker.obj
 0001:000094c0       ??9const_iterator@?$QMap@VQString@@I@@QBE_NABV01@@Z 1000a4c0 f i WevoteWorker.obj
 0001:000094e0       ??A?$QMap@VQString@@VQScriptValue@@@@QAEAAVQScriptValue@@ABVQString@@@Z 1000a4e0 f i WevoteWorker.obj
 0001:000095b0       ??A?$QMap@VQString@@VQVariant@@@@QAEAAVQVariant@@ABVQString@@@Z 1000a5b0 f i WevoteWorker.obj
 0001:00009680       ??Dconst_iterator@?$QList@VDescriptor@U2@@@@QBEABVDescriptor@U2@@XZ 1000a680 f i WevoteWorker.obj
 0001:00009690       ??Diterator@?$QMap@VQString@@VQScriptValue@@@@QBEAAVQScriptValue@@XZ 1000a690 f i WevoteWorker.obj
 0001:000096a0       ??Diterator@?$QMap@VQString@@VQVariant@@@@QBEAAVQVariant@@XZ 1000a6a0 f i WevoteWorker.obj
 0001:000096b0       ??Econst_iterator@?$QList@VDescriptor@U2@@@@QAEAAV01@XZ 1000a6b0 f i WevoteWorker.obj
 0001:000096c0       ??Econst_iterator@?$QMap@VDescriptor@U2@@VQVariant@@@@QAEAAV01@XZ 1000a6c0 f i WevoteWorker.obj
 0001:000096e0       ??Econst_iterator@?$QMap@VQString@@I@@QAEAAV01@XZ 1000a6e0 f i WevoteWorker.obj
 0001:00009700       ??Fconst_iterator@?$QMap@VQString@@I@@QAEAAV01@XZ 1000a700 f i WevoteWorker.obj
 0001:00009720       ??R?$QAssociativeIterableConvertFunctor@V?$QMap@VQString@@I@@@QtMetaTypePrivate@@QBE?AVQAssociativeIterableImpl@1@ABV?$QMap@VQString@@I@@@Z 1000a720 f i WevoteWorker.obj
 0001:00009740       ??_5?$QFlags@W4TypeFlag@QMetaType@@@@QAEAAV0@W4TypeFlag@QMetaType@@@Z 1000a740 f i WevoteWorker.obj
 0001:0000974e       ??_EWevoteWorker@LocalWorkflow@U2@@W7AEPAXI@Z 1000a74e f i WevoteWorker.obj
 0001:00009756       ??_EWevoteWorker@LocalWorkflow@U2@@WBA@AEPAXI@Z 1000a756 f i WevoteWorker.obj
 0001:00009760       ??_G?$QMap@VQString@@I@@QAEPAXI@Z 1000a760 f i WevoteWorker.obj
 0001:00009790       ??_GDescriptor@U2@@UAEPAXI@Z 1000a790 f i WevoteWorker.obj
 0001:00009790       ??_EDescriptor@U2@@UAEPAXI@Z 1000a790 f i WevoteWorker.obj
 0001:000097c0       ??_EFailTask@U2@@UAEPAXI@Z 1000a7c0 f i WevoteWorker.obj
 0001:000097c0       ??_GFailTask@U2@@UAEPAXI@Z 1000a7c0 f i WevoteWorker.obj
 0001:000097f0       ??_GQScriptValue@@QAEPAXI@Z 1000a7f0 f i WevoteWorker.obj
 0001:00009820       ??_GQVariant@@QAEPAXI@Z    1000a820 f i WevoteWorker.obj
 0001:00009850       ??_GTaskSignalMapper@U2@@UAEPAXI@Z 1000a850 f i WevoteWorker.obj
 0001:00009850       ??_ETaskSignalMapper@U2@@UAEPAXI@Z 1000a850 f i WevoteWorker.obj
 0001:00009880       ??_GWevoteWorker@LocalWorkflow@U2@@UAEPAXI@Z 1000a880 f i WevoteWorker.obj
 0001:00009880       ??_EWevoteWorker@LocalWorkflow@U2@@UAEPAXI@Z 1000a880 f i WevoteWorker.obj
 0001:000098b0       ?Construct@?$QMetaTypeFunctionHelper@V?$QMap@VQString@@I@@$00@QtMetaTypePrivate@@SAPAXPAXPBX@Z 1000a8b0 f i WevoteWorker.obj
 0001:00009940       ?Construct@?$QMetaTypeFunctionHelper@VQAssociativeIterableImpl@QtMetaTypePrivate@@$00@QtMetaTypePrivate@@SAPAXPAXPBX@Z 1000a940 f i WevoteWorker.obj
 0001:00009990       ?Create@?$QMetaTypeFunctionHelper@V?$QMap@VQString@@I@@$00@QtMetaTypePrivate@@SAPAXPBX@Z 1000a990 f i WevoteWorker.obj
 0001:00009a30       ?Create@?$QMetaTypeFunctionHelper@VQAssociativeIterableImpl@QtMetaTypePrivate@@$00@QtMetaTypePrivate@@SAPAXPBX@Z 1000aa30 f i WevoteWorker.obj
 0001:00009a90       ?Delete@?$QMetaTypeFunctionHelper@V?$QMap@VQString@@I@@$00@QtMetaTypePrivate@@SAXPAX@Z 1000aa90 f i WevoteWorker.obj
 0001:00009ab0       ?Delete@?$QMetaTypeFunctionHelper@VQAssociativeIterableImpl@QtMetaTypePrivate@@$00@QtMetaTypePrivate@@SAXPAX@Z 1000aab0 f i WevoteWorker.obj
 0001:00009ac0       ?Destruct@?$QMetaTypeFunctionHelper@V?$QMap@VQString@@I@@$00@QtMetaTypePrivate@@SAXPAX@Z 1000aac0 f i WevoteWorker.obj
 0001:00009ad0       ?Destruct@?$QMetaTypeFunctionHelper@VQAssociativeIterableImpl@QtMetaTypePrivate@@$00@QtMetaTypePrivate@@SAXPAX@Z 1000aad0 f i WevoteWorker.obj
 0001:00009ae0       ?append@?$QList@VDescriptor@U2@@@@QAEXABVDescriptor@U2@@@Z 1000aae0 f i WevoteWorker.obj
 0001:00009bd0       ?assign@?$IteratorOwnerCommon@Vconst_iterator@?$QMap@VQString@@I@@@QtMetaTypePrivate@@SAXPAPAXPBQAX@Z 1000abd0 f i WevoteWorker.obj
 0001:00009c00       ?assign@?$IteratorOwnerCommon@Vconst_iterator@?$QMap@VQString@@I@@@QtMetaTypePrivate@@SAXPAPAXVconst_iterator@?$QMap@VQString@@I@@@Z 1000ac00 f i WevoteWorker.obj
 0001:00009c30       ?begin@?$QList@VDescriptor@U2@@@@QBE?AVconst_iterator@1@XZ 1000ac30 f i WevoteWorker.obj
 0001:00009c50       ?begin@?$QMap@VDescriptor@U2@@VQVariant@@@@QBE?AVconst_iterator@1@XZ 1000ac50 f i WevoteWorker.obj
 0001:00009c70       ?begin@?$QMap@VQString@@I@@QBE?AVconst_iterator@1@XZ 1000ac70 f i WevoteWorker.obj
 0001:00009c90       ?begin@?$QMapData@VDescriptor@U2@@VQVariant@@@@QAEPAU?$QMapNode@VDescriptor@U2@@VQVariant@@@@XZ 1000ac90 f i WevoteWorker.obj
 0001:00009ca0       ?begin@?$QMapData@VQString@@I@@QAEPAU?$QMapNode@VQString@@I@@XZ 1000aca0 f i WevoteWorker.obj
 0001:00009cb0       ?cleanup@WevoteWorker@LocalWorkflow@U2@@UAEXXZ 1000acb0 f   WevoteWorker.obj
 0001:00009cc0       ?constFind@?$QMap@VQString@@I@@QBE?AVconst_iterator@1@ABVQString@@@Z 1000acc0 f i WevoteWorker.obj
 0001:00009d10       ?convert@?$ConverterFunctor@V?$QMap@VQString@@I@@VQAssociativeIterableImpl@QtMetaTypePrivate@@U?$QAssociativeIterableConvertFunctor@V?$QMap@VQString@@I@@@3@@QtPrivate@@SA_NPBUAbstractConverterFunction@2@PBXPAX@Z 1000ad10 f i WevoteWorker.obj
 0001:00009d60       ?copy@?$QMapNode@VQString@@VQScriptValue@@@@QBEPAU1@PAU?$QMapData@VQString@@VQScriptValue@@@@@Z 1000ad60 f i WevoteWorker.obj
 0001:00009df0       ?copy@?$QMapNode@VQString@@VQVariant@@@@QBEPAU1@PAU?$QMapData@VQString@@VQVariant@@@@@Z 1000adf0 f i WevoteWorker.obj
 0001:00009e80       ?create@?$QMapData@VQString@@VQScriptValue@@@@SAPAU1@XZ 1000ae80 f i WevoteWorker.obj
 0001:00009e90       ?create@?$QMapData@VQString@@VQVariant@@@@SAPAU1@XZ 1000ae90 f i WevoteWorker.obj
 0001:00009ea0       ?createNode@?$QMapData@VQString@@VQScriptValue@@@@QAEPAU?$QMapNode@VQString@@VQScriptValue@@@@ABVQString@@ABVQScriptValue@@PAU2@_N@Z 1000aea0 f i WevoteWorker.obj
 0001:00009f60       ?createNode@?$QMapData@VQString@@VQVariant@@@@QAEPAU?$QMapNode@VQString@@VQVariant@@@@ABVQString@@ABVQVariant@@PAU2@_N@Z 1000af60 f i WevoteWorker.obj
 0001:0000a020       ?dataFinished@WevoteWorker@LocalWorkflow@U2@@ABE_NXZ 1000b020 f   WevoteWorker.obj
 0001:0000a030       ?dealloc@?$QList@PAVExternalToolListener@U2@@@@AAEXPAUData@QListData@@@Z 1000b030 f i WevoteWorker.obj
 0001:0000a050       ?dealloc@?$QList@VDescriptor@U2@@@@AAEXPAUData@QListData@@@Z 1000b050 f i WevoteWorker.obj
 0001:0000a0a0       ?destroy@?$IteratorOwnerCommon@Vconst_iterator@?$QMap@VQString@@I@@@QtMetaTypePrivate@@SAXPAPAX@Z 1000b0a0 f i WevoteWorker.obj
 0001:0000a0c0       ?destroy@?$QMapData@VQString@@VQScriptValue@@@@QAEXXZ 1000b0c0 f i WevoteWorker.obj
 0001:0000a0f0       ?destroy@?$QMapData@VQString@@VQVariant@@@@QAEXXZ 1000b0f0 f i WevoteWorker.obj
 0001:0000a120       ?destroySubTree@?$QMapNode@VQString@@VQScriptValue@@@@QAEXXZ 1000b120 f i WevoteWorker.obj
 0001:0000a160       ?destroySubTree@?$QMapNode@VQString@@VQVariant@@@@QAEXXZ 1000b160 f i WevoteWorker.obj
 0001:0000a1a0       ?detach@?$QMap@VQString@@VQScriptValue@@@@QAEXXZ 1000b1a0 f i WevoteWorker.obj
 0001:0000a1c0       ?detach@?$QMap@VQString@@VQVariant@@@@QAEXXZ 1000b1c0 f i WevoteWorker.obj
 0001:0000a1e0       ?detach_helper@?$QList@VDescriptor@U2@@@@AAEXH@Z 1000b1e0 f i WevoteWorker.obj
 0001:0000a2b0       ?detach_helper@?$QMap@VQString@@VQScriptValue@@@@AAEXXZ 1000b2b0 f i WevoteWorker.obj
 0001:0000a330       ?detach_helper@?$QMap@VQString@@VQVariant@@@@AAEXXZ 1000b330 f i WevoteWorker.obj
 0001:0000a3b0       ?detach_helper_grow@?$QList@VDescriptor@U2@@@@AAEPAUNode@1@HH@Z 1000b3b0 f i WevoteWorker.obj
 0001:0000a500       ?end@?$QList@VDescriptor@U2@@@@QBE?AVconst_iterator@1@XZ 1000b500 f i WevoteWorker.obj
 0001:0000a520       ?end@?$QMap@VDescriptor@U2@@VQVariant@@@@QBE?AVconst_iterator@1@XZ 1000b520 f i WevoteWorker.obj
 0001:0000a540       ?end@?$QMap@VQString@@I@@QBE?AVconst_iterator@1@XZ 1000b540 f i WevoteWorker.obj
 0001:0000a560       ?end@?$QMapData@VDescriptor@U2@@VQVariant@@@@QAEPAU?$QMapNode@VDescriptor@U2@@VQVariant@@@@XZ 1000b560 f i WevoteWorker.obj
 0001:0000a570       ?end@?$QMapData@VQString@@VQScriptValue@@@@QAEPAU?$QMapNode@VQString@@VQScriptValue@@@@XZ 1000b570 f i WevoteWorker.obj
 0001:0000a580       ?end@?$QMapData@VQString@@VQVariant@@@@QAEPAU?$QMapNode@VQString@@VQVariant@@@@XZ 1000b580 f i WevoteWorker.obj
 0001:0000a590       ?equal@?$IteratorOwnerCommon@Vconst_iterator@?$QMap@VQString@@I@@@QtMetaTypePrivate@@SA_NPBQAX0@Z 1000b590 f i WevoteWorker.obj
 0001:0000a5b0       ?find@?$QMap@VQString@@I@@QBE?AVconst_iterator@1@ABVQString@@@Z 1000b5b0 f i WevoteWorker.obj
 0001:0000a600       ?findNode@?$QMapData@VDescriptor@U2@@VQVariant@@@@QBEPAU?$QMapNode@VDescriptor@U2@@VQVariant@@@@ABVDescriptor@U2@@@Z 1000b600 f i WevoteWorker.obj
 0001:0000a640       ?findNode@?$QMapData@VQString@@I@@QBEPAU?$QMapNode@VQString@@I@@ABVQString@@@Z 1000b640 f i WevoteWorker.obj
 0001:0000a680       ?findNode@?$QMapData@VQString@@PAVIntegralBus@Workflow@U2@@@@QBEPAU?$QMapNode@VQString@@PAVIntegralBus@Workflow@U2@@@@ABVQString@@@Z 1000b680 f i WevoteWorker.obj
 0001:0000a6c0       ?findNode@?$QMapData@VQString@@VQScriptValue@@@@QBEPAU?$QMapNode@VQString@@VQScriptValue@@@@ABVQString@@@Z 1000b6c0 f i WevoteWorker.obj
 0001:0000a700       ?findNode@?$QMapData@VQString@@VQVariant@@@@QBEPAU?$QMapNode@VQString@@VQVariant@@@@ABVQString@@@Z 1000b700 f i WevoteWorker.obj
 0001:0000a740       ?getKey@?$AssociativeContainerAccessor@V?$QMap@VQString@@I@@$00@QtMetaTypePrivate@@SAABVQString@@ABVconst_iterator@?$QMap@VQString@@I@@@Z 1000b740 f i WevoteWorker.obj
 0001:0000a750       ?getSettings@WevoteWorker@LocalWorkflow@U2@@AAE?AUWevoteTaskSettings@3@AAVU2OpStatus@3@@Z 1000b750 f   WevoteWorker.obj
 0001:0000aca0       ?getValue@?$AssociativeContainerAccessor@V?$QMap@VQString@@I@@$00@QtMetaTypePrivate@@SAABIABVconst_iterator@?$QMap@VQString@@I@@@Z 1000bca0 f i WevoteWorker.obj
 0001:0000acb0       ?init@WevoteWorker@LocalWorkflow@U2@@UAEXXZ 1000bcb0 f   WevoteWorker.obj
 0001:0000aff0       ?insert@?$QMap@VQString@@VQScriptValue@@@@QAE?AViterator@1@ABVQString@@ABVQScriptValue@@@Z 1000bff0 f i WevoteWorker.obj
 0001:0000b0b0       ?insert@?$QMap@VQString@@VQVariant@@@@QAE?AViterator@1@ABVQString@@ABVQVariant@@@Z 1000c0b0 f i WevoteWorker.obj
 0001:0000b170       ?invoke@?$MetaTypeInvoker@U?$QVariantValueHelper@H@QtPrivate@@ABVQVariant@@H@QtPrivate@@SAHABVQVariant@@@Z 1000c170 f i WevoteWorker.obj
 0001:0000b1b0       ?invoke@?$MetaTypeInvoker@U?$QVariantValueHelper@VQString@@@QtPrivate@@ABVQVariant@@VQString@@@QtPrivate@@SA?AVQString@@ABVQVariant@@@Z 1000c1b0 f i WevoteWorker.obj
 0001:0000b1d0       ?isReadyToRun@WevoteWorker@LocalWorkflow@U2@@ABE_NXZ 1000c1d0 f   WevoteWorker.obj
 0001:0000b1f0       ?key@const_iterator@?$QMap@VDescriptor@U2@@VQVariant@@@@QBEABVDescriptor@U2@@XZ 1000c1f0 f i WevoteWorker.obj
 0001:0000b200       ?key@const_iterator@?$QMap@VQString@@I@@QBEABVQString@@XZ 1000c200 f i WevoteWorker.obj
 0001:0000b210       ?leftNode@?$QMapNode@VDescriptor@U2@@VQVariant@@@@QBEPAU1@XZ 1000c210 f i WevoteWorker.obj
 0001:0000b220       ?leftNode@?$QMapNode@VQString@@PAVIntegralBus@Workflow@U2@@@@QBEPAU1@XZ 1000c220 f i WevoteWorker.obj
 0001:0000b230       ?leftNode@?$QMapNode@VQString@@VQScriptValue@@@@QBEPAU1@XZ 1000c230 f i WevoteWorker.obj
 0001:0000b240       ?leftNode@?$QMapNode@VQString@@VQVariant@@@@QBEPAU1@XZ 1000c240 f i WevoteWorker.obj
 0001:0000b250       ?loadAcquire@?$QBasicAtomicInteger@H@@QBEHXZ 1000c250 f i WevoteWorker.obj
 0001:0000b260       ?lowerBound@?$QMapNode@VDescriptor@U2@@VQVariant@@@@QAEPAU1@ABVDescriptor@U2@@@Z 1000c260 f i WevoteWorker.obj
 0001:0000b2a0       ?lowerBound@?$QMapNode@VQString@@I@@QAEPAU1@ABVQString@@@Z 1000c2a0 f i WevoteWorker.obj
 0001:0000b2e0       ?lowerBound@?$QMapNode@VQString@@PAVIntegralBus@Workflow@U2@@@@QAEPAU1@ABVQString@@@Z 1000c2e0 f i WevoteWorker.obj
 0001:0000b320       ?lowerBound@?$QMapNode@VQString@@VQScriptValue@@@@QAEPAU1@ABVQString@@@Z 1000c320 f i WevoteWorker.obj
 0001:0000b360       ?lowerBound@?$QMapNode@VQString@@VQVariant@@@@QAEPAU1@ABVQString@@@Z 1000c360 f i WevoteWorker.obj
 0001:0000b3a0       ?metaType@?$QVariantValueHelper@H@QtPrivate@@SAHABVQVariant@@@Z 1000c3a0 f i WevoteWorker.obj
 0001:0000b3e0       ?metaType@?$QVariantValueHelper@VQString@@@QtPrivate@@SA?AVQString@@ABVQVariant@@@Z 1000c3e0 f i WevoteWorker.obj
 0001:0000b4a0       ?nextNode@?$QMapNode@VDescriptor@U2@@VQVariant@@@@QBEPBU1@XZ 1000c4a0 f i WevoteWorker.obj
 0001:0000b4b0       ?nextNode@?$QMapNode@VQString@@I@@QBEPBU1@XZ 1000c4b0 f i WevoteWorker.obj
 0001:0000b4c0       ?node_construct@?$QList@VDescriptor@U2@@@@AAEXPAUNode@1@ABVDescriptor@U2@@@Z 1000c4c0 f i WevoteWorker.obj
 0001:0000b550       ?node_copy@?$QList@VDescriptor@U2@@@@AAEXPAUNode@1@00@Z 1000c550 f i WevoteWorker.obj
 0001:0000b620       ?node_destruct@?$QList@PAVExternalToolListener@U2@@@@AAEXPAUNode@1@0@Z 1000c620 f i WevoteWorker.obj
 0001:0000b630       ?node_destruct@?$QList@VDescriptor@U2@@@@AAEXPAUNode@1@0@Z 1000c630 f i WevoteWorker.obj
 0001:0000b660       ?node_destruct@?$QList@VDescriptor@U2@@@@AAEXPAUNode@1@@Z 1000c660 f i WevoteWorker.obj
 0001:0000b680       ?previousNode@?$QMapNode@VQString@@I@@QBEPBU1@XZ 1000c680 f i WevoteWorker.obj
 0001:0000b690       ?qt_metatype_id@?$QMetaTypeId2@H@@SAHXZ 1000c690 f i WevoteWorker.obj
 0001:0000b6a0       ?qt_metatype_id@?$QMetaTypeId2@I@@SAHXZ 1000c6a0 f i WevoteWorker.obj
 0001:0000b6b0       ?qt_metatype_id@?$QMetaTypeId2@V?$QMap@VQString@@I@@@@SAHXZ 1000c6b0 f i WevoteWorker.obj
 0001:0000b6c0       ?qt_metatype_id@?$QMetaTypeId2@VQAssociativeIterableImpl@QtMetaTypePrivate@@@@SAHXZ 1000c6c0 f i WevoteWorker.obj
 0001:0000b6d0       ?qt_metatype_id@?$QMetaTypeId2@VQString@@@@SAHXZ 1000c6d0 f i WevoteWorker.obj
 0001:0000b6e0       ?qt_metatype_id@?$QMetaTypeId@V?$QMap@VQString@@I@@@@SAHXZ 1000c6e0 f i WevoteWorker.obj
 0001:0000b790       ?qt_metatype_id@?$QMetaTypeId@VQAssociativeIterableImpl@QtMetaTypePrivate@@@@SAHXZ 1000c790 f i WevoteWorker.obj
 0001:0000b830       ?qt_metatype_id@?$QMetaTypeIdHelper@V?$QMap@VQString@@I@@$00@QtPrivate@@SAHXZ 1000c830 f i WevoteWorker.obj
 0001:0000b840       ?qt_metatype_id@?$QMetaTypeIdHelper@VQAssociativeIterableImpl@QtMetaTypePrivate@@$00@QtPrivate@@SAHXZ 1000c840 f i WevoteWorker.obj
 0001:0000b850       ?registerConverter@?$AssociativeContainerConverterHelper@VQAssociativeIterableImpl@QtMetaTypePrivate@@$0A@@QtPrivate@@SA_NH@Z 1000c850 f i WevoteWorker.obj
 0001:0000b860       ?registerConverter@?$AssociativeValueTypeIsMetaType@V?$QMap@VQString@@I@@$00@QtPrivate@@SA_NH@Z 1000c860 f i WevoteWorker.obj
 0001:0000b8d0       ?registerConverter@?$IsPair@V?$QMap@VQString@@I@@@QtPrivate@@SA_NH@Z 1000c8d0 f i WevoteWorker.obj
 0001:0000b8e0       ?registerConverter@?$IsPair@VQAssociativeIterableImpl@QtMetaTypePrivate@@@QtPrivate@@SA_NH@Z 1000c8e0 f i WevoteWorker.obj
 0001:0000b8f0       ?registerConverter@?$MetaTypeSmartPointerHelper@V?$QMap@VQString@@I@@X@QtPrivate@@SA_NH@Z 1000c8f0 f i WevoteWorker.obj
 0001:0000b900       ?registerConverter@?$MetaTypeSmartPointerHelper@VQAssociativeIterableImpl@QtMetaTypePrivate@@X@QtPrivate@@SA_NH@Z 1000c900 f i WevoteWorker.obj
 0001:0000b910       ?registerConverter@?$SequentialContainerConverterHelper@V?$QMap@VQString@@I@@$0A@@QtPrivate@@SA_NH@Z 1000c910 f i WevoteWorker.obj
 0001:0000b920       ?registerConverter@?$SequentialContainerConverterHelper@VQAssociativeIterableImpl@QtMetaTypePrivate@@$0A@@QtPrivate@@SA_NH@Z 1000c920 f i WevoteWorker.obj
 0001:0000b930       ?reserve@?$QList@VDescriptor@U2@@@@QAEXH@Z 1000c930 f i WevoteWorker.obj
 0001:0000b960       ?rightNode@?$QMapNode@VDescriptor@U2@@VQVariant@@@@QBEPAU1@XZ 1000c960 f i WevoteWorker.obj
 0001:0000b970       ?rightNode@?$QMapNode@VQString@@PAVIntegralBus@Workflow@U2@@@@QBEPAU1@XZ 1000c970 f i WevoteWorker.obj
 0001:0000b980       ?rightNode@?$QMapNode@VQString@@VQScriptValue@@@@QBEPAU1@XZ 1000c980 f i WevoteWorker.obj
 0001:0000b990       ?rightNode@?$QMapNode@VQString@@VQVariant@@@@QBEPAU1@XZ 1000c990 f i WevoteWorker.obj
 0001:0000b9a0       ?root@?$QMapData@VDescriptor@U2@@VQVariant@@@@QBEPAU?$QMapNode@VDescriptor@U2@@VQVariant@@@@XZ 1000c9a0 f i WevoteWorker.obj
 0001:0000b9b0       ?root@?$QMapData@VQString@@PAVIntegralBus@Workflow@U2@@@@QBEPAU?$QMapNode@VQString@@PAVIntegralBus@Workflow@U2@@@@XZ 1000c9b0 f i WevoteWorker.obj
 0001:0000b9c0       ?root@?$QMapData@VQString@@VQScriptValue@@@@QBEPAU?$QMapNode@VQString@@VQScriptValue@@@@XZ 1000c9c0 f i WevoteWorker.obj
 0001:0000b9d0       ?root@?$QMapData@VQString@@VQVariant@@@@QBEPAU?$QMapNode@VQString@@VQVariant@@@@XZ 1000c9d0 f i WevoteWorker.obj
 0001:0000b9e0       ?size@?$QMap@VDescriptor@U2@@VQVariant@@@@QBEHXZ 1000c9e0 f i WevoteWorker.obj
 0001:0000b9f0       ?size@?$QMap@VQString@@I@@QBEHXZ 1000c9f0 f i WevoteWorker.obj
 0001:0000ba00       ?sl_taskFinished@WevoteWorker@LocalWorkflow@U2@@AAEXPAVTask@3@@Z 1000ca00 f   WevoteWorker.obj
 0001:0000bcb0       ?storeRelease@?$QBasicAtomicInteger@H@@QAEXH@Z 1000ccb0 f i WevoteWorker.obj
 0001:0000bcc0       ?t@Node@?$QList@VDescriptor@U2@@@@QAEAAVDescriptor@U2@@XZ 1000ccc0 f i WevoteWorker.obj
 0001:0000bcd0       ?tick@WevoteWorker@LocalWorkflow@U2@@UAEPAVTask@3@XZ 1000ccd0 f   WevoteWorker.obj
 0001:0000bf00       ?tr@WevoteWorker@LocalWorkflow@U2@@SA?AVQString@@PBD0H@Z 1000cf00 f i WevoteWorker.obj
 0001:0000bf30       ?uniqueKeys@?$QMap@VDescriptor@U2@@VQVariant@@@@QBE?AV?$QList@VDescriptor@U2@@@@XZ 1000cf30 f i WevoteWorker.obj
 0001:0000c030       ?value@?$MetaObjectForType@V?$QMap@VQString@@I@@$0A@@QtPrivate@@SAPBUQMetaObject@@XZ 1000d030 f i WevoteWorker.obj
 0001:0000c040       ?value@?$MetaObjectForType@VQAssociativeIterableImpl@QtMetaTypePrivate@@$0A@@QtPrivate@@SAPBUQMetaObject@@XZ 1000d040 f i WevoteWorker.obj
 0001:0000c050       ?value@?$QMap@VDescriptor@U2@@VQVariant@@@@QBE?BVQVariant@@ABVDescriptor@U2@@ABV2@@Z 1000d050 f i WevoteWorker.obj
 0001:0000c0b0       ?value@?$QMap@VQString@@PAVIntegralBus@Workflow@U2@@@@QBEQAVIntegralBus@Workflow@U2@@ABVQString@@ABQAV234@@Z 1000d0b0 f i WevoteWorker.obj
 0001:0000c100       ?value@const_iterator@?$QMap@VQString@@I@@QBEABIXZ 1000d100 f i WevoteWorker.obj
 0001:0000c110       ??$_Move@AAPAVDataType@U2@@@std@@YA$$QAPAVDataType@U2@@AAPAV12@@Z 1000d110 f i WevoteWorkerFactory.obj
 0001:0000c120       ??$qSwap@PAVDataType@U2@@@@YAXAAPAVDataType@U2@@0@Z 1000d120 f i WevoteWorkerFactory.obj
 0001:0000c140       ??$swap@PAVDataType@U2@@@std@@YAXAAPAVDataType@U2@@0@Z 1000d140 f i WevoteWorkerFactory.obj
 0001:0000c160       ??0?$QExplicitlySharedDataPointer@VDataType@U2@@@@QAE@ABV0@@Z 1000d160 f i WevoteWorkerFactory.obj
 0001:0000c180       ??0?$QExplicitlySharedDataPointer@VDataType@U2@@@@QAE@PAVDataType@U2@@@Z 1000d180 f i WevoteWorkerFactory.obj
 0001:0000c1a0       ??0?$QExplicitlySharedDataPointer@VDataType@U2@@@@QAE@XZ 1000d1a0 f i WevoteWorkerFactory.obj
 0001:0000c1b0       ??0?$QFlags@W4Flag@Attribute@U2@@@@QAE@VQFlag@@@Z 1000d1b0 f i WevoteWorkerFactory.obj
 0001:0000c1c0       ??0?$QFlags@W4Flag@Attribute@U2@@@@QAE@W4Flag@Attribute@U2@@@Z 1000d1c0 f i WevoteWorkerFactory.obj
 0001:0000c1d0       ??0?$QList@PAVAttribute@U2@@@@QAE@XZ 1000d1d0 f i WevoteWorkerFactory.obj
 0001:0000c1e0       ??0?$QList@PAVPortDescriptor@Workflow@U2@@@@QAE@XZ 1000d1e0 f i WevoteWorkerFactory.obj
 0001:0000c1f0       ??0?$QMap@VDescriptor@U2@@V?$QExplicitlySharedDataPointer@VDataType@U2@@@@@@QAE@XZ 1000d1f0 f i WevoteWorkerFactory.obj
 0001:0000c200       ??0?$QMap@VQString@@PAVPropertyDelegate@U2@@@@QAE@XZ 1000d200 f i WevoteWorkerFactory.obj
 0001:0000c210       ??0QStringList@@QAE@ABVQString@@@Z 1000d210 f i WevoteWorkerFactory.obj
 0001:0000c270       ??0WevoteValidator@Workflow@U2@@QAE@XZ 1000d270 f i WevoteWorkerFactory.obj
 0001:0000c280       ??0WevoteWorkerFactory@LocalWorkflow@U2@@QAE@XZ 1000d280 f   WevoteWorkerFactory.obj
 0001:0000c2a0       ??0iterator@?$QMap@VDescriptor@U2@@V?$QExplicitlySharedDataPointer@VDataType@U2@@@@@@QAE@PAU?$QMapNode@VDescriptor@U2@@V?$QExplicitlySharedDataPointer@VDataType@U2@@@@@@@Z 1000d2a0 f i WevoteWorkerFactory.obj
 0001:0000c2b0       ??0iterator@?$QMap@VQString@@PAVPropertyDelegate@U2@@@@QAE@PAU?$QMapNode@VQString@@PAVPropertyDelegate@U2@@@@@Z 1000d2b0 f i WevoteWorkerFactory.obj
 0001:0000c2c0       ??1?$QList@PAVAttribute@U2@@@@QAE@XZ 1000d2c0 f i WevoteWorkerFactory.obj
 0001:0000c2f0       ??1?$QList@PAVPortDescriptor@Workflow@U2@@@@QAE@XZ 1000d2f0 f i WevoteWorkerFactory.obj
 0001:0000c320       ??1?$QMap@VDescriptor@U2@@V?$QExplicitlySharedDataPointer@VDataType@U2@@@@@@QAE@XZ 1000d320 f i WevoteWorkerFactory.obj
 0001:0000c370       ??1?$QMap@VQString@@PAVPropertyDelegate@U2@@@@QAE@XZ 1000d370 f i WevoteWorkerFactory.obj
 0001:0000c3e0       ??1WevoteValidator@Workflow@U2@@UAE@XZ 1000d3e0 f i WevoteWorkerFactory.obj
 0001:0000c3f0       ??1WevoteWorkerFactory@LocalWorkflow@U2@@UAE@XZ 1000d3f0 f i WevoteWorkerFactory.obj
 0001:0000c400       ??4?$QExplicitlySharedDataPointer@VDataType@U2@@@@QAEAAV0@$$QAV0@@Z 1000d400 f i WevoteWorkerFactory.obj
 0001:0000c420       ??4?$QExplicitlySharedDataPointer@VDataType@U2@@@@QAEAAV0@ABV0@@Z 1000d420 f i WevoteWorkerFactory.obj
 0001:0000c470       ??6?$QList@PAVAttribute@U2@@@@QAEAAV0@ABQAVAttribute@U2@@@Z 1000d470 f i WevoteWorkerFactory.obj
 0001:0000c490       ??6?$QList@PAVPortDescriptor@Workflow@U2@@@@QAEAAV0@ABQAVPortDescriptor@Workflow@U2@@@Z 1000d490 f i WevoteWorkerFactory.obj
 0001:0000c4b0       ??A?$QMap@VDescriptor@U2@@V?$QExplicitlySharedDataPointer@VDataType@U2@@@@@@QAEAAV?$QExplicitlySharedDataPointer@VDataType@U2@@@@ABVDescriptor@U2@@@Z 1000d4b0 f i WevoteWorkerFactory.obj
 0001:0000c570       ??A?$QMap@VQString@@PAVPropertyDelegate@U2@@@@QAEAAPAVPropertyDelegate@U2@@ABVQString@@@Z 1000d570 f i WevoteWorkerFactory.obj
 0001:0000c5f0       ??Diterator@?$QMap@VDescriptor@U2@@V?$QExplicitlySharedDataPointer@VDataType@U2@@@@@@QBEAAV?$QExplicitlySharedDataPointer@VDataType@U2@@@@XZ 1000d5f0 f i WevoteWorkerFactory.obj
 0001:0000c600       ??Diterator@?$QMap@VQString@@PAVPropertyDelegate@U2@@@@QBEAAPAVPropertyDelegate@U2@@XZ 1000d600 f i WevoteWorkerFactory.obj
 0001:0000c610       ??U?$QFlags@W4Flag@Attribute@U2@@@@QBE?AV0@W4Flag@Attribute@U2@@@Z 1000d610 f i WevoteWorkerFactory.obj
 0001:0000c630       ??U@YA?AV?$QFlags@W4Flag@Attribute@U2@@@@W4Flag@Attribute@U2@@0@Z 1000d630 f i WevoteWorkerFactory.obj
 0001:0000c640       ??_EWevoteWorkerFactory@LocalWorkflow@U2@@W7AEPAXI@Z 1000d640 f i WevoteWorkerFactory.obj
 0001:0000c650       ??_G?$QExplicitlySharedDataPointer@VDataType@U2@@@@QAEPAXI@Z 1000d650 f i WevoteWorkerFactory.obj
 0001:0000c690       ??_GAttribute@U2@@UAEPAXI@Z 1000d690 f i WevoteWorkerFactory.obj
 0001:0000c690       ??_EAttribute@U2@@UAEPAXI@Z 1000d690 f i WevoteWorkerFactory.obj
 0001:0000c6c0       ??_GDelegateEditor@U2@@UAEPAXI@Z 1000d6c0 f i WevoteWorkerFactory.obj
 0001:0000c6c0       ??_EDelegateEditor@U2@@UAEPAXI@Z 1000d6c0 f i WevoteWorkerFactory.obj
 0001:0000c6f0       ??_GIntegralBusActorPrototype@Workflow@U2@@UAEPAXI@Z 1000d6f0 f i WevoteWorkerFactory.obj
 0001:0000c6f0       ??_EIntegralBusActorPrototype@Workflow@U2@@UAEPAXI@Z 1000d6f0 f i WevoteWorkerFactory.obj
 0001:0000c720       ??_GMapDataType@U2@@UAEPAXI@Z 1000d720 f i WevoteWorkerFactory.obj
 0001:0000c720       ??_EMapDataType@U2@@UAEPAXI@Z 1000d720 f i WevoteWorkerFactory.obj
 0001:0000c750       ??_EPortDescriptor@Workflow@U2@@UAEPAXI@Z 1000d750 f i WevoteWorkerFactory.obj
 0001:0000c750       ??_GPortDescriptor@Workflow@U2@@UAEPAXI@Z 1000d750 f i WevoteWorkerFactory.obj
 0001:0000c780       ??_ESpinBoxDelegate@U2@@UAEPAXI@Z 1000d780 f i WevoteWorkerFactory.obj
 0001:0000c780       ??_GSpinBoxDelegate@U2@@UAEPAXI@Z 1000d780 f i WevoteWorkerFactory.obj
 0001:0000c7b0       ??_GURLDelegate@U2@@UAEPAXI@Z 1000d7b0 f i WevoteWorkerFactory.obj
 0001:0000c7b0       ??_EURLDelegate@U2@@UAEPAXI@Z 1000d7b0 f i WevoteWorkerFactory.obj
 0001:0000c7e0       ??_EWevoteValidator@Workflow@U2@@UAEPAXI@Z 1000d7e0 f i WevoteWorkerFactory.obj
 0001:0000c7e0       ??_GWevoteValidator@Workflow@U2@@UAEPAXI@Z 1000d7e0 f i WevoteWorkerFactory.obj
 0001:0000c810       ??_GWevoteWorkerFactory@LocalWorkflow@U2@@UAEPAXI@Z 1000d810 f i WevoteWorkerFactory.obj
 0001:0000c810       ??_EWevoteWorkerFactory@LocalWorkflow@U2@@UAEPAXI@Z 1000d810 f i WevoteWorkerFactory.obj
 0001:0000c840       ?append@?$QList@PAVAttribute@U2@@@@QAEXABQAVAttribute@U2@@@Z 1000d840 f i WevoteWorkerFactory.obj
 0001:0000c8d0       ?append@?$QList@PAVPortDescriptor@Workflow@U2@@@@QAEXABQAVPortDescriptor@Workflow@U2@@@Z 1000d8d0 f i WevoteWorkerFactory.obj
 0001:0000c960       ?cleanup@WevoteWorkerFactory@LocalWorkflow@U2@@SAXXZ 1000d960 f   WevoteWorkerFactory.obj
 0001:0000c9b0       ?copy@?$QMapNode@VDescriptor@U2@@V?$QExplicitlySharedDataPointer@VDataType@U2@@@@@@QBEPAU1@PAU?$QMapData@VDescriptor@U2@@V?$QExplicitlySharedDataPointer@VDataType@U2@@@@@@@Z 1000d9b0 f i WevoteWorkerFactory.obj
 0001:0000ca40       ?copy@?$QMapNode@VQString@@PAVPropertyDelegate@U2@@@@QBEPAU1@PAU?$QMapData@VQString@@PAVPropertyDelegate@U2@@@@@Z 1000da40 f i WevoteWorkerFactory.obj
 0001:0000cad0       ?create@?$QMapData@VDescriptor@U2@@V?$QExplicitlySharedDataPointer@VDataType@U2@@@@@@SAPAU1@XZ 1000dad0 f i WevoteWorkerFactory.obj
 0001:0000cae0       ?create@?$QMapData@VQString@@PAVPropertyDelegate@U2@@@@SAPAU1@XZ 1000dae0 f i WevoteWorkerFactory.obj
 0001:0000caf0       ?createNode@?$QMapData@VDescriptor@U2@@V?$QExplicitlySharedDataPointer@VDataType@U2@@@@@@QAEPAU?$QMapNode@VDescriptor@U2@@V?$QExplicitlySharedDataPointer@VDataType@U2@@@@@@ABVDescriptor@U2@@ABV?$QExplicitlySharedDataPointer@VDataType@U2@@@@PAU2@_N@Z 1000daf0 f i WevoteWorkerFactory.obj
 0001:0000cbb0       ?createNode@?$QMapData@VQString@@PAVPropertyDelegate@U2@@@@QAEPAU?$QMapNode@VQString@@PAVPropertyDelegate@U2@@@@ABVQString@@ABQAVPropertyDelegate@U2@@PAU2@_N@Z 1000dbb0 f i WevoteWorkerFactory.obj
 0001:0000cc50       ?createWorker@WevoteWorkerFactory@LocalWorkflow@U2@@UAEPAVWorker@Workflow@3@PAVActor@53@@Z 1000dc50 f   WevoteWorkerFactory.obj
 0001:0000ccc0       ?dealloc@?$QList@PAVAttribute@U2@@@@AAEXPAUData@QListData@@@Z 1000dcc0 f i WevoteWorkerFactory.obj
 0001:0000cce0       ?dealloc@?$QList@PAVPortDescriptor@Workflow@U2@@@@AAEXPAUData@QListData@@@Z 1000dce0 f i WevoteWorkerFactory.obj
 0001:0000cd00       ?destroy@?$QMapData@VDescriptor@U2@@V?$QExplicitlySharedDataPointer@VDataType@U2@@@@@@QAEXXZ 1000dd00 f i WevoteWorkerFactory.obj
 0001:0000cd30       ?destroy@?$QMapData@VQString@@PAVPropertyDelegate@U2@@@@QAEXXZ 1000dd30 f i WevoteWorkerFactory.obj
 0001:0000cd80       ?destroySubTree@?$QMapNode@VDescriptor@U2@@V?$QExplicitlySharedDataPointer@VDataType@U2@@@@@@QAEXXZ 1000dd80 f i WevoteWorkerFactory.obj
 0001:0000cdd0       ?destroySubTree@?$QMapNode@VQString@@PAVPropertyDelegate@U2@@@@QAEXXZ 1000ddd0 f i WevoteWorkerFactory.obj
 0001:0000ce00       ?detach@?$QMap@VDescriptor@U2@@V?$QExplicitlySharedDataPointer@VDataType@U2@@@@@@QAEXXZ 1000de00 f i WevoteWorkerFactory.obj
 0001:0000ce20       ?detach@?$QMap@VQString@@PAVPropertyDelegate@U2@@@@QAEXXZ 1000de20 f i WevoteWorkerFactory.obj
 0001:0000ce40       ?detach_helper@?$QMap@VDescriptor@U2@@V?$QExplicitlySharedDataPointer@VDataType@U2@@@@@@AAEXXZ 1000de40 f i WevoteWorkerFactory.obj
 0001:0000cec0       ?detach_helper@?$QMap@VQString@@PAVPropertyDelegate@U2@@@@AAEXXZ 1000dec0 f i WevoteWorkerFactory.obj
 0001:0000cf70       ?detach_helper_grow@?$QList@PAVAttribute@U2@@@@AAEPAUNode@1@HH@Z 1000df70 f i WevoteWorkerFactory.obj
 0001:0000d080       ?detach_helper_grow@?$QList@PAVPortDescriptor@Workflow@U2@@@@AAEPAUNode@1@HH@Z 1000e080 f i WevoteWorkerFactory.obj
 0001:0000d190       ?end@?$QMapData@VDescriptor@U2@@V?$QExplicitlySharedDataPointer@VDataType@U2@@@@@@QAEPAU?$QMapNode@VDescriptor@U2@@V?$QExplicitlySharedDataPointer@VDataType@U2@@@@@@XZ 1000e190 f i WevoteWorkerFactory.obj
 0001:0000d1a0       ?end@?$QMapData@VQString@@PAVPropertyDelegate@U2@@@@QAEPAU?$QMapNode@VQString@@PAVPropertyDelegate@U2@@@@XZ 1000e1a0 f i WevoteWorkerFactory.obj
 0001:0000d1b0       ?findNode@?$QMapData@VDescriptor@U2@@V?$QExplicitlySharedDataPointer@VDataType@U2@@@@@@QBEPAU?$QMapNode@VDescriptor@U2@@V?$QExplicitlySharedDataPointer@VDataType@U2@@@@@@ABVDescriptor@U2@@@Z 1000e1b0 f i WevoteWorkerFactory.obj
 0001:0000d1f0       ?findNode@?$QMapData@VQString@@PAVPropertyDelegate@U2@@@@QBEPAU?$QMapNode@VQString@@PAVPropertyDelegate@U2@@@@ABVQString@@@Z 1000e1f0 f i WevoteWorkerFactory.obj
 0001:0000d230       ?init@WevoteWorkerFactory@LocalWorkflow@U2@@SAXXZ 1000e230 f   WevoteWorkerFactory.obj
 0001:0000e600       ?insert@?$QMap@VDescriptor@U2@@V?$QExplicitlySharedDataPointer@VDataType@U2@@@@@@QAE?AViterator@1@ABVDescriptor@U2@@ABV?$QExplicitlySharedDataPointer@VDataType@U2@@@@@Z 1000f600 f i WevoteWorkerFactory.obj
 0001:0000e700       ?insert@?$QMap@VQString@@PAVPropertyDelegate@U2@@@@QAE?AViterator@1@ABVQString@@ABQAVPropertyDelegate@U2@@@Z 1000f700 f i WevoteWorkerFactory.obj
 0001:0000e7c0       ?leftNode@?$QMapNode@VDescriptor@U2@@V?$QExplicitlySharedDataPointer@VDataType@U2@@@@@@QBEPAU1@XZ 1000f7c0 f i WevoteWorkerFactory.obj
 0001:0000e7d0       ?leftNode@?$QMapNode@VQString@@PAVPropertyDelegate@U2@@@@QBEPAU1@XZ 1000f7d0 f i WevoteWorkerFactory.obj
 0001:0000e7e0       ?lowerBound@?$QMapNode@VDescriptor@U2@@V?$QExplicitlySharedDataPointer@VDataType@U2@@@@@@QAEPAU1@ABVDescriptor@U2@@@Z 1000f7e0 f i WevoteWorkerFactory.obj
 0001:0000e820       ?lowerBound@?$QMapNode@VQString@@PAVPropertyDelegate@U2@@@@QAEPAU1@ABVQString@@@Z 1000f820 f i WevoteWorkerFactory.obj
 0001:0000e860       ?max@?$numeric_limits@H@std@@SAHXZ 1000f860 f i WevoteWorkerFactory.obj
 0001:0000e870       ?node_construct@?$QList@PAVAttribute@U2@@@@AAEXPAUNode@1@ABQAVAttribute@U2@@@Z 1000f870 f i WevoteWorkerFactory.obj
 0001:0000e890       ?node_construct@?$QList@PAVPortDescriptor@Workflow@U2@@@@AAEXPAUNode@1@ABQAVPortDescriptor@Workflow@U2@@@Z 1000f890 f i WevoteWorkerFactory.obj
 0001:0000e8b0       ?node_copy@?$QList@PAVAttribute@U2@@@@AAEXPAUNode@1@00@Z 1000f8b0 f i WevoteWorkerFactory.obj
 0001:0000e8e0       ?node_copy@?$QList@PAVPortDescriptor@Workflow@U2@@@@AAEXPAUNode@1@00@Z 1000f8e0 f i WevoteWorkerFactory.obj
 0001:0000e910       ?node_destruct@?$QList@PAVAttribute@U2@@@@AAEXPAUNode@1@0@Z 1000f910 f i WevoteWorkerFactory.obj
 0001:0000e920       ?node_destruct@?$QList@PAVAttribute@U2@@@@AAEXPAUNode@1@@Z 1000f920 f i WevoteWorkerFactory.obj
 0001:0000e930       ?node_destruct@?$QList@PAVPortDescriptor@Workflow@U2@@@@AAEXPAUNode@1@0@Z 1000f930 f i WevoteWorkerFactory.obj
 0001:0000e940       ?node_destruct@?$QList@PAVPortDescriptor@Workflow@U2@@@@AAEXPAUNode@1@@Z 1000f940 f i WevoteWorkerFactory.obj
 0001:0000e950       ?rightNode@?$QMapNode@VDescriptor@U2@@V?$QExplicitlySharedDataPointer@VDataType@U2@@@@@@QBEPAU1@XZ 1000f950 f i WevoteWorkerFactory.obj
 0001:0000e960       ?rightNode@?$QMapNode@VQString@@PAVPropertyDelegate@U2@@@@QBEPAU1@XZ 1000f960 f i WevoteWorkerFactory.obj
 0001:0000e970       ?root@?$QMapData@VDescriptor@U2@@V?$QExplicitlySharedDataPointer@VDataType@U2@@@@@@QBEPAU?$QMapNode@VDescriptor@U2@@V?$QExplicitlySharedDataPointer@VDataType@U2@@@@@@XZ 1000f970 f i WevoteWorkerFactory.obj
 0001:0000e980       ?root@?$QMapData@VQString@@PAVPropertyDelegate@U2@@@@QBEPAU?$QMapNode@VQString@@PAVPropertyDelegate@U2@@@@XZ 1000f980 f i WevoteWorkerFactory.obj
 0001:0000e990       ??C?$QScopedPointer@VQObjectData@@U?$QScopedPointerDeleter@VQObjectData@@@@@@QBEPAVQObjectData@@XZ 1000f990 f i moc_WevotePrompter.obj
 0001:0000e9a0       ?metaObject@WevotePrompter@LocalWorkflow@U2@@UBEPBUQMetaObject@@XZ 1000f9a0 f   moc_WevotePrompter.obj
 0001:0000e9c0       ?qt_metacall@WevotePrompter@LocalWorkflow@U2@@UAEHW4Call@QMetaObject@@HPAPAX@Z 1000f9c0 f   moc_WevotePrompter.obj
 0001:0000e9d0       ?qt_metacast@WevotePrompter@LocalWorkflow@U2@@UAEPAXPBD@Z 1000f9d0 f   moc_WevotePrompter.obj
 0001:0000ea30       ?qt_static_metacall@WevotePrompter@LocalWorkflow@U2@@CAXPAVQObject@@W4Call@QMetaObject@@HPAPAX@Z 1000fa30 f   moc_WevotePrompter.obj
 0001:0000ea40       ?metaObject@WevoteSupportPlugin@U2@@UBEPBUQMetaObject@@XZ 1000fa40 f   moc_WevoteSupportPlugin.obj
 0001:0000ea60       ?qt_metacall@WevoteSupportPlugin@U2@@UAEHW4Call@QMetaObject@@HPAPAX@Z 1000fa60 f   moc_WevoteSupportPlugin.obj
 0001:0000ea70       ?qt_metacast@WevoteSupportPlugin@U2@@UAEPAXPBD@Z 1000fa70 f   moc_WevoteSupportPlugin.obj
 0001:0000ead0       ?qt_static_metacall@WevoteSupportPlugin@U2@@CAXPAVQObject@@W4Call@QMetaObject@@HPAPAX@Z 1000fad0 f   moc_WevoteSupportPlugin.obj
 0001:0000eae0       ?metaObject@WevoteTask@U2@@UBEPBUQMetaObject@@XZ 1000fae0 f   moc_WevoteTask.obj
 0001:0000eb00       ?qt_metacall@WevoteTask@U2@@UAEHW4Call@QMetaObject@@HPAPAX@Z 1000fb00 f   moc_WevoteTask.obj
 0001:0000eb10       ?qt_metacast@WevoteTask@U2@@UAEPAXPBD@Z 1000fb10 f   moc_WevoteTask.obj
 0001:0000eb70       ?qt_static_metacall@WevoteTask@U2@@CAXPAVQObject@@W4Call@QMetaObject@@HPAPAX@Z 1000fb70 f   moc_WevoteTask.obj
 0001:0000eb80       ??$qMetaTypeId@PAVTask@U2@@@@YAHXZ 1000fb80 f i moc_WevoteWorker.obj
 0001:0000eb90       ??$qRegisterMetaType@PAVTask@U2@@@@YAHXZ 1000fb90 f i moc_WevoteWorker.obj
 0001:0000eba0       ??$qRegisterNormalizedMetaType@PAVTask@U2@@@@YAHABVQByteArray@@PAPAVTask@U2@@W4DefinedType@?$MetaTypeDefinedHelper@PAVTask@U2@@$00@QtPrivate@@@Z 1000fba0 f i moc_WevoteWorker.obj
 0001:0000ec00       ?Construct@?$QMetaTypeFunctionHelper@PAVTask@U2@@$00@QtMetaTypePrivate@@SAPAXPAXPBX@Z 1000fc00 f i moc_WevoteWorker.obj
 0001:0000ec30       ?Create@?$QMetaTypeFunctionHelper@PAVTask@U2@@$00@QtMetaTypePrivate@@SAPAXPBX@Z 1000fc30 f i moc_WevoteWorker.obj
 0001:0000ec70       ?Delete@?$QMetaTypeFunctionHelper@PAVTask@U2@@$00@QtMetaTypePrivate@@SAXPAX@Z 1000fc70 f i moc_WevoteWorker.obj
 0001:0000ec80       ?Destruct@?$QMetaTypeFunctionHelper@PAVTask@U2@@$00@QtMetaTypePrivate@@SAXPAX@Z 1000fc80 f i moc_WevoteWorker.obj
 0001:0000ec90       ?metaObject@WevoteWorker@LocalWorkflow@U2@@UBEPBUQMetaObject@@XZ 1000fc90 f   moc_WevoteWorker.obj
 0001:0000ecb0       ?qt_metacall@WevoteWorker@LocalWorkflow@U2@@UAEHW4Call@QMetaObject@@HPAPAX@Z 1000fcb0 f   moc_WevoteWorker.obj
 0001:0000ed10       ?qt_metacast@WevoteWorker@LocalWorkflow@U2@@UAEPAXPBD@Z 1000fd10 f   moc_WevoteWorker.obj
 0001:0000ed70       ?qt_metatype_id@?$QMetaTypeId2@PAVTask@U2@@@@SAHXZ 1000fd70 f i moc_WevoteWorker.obj
 0001:0000ed80       ?qt_metatype_id@?$QMetaTypeIdHelper@PAVTask@U2@@$00@QtPrivate@@SAHXZ 1000fd80 f i moc_WevoteWorker.obj
 0001:0000ed90       ?qt_metatype_id@?$QMetaTypeIdQObject@PAVTask@U2@@$00@@SAHXZ 1000fd90 f i moc_WevoteWorker.obj
 0001:0000ee70       ?qt_static_metacall@WevoteWorker@LocalWorkflow@U2@@CAXPAVQObject@@W4Call@QMetaObject@@HPAPAX@Z 1000fe70 f   moc_WevoteWorker.obj
 0001:0000eed0       ?registerConverter@?$AssociativeContainerConverterHelper@PAVTask@U2@@$0A@@QtPrivate@@SA_NH@Z 1000fed0 f i moc_WevoteWorker.obj
 0001:0000eee0       ?registerConverter@?$IsPair@PAVTask@U2@@@QtPrivate@@SA_NH@Z 1000fee0 f i moc_WevoteWorker.obj
 0001:0000eef0       ?registerConverter@?$MetaTypeSmartPointerHelper@PAVTask@U2@@X@QtPrivate@@SA_NH@Z 1000fef0 f i moc_WevoteWorker.obj
 0001:0000ef00       ?registerConverter@?$SequentialContainerConverterHelper@PAVTask@U2@@$0A@@QtPrivate@@SA_NH@Z 1000ff00 f i moc_WevoteWorker.obj
 0001:0000ef10       ?value@?$MetaObjectForType@PAVTask@U2@@$00@QtPrivate@@SAPBUQMetaObject@@XZ 1000ff10 f i moc_WevoteWorker.obj
 0001:0000ef16       ?countClassified@NgsReadsClassificationUtils@U2@@SAHABV?$QMap@VQString@@I@@@Z 1000ff16 f   ngs_reads_classification:ngs_reads_classification.dll
 0001:0000ef1c       ?TAXONOMY_CLASSIFICATION_SLOT@TaxonomySupport@LocalWorkflow@U2@@SA?BVDescriptor@3@XZ 1000ff1c f   ngs_reads_classification:ngs_reads_classification.dll
 0001:0000ef22       ?TAXONOMY_CLASSIFICATION_TYPE@TaxonomySupport@LocalWorkflow@U2@@SA?AV?$QExplicitlySharedDataPointer@VDataType@U2@@@@XZ 1000ff22 f   ngs_reads_classification:ngs_reads_classification.dll
 0001:0000ef28       ?getDataPathRegistry@AppContext@U2@@SAPAVU2DataPathRegistry@2@XZ 1000ff28 f   U2Core:U2Core.dll
 0001:0000ef2e       ?getAppFileStorage@AppContext@U2@@SAPAVAppFileStorage@2@XZ 1000ff2e f   U2Core:U2Core.dll
 0001:0000ef34       ??0GUrl@U2@@QAE@ABVQString@@@Z 1000ff34 f   U2Core:U2Core.dll
 0001:0000ef3a       ??1GUrl@U2@@QAE@XZ         1000ff3a f   U2Core:U2Core.dll
 0001:0000ef40       ??0FileInfo@FileStorage@U2@@QAE@ABVQString@@00@Z 1000ff40 f   U2Core:U2Core.dll
 0001:0000ef46       ??1FileInfo@FileStorage@U2@@QAE@XZ 1000ff46 f   U2Core:U2Core.dll
 0001:0000ef4c       ?getStorageDir@AppFileStorage@U2@@QBE?AVQString@@XZ 1000ff4c f   U2Core:U2Core.dll
 0001:0000ef52       ?isValid@U2DataPath@U2@@QBE_NXZ 1000ff52 f   U2Core:U2Core.dll
 0001:0000ef58       ?getPathByName@U2DataPath@U2@@QBE?AVQString@@ABV3@@Z 1000ff58 f   U2Core:U2Core.dll
 0001:0000ef5e       ?getDataPathByName@U2DataPathRegistry@U2@@QAEPAVU2DataPath@2@ABVQString@@@Z 1000ff5e f   U2Core:U2Core.dll
 0001:0000ef64       ?getFileToFileInfo@FileStorageUtils@U2@@SA?AVQString@@ABV3@0AAVWorkflowProcess@FileStorage@2@@Z 1000ff64 f   U2Core:U2Core.dll
 0001:0000ef6a       ?addFileToFileInfo@FileStorageUtils@U2@@SAXABVFileInfo@FileStorage@2@AAVWorkflowProcess@42@@Z 1000ff6a f   U2Core:U2Core.dll
 0001:0000ef70       ?errorOpeningFileRead@L10N@U2@@SA?AVQString@@ABVGUrl@2@@Z 1000ff70 f   U2Core:U2Core.dll
 0001:0000ef76       ?errorOpeningFileWrite@L10N@U2@@SA?AVQString@@ABVGUrl@2@@Z 1000ff76 f   U2Core:U2Core.dll
 0001:0000ef7c       ??0Logger@U2@@QAE@ABVQString@@@Z 1000ff7c f   U2Core:U2Core.dll
 0001:0000ef82       ??1Logger@U2@@UAE@XZ       1000ff82 f   U2Core:U2Core.dll
 0001:0000ef88       ?details@Logger@U2@@QAEXABVQString@@@Z 1000ff88 f   U2Core:U2Core.dll
 0001:0000ef8e       ?tr@Task@U2@@SA?AVQString@@PBD0H@Z 1000ff8e f   U2Core:U2Core.dll
 0001:0000ef94       ??0Task@U2@@QAE@ABVQString@@V?$QFlags@W4TaskFlag@U2@@@@@Z 1000ff94 f   U2Core:U2Core.dll
 0001:0000ef9a       ?setError@Task@U2@@QAEXABVQString@@@Z 1000ff9a f   U2Core:U2Core.dll
 0001:0000efa0       ??1Task@U2@@UAE@XZ         1000ffa0 f   U2Core:U2Core.dll
 0001:0000efa6       ?cleanup@Task@U2@@UAEXXZ   1000ffa6 f   U2Core:U2Core.dll
 0001:0000efac       ?generateReport@Task@U2@@UBE?AVQString@@XZ 1000ffac f   U2Core:U2Core.dll
 0001:0000efb2       ?getNumParallelSubtasks@Task@U2@@UBEHXZ 1000ffb2 f   U2Core:U2Core.dll
 0001:0000efb8       ?getParentTask@Task@U2@@UBEPAV12@XZ 1000ffb8 f   U2Core:U2Core.dll
 0001:0000efbe       ?getSubtaskWithErrors@Task@U2@@UBEPAV12@XZ 1000ffbe f   U2Core:U2Core.dll
 0001:0000efc4       ?getTaskId@Task@U2@@UBE_JXZ 1000ffc4 f   U2Core:U2Core.dll
 0001:0000efca       ?getTopLevelParentTask@Task@U2@@UAEPAV12@XZ 1000ffca f   U2Core:U2Core.dll
 0001:0000efd0       ?getWarnings@Task@U2@@UBE?AVQStringList@@XZ 1000ffd0 f   U2Core:U2Core.dll
 0001:0000efd6       ?hasSubtasksWithErrors@Task@U2@@UBE_NXZ 1000ffd6 f   U2Core:U2Core.dll
 0001:0000efdc       ?hasWarning@Task@U2@@UBE_NXZ 1000ffdc f   U2Core:U2Core.dll
 0001:0000efe2       ?isNotificationReport@Task@U2@@UBE_NXZ 1000ffe2 f   U2Core:U2Core.dll
 0001:0000efe8       ?isReportingEnabled@Task@U2@@UBE_NXZ 1000ffe8 f   U2Core:U2Core.dll
 0001:0000efee       ?isReportingSupported@Task@U2@@UBE_NXZ 1000ffee f   U2Core:U2Core.dll
 0001:0000eff4       ?isTopLevelTask@Task@U2@@UBE_NXZ 1000fff4 f   U2Core:U2Core.dll
 0001:0000effa       ?metaObject@Task@U2@@UBEPBUQMetaObject@@XZ 1000fffa f   U2Core:U2Core.dll
 0001:0000f000       ?onSubTaskFinished@Task@U2@@MAE?AV?$QList@PAVTask@U2@@@@PAV12@@Z 10010000 f   U2Core:U2Core.dll
 0001:0000f006       ?prepare@Task@U2@@UAEXXZ   10010006 f   U2Core:U2Core.dll
 0001:0000f00c       ?propagateSubtaskError@Task@U2@@UAE_NXZ 1001000c f   U2Core:U2Core.dll
 0001:0000f012       ?qt_metacall@Task@U2@@UAEHW4Call@QMetaObject@@HPAPAX@Z 10010012 f   U2Core:U2Core.dll
 0001:0000f018       ?qt_metacast@Task@U2@@UAEPAXPBD@Z 10010018 f   U2Core:U2Core.dll
 0001:0000f01e       ?setCollectChildrensWarningsFlag@Task@U2@@UAEX_N@Z 1001001e f   U2Core:U2Core.dll
 0001:0000f024       ?setNoAutoDelete@Task@U2@@UAEX_N@Z 10010024 f   U2Core:U2Core.dll
 0001:0000f02a       ?setNotificationReport@Task@U2@@UAEX_N@Z 1001002a f   U2Core:U2Core.dll
 0001:0000f030       ?setReportingEnabled@Task@U2@@UAEX_N@Z 10010030 f   U2Core:U2Core.dll
 0001:0000f036       ?setReportingSupported@Task@U2@@UAEX_N@Z 10010036 f   U2Core:U2Core.dll
 0001:0000f03c       ?tr@ExternalTool@U2@@SA?AVQString@@PBD0H@Z 1001003c f   U2Core:U2Core.dll
 0001:0000f042       ??0ExternalTool@U2@@QAE@VQString@@0@Z 10010042 f   U2Core:U2Core.dll
 0001:0000f048       ??1ExternalTool@U2@@UAE@XZ 10010048 f   U2Core:U2Core.dll
 0001:0000f04e       ?getAdditionalParameters@ExternalTool@U2@@UAEXABVQString@@@Z 1001004e f   U2Core:U2Core.dll
 0001:0000f054       ?getAdditionalPaths@ExternalTool@U2@@UBE?AVQStringList@@XZ 10010054 f   U2Core:U2Core.dll
 0001:0000f05a       ?getToolRunnerAdditionalOptions@ExternalTool@U2@@UAE?BVQStringList@@XZ 1001005a f   U2Core:U2Core.dll
 0001:0000f060       ?metaObject@ExternalTool@U2@@UBEPBUQMetaObject@@XZ 10010060 f   U2Core:U2Core.dll
 0001:0000f066       ?performAdditionalChecks@ExternalTool@U2@@UAEXABVQString@@@Z 10010066 f   U2Core:U2Core.dll
 0001:0000f06c       ?qt_metacall@ExternalTool@U2@@UAEHW4Call@QMetaObject@@HPAPAX@Z 1001006c f   U2Core:U2Core.dll
 0001:0000f072       ?qt_metacast@ExternalTool@U2@@UAEPAXPBD@Z 10010072 f   U2Core:U2Core.dll
 0001:0000f078       ?getExternalToolRegistry@AppContext@U2@@SAPAVExternalToolRegistry@2@XZ 10010078 f   U2Core:U2Core.dll
 0001:0000f07e       ?registerEntry@ExternalToolRegistry@U2@@QAE_NPAVExternalTool@2@@Z 1001007e f   U2Core:U2Core.dll
 0001:0000f084       ?unregisterEntry@ExternalToolRegistry@U2@@QAEXABVQString@@@Z 10010084 f   U2Core:U2Core.dll
 0001:0000f08a       ??0Plugin@U2@@QAE@ABVQString@@0_NW4PluginState@1@@Z 1001008a f   U2Core:U2Core.dll
 0001:0000f090       ??1Plugin@U2@@UAE@XZ       10010090 f   U2Core:U2Core.dll
 0001:0000f096       ?open@IOAdapterUtils@U2@@SAPAVIOAdapter@2@ABVGUrl@2@AAVU2OpStatus@2@W4IOAdapterMode@2@PAVIOAdapterFactory@2@@Z 10010096 f   U2Core:U2Core.dll
 0001:0000f09c       ?addSubTask@Task@U2@@QAEXPAV12@@Z 1001009c f   U2Core:U2Core.dll
 0001:0000f0a2       ??0ExternalToolRunTask@U2@@QAE@ABVQString@@ABVQStringList@@PAVExternalToolLogParser@1@010_N@Z 100100a2 f   U2Core:U2Core.dll
 0001:0000f0a8       ??1ExternalToolRunTask@U2@@UAE@XZ 100100a8 f   U2Core:U2Core.dll
 0001:0000f0ae       ??0ExternalToolSupportTask@U2@@QAE@ABVQString@@V?$QFlags@W4TaskFlag@U2@@@@@Z 100100ae f   U2Core:U2Core.dll
 0001:0000f0b4       ??1ExternalToolSupportTask@U2@@UAE@XZ 100100b4 f   U2Core:U2Core.dll
 0001:0000f0ba       ??0ExternalToolLogParser@U2@@QAE@XZ 100100ba f   U2Core:U2Core.dll
 0001:0000f0c0       ??1ExternalToolLogParser@U2@@UAE@XZ 100100c0 f   U2Core:U2Core.dll
 0001:0000f0c6       ?getProgress@ExternalToolLogParser@U2@@UAEHXZ 100100c6 f   U2Core:U2Core.dll
 0001:0000f0cc       ?isError@ExternalToolLogParser@U2@@MBE_NABVQString@@@Z 100100cc f   U2Core:U2Core.dll
 0001:0000f0d2       ?metaObject@ExternalToolLogParser@U2@@UBEPBUQMetaObject@@XZ 100100d2 f   U2Core:U2Core.dll
 0001:0000f0d8       ?metaObject@ExternalToolRunTask@U2@@UBEPBUQMetaObject@@XZ 100100d8 f   U2Core:U2Core.dll
 0001:0000f0de       ?parseErrOutput@ExternalToolLogParser@U2@@UAEXABVQString@@@Z 100100de f   U2Core:U2Core.dll
 0001:0000f0e4       ?parseOutput@ExternalToolLogParser@U2@@UAEXABVQString@@@Z 100100e4 f   U2Core:U2Core.dll
 0001:0000f0ea       ?processErrLine@ExternalToolLogParser@U2@@MAEXABVQString@@@Z 100100ea f   U2Core:U2Core.dll
 0001:0000f0f0       ?processLine@ExternalToolLogParser@U2@@MAEXABVQString@@@Z 100100f0 f   U2Core:U2Core.dll
 0001:0000f0f6       ?qt_metacall@ExternalToolLogParser@U2@@UAEHW4Call@QMetaObject@@HPAPAX@Z 100100f6 f   U2Core:U2Core.dll
 0001:0000f0fc       ?qt_metacall@ExternalToolRunTask@U2@@UAEHW4Call@QMetaObject@@HPAPAX@Z 100100fc f   U2Core:U2Core.dll
 0001:0000f102       ?qt_metacast@ExternalToolLogParser@U2@@UAEPAXPBD@Z 10010102 f   U2Core:U2Core.dll
 0001:0000f108       ?qt_metacast@ExternalToolRunTask@U2@@UAEPAXPBD@Z 10010108 f   U2Core:U2Core.dll
 0001:0000f10e       ?report@Task@U2@@UAE?AW4ReportResult@12@XZ 1001010e f   U2Core:U2Core.dll
 0001:0000f114       ?run@ExternalToolRunTask@U2@@UAEXXZ 10010114 f   U2Core:U2Core.dll
 0001:0000f11a       ?setLastError@ExternalToolLogParser@U2@@MAEXABVQString@@@Z 1001011a f   U2Core:U2Core.dll
 0001:0000f120       ?setListenerForHelper@ExternalToolSupportTask@U2@@MAEXPAVExternalToolRunTaskHelper@2@H@Z 10010120 f   U2Core:U2Core.dll
 0001:0000f126       ?setListenerForTask@ExternalToolSupportTask@U2@@MAEXPAVExternalToolRunTask@2@H@Z 10010126 f   U2Core:U2Core.dll
 0001:0000f12c       ?error@Logger@U2@@QAEXABVQString@@@Z 1001012c f   U2Core:U2Core.dll
 0001:0000f132       ??0TaskStateInfo@U2@@QAE@XZ 10010132 f   U2Core:U2Core.dll
 0001:0000f138       ?getError@TaskStateInfo@U2@@UBE?AVQString@@XZ 10010138 f   U2Core:U2Core.dll
 0001:0000f13e       ?setError@TaskStateInfo@U2@@UAEXABVQString@@@Z 1001013e f   U2Core:U2Core.dll
 0001:0000f144       ??1TaskStateInfo@U2@@UAE@XZ 10010144 f   U2Core:U2Core.dll
 0001:0000f14a       ?hasError@Task@U2@@QBE_NXZ 1001014a f   U2Core:U2Core.dll
 0001:0000f150       ??0FailTask@U2@@QAE@ABVQString@@@Z 10010150 f   U2Core:U2Core.dll
 0001:0000f156       ??1FailTask@U2@@UAE@XZ     10010156 f   U2Core:U2Core.dll
 0001:0000f15c       ?createWorkingDir@FileAndDirectoryUtils@U2@@SA?AVQString@@ABV3@H00@Z 1001015c f   U2Core:U2Core.dll
 0001:0000f162       ?createDirectory@GUrlUtils@U2@@SA?AVQString@@ABV3@0AAVU2OpStatus@2@@Z 10010162 f   U2Core:U2Core.dll
 0001:0000f168       ??0TaskSignalMapper@U2@@QAE@PAVTask@1@@Z 10010168 f   U2Core:U2Core.dll
 0001:0000f16e       ?getError@U2OpStatusImpl@U2@@UBE?AVQString@@XZ 1001016e f   U2Core:U2Core.dll
 0001:0000f174       ??0U2OpStatus2Log@U2@@QAE@W4LogLevel@1@@Z 10010174 f   U2Core:U2Core.dll
 0001:0000f17a       ??1U2OpStatus2Log@U2@@UAE@XZ 1001017a f   U2Core:U2Core.dll
 0001:0000f180       ?addListeners@ExternalToolSupportTask@U2@@QAEXABV?$QList@PAVExternalToolListener@U2@@@@@Z 10010180 f   U2Core:U2Core.dll
 0001:0000f186       ?runScript@ScriptTask@U2@@SA?AVQScriptValue@@PAVQScriptEngine@@ABV?$QMap@VQString@@VQScriptValue@@@@ABVQString@@AAVTaskStateInfo@2@@Z 10010186 f   U2Core:U2Core.dll
 0001:0000f18c       ?metaObject@FailTask@U2@@UBEPBUQMetaObject@@XZ 1001018c f   U2Core:U2Core.dll
 0001:0000f192       ?metaObject@TaskSignalMapper@U2@@UBEPBUQMetaObject@@XZ 10010192 f   U2Core:U2Core.dll
 0001:0000f198       ?qt_metacall@FailTask@U2@@UAEHW4Call@QMetaObject@@HPAPAX@Z 10010198 f   U2Core:U2Core.dll
 0001:0000f19e       ?qt_metacall@TaskSignalMapper@U2@@UAEHW4Call@QMetaObject@@HPAPAX@Z 1001019e f   U2Core:U2Core.dll
 0001:0000f1a4       ?qt_metacast@FailTask@U2@@UAEPAXPBD@Z 100101a4 f   U2Core:U2Core.dll
 0001:0000f1aa       ?qt_metacast@TaskSignalMapper@U2@@UAEPAXPBD@Z 100101aa f   U2Core:U2Core.dll
 0001:0000f1b0       ?run@Task@U2@@UAEXXZ       100101b0 f   U2Core:U2Core.dll
 0001:0000f1b6       ?getAppSettings@AppContext@U2@@SAPAVAppSettings@2@XZ 100101b6 f   U2Core:U2Core.dll
 0001:0000f1bc       ?qt_metacast@Plugin@U2@@UAEPAXPBD@Z 100101bc f   U2Core:U2Core.dll
 0001:0000f1c2       ?qt_metacall@Plugin@U2@@UAEHW4Call@QMetaObject@@HPAPAX@Z 100101c2 f   U2Core:U2Core.dll
 0001:0000f1c8       ??0TabulatedFormatReader@U2@@QAE@AAVU2OpStatus@1@PAVIOAdapter@1@@Z 100101c8 f   U2Formats:U2Formats.dll
 0001:0000f1ce       ?hasNextLine@TabulatedFormatReader@U2@@QBE_NXZ 100101ce f   U2Formats:U2Formats.dll
 0001:0000f1d4       ?getNextLine@TabulatedFormatReader@U2@@QAE?AVQStringList@@XZ 100101d4 f   U2Formats:U2Formats.dll
 0001:0000f1da       ??1TabulatedFormatReader@U2@@UAE@XZ 100101da f   U2Formats:U2Formats.dll
 0001:0000f1e0       ?prepareDocumentsFileFilter@DialogUtils@U2@@SA?AVQString@@ABV3@_NABVQStringList@@@Z 100101e0 f   U2Gui:U2Gui.dll
 0001:0000f1e6       ?getInputPorts@Actor@Workflow@U2@@QBE?AV?$QList@PAVPort@Workflow@U2@@@@XZ 100101e6 f   U2Lang:U2Lang.dll
 0001:0000f1ec       ?getOutputPorts@Actor@Workflow@U2@@QBE?AV?$QList@PAVPort@Workflow@U2@@@@XZ 100101ec f   U2Lang:U2Lang.dll
 0001:0000f1f2       ??0PrompterBaseImpl@U2@@QAE@PAVActor@Workflow@1@@Z 100101f2 f   U2Lang:U2Lang.dll
 0001:0000f1f8       ??1PrompterBaseImpl@U2@@UAE@XZ 100101f8 f   U2Lang:U2Lang.dll
 0001:0000f1fe       ?metaObject@PrompterBaseImpl@U2@@UBEPBUQMetaObject@@XZ 100101fe f   U2Lang:U2Lang.dll
 0001:0000f204       ?qt_metacall@PrompterBaseImpl@U2@@UAEHW4Call@QMetaObject@@HPAPAX@Z 10010204 f   U2Lang:U2Lang.dll
 0001:0000f20a       ?qt_metacast@PrompterBaseImpl@U2@@UAEPAXPBD@Z 1001020a f   U2Lang:U2Lang.dll
 0001:0000f210       ?sl_actorModified@PrompterBaseImpl@U2@@MAEXXZ 10010210 f   U2Lang:U2Lang.dll
 0001:0000f216       ?update@PrompterBaseImpl@U2@@UAEXABV?$QMap@VQString@@VQVariant@@@@@Z 10010216 f   U2Lang:U2Lang.dll
 0001:0000f21c       ??0WorkflowNotification@U2@@QAE@ABVQString@@00@Z 1001021c f   U2Lang:U2Lang.dll
 0001:0000f222       ??1WorkflowNotification@U2@@QAE@XZ 10010222 f   U2Lang:U2Lang.dll
 0001:0000f228       ??0WorkflowNotification@U2@@QAE@ABV01@@Z 10010228 f   U2Lang:U2Lang.dll
 0001:0000f22e       ?getId@Actor@Workflow@U2@@QBE?AVQString@@XZ 1001022e f   U2Lang:U2Lang.dll
 0001:0000f234       ??1Descriptor@U2@@UAE@XZ   10010234 f   U2Lang:U2Lang.dll
 0001:0000f23a       ?getId@Descriptor@U2@@QBE?AVQString@@XZ 1001023a f   U2Lang:U2Lang.dll
 0001:0000f240       ??0Descriptor@U2@@QAE@ABV01@@Z 10010240 f   U2Lang:U2Lang.dll
 0001:0000f246       ?URL_SLOT@BaseSlots@Workflow@U2@@SA?BVDescriptor@3@XZ 10010246 f   U2Lang:U2Lang.dll
 0001:0000f24c       ?initEngine@WorkflowScriptLibrary@U2@@SAXPAVWorkflowScriptEngine@2@@Z 1001024c f   U2Lang:U2Lang.dll
 0001:0000f252       ?getFileUrl@MessageMetadata@U2@@QBEABVQString@@XZ 10010252 f   U2Lang:U2Lang.dll
 0001:0000f258       ??1MessageMetadata@U2@@QAE@XZ 10010258 f   U2Lang:U2Lang.dll
 0001:0000f25e       ?get@MessageMetadataStorage@U2@@QBE?AVMessageMetadata@2@H@Z 1001025e f   U2Lang:U2Lang.dll
 0001:0000f264       ?getMonitor@WorkflowContext@Workflow@U2@@QAEPAVWorkflowMonitor@23@XZ 10010264 f   U2Lang:U2Lang.dll
 0001:0000f26a       ?getWorkflowProcess@WorkflowContext@Workflow@U2@@QAEAAVWorkflowProcess@FileStorage@3@XZ 1001026a f   U2Lang:U2Lang.dll
 0001:0000f270       ?workingDir@WorkflowContext@Workflow@U2@@QBE?AVQString@@XZ 10010270 f   U2Lang:U2Lang.dll
 0001:0000f276       ?absolutePath@WorkflowContext@Workflow@U2@@QBE?AVQString@@ABV4@@Z 10010276 f   U2Lang:U2Lang.dll
 0001:0000f27c       ?getMetadataStorage@WorkflowContext@Workflow@U2@@QAEAAVMessageMetadataStorage@3@XZ 1001027c f   U2Lang:U2Lang.dll
 0001:0000f282       ??0WorkflowScriptEngine@U2@@QAE@PAVWorkflowContext@Workflow@1@@Z 10010282 f   U2Lang:U2Lang.dll
 0001:0000f288       ??1WorkflowScriptEngine@U2@@UAE@XZ 10010288 f   U2Lang:U2Lang.dll
 0001:0000f28e       ?isEmpty@AttributeScript@U2@@QBE_NXZ 1001028e f   U2Lang:U2Lang.dll
 0001:0000f294       ?getScriptText@AttributeScript@U2@@QBEABVQString@@XZ 10010294 f   U2Lang:U2Lang.dll
 0001:0000f29a       ?getScriptVars@AttributeScript@U2@@QBEABV?$QMap@VDescriptor@U2@@VQVariant@@@@XZ 1001029a f   U2Lang:U2Lang.dll
 0001:0000f2a0       ??0Message@Workflow@U2@@QAE@V?$QExplicitlySharedDataPointer@VDataType@U2@@@@ABVQVariant@@H@Z 100102a0 f   U2Lang:U2Lang.dll
 0001:0000f2a6       ?getData@Message@Workflow@U2@@QBE?AVQVariant@@XZ 100102a6 f   U2Lang:U2Lang.dll
 0001:0000f2ac       ?getMetadataId@Message@Workflow@U2@@QBEHXZ 100102ac f   U2Lang:U2Lang.dll
 0001:0000f2b2       ??1Message@Workflow@U2@@QAE@XZ 100102b2 f   U2Lang:U2Lang.dll
 0001:0000f2b8       ?addOutputFile@WorkflowMonitor@Workflow@U2@@QAEXABVQString@@0_N@Z 100102b8 f   U2Lang:U2Lang.dll
 0001:0000f2be       ?addInfo@WorkflowMonitor@Workflow@U2@@QAEXABVQString@@00@Z 100102be f   U2Lang:U2Lang.dll
 0001:0000f2c4       ?isOutUrlAttribute@RFSUtils@U2@@SA_NPAVAttribute@2@PAVActor@Workflow@2@AA_N@Z 100102c4 f   U2Lang:U2Lang.dll
 0001:0000f2ca       ?getBusType@IntegralBus@Workflow@U2@@QBE?AV?$QExplicitlySharedDataPointer@VDataType@U2@@@@XZ 100102ca f   U2Lang:U2Lang.dll
 0001:0000f2d0       ??0BaseWorker@LocalWorkflow@U2@@QAE@PAVActor@Workflow@2@_N@Z 100102d0 f   U2Lang:U2Lang.dll
 0001:0000f2d6       ??1BaseWorker@LocalWorkflow@U2@@UAE@XZ 100102d6 f   U2Lang:U2Lang.dll
 0001:0000f2dc       ?createLogListeners@BaseWorker@LocalWorkflow@U2@@QAE?AV?$QList@PAVExternalToolListener@U2@@@@H@Z 100102dc f   U2Lang:U2Lang.dll
 0001:0000f2e2       ?addCommunication@BaseWorker@LocalWorkflow@U2@@UAE_NABVQString@@PAVCommunicationChannel@Workflow@3@@Z 100102e2 f   U2Lang:U2Lang.dll
 0001:0000f2e8       ?canTaskBeCanceled@BaseWorker@LocalWorkflow@U2@@MBE_NPAVTask@3@@Z 100102e8 f   U2Lang:U2Lang.dll
 0001:0000f2ee       ?getActorId@BaseWorker@LocalWorkflow@U2@@UBE?AVQString@@XZ 100102ee f   U2Lang:U2Lang.dll
 0001:0000f2f4       ?getCommunication@BaseWorker@LocalWorkflow@U2@@UAEPAVCommunicationChannel@Workflow@3@ABVQString@@@Z 100102f4 f   U2Lang:U2Lang.dll
 0001:0000f2fa       ?getMessageAndSetupScriptValues@BaseWorker@LocalWorkflow@U2@@UAE?AVMessage@Workflow@3@PAVCommunicationChannel@53@@Z 100102fa f   U2Lang:U2Lang.dll
 0001:0000f300       ?getOutputFiles@BaseWorker@LocalWorkflow@U2@@UAE?AVQStringList@@XZ 10010300 f   U2Lang:U2Lang.dll
 0001:0000f306       ?isDone@BaseWorker@LocalWorkflow@U2@@UBE_NXZ 10010306 f   U2Lang:U2Lang.dll
 0001:0000f30c       ?isReady@BaseWorker@LocalWorkflow@U2@@UBE_NXZ 1001030c f   U2Lang:U2Lang.dll
 0001:0000f312       ?setDone@BaseWorker@LocalWorkflow@U2@@UAEXXZ 10010312 f   U2Lang:U2Lang.dll
 0001:0000f318       ??0Descriptor@U2@@QAE@ABVQString@@00@Z 10010318 f   U2Lang:U2Lang.dll
 0001:0000f31e       ??0Descriptor@U2@@QAE@ABVQString@@@Z 1001031e f   U2Lang:U2Lang.dll
 0001:0000f324       ??0MapDataType@U2@@QAE@ABVDescriptor@1@ABV?$QMap@VDescriptor@U2@@V?$QExplicitlySharedDataPointer@VDataType@U2@@@@@@@Z 10010324 f   U2Lang:U2Lang.dll
 0001:0000f32a       ??1MapDataType@U2@@UAE@XZ  1001032a f   U2Lang:U2Lang.dll
 0001:0000f330       ??0Attribute@U2@@QAE@ABVDescriptor@1@V?$QExplicitlySharedDataPointer@VDataType@U2@@@@V?$QFlags@W4Flag@Attribute@U2@@@@ABVQVariant@@@Z 10010330 f   U2Lang:U2Lang.dll
 0001:0000f336       ??0Attribute@U2@@QAE@ABVDescriptor@1@V?$QExplicitlySharedDataPointer@VDataType@U2@@@@_NABVQVariant@@@Z 10010336 f   U2Lang:U2Lang.dll
 0001:0000f33c       ??1Attribute@U2@@UAE@XZ    1001033c f   U2Lang:U2Lang.dll
 0001:0000f342       ??0DelegateTags@U2@@QAE@PAVQObject@@@Z 10010342 f   U2Lang:U2Lang.dll
 0001:0000f348       ?set@DelegateTags@U2@@QAEXABVQString@@ABVQVariant@@@Z 10010348 f   U2Lang:U2Lang.dll
 0001:0000f34e       ??1DelegateTags@U2@@UAE@XZ 1001034e f   U2Lang:U2Lang.dll
 0001:0000f354       ??0PortDescriptor@Workflow@U2@@QAE@ABVDescriptor@2@V?$QExplicitlySharedDataPointer@VDataType@U2@@@@_N2I@Z 10010354 f   U2Lang:U2Lang.dll
 0001:0000f35a       ??1PortDescriptor@Workflow@U2@@UAE@XZ 1001035a f   U2Lang:U2Lang.dll
 0001:0000f360       ??0ActorPrototype@Workflow@U2@@QAE@ABVDescriptor@2@ABV?$QList@PAVPortDescriptor@Workflow@U2@@@@ABV?$QList@PAVAttribute@U2@@@@@Z 10010360 f   U2Lang:U2Lang.dll
 0001:0000f366       ??1ActorPrototype@Workflow@U2@@UAE@XZ 10010366 f   U2Lang:U2Lang.dll
 0001:0000f36c       ?setEditor@ActorPrototype@Workflow@U2@@QAEXPAVConfigurationEditor@3@@Z 1001036c f   U2Lang:U2Lang.dll
 0001:0000f372       ?setValidator@ActorPrototype@Workflow@U2@@QAEXPAVConfigurationValidator@3@@Z 10010372 f   U2Lang:U2Lang.dll
 0001:0000f378       ?setPrompter@ActorPrototype@Workflow@U2@@QAEXPAVPrompter@23@@Z 10010378 f   U2Lang:U2Lang.dll
 0001:0000f37e       ?addExternalTool@ActorPrototype@Workflow@U2@@QAEXABVQString@@0@Z 1001037e f   U2Lang:U2Lang.dll
 0001:0000f384       ?registerProto@ActorPrototypeRegistry@Workflow@U2@@QAEXABVDescriptor@3@PAVActorPrototype@23@@Z 10010384 f   U2Lang:U2Lang.dll
 0001:0000f38a       ?unregisterProto@ActorPrototypeRegistry@Workflow@U2@@QAEPAVActorPrototype@23@ABVQString@@@Z 1001038a f   U2Lang:U2Lang.dll
 0001:0000f390       ?STRING_TYPE@BaseTypes@U2@@SA?AV?$QExplicitlySharedDataPointer@VDataType@U2@@@@XZ 10010390 f   U2Lang:U2Lang.dll
 0001:0000f396       ?NUM_TYPE@BaseTypes@U2@@SA?AV?$QExplicitlySharedDataPointer@VDataType@U2@@@@XZ 10010396 f   U2Lang:U2Lang.dll
 0001:0000f39c       ?getInstance@WorkflowEnv@Workflow@U2@@KAPAV123@XZ 1001039c f   U2Lang:U2Lang.dll
 0001:0000f3a2       ??0DomainFactory@Workflow@U2@@QAE@ABVQString@@@Z 100103a2 f   U2Lang:U2Lang.dll
 0001:0000f3a8       ??1DomainFactory@Workflow@U2@@UAE@XZ 100103a8 f   U2Lang:U2Lang.dll
 0001:0000f3ae       ?clone@Attribute@U2@@UAEPAV12@XZ 100103ae f   U2Lang:U2Lang.dll
 0001:0000f3b4       ?createConnection@DomainFactory@Workflow@U2@@UAEPAVCommunicationChannel@23@PAVLink@23@@Z 100103b4 f   U2Lang:U2Lang.dll
 0001:0000f3ba       ?createInstance@ActorPrototype@Workflow@U2@@UAEPAVActor@23@ABVQString@@PAVAttributeScript@3@ABV?$QMap@VQString@@VQVariant@@@@@Z 100103ba f   U2Lang:U2Lang.dll
 0001:0000f3c0       ?createPort@IntegralBusActorPrototype@Workflow@U2@@UAEPAVPort@23@ABVPortDescriptor@23@PAVActor@23@@Z 100103c0 f   U2Lang:U2Lang.dll
 0001:0000f3c6       ?createScheduler@DomainFactory@Workflow@U2@@UAEPAVScheduler@23@PAVSchema@23@@Z 100103c6 f   U2Lang:U2Lang.dll
 0001:0000f3cc       ?destroy@DomainFactory@Workflow@U2@@UAEXPAVScheduler@23@PAVSchema@23@@Z 100103cc f   U2Lang:U2Lang.dll
 0001:0000f3d2       ?getAllDescriptors@MapDataType@U2@@UBE?AV?$QList@VDescriptor@U2@@@@XZ 100103d2 f   U2Lang:U2Lang.dll
 0001:0000f3d8       ?getAllEntries@?$IdRegistry@VDomainFactory@Workflow@U2@@@U2@@UBE?AV?$QList@PAVDomainFactory@Workflow@U2@@@@XZ 100103d8 f   U2Lang:U2Lang.dll
 0001:0000f3de       ?getAllIds@?$IdRegistry@VDomainFactory@Workflow@U2@@@U2@@UBE?AV?$QList@VQString@@@@XZ 100103de f   U2Lang:U2Lang.dll
 0001:0000f3e4       ?getAttributePureValue@Attribute@U2@@UBEABVQVariant@@XZ 100103e4 f   U2Lang:U2Lang.dll
 0001:0000f3ea       ?getById@?$IdRegistry@VDomainFactory@Workflow@U2@@@U2@@UAEPAVDomainFactory@Workflow@2@ABVQString@@@Z 100103ea f   U2Lang:U2Lang.dll
 0001:0000f3f0       ?getDatatypeByDescriptor@MapDataType@U2@@UBE?AV?$QExplicitlySharedDataPointer@VDataType@U2@@@@ABVDescriptor@2@@Z 100103f0 f   U2Lang:U2Lang.dll
 0001:0000f3f6       ?getDatatypesMap@MapDataType@U2@@UBE?AV?$QMap@VDescriptor@U2@@V?$QExplicitlySharedDataPointer@VDataType@U2@@@@@@XZ 100103f6 f   U2Lang:U2Lang.dll
 0001:0000f3fc       ?getDefaultPureValue@Attribute@U2@@UBEABVQVariant@@XZ 100103fc f   U2Lang:U2Lang.dll
 0001:0000f402       ?getGroup@Attribute@U2@@UAE?AW4AttributeGroup@2@XZ 10010402 f   U2Lang:U2Lang.dll
 0001:0000f408       ?getItems@PropertyDelegate@U2@@UBEXAAV?$QMap@VQString@@VQVariant@@@@@Z 10010408 f   U2Lang:U2Lang.dll
 0001:0000f40e       ?getType@PortDescriptor@Workflow@U2@@UBE?AV?$QExplicitlySharedDataPointer@VDataType@U2@@@@XZ 1001040e f   U2Lang:U2Lang.dll
 0001:0000f414       ?getWidget@ConfigurationEditor@U2@@UAEPAVQWidget@@XZ 10010414 f   U2Lang:U2Lang.dll
 0001:0000f41a       ?isAcceptableDrop@ActorPrototype@Workflow@U2@@UBE_NPBVQMimeData@@PAV?$QMap@VQString@@VQVariant@@@@@Z 1001041a f   U2Lang:U2Lang.dll
 0001:0000f420       ?isDefaultValue@Attribute@U2@@UBE_NXZ 10010420 f   U2Lang:U2Lang.dll
 0001:0000f426       ?isEmpty@Attribute@U2@@UBE_NXZ 10010426 f   U2Lang:U2Lang.dll
 0001:0000f42c       ?isEmpty@ConfigurationEditor@U2@@UBE_NXZ 1001042c f   U2Lang:U2Lang.dll
 0001:0000f432       ?kind@MapDataType@U2@@UBE?AW4Kind@DataType@2@XZ 10010432 f   U2Lang:U2Lang.dll
 0001:0000f438       ?registerEntry@?$IdRegistry@VDomainFactory@Workflow@U2@@@U2@@UAE_NPAVDomainFactory@Workflow@2@@Z 10010438 f   U2Lang:U2Lang.dll
 0001:0000f43e       ?setAttributeValue@Attribute@U2@@UAEXABVQVariant@@@Z 1001043e f   U2Lang:U2Lang.dll
 0001:0000f444       ?setVisibleSlot@PortDescriptor@Workflow@U2@@UAEXABVQString@@_N@Z 10010444 f   U2Lang:U2Lang.dll
 0001:0000f44a       ?type@PropertyDelegate@U2@@UBE?AW4Type@12@XZ 1001044a f   U2Lang:U2Lang.dll
 0001:0000f450       ?unregisterEntry@?$IdRegistry@VDomainFactory@Workflow@U2@@@U2@@UAEPAVDomainFactory@Workflow@2@ABVQString@@@Z 10010450 f   U2Lang:U2Lang.dll
 0001:0000f456       ?update@PropertyDelegate@U2@@UAEXXZ 10010456 f   U2Lang:U2Lang.dll
 0001:0000f45c       ?updateActorIds@Attribute@U2@@UAEXABV?$QMap@VQString@@V1@@@@Z 1001045c f   U2Lang:U2Lang.dll
 0001:0000f462       ?validate@ActorValidator@Workflow@U2@@UBE_NPBVConfiguration@3@AAV?$QList@VWorkflowNotification@U2@@@@@Z 10010462 f   U2Lang:U2Lang.dll
 0001:0000f468       ?validate@Attribute@U2@@UAE_NAAV?$QList@VWorkflowNotification@U2@@@@@Z 10010468 f   U2Lang:U2Lang.dll
 0001:0000f46e       ?qt_metacast@BaseWorker@LocalWorkflow@U2@@UAEPAXPBD@Z 1001046e f   U2Lang:U2Lang.dll
 0001:0000f474       ?qt_metacall@BaseWorker@LocalWorkflow@U2@@UAEHW4Call@QMetaObject@@HPAPAX@Z 10010474 f   U2Lang:U2Lang.dll
 0001:0000f47a       ??0DelegateEditor@U2@@QAE@ABV?$QMap@VQString@@PAVPropertyDelegate@U2@@@@@Z 1001047a f   U2Designer:U2Designer.dll
 0001:0000f480       ??1DelegateEditor@U2@@UAE@XZ 10010480 f   U2Designer:U2Designer.dll
 0001:0000f486       ??0URLDelegate@U2@@QAE@ABVDelegateTags@1@ABVQString@@_N22PAVQObject@@2@Z 10010486 f   U2Designer:U2Designer.dll
 0001:0000f48c       ??1URLDelegate@U2@@UAE@XZ  1001048c f   U2Designer:U2Designer.dll
 0001:0000f492       ??0SpinBoxDelegate@U2@@QAE@ABV?$QMap@VQString@@VQVariant@@@@PAVQObject@@@Z 10010492 f   U2Designer:U2Designer.dll
 0001:0000f498       ??1SpinBoxDelegate@U2@@UAE@XZ 10010498 f   U2Designer:U2Designer.dll
 0001:0000f49e       ?addDelegate@DelegateEditor@U2@@UAEXPAVPropertyDelegate@2@ABVQString@@@Z 1001049e f   U2Designer:U2Designer.dll
 0001:0000f4a4       ?clone@DelegateEditor@U2@@UAEPAVConfigurationEditor@2@XZ 100104a4 f   U2Designer:U2Designer.dll
 0001:0000f4aa       ?clone@SpinBoxDelegate@U2@@UAEPAVPropertyDelegate@2@XZ 100104aa f   U2Designer:U2Designer.dll
 0001:0000f4b0       ?clone@URLDelegate@U2@@UAEPAVPropertyDelegate@2@XZ 100104b0 f   U2Designer:U2Designer.dll
 0001:0000f4b6       ?commit@DelegateEditor@U2@@UAEXXZ 100104b6 f   U2Designer:U2Designer.dll
 0001:0000f4bc       ?createEditor@SpinBoxDelegate@U2@@UBEPAVQWidget@@PAV3@ABVQStyleOptionViewItem@@ABVQModelIndex@@@Z 100104bc f   U2Designer:U2Designer.dll
 0001:0000f4c2       ?createEditor@URLDelegate@U2@@UBEPAVQWidget@@PAV3@ABVQStyleOptionViewItem@@ABVQModelIndex@@@Z 100104c2 f   U2Designer:U2Designer.dll
 0001:0000f4c8       ?createWizardWidget@SpinBoxDelegate@U2@@UBEPAVPropertyWidget@2@AAVU2OpStatus@2@PAVQWidget@@@Z 100104c8 f   U2Designer:U2Designer.dll
 0001:0000f4ce       ?createWizardWidget@URLDelegate@U2@@UBEPAVPropertyWidget@2@AAVU2OpStatus@2@PAVQWidget@@@Z 100104ce f   U2Designer:U2Designer.dll
 0001:0000f4d4       ?getDelegate@DelegateEditor@U2@@UAEPAVPropertyDelegate@2@ABVQString@@@Z 100104d4 f   U2Designer:U2Designer.dll
 0001:0000f4da       ?getDisplayValue@SpinBoxDelegate@U2@@UBE?AVQVariant@@ABV3@@Z 100104da f   U2Designer:U2Designer.dll
 0001:0000f4e0       ?getDisplayValue@URLDelegate@U2@@UBE?AVQVariant@@ABV3@@Z 100104e0 f   U2Designer:U2Designer.dll
 0001:0000f4e6       ?getItems@SpinBoxDelegate@U2@@UBEXAAV?$QMap@VQString@@VQVariant@@@@@Z 100104e6 f   U2Designer:U2Designer.dll
 0001:0000f4ec       ?metaObject@DelegateEditor@U2@@UBEPBUQMetaObject@@XZ 100104ec f   U2Designer:U2Designer.dll
 0001:0000f4f2       ?metaObject@SpinBoxDelegate@U2@@UBEPBUQMetaObject@@XZ 100104f2 f   U2Designer:U2Designer.dll
 0001:0000f4f8       ?metaObject@URLDelegate@U2@@UBEPBUQMetaObject@@XZ 100104f8 f   U2Designer:U2Designer.dll
 0001:0000f4fe       ?qt_metacall@DelegateEditor@U2@@UAEHW4Call@QMetaObject@@HPAPAX@Z 100104fe f   U2Designer:U2Designer.dll
 0001:0000f504       ?qt_metacall@SpinBoxDelegate@U2@@UAEHW4Call@QMetaObject@@HPAPAX@Z 10010504 f   U2Designer:U2Designer.dll
 0001:0000f50a       ?qt_metacall@URLDelegate@U2@@UAEHW4Call@QMetaObject@@HPAPAX@Z 1001050a f   U2Designer:U2Designer.dll
 0001:0000f510       ?qt_metacast@DelegateEditor@U2@@UAEPAXPBD@Z 10010510 f   U2Designer:U2Designer.dll
 0001:0000f516       ?qt_metacast@SpinBoxDelegate@U2@@UAEPAXPBD@Z 10010516 f   U2Designer:U2Designer.dll
 0001:0000f51c       ?qt_metacast@URLDelegate@U2@@UAEPAXPBD@Z 1001051c f   U2Designer:U2Designer.dll
 0001:0000f522       ?removeDelegate@DelegateEditor@U2@@UAEPAVPropertyDelegate@2@ABVQString@@@Z 10010522 f   U2Designer:U2Designer.dll
 0001:0000f528       ?setEditorData@SpinBoxDelegate@U2@@UBEXPAVQWidget@@ABVQModelIndex@@@Z 10010528 f   U2Designer:U2Designer.dll
 0001:0000f52e       ?setEditorData@URLDelegate@U2@@UBEXPAVQWidget@@ABVQModelIndex@@@Z 1001052e f   U2Designer:U2Designer.dll
 0001:0000f534       ?setModelData@SpinBoxDelegate@U2@@UBEXPAVQWidget@@PAVQAbstractItemModel@@ABVQModelIndex@@@Z 10010534 f   U2Designer:U2Designer.dll
 0001:0000f53a       ?setModelData@URLDelegate@U2@@UBEXPAVQWidget@@PAVQAbstractItemModel@@ABVQModelIndex@@@Z 1001053a f   U2Designer:U2Designer.dll
 0001:0000f540       ?type@URLDelegate@U2@@UBE?AW4Type@PropertyDelegate@2@XZ 10010540 f   U2Designer:U2Designer.dll
 0001:0000f546       ?updateDelegate@DelegateEditor@U2@@UAEXABVQString@@@Z 10010546 f   U2Designer:U2Designer.dll
 0001:0000f54c       ?updateDelegates@DelegateEditor@U2@@UAEXXZ 1001054c f   U2Designer:U2Designer.dll
 0001:0000f552       ?destroyEditor@QAbstractItemDelegate@@UBEXPAVQWidget@@ABVQModelIndex@@@Z 10010552 f   Qt5Widgets:Qt5Widgets.dll
 0001:0000f558       ?drawCheck@QItemDelegate@@MBEXPAVQPainter@@ABVQStyleOptionViewItem@@ABVQRect@@W4CheckState@Qt@@@Z 10010558 f   Qt5Widgets:Qt5Widgets.dll
 0001:0000f55e       ?drawDecoration@QItemDelegate@@MBEXPAVQPainter@@ABVQStyleOptionViewItem@@ABVQRect@@ABVQPixmap@@@Z 1001055e f   Qt5Widgets:Qt5Widgets.dll
 0001:0000f564       ?drawDisplay@QItemDelegate@@MBEXPAVQPainter@@ABVQStyleOptionViewItem@@ABVQRect@@ABVQString@@@Z 10010564 f   Qt5Widgets:Qt5Widgets.dll
 0001:0000f56a       ?drawFocus@QItemDelegate@@MBEXPAVQPainter@@ABVQStyleOptionViewItem@@ABVQRect@@@Z 1001056a f   Qt5Widgets:Qt5Widgets.dll
 0001:0000f570       ?editorEvent@QItemDelegate@@MAE_NPAVQEvent@@PAVQAbstractItemModel@@ABVQStyleOptionViewItem@@ABVQModelIndex@@@Z 10010570 f   Qt5Widgets:Qt5Widgets.dll
 0001:0000f576       ?eventFilter@QItemDelegate@@MAE_NPAVQObject@@PAVQEvent@@@Z 10010576 f   Qt5Widgets:Qt5Widgets.dll
 0001:0000f57c       ?helpEvent@QAbstractItemDelegate@@UAE_NPAVQHelpEvent@@PAVQAbstractItemView@@ABVQStyleOptionViewItem@@ABVQModelIndex@@@Z 1001057c f   Qt5Widgets:Qt5Widgets.dll
 0001:0000f582       ?paint@QItemDelegate@@UBEXPAVQPainter@@ABVQStyleOptionViewItem@@ABVQModelIndex@@@Z 10010582 f   Qt5Widgets:Qt5Widgets.dll
 0001:0000f588       ?paintingRoles@QAbstractItemDelegate@@UBE?AV?$QVector@H@@XZ 10010588 f   Qt5Widgets:Qt5Widgets.dll
 0001:0000f58e       ?sizeHint@QItemDelegate@@UBE?AVQSize@@ABVQStyleOptionViewItem@@ABVQModelIndex@@@Z 1001058e f   Qt5Widgets:Qt5Widgets.dll
 0001:0000f594       ?updateEditorGeometry@QItemDelegate@@UBEXPAVQWidget@@ABVQStyleOptionViewItem@@ABVQModelIndex@@@Z 10010594 f   Qt5Widgets:Qt5Widgets.dll
 0001:0000f59a       ?clear@QTextDocument@@UAEXXZ 1001059a f   Qt5Gui:Qt5Gui.dll
 0001:0000f5a0       ?createObject@QTextDocument@@MAEPAVQTextObject@@ABVQTextFormat@@@Z 100105a0 f   Qt5Gui:Qt5Gui.dll
 0001:0000f5a6       ?loadResource@QTextDocument@@MAE?AVQVariant@@HABVQUrl@@@Z 100105a6 f   Qt5Gui:Qt5Gui.dll
 0001:0000f5ac       ??0QScriptValue@@QAE@XZ    100105ac f   Qt5Script:Qt5Script.dll
 0001:0000f5b2       ??1QScriptValue@@QAE@XZ    100105b2 f   Qt5Script:Qt5Script.dll
 0001:0000f5b8       ??0QScriptValue@@QAE@ABV0@@Z 100105b8 f   Qt5Script:Qt5Script.dll
 0001:0000f5be       ??4QScriptValue@@QAEAAV0@ABV0@@Z 100105be f   Qt5Script:Qt5Script.dll
 0001:0000f5c4       ?isNumber@QScriptValue@@QBE_NXZ 100105c4 f   Qt5Script:Qt5Script.dll
 0001:0000f5ca       ?isString@QScriptValue@@QBE_NXZ 100105ca f   Qt5Script:Qt5Script.dll
 0001:0000f5d0       ?toString@QScriptValue@@QBE?AVQString@@XZ 100105d0 f   Qt5Script:Qt5Script.dll
 0001:0000f5d6       ?toInt32@QScriptValue@@QBEHXZ 100105d6 f   Qt5Script:Qt5Script.dll
 0001:0000f5dc       ??1QScriptEngine@@UAE@XZ   100105dc f   Qt5Script:Qt5Script.dll
 0001:0000f5e2       ?newVariant@QScriptEngine@@QAE?AVQScriptValue@@ABVQVariant@@@Z 100105e2 f   Qt5Script:Qt5Script.dll
 0001:0000f5e8       ??0QChar@@QAE@UQLatin1Char@@@Z 100105e8 f   Qt5Core:Qt5Core.dll
 0001:0000f5ee       ??0QString@@QAE@XZ         100105ee f   Qt5Core:Qt5Core.dll
 0001:0000f5f4       ??0QString@@QAE@ABV0@@Z    100105f4 f   Qt5Core:Qt5Core.dll
 0001:0000f5fa       ??1QString@@QAE@XZ         100105fa f   Qt5Core:Qt5Core.dll
 0001:0000f600       ??4QString@@QAEAAV0@ABV0@@Z 10010600 f   Qt5Core:Qt5Core.dll
 0001:0000f606       ??4QString@@QAEAAV0@$$QAV0@@Z 10010606 f   Qt5Core:Qt5Core.dll
 0001:0000f60c       ?arg@QString@@QBE?AV1@ABV1@HVQChar@@@Z 1001060c f   Qt5Core:Qt5Core.dll
 0001:0000f612       ?indexOf@QString@@QBEHABV1@HW4CaseSensitivity@Qt@@@Z 10010612 f   Qt5Core:Qt5Core.dll
 0001:0000f618       ?append@QString@@QAEAAV1@ABV1@@Z 10010618 f   Qt5Core:Qt5Core.dll
 0001:0000f61e       ?replace@QString@@QAEAAV1@VQChar@@0W4CaseSensitivity@Qt@@@Z 1001061e f   Qt5Core:Qt5Core.dll
 0001:0000f624       ?fromUtf8@QString@@SA?AV1@PBDH@Z 10010624 f   Qt5Core:Qt5Core.dll
 0001:0000f62a       ?fromAscii_helper@QString@@CAPAU?$QTypedArrayData@G@@PBDH@Z 1001062a f   Qt5Core:Qt5Core.dll
 0001:0000f630       ??0QTextStream@@QAE@PAVQIODevice@@@Z 10010630 f   Qt5Core:Qt5Core.dll
 0001:0000f636       ??1QTextStream@@UAE@XZ     10010636 f   Qt5Core:Qt5Core.dll
 0001:0000f63c       ?atEnd@QTextStream@@QBE_NXZ 1001063c f   Qt5Core:Qt5Core.dll
 0001:0000f642       ?readLine@QTextStream@@QAE?AVQString@@_J@Z 10010642 f   Qt5Core:Qt5Core.dll
 0001:0000f648       ?read@QTextStream@@QAE?AVQString@@_J@Z 10010648 f   Qt5Core:Qt5Core.dll
 0001:0000f64e       ??6QTextStream@@QAEAAV0@D@Z 1001064e f   Qt5Core:Qt5Core.dll
 0001:0000f654       ??6QTextStream@@QAEAAV0@ABVQString@@@Z 10010654 f   Qt5Core:Qt5Core.dll
 0001:0000f65a       ??0QFile@@QAE@ABVQString@@@Z 1001065a f   Qt5Core:Qt5Core.dll
 0001:0000f660       ??1QFile@@UAE@XZ           10010660 f   Qt5Core:Qt5Core.dll
 0001:0000f666       ?fileName@QFile@@UBE?AVQString@@XZ 10010666 f   Qt5Core:Qt5Core.dll
 0001:0000f66c       ?remove@QFile@@QAE_NXZ     1001066c f   Qt5Core:Qt5Core.dll
 0001:0000f672       ?open@QFile@@UAE_NV?$QFlags@W4OpenModeFlag@QIODevice@@@@@Z 10010672 f   Qt5Core:Qt5Core.dll
 0001:0000f678       ??0QDir@@QAE@ABVQString@@@Z 10010678 f   Qt5Core:Qt5Core.dll
 0001:0000f67e       ??1QDir@@QAE@XZ            1001067e f   Qt5Core:Qt5Core.dll
 0001:0000f684       ?mkpath@QDir@@QBE_NABVQString@@@Z 10010684 f   Qt5Core:Qt5Core.dll
 0001:0000f68a       ?childEvent@QObject@@MAEXPAVQChildEvent@@@Z 1001068a f   Qt5Core:Qt5Core.dll
 0001:0000f690       ?connectNotify@QObject@@MAEXABVQMetaMethod@@@Z 10010690 f   Qt5Core:Qt5Core.dll
 0001:0000f696       ?customEvent@QObject@@MAEXPAVQEvent@@@Z 10010696 f   Qt5Core:Qt5Core.dll
 0001:0000f69c       ?disconnectNotify@QObject@@MAEXABVQMetaMethod@@@Z 1001069c f   Qt5Core:Qt5Core.dll
 0001:0000f6a2       ?event@QObject@@UAE_NPAVQEvent@@@Z 100106a2 f   Qt5Core:Qt5Core.dll
 0001:0000f6a8       ?eventFilter@QObject@@UAE_NPAV1@PAVQEvent@@@Z 100106a8 f   Qt5Core:Qt5Core.dll
 0001:0000f6ae       ?timerEvent@QObject@@MAEXPAVQTimerEvent@@@Z 100106ae f   Qt5Core:Qt5Core.dll
 0001:0000f6b4       ?tr@QMetaObject@@QBE?AVQString@@PBD0H@Z 100106b4 f   Qt5Core:Qt5Core.dll
 0001:0000f6ba       ??1Connection@QMetaObject@@QAE@XZ 100106ba f   Qt5Core:Qt5Core.dll
 0001:0000f6c0       ?detach@QListData@@QAEPAUData@1@H@Z 100106c0 f   Qt5Core:Qt5Core.dll
 0001:0000f6c6       ?dispose@QListData@@SAXPAUData@1@@Z 100106c6 f   Qt5Core:Qt5Core.dll
 0001:0000f6cc       ?connect@QObject@@QBE?AVConnection@QMetaObject@@PBV1@PBD1W4ConnectionType@Qt@@@Z 100106cc f   Qt5Core:Qt5Core.dll
 0001:0000f6d2       ??4QString@@QAEAAV0@PBD@Z  100106d2 f   Qt5Core:Qt5Core.dll
 0001:0000f6d8       ?tr@QObject@@SA?AVQString@@PBD0H@Z 100106d8 f   Qt5Core:Qt5Core.dll
 0001:0000f6de       ?toUInt@QString@@QBEIPA_NH@Z 100106de f   Qt5Core:Qt5Core.dll
 0001:0000f6e4       ?number@QString@@SA?AV1@HH@Z 100106e4 f   Qt5Core:Qt5Core.dll
 0001:0000f6ea       ??8@YA_NABVQString@@0@Z    100106ea f   Qt5Core:Qt5Core.dll
 0001:0000f6f0       ??M@YA_NABVQString@@0@Z    100106f0 f   Qt5Core:Qt5Core.dll
 0001:0000f6f6       ?detach_grow@QListData@@QAEPAUData@1@PAHH@Z 100106f6 f   Qt5Core:Qt5Core.dll
 0001:0000f6fc       ?append@QListData@@QAEPAPAXXZ 100106fc f   Qt5Core:Qt5Core.dll
 0001:0000f702       ?freeNodeAndRebalance@QMapDataBase@@QAEXPAUQMapNodeBase@@@Z 10010702 f   Qt5Core:Qt5Core.dll
 0001:0000f708       ?recalcMostLeftNode@QMapDataBase@@QAEXXZ 10010708 f   Qt5Core:Qt5Core.dll
 0001:0000f70e       ?createNode@QMapDataBase@@QAEPAUQMapNodeBase@@HHPAU2@_N@Z 1001070e f   Qt5Core:Qt5Core.dll
 0001:0000f714       ?freeTree@QMapDataBase@@QAEXPAUQMapNodeBase@@H@Z 10010714 f   Qt5Core:Qt5Core.dll
 0001:0000f71a       ?createData@QMapDataBase@@SAPAU1@XZ 1001071a f   Qt5Core:Qt5Core.dll
 0001:0000f720       ?freeData@QMapDataBase@@SAXPAU1@@Z 10010720 f   Qt5Core:Qt5Core.dll
 0001:0000f726       ?rename@QFile@@SA_NABVQString@@0@Z 10010726 f   Qt5Core:Qt5Core.dll
 0001:0000f72c       ??0QFileInfo@@QAE@ABVQString@@@Z 1001072c f   Qt5Core:Qt5Core.dll
 0001:0000f732       ??1QFileInfo@@QAE@XZ       10010732 f   Qt5Core:Qt5Core.dll
 0001:0000f738       ?exists@QFileInfo@@QBE_NXZ 10010738 f   Qt5Core:Qt5Core.dll
 0001:0000f73e       ?completeBaseName@QFileInfo@@QBE?AVQString@@XZ 1001073e f   Qt5Core:Qt5Core.dll
 0001:0000f744       ?translate@QCoreApplication@@SA?AVQString@@PBD00H@Z 10010744 f   Qt5Core:Qt5Core.dll
 0001:0000f74a       ?cast@QMetaObject@@QBEPAVQObject@@PAV2@@Z 1001074a f   Qt5Core:Qt5Core.dll
 0001:0000f750       ?normalizedType@QMetaObject@@SA?AVQByteArray@@PBD@Z 10010750 f   Qt5Core:Qt5Core.dll
 0001:0000f756       ??1QByteArray@@QAE@XZ      10010756 f   Qt5Core:Qt5Core.dll
 0001:0000f75c       ??0QString@@QAE@$$QAV0@@Z  1001075c f   Qt5Core:Qt5Core.dll
 0001:0000f762       ?arg@QString@@QBE?AV1@HHHVQChar@@@Z 10010762 f   Qt5Core:Qt5Core.dll
 0001:0000f768       ?realloc@QListData@@QAEXH@Z 10010768 f   Qt5Core:Qt5Core.dll
 0001:0000f76e       ?registerNormalizedType@QMetaType@@SAHABVQByteArray@@P6AXPAX@ZP6APAXPBX@Z2P6APAX13@ZHV?$QFlags@W4TypeFlag@QMetaType@@@@PBUQMetaObject@@@Z 1001076e f   Qt5Core:Qt5Core.dll
 0001:0000f774       ?registerNormalizedTypedef@QMetaType@@SAHABVQByteArray@@H@Z 10010774 f   Qt5Core:Qt5Core.dll
 0001:0000f77a       ?hasRegisteredConverterFunction@QMetaType@@SA_NHH@Z 1001077a f   Qt5Core:Qt5Core.dll
 0001:0000f780       ?registerConverterFunction@QMetaType@@SA_NPBUAbstractConverterFunction@QtPrivate@@HH@Z 10010780 f   Qt5Core:Qt5Core.dll
 0001:0000f786       ?unregisterConverterFunction@QMetaType@@SAXHH@Z 10010786 f   Qt5Core:Qt5Core.dll
 0001:0000f78c       ??1QObject@@UAE@XZ         1001078c f   Qt5Core:Qt5Core.dll
 0001:0000f792       ?nextNode@QMapNodeBase@@QBEPBU1@XZ 10010792 f   Qt5Core:Qt5Core.dll
 0001:0000f798       ?previousNode@QMapNodeBase@@QBEPBU1@XZ 10010798 f   Qt5Core:Qt5Core.dll
 0001:0000f79e       ??0QVariant@@QAE@XZ        1001079e f   Qt5Core:Qt5Core.dll
 0001:0000f7a4       ??1QVariant@@QAE@XZ        100107a4 f   Qt5Core:Qt5Core.dll
 0001:0000f7aa       ??0QVariant@@QAE@HPBXI@Z   100107aa f   Qt5Core:Qt5Core.dll
 0001:0000f7b0       ??0QVariant@@QAE@ABV0@@Z   100107b0 f   Qt5Core:Qt5Core.dll
 0001:0000f7b6       ??0QVariant@@QAE@ABV?$QMap@VQString@@VQVariant@@@@@Z 100107b6 f   Qt5Core:Qt5Core.dll
 0001:0000f7bc       ??4QVariant@@QAEAAV0@ABV0@@Z 100107bc f   Qt5Core:Qt5Core.dll
 0001:0000f7c2       ??4QVariant@@QAEAAV0@$$QAV0@@Z 100107c2 f   Qt5Core:Qt5Core.dll
 0001:0000f7c8       ?userType@QVariant@@QBEHXZ 100107c8 f   Qt5Core:Qt5Core.dll
 0001:0000f7ce       ?toString@QVariant@@QBE?AVQString@@XZ 100107ce f   Qt5Core:Qt5Core.dll
 0001:0000f7d4       ?toMap@QVariant@@QBE?AV?$QMap@VQString@@VQVariant@@@@XZ 100107d4 f   Qt5Core:Qt5Core.dll
 0001:0000f7da       ?constData@QVariant@@QBEPBXXZ 100107da f   Qt5Core:Qt5Core.dll
 0001:0000f7e0       ?convert@QVariant@@QBE_NHPAX@Z 100107e0 f   Qt5Core:Qt5Core.dll
 0001:0000f7e6       ?idealThreadCount@QThread@@SAHXZ 100107e6 f   Qt5Core:Qt5Core.dll
 0001:0000f7ec       ??0QVariant@@QAE@H@Z       100107ec f   Qt5Core:Qt5Core.dll
 0001:0000f7f2       ??0QVariant@@QAE@ABVQString@@@Z 100107f2 f   Qt5Core:Qt5Core.dll
 0001:0000f7f8       ?dynamicMetaObject@QObjectData@@QBEPAUQMetaObject@@XZ 100107f8 f   Qt5Core:Qt5Core.dll
 0001:0000f7fe       ?className@QMetaObject@@QBEPBDXZ 100107fe f   Qt5Core:Qt5Core.dll
 0001:0000f804       ??0QByteArray@@QAE@XZ      10010804 f   Qt5Core:Qt5Core.dll
 0001:0000f80a       ?reserve@QByteArray@@QAEXH@Z 1001080a f   Qt5Core:Qt5Core.dll
 0001:0000f810       ?append@QByteArray@@QAEAAV1@D@Z 10010810 f   Qt5Core:Qt5Core.dll
 0001:0000f816       ?append@QByteArray@@QAEAAV1@PBD@Z 10010816 f   Qt5Core:Qt5Core.dll
 0001:0000f81c       ?_Xbad_alloc@std@@YAXXZ    1001081c f   msvcprt:MSVCP120.dll
 0001:0000f822       ?_Xlength_error@std@@YAXPBD@Z 10010822 f   msvcprt:MSVCP120.dll
 0001:0000f828       ?_Xout_of_range@std@@YAXPBD@Z 10010828 f   msvcprt:MSVCP120.dll
 0001:0000f82e       ?_Syserror_map@std@@YAPBDH@Z 1001082e f   msvcprt:MSVCP120.dll
 0001:0000f834       ?_Winerror_map@std@@YAPBDH@Z 10010834 f   msvcprt:MSVCP120.dll
 0001:0000f83a       __purecall                 1001083a f   MSVCRT:MSVCR120.dll
 0001:0000f840       ??2@YAPAXI@Z               10010840 f   MSVCRT:MSVCR120.dll
 0001:0000f846       ??3@YAXPAX@Z               10010846 f   MSVCRT:MSVCR120.dll
 0001:0000f84c       ___atonexitinit            1001084c f   MSVCRT:atonexit.obj
 0001:0000f888       __onexit                   10010888 f   MSVCRT:atonexit.obj
 0001:0000f931       _atexit                    10010931 f   MSVCRT:atonexit.obj
 0001:0000f946       _memmove                   10010946 f   MSVCRT:MSVCR120.dll
 0001:0000f94c       __hypot                    1001094c f   MSVCRT:MSVCR120.dll
 0001:0000f952       @__security_check_cookie@4 10010952 f   MSVCRT:secchk.obj
 0001:0000f962       __CxxThrowException@8      10010962 f   MSVCRT:MSVCR120.dll
 0001:0000f968       ___CxxFrameHandler3        10010968 f   MSVCRT:MSVCR120.dll
 0001:0000f96e       _memcpy                    1001096e f   MSVCRT:MSVCR120.dll
 0001:0000f974       ??0type_info@@AAE@ABV0@@Z  10010974 f   MSVCRT:ti_inst.obj
 0001:0000f97f       ??4type_info@@AAEAAV0@ABV0@@Z 1001097f f   MSVCRT:ti_inst.obj
 0001:0000f984       ??_Etype_info@@UAEPAXI@Z   10010984 f i MSVCRT:ti_inst.obj
 0001:0000f9d0       __chkstk                   100109d0 f   MSVCRT:chkstk.obj
 0001:0000f9d0       __alloca_probe             100109d0 f   MSVCRT:chkstk.obj
 0001:0000fa47       _NtCurrentTeb              10010a47 f i MSVCRT:crtdll.obj
 0001:0000fa4e       __CRT_INIT@12              10010a4e f   MSVCRT:crtdll.obj
 0001:0000fc45       __DllMainCRTStartup@12     10010c45 f   MSVCRT:crtdll.obj
 0001:0000fd9c       __lock                     10010d9c f   MSVCRT:MSVCR120.dll
 0001:0000fda2       __unlock                   10010da2 f   MSVCRT:MSVCR120.dll
 0001:0000fda8       __calloc_crt               10010da8 f   MSVCRT:MSVCR120.dll
 0001:0000fdae       ___dllonexit               10010dae f   MSVCRT:MSVCR120.dll
 0001:0000fdc0       __SEH_prolog4              10010dc0 f   MSVCRT:sehprolg4.obj
 0001:0000fe05       __SEH_epilog4              10010e05 f   MSVCRT:sehprolg4.obj
 0001:0000fe19       __except_handler4          10010e19 f   MSVCRT:chandler4gs.obj
 0001:0000fe3c       ___raise_securityfailure   10010e3c f   MSVCRT:gs_report.obj
 0001:0000fe79       ___report_gsfailure        10010e79 f   MSVCRT:gs_report.obj
 0001:0000ff74       ___report_rangecheckfailure 10010f74 f   MSVCRT:gs_report.obj
 0001:0000ff80       ___report_securityfailure  10010f80 f   MSVCRT:gs_report.obj
 0001:00010050       ___report_securityfailureEx 10011050 f   MSVCRT:gs_report.obj
 0001:00010166       ??_M@YGXPAXIHP6EX0@Z@Z     10011166 f   MSVCRT:ehvecdtr.obj
 0001:000101ee       ?__ArrayUnwind@@YGXPAXIHP6EX0@Z@Z 100111ee f   MSVCRT:ehvecdtr.obj
 0001:0001024c       ??1type_info@@UAE@XZ       1001124c f   MSVCRT:MSVCR120.dll
 0001:00010252       ___CppXcptFilter           10011252 f   MSVCRT:MSVCR120.dll
 0001:00010258       __amsg_exit                10011258 f   MSVCRT:MSVCR120.dll
 0001:00010260       __FindPESection            10011260 f   MSVCRT:pesect.obj
 0001:000102b0       __IsNonwritableInCurrentImage 100112b0 f   MSVCRT:pesect.obj
 0001:00010370       __ValidateImageBase        10011370 f   MSVCRT:pesect.obj
 0001:000103a2       _free                      100113a2 f   MSVCRT:MSVCR120.dll
 0001:000103a8       ___security_init_cookie    100113a8 f   MSVCRT:gs_support.obj
 0001:00010444       _DllMain@12                10011444 f   MSVCRT:dllmain.obj
 0001:00010466       __malloc_crt               10011466 f   MSVCRT:MSVCR120.dll
 0001:0001046c       __RTC_Initialize           1001146c f   MSVCRT:initsect.obj
 0001:0001048c       __RTC_Terminate            1001148c f   MSVCRT:initsect.obj
 0001:000104ac       __initterm                 100114ac f   MSVCRT:MSVCR120.dll
 0001:000104b2       __initterm_e               100114b2 f   MSVCRT:MSVCR120.dll
 0001:000104b8       ___clean_type_info_names   100114b8 f   MSVCRT:tncleanup.obj
 0001:000104c4       __except_handler4_common   100114c4 f   MSVCRT:MSVCR120.dll
 0001:000104ca       __crt_debugger_hook        100114ca f   MSVCRT:MSVCR120.dll
 0001:000104d0       ___crtUnhandledException   100114d0 f   MSVCRT:MSVCR120.dll
 0001:000104d6       ___crtTerminateProcess     100114d6 f   MSVCRT:MSVCR120.dll
 0001:000104dc       ?terminate@@YAXXZ          100114dc f   MSVCRT:MSVCR120.dll
 0001:000104e2       ___clean_type_info_names_internal 100114e2 f   MSVCRT:MSVCR120.dll
 0001:000104e8       _EncodePointer@4           100114e8 f   kernel32:KERNEL32.dll
 0001:000104ee       _DecodePointer@4           100114ee f   kernel32:KERNEL32.dll
 0001:000104f4       _IsDebuggerPresent@0       100114f4 f   kernel32:KERNEL32.dll
 0001:000104fa       _IsProcessorFeaturePresent@4 100114fa f   kernel32:KERNEL32.dll
 0001:00010500       _QueryPerformanceCounter@4 10011500 f   kernel32:KERNEL32.dll
 0001:00010506       _GetCurrentProcessId@0     10011506 f   kernel32:KERNEL32.dll
 0001:0001050c       _GetCurrentThreadId@0      1001150c f   kernel32:KERNEL32.dll
 0001:00010512       _GetSystemTimeAsFileTime@4 10011512 f   kernel32:KERNEL32.dll
 0001:00010518       _DisableThreadLibraryCalls@4 10011518 f   kernel32:KERNEL32.dll
 0001:00013640       ??__Ff@?4??registerConverter@?$AssociativeValueTypeIsMetaType@V?$QMap@VQString@@I@@$00@QtPrivate@@SA_NH@Z@YAXXZ 10014640 f i WevoteWorker.obj
 0002:00000000       __imp__DisableThreadLibraryCalls@4 10015000     kernel32:KERNEL32.dll
 0002:00000004       __imp__GetSystemTimeAsFileTime@4 10015004     kernel32:KERNEL32.dll
 0002:00000008       __imp__GetCurrentThreadId@0 10015008     kernel32:KERNEL32.dll
 0002:0000000c       __imp__GetCurrentProcessId@0 1001500c     kernel32:KERNEL32.dll
 0002:00000010       __imp__QueryPerformanceCounter@4 10015010     kernel32:KERNEL32.dll
 0002:00000014       __imp__IsProcessorFeaturePresent@4 10015014     kernel32:KERNEL32.dll
 0002:00000018       __imp__IsDebuggerPresent@0 10015018     kernel32:KERNEL32.dll
 0002:0000001c       __imp__DecodePointer@4     1001501c     kernel32:KERNEL32.dll
 0002:00000020       __imp__EncodePointer@4     10015020     kernel32:KERNEL32.dll
 0002:00000024       \177KERNEL32_NULL_THUNK_DATA 10015024     kernel32:KERNEL32.dll
 0002:00000028       __imp_?_Xlength_error@std@@YAXPBD@Z 10015028     msvcprt:MSVCP120.dll
 0002:0000002c       __imp_?_Xout_of_range@std@@YAXPBD@Z 1001502c     msvcprt:MSVCP120.dll
 0002:00000030       __imp_?_Syserror_map@std@@YAPBDH@Z 10015030     msvcprt:MSVCP120.dll
 0002:00000034       __imp_?_Winerror_map@std@@YAPBDH@Z 10015034     msvcprt:MSVCP120.dll
 0002:00000038       __imp_?_Xbad_alloc@std@@YAXXZ 10015038     msvcprt:MSVCP120.dll
 0002:0000003c       \177MSVCP120_NULL_THUNK_DATA 1001503c     msvcprt:MSVCP120.dll
 0002:00000040       __imp___initterm_e         10015040     MSVCRT:MSVCR120.dll
 0002:00000044       __imp___initterm           10015044     MSVCRT:MSVCR120.dll
 0002:00000048       __imp___malloc_crt         10015048     MSVCRT:MSVCR120.dll
 0002:0000004c       __imp__free                1001504c     MSVCRT:MSVCR120.dll
 0002:00000050       __imp___amsg_exit          10015050     MSVCRT:MSVCR120.dll
 0002:00000054       __imp_??1type_info@@UAE@XZ 10015054     MSVCRT:MSVCR120.dll
 0002:00000058       __imp___onexit             10015058     MSVCRT:MSVCR120.dll
 0002:0000005c       __imp____dllonexit         1001505c     MSVCRT:MSVCR120.dll
 0002:00000060       __imp___calloc_crt         10015060     MSVCRT:MSVCR120.dll
 0002:00000064       __imp___unlock             10015064     MSVCRT:MSVCR120.dll
 0002:00000068       __imp___lock               10015068     MSVCRT:MSVCR120.dll
 0002:0000006c       __imp__memcpy              1001506c     MSVCRT:MSVCR120.dll
 0002:00000070       __imp____CxxFrameHandler3  10015070     MSVCRT:MSVCR120.dll
 0002:00000074       __imp___CxxThrowException@8 10015074     MSVCRT:MSVCR120.dll
 0002:00000078       __imp___hypot              10015078     MSVCRT:MSVCR120.dll
 0002:0000007c       __imp__memmove             1001507c     MSVCRT:MSVCR120.dll
 0002:00000080       __imp_??3@YAXPAX@Z         10015080     MSVCRT:MSVCR120.dll
 0002:00000084       __imp_??2@YAPAXI@Z         10015084     MSVCRT:MSVCR120.dll
 0002:00000088       __imp___purecall           10015088     MSVCRT:MSVCR120.dll
 0002:0000008c       __imp___except_handler4_common 1001508c     MSVCRT:MSVCR120.dll
 0002:00000090       __imp___crt_debugger_hook  10015090     MSVCRT:MSVCR120.dll
 0002:00000094       __imp____crtUnhandledException 10015094     MSVCRT:MSVCR120.dll
 0002:00000098       __imp____crtTerminateProcess 10015098     MSVCRT:MSVCR120.dll
 0002:0000009c       __imp_?terminate@@YAXXZ    1001509c     MSVCRT:MSVCR120.dll
 0002:000000a0       __imp____CppXcptFilter     100150a0     MSVCRT:MSVCR120.dll
 0002:000000a4       __imp____clean_type_info_names_internal 100150a4     MSVCRT:MSVCR120.dll
 0002:000000a8       \177MSVCR120_NULL_THUNK_DATA 100150a8     MSVCRT:MSVCR120.dll
 0002:000000ac       __imp_?dynamicMetaObject@QObjectData@@QBEPAUQMetaObject@@XZ 100150ac     Qt5Core:Qt5Core.dll
 0002:000000b0       __imp_??0QVariant@@QAE@H@Z 100150b0     Qt5Core:Qt5Core.dll
 0002:000000b4       __imp_??0QVariant@@QAE@ABVQString@@@Z 100150b4     Qt5Core:Qt5Core.dll
 0002:000000b8       __imp_?className@QMetaObject@@QBEPBDXZ 100150b8     Qt5Core:Qt5Core.dll
 0002:000000bc       __imp_??0QByteArray@@QAE@XZ 100150bc     Qt5Core:Qt5Core.dll
 0002:000000c0       __imp_?reserve@QByteArray@@QAEXH@Z 100150c0     Qt5Core:Qt5Core.dll
 0002:000000c4       __imp_?append@QByteArray@@QAEAAV1@D@Z 100150c4     Qt5Core:Qt5Core.dll
 0002:000000c8       __imp_?append@QByteArray@@QAEAAV1@PBD@Z 100150c8     Qt5Core:Qt5Core.dll
 0002:000000cc       __imp_?convert@QVariant@@QBE_NHPAX@Z 100150cc     Qt5Core:Qt5Core.dll
 0002:000000d0       __imp_?constData@QVariant@@QBEPBXXZ 100150d0     Qt5Core:Qt5Core.dll
 0002:000000d4       __imp_?toMap@QVariant@@QBE?AV?$QMap@VQString@@VQVariant@@@@XZ 100150d4     Qt5Core:Qt5Core.dll
 0002:000000d8       __imp_?toString@QVariant@@QBE?AVQString@@XZ 100150d8     Qt5Core:Qt5Core.dll
 0002:000000dc       __imp_?userType@QVariant@@QBEHXZ 100150dc     Qt5Core:Qt5Core.dll
 0002:000000e0       __imp_??4QVariant@@QAEAAV0@$$QAV0@@Z 100150e0     Qt5Core:Qt5Core.dll
 0002:000000e4       __imp_??4QVariant@@QAEAAV0@ABV0@@Z 100150e4     Qt5Core:Qt5Core.dll
 0002:000000e8       __imp_??0QVariant@@QAE@ABV?$QMap@VQString@@VQVariant@@@@@Z 100150e8     Qt5Core:Qt5Core.dll
 0002:000000ec       __imp_??0QVariant@@QAE@ABV0@@Z 100150ec     Qt5Core:Qt5Core.dll
 0002:000000f0       __imp_??0QVariant@@QAE@HPBXI@Z 100150f0     Qt5Core:Qt5Core.dll
 0002:000000f4       __imp_??1QVariant@@QAE@XZ  100150f4     Qt5Core:Qt5Core.dll
 0002:000000f8       __imp_??0QVariant@@QAE@XZ  100150f8     Qt5Core:Qt5Core.dll
 0002:000000fc       __imp_?previousNode@QMapNodeBase@@QBEPBU1@XZ 100150fc     Qt5Core:Qt5Core.dll
 0002:00000100       __imp_?nextNode@QMapNodeBase@@QBEPBU1@XZ 10015100     Qt5Core:Qt5Core.dll
 0002:00000104       __imp_??1QObject@@UAE@XZ   10015104     Qt5Core:Qt5Core.dll
 0002:00000108       __imp_?unregisterConverterFunction@QMetaType@@SAXHH@Z 10015108     Qt5Core:Qt5Core.dll
 0002:0000010c       __imp_?registerConverterFunction@QMetaType@@SA_NPBUAbstractConverterFunction@QtPrivate@@HH@Z 1001510c     Qt5Core:Qt5Core.dll
 0002:00000110       __imp_?hasRegisteredConverterFunction@QMetaType@@SA_NHH@Z 10015110     Qt5Core:Qt5Core.dll
 0002:00000114       __imp_?registerNormalizedTypedef@QMetaType@@SAHABVQByteArray@@H@Z 10015114     Qt5Core:Qt5Core.dll
 0002:00000118       __imp_??0QChar@@QAE@UQLatin1Char@@@Z 10015118     Qt5Core:Qt5Core.dll
 0002:0000011c       __imp_??0QString@@QAE@XZ   1001511c     Qt5Core:Qt5Core.dll
 0002:00000120       __imp_??0QString@@QAE@ABV0@@Z 10015120     Qt5Core:Qt5Core.dll
 0002:00000124       __imp_??1QString@@QAE@XZ   10015124     Qt5Core:Qt5Core.dll
 0002:00000128       __imp_??4QString@@QAEAAV0@ABV0@@Z 10015128     Qt5Core:Qt5Core.dll
 0002:0000012c       __imp_??4QString@@QAEAAV0@$$QAV0@@Z 1001512c     Qt5Core:Qt5Core.dll
 0002:00000130       __imp_?arg@QString@@QBE?AV1@ABV1@HVQChar@@@Z 10015130     Qt5Core:Qt5Core.dll
 0002:00000134       __imp_?indexOf@QString@@QBEHABV1@HW4CaseSensitivity@Qt@@@Z 10015134     Qt5Core:Qt5Core.dll
 0002:00000138       __imp_?append@QString@@QAEAAV1@ABV1@@Z 10015138     Qt5Core:Qt5Core.dll
 0002:0000013c       __imp_?replace@QString@@QAEAAV1@VQChar@@0W4CaseSensitivity@Qt@@@Z 1001513c     Qt5Core:Qt5Core.dll
 0002:00000140       __imp_?fromUtf8@QString@@SA?AV1@PBDH@Z 10015140     Qt5Core:Qt5Core.dll
 0002:00000144       __imp_?fromAscii_helper@QString@@CAPAU?$QTypedArrayData@G@@PBDH@Z 10015144     Qt5Core:Qt5Core.dll
 0002:00000148       __imp_??0QTextStream@@QAE@PAVQIODevice@@@Z 10015148     Qt5Core:Qt5Core.dll
 0002:0000014c       __imp_??1QTextStream@@UAE@XZ 1001514c     Qt5Core:Qt5Core.dll
 0002:00000150       __imp_?atEnd@QTextStream@@QBE_NXZ 10015150     Qt5Core:Qt5Core.dll
 0002:00000154       __imp_?readLine@QTextStream@@QAE?AVQString@@_J@Z 10015154     Qt5Core:Qt5Core.dll
 0002:00000158       __imp_?read@QTextStream@@QAE?AVQString@@_J@Z 10015158     Qt5Core:Qt5Core.dll
 0002:0000015c       __imp_??6QTextStream@@QAEAAV0@D@Z 1001515c     Qt5Core:Qt5Core.dll
 0002:00000160       __imp_??6QTextStream@@QAEAAV0@ABVQString@@@Z 10015160     Qt5Core:Qt5Core.dll
 0002:00000164       __imp_??0QFile@@QAE@ABVQString@@@Z 10015164     Qt5Core:Qt5Core.dll
 0002:00000168       __imp_??1QFile@@UAE@XZ     10015168     Qt5Core:Qt5Core.dll
 0002:0000016c       __imp_?fileName@QFile@@UBE?AVQString@@XZ 1001516c     Qt5Core:Qt5Core.dll
 0002:00000170       __imp_?remove@QFile@@QAE_NXZ 10015170     Qt5Core:Qt5Core.dll
 0002:00000174       __imp_?open@QFile@@UAE_NV?$QFlags@W4OpenModeFlag@QIODevice@@@@@Z 10015174     Qt5Core:Qt5Core.dll
 0002:00000178       __imp_??0QDir@@QAE@ABVQString@@@Z 10015178     Qt5Core:Qt5Core.dll
 0002:0000017c       __imp_??1QDir@@QAE@XZ      1001517c     Qt5Core:Qt5Core.dll
 0002:00000180       __imp_?mkpath@QDir@@QBE_NABVQString@@@Z 10015180     Qt5Core:Qt5Core.dll
 0002:00000184       __imp_?childEvent@QObject@@MAEXPAVQChildEvent@@@Z 10015184     Qt5Core:Qt5Core.dll
 0002:00000188       __imp_?connectNotify@QObject@@MAEXABVQMetaMethod@@@Z 10015188     Qt5Core:Qt5Core.dll
 0002:0000018c       __imp_?customEvent@QObject@@MAEXPAVQEvent@@@Z 1001518c     Qt5Core:Qt5Core.dll
 0002:00000190       __imp_?disconnectNotify@QObject@@MAEXABVQMetaMethod@@@Z 10015190     Qt5Core:Qt5Core.dll
 0002:00000194       __imp_?event@QObject@@UAE_NPAVQEvent@@@Z 10015194     Qt5Core:Qt5Core.dll
 0002:00000198       __imp_?eventFilter@QObject@@UAE_NPAV1@PAVQEvent@@@Z 10015198     Qt5Core:Qt5Core.dll
 0002:0000019c       __imp_?timerEvent@QObject@@MAEXPAVQTimerEvent@@@Z 1001519c     Qt5Core:Qt5Core.dll
 0002:000001a0       __imp_?tr@QMetaObject@@QBE?AVQString@@PBD0H@Z 100151a0     Qt5Core:Qt5Core.dll
 0002:000001a4       __imp_??1Connection@QMetaObject@@QAE@XZ 100151a4     Qt5Core:Qt5Core.dll
 0002:000001a8       __imp_?detach@QListData@@QAEPAUData@1@H@Z 100151a8     Qt5Core:Qt5Core.dll
 0002:000001ac       __imp_?dispose@QListData@@SAXPAUData@1@@Z 100151ac     Qt5Core:Qt5Core.dll
 0002:000001b0       __imp_?connect@QObject@@QBE?AVConnection@QMetaObject@@PBV1@PBD1W4ConnectionType@Qt@@@Z 100151b0     Qt5Core:Qt5Core.dll
 0002:000001b4       __imp_??4QString@@QAEAAV0@PBD@Z 100151b4     Qt5Core:Qt5Core.dll
 0002:000001b8       __imp_?tr@QObject@@SA?AVQString@@PBD0H@Z 100151b8     Qt5Core:Qt5Core.dll
 0002:000001bc       __imp_?toUInt@QString@@QBEIPA_NH@Z 100151bc     Qt5Core:Qt5Core.dll
 0002:000001c0       __imp_?number@QString@@SA?AV1@HH@Z 100151c0     Qt5Core:Qt5Core.dll
 0002:000001c4       __imp_??8@YA_NABVQString@@0@Z 100151c4     Qt5Core:Qt5Core.dll
 0002:000001c8       __imp_??M@YA_NABVQString@@0@Z 100151c8     Qt5Core:Qt5Core.dll
 0002:000001cc       __imp_?detach_grow@QListData@@QAEPAUData@1@PAHH@Z 100151cc     Qt5Core:Qt5Core.dll
 0002:000001d0       __imp_?append@QListData@@QAEPAPAXXZ 100151d0     Qt5Core:Qt5Core.dll
 0002:000001d4       __imp_?freeNodeAndRebalance@QMapDataBase@@QAEXPAUQMapNodeBase@@@Z 100151d4     Qt5Core:Qt5Core.dll
 0002:000001d8       __imp_?recalcMostLeftNode@QMapDataBase@@QAEXXZ 100151d8     Qt5Core:Qt5Core.dll
 0002:000001dc       __imp_?createNode@QMapDataBase@@QAEPAUQMapNodeBase@@HHPAU2@_N@Z 100151dc     Qt5Core:Qt5Core.dll
 0002:000001e0       __imp_?freeTree@QMapDataBase@@QAEXPAUQMapNodeBase@@H@Z 100151e0     Qt5Core:Qt5Core.dll
 0002:000001e4       __imp_?createData@QMapDataBase@@SAPAU1@XZ 100151e4     Qt5Core:Qt5Core.dll
 0002:000001e8       __imp_?freeData@QMapDataBase@@SAXPAU1@@Z 100151e8     Qt5Core:Qt5Core.dll
 0002:000001ec       __imp_?rename@QFile@@SA_NABVQString@@0@Z 100151ec     Qt5Core:Qt5Core.dll
 0002:000001f0       __imp_??0QFileInfo@@QAE@ABVQString@@@Z 100151f0     Qt5Core:Qt5Core.dll
 0002:000001f4       __imp_??1QFileInfo@@QAE@XZ 100151f4     Qt5Core:Qt5Core.dll
 0002:000001f8       __imp_?exists@QFileInfo@@QBE_NXZ 100151f8     Qt5Core:Qt5Core.dll
 0002:000001fc       __imp_?completeBaseName@QFileInfo@@QBE?AVQString@@XZ 100151fc     Qt5Core:Qt5Core.dll
 0002:00000200       __imp_?shared_null@QListData@@2UData@1@B 10015200     Qt5Core:Qt5Core.dll
 0002:00000204       __imp_?shared_null@QMapDataBase@@2U1@B 10015204     Qt5Core:Qt5Core.dll
 0002:00000208       __imp_?translate@QCoreApplication@@SA?AVQString@@PBD00H@Z 10015208     Qt5Core:Qt5Core.dll
 0002:0000020c       __imp_?cast@QMetaObject@@QBEPAVQObject@@PAV2@@Z 1001520c     Qt5Core:Qt5Core.dll
 0002:00000210       __imp_?normalizedType@QMetaObject@@SA?AVQByteArray@@PBD@Z 10015210     Qt5Core:Qt5Core.dll
 0002:00000214       __imp_??1QByteArray@@QAE@XZ 10015214     Qt5Core:Qt5Core.dll
 0002:00000218       __imp_??0QString@@QAE@$$QAV0@@Z 10015218     Qt5Core:Qt5Core.dll
 0002:0000021c       __imp_?arg@QString@@QBE?AV1@HHHVQChar@@@Z 1001521c     Qt5Core:Qt5Core.dll
 0002:00000220       __imp_?realloc@QListData@@QAEXH@Z 10015220     Qt5Core:Qt5Core.dll
 0002:00000224       __imp_?registerNormalizedType@QMetaType@@SAHABVQByteArray@@P6AXPAX@ZP6APAXPBX@Z2P6APAX13@ZHV?$QFlags@W4TypeFlag@QMetaType@@@@PBUQMetaObject@@@Z 10015224     Qt5Core:Qt5Core.dll
 0002:00000228       __imp_?idealThreadCount@QThread@@SAHXZ 10015228     Qt5Core:Qt5Core.dll
 0002:0000022c       \177Qt5Core_NULL_THUNK_DATA 1001522c     Qt5Core:Qt5Core.dll
 0002:00000230       __imp_?clear@QTextDocument@@UAEXXZ 10015230     Qt5Gui:Qt5Gui.dll
 0002:00000234       __imp_?createObject@QTextDocument@@MAEPAVQTextObject@@ABVQTextFormat@@@Z 10015234     Qt5Gui:Qt5Gui.dll
 0002:00000238       __imp_?loadResource@QTextDocument@@MAE?AVQVariant@@HABVQUrl@@@Z 10015238     Qt5Gui:Qt5Gui.dll
 0002:0000023c       \177Qt5Gui_NULL_THUNK_DATA 1001523c     Qt5Gui:Qt5Gui.dll
 0002:00000240       __imp_?isString@QScriptValue@@QBE_NXZ 10015240     Qt5Script:Qt5Script.dll
 0002:00000244       __imp_?isNumber@QScriptValue@@QBE_NXZ 10015244     Qt5Script:Qt5Script.dll
 0002:00000248       __imp_??4QScriptValue@@QAEAAV0@ABV0@@Z 10015248     Qt5Script:Qt5Script.dll
 0002:0000024c       __imp_??0QScriptValue@@QAE@ABV0@@Z 1001524c     Qt5Script:Qt5Script.dll
 0002:00000250       __imp_??1QScriptValue@@QAE@XZ 10015250     Qt5Script:Qt5Script.dll
 0002:00000254       __imp_??0QScriptValue@@QAE@XZ 10015254     Qt5Script:Qt5Script.dll
 0002:00000258       __imp_?toString@QScriptValue@@QBE?AVQString@@XZ 10015258     Qt5Script:Qt5Script.dll
 0002:0000025c       __imp_?toInt32@QScriptValue@@QBEHXZ 1001525c     Qt5Script:Qt5Script.dll
 0002:00000260       __imp_??1QScriptEngine@@UAE@XZ 10015260     Qt5Script:Qt5Script.dll
 0002:00000264       __imp_?newVariant@QScriptEngine@@QAE?AVQScriptValue@@ABVQVariant@@@Z 10015264     Qt5Script:Qt5Script.dll
 0002:00000268       \177Qt5Script_NULL_THUNK_DATA 10015268     Qt5Script:Qt5Script.dll
 0002:0000026c       __imp_?updateEditorGeometry@QItemDelegate@@UBEXPAVQWidget@@ABVQStyleOptionViewItem@@ABVQModelIndex@@@Z 1001526c     Qt5Widgets:Qt5Widgets.dll
 0002:00000270       __imp_?paintingRoles@QAbstractItemDelegate@@UBE?AV?$QVector@H@@XZ 10015270     Qt5Widgets:Qt5Widgets.dll
 0002:00000274       __imp_?paint@QItemDelegate@@UBEXPAVQPainter@@ABVQStyleOptionViewItem@@ABVQModelIndex@@@Z 10015274     Qt5Widgets:Qt5Widgets.dll
 0002:00000278       __imp_?helpEvent@QAbstractItemDelegate@@UAE_NPAVQHelpEvent@@PAVQAbstractItemView@@ABVQStyleOptionViewItem@@ABVQModelIndex@@@Z 10015278     Qt5Widgets:Qt5Widgets.dll
 0002:0000027c       __imp_?eventFilter@QItemDelegate@@MAE_NPAVQObject@@PAVQEvent@@@Z 1001527c     Qt5Widgets:Qt5Widgets.dll
 0002:00000280       __imp_?editorEvent@QItemDelegate@@MAE_NPAVQEvent@@PAVQAbstractItemModel@@ABVQStyleOptionViewItem@@ABVQModelIndex@@@Z 10015280     Qt5Widgets:Qt5Widgets.dll
 0002:00000284       __imp_?drawFocus@QItemDelegate@@MBEXPAVQPainter@@ABVQStyleOptionViewItem@@ABVQRect@@@Z 10015284     Qt5Widgets:Qt5Widgets.dll
 0002:00000288       __imp_?drawDisplay@QItemDelegate@@MBEXPAVQPainter@@ABVQStyleOptionViewItem@@ABVQRect@@ABVQString@@@Z 10015288     Qt5Widgets:Qt5Widgets.dll
 0002:0000028c       __imp_?destroyEditor@QAbstractItemDelegate@@UBEXPAVQWidget@@ABVQModelIndex@@@Z 1001528c     Qt5Widgets:Qt5Widgets.dll
 0002:00000290       __imp_?drawDecoration@QItemDelegate@@MBEXPAVQPainter@@ABVQStyleOptionViewItem@@ABVQRect@@ABVQPixmap@@@Z 10015290     Qt5Widgets:Qt5Widgets.dll
 0002:00000294       __imp_?drawCheck@QItemDelegate@@MBEXPAVQPainter@@ABVQStyleOptionViewItem@@ABVQRect@@W4CheckState@Qt@@@Z 10015294     Qt5Widgets:Qt5Widgets.dll
 0002:00000298       __imp_?sizeHint@QItemDelegate@@UBE?AVQSize@@ABVQStyleOptionViewItem@@ABVQModelIndex@@@Z 10015298     Qt5Widgets:Qt5Widgets.dll
 0002:0000029c       \177Qt5Widgets_NULL_THUNK_DATA 1001529c     Qt5Widgets:Qt5Widgets.dll
 0002:000002a0       __imp_?isNotificationReport@Task@U2@@UBE_NXZ 100152a0     U2Core:U2Core.dll
 0002:000002a4       __imp_?hasWarning@Task@U2@@UBE_NXZ 100152a4     U2Core:U2Core.dll
 0002:000002a8       __imp_?hasSubtasksWithErrors@Task@U2@@UBE_NXZ 100152a8     U2Core:U2Core.dll
 0002:000002ac       __imp_?getWarnings@Task@U2@@UBE?AVQStringList@@XZ 100152ac     U2Core:U2Core.dll
 0002:000002b0       __imp_?getTopLevelParentTask@Task@U2@@UAEPAV12@XZ 100152b0     U2Core:U2Core.dll
 0002:000002b4       __imp_?getTaskId@Task@U2@@UBE_JXZ 100152b4     U2Core:U2Core.dll
 0002:000002b8       __imp_?getSubtaskWithErrors@Task@U2@@UBEPAV12@XZ 100152b8     U2Core:U2Core.dll
 0002:000002bc       __imp_?getParentTask@Task@U2@@UBEPAV12@XZ 100152bc     U2Core:U2Core.dll
 0002:000002c0       __imp_?getNumParallelSubtasks@Task@U2@@UBEHXZ 100152c0     U2Core:U2Core.dll
 0002:000002c4       __imp_?generateReport@Task@U2@@UBE?AVQString@@XZ 100152c4     U2Core:U2Core.dll
 0002:000002c8       __imp_?cleanup@Task@U2@@UAEXXZ 100152c8     U2Core:U2Core.dll
 0002:000002cc       __imp_??1Task@U2@@UAE@XZ   100152cc     U2Core:U2Core.dll
 0002:000002d0       __imp_?setError@Task@U2@@QAEXABVQString@@@Z 100152d0     U2Core:U2Core.dll
 0002:000002d4       __imp_??0Task@U2@@QAE@ABVQString@@V?$QFlags@W4TaskFlag@U2@@@@@Z 100152d4     U2Core:U2Core.dll
 0002:000002d8       __imp_?tr@Task@U2@@SA?AVQString@@PBD0H@Z 100152d8     U2Core:U2Core.dll
 0002:000002dc       __imp_?details@Logger@U2@@QAEXABVQString@@@Z 100152dc     U2Core:U2Core.dll
 0002:000002e0       __imp_??1Logger@U2@@UAE@XZ 100152e0     U2Core:U2Core.dll
 0002:000002e4       __imp_??0Logger@U2@@QAE@ABVQString@@@Z 100152e4     U2Core:U2Core.dll
 0002:000002e8       __imp_?errorOpeningFileWrite@L10N@U2@@SA?AVQString@@ABVGUrl@2@@Z 100152e8     U2Core:U2Core.dll
 0002:000002ec       __imp_?errorOpeningFileRead@L10N@U2@@SA?AVQString@@ABVGUrl@2@@Z 100152ec     U2Core:U2Core.dll
 0002:000002f0       __imp_?addFileToFileInfo@FileStorageUtils@U2@@SAXABVFileInfo@FileStorage@2@AAVWorkflowProcess@42@@Z 100152f0     U2Core:U2Core.dll
 0002:000002f4       __imp_?getFileToFileInfo@FileStorageUtils@U2@@SA?AVQString@@ABV3@0AAVWorkflowProcess@FileStorage@2@@Z 100152f4     U2Core:U2Core.dll
 0002:000002f8       __imp_?getDataPathByName@U2DataPathRegistry@U2@@QAEPAVU2DataPath@2@ABVQString@@@Z 100152f8     U2Core:U2Core.dll
 0002:000002fc       __imp_?getPathByName@U2DataPath@U2@@QBE?AVQString@@ABV3@@Z 100152fc     U2Core:U2Core.dll
 0002:00000300       __imp_?isValid@U2DataPath@U2@@QBE_NXZ 10015300     U2Core:U2Core.dll
 0002:00000304       __imp_?getStorageDir@AppFileStorage@U2@@QBE?AVQString@@XZ 10015304     U2Core:U2Core.dll
 0002:00000308       __imp_??1FileInfo@FileStorage@U2@@QAE@XZ 10015308     U2Core:U2Core.dll
 0002:0000030c       __imp_??0FileInfo@FileStorage@U2@@QAE@ABVQString@@00@Z 1001530c     U2Core:U2Core.dll
 0002:00000310       __imp_??1GUrl@U2@@QAE@XZ   10015310     U2Core:U2Core.dll
 0002:00000314       __imp_??0GUrl@U2@@QAE@ABVQString@@@Z 10015314     U2Core:U2Core.dll
 0002:00000318       __imp_?getAppFileStorage@AppContext@U2@@SAPAVAppFileStorage@2@XZ 10015318     U2Core:U2Core.dll
 0002:0000031c       __imp_?staticMetaObject@Task@U2@@2UQMetaObject@@B 1001531c     U2Core:U2Core.dll
 0002:00000320       __imp_?staticMetaObject@Plugin@U2@@2UQMetaObject@@B 10015320     U2Core:U2Core.dll
 0002:00000324       __imp_?qt_metacall@Plugin@U2@@UAEHW4Call@QMetaObject@@HPAPAX@Z 10015324     U2Core:U2Core.dll
 0002:00000328       __imp_?qt_metacast@Plugin@U2@@UAEPAXPBD@Z 10015328     U2Core:U2Core.dll
 0002:0000032c       __imp_?PLAIN_TEXT@BaseDocumentFormats@U2@@2VQString@@B 1001532c     U2Core:U2Core.dll
 0002:00000330       __imp_?getAppSettings@AppContext@U2@@SAPAVAppSettings@2@XZ 10015330     U2Core:U2Core.dll
 0002:00000334       __imp_?run@Task@U2@@UAEXXZ 10015334     U2Core:U2Core.dll
 0002:00000338       __imp_?qt_metacast@TaskSignalMapper@U2@@UAEPAXPBD@Z 10015338     U2Core:U2Core.dll
 0002:0000033c       __imp_?qt_metacast@FailTask@U2@@UAEPAXPBD@Z 1001533c     U2Core:U2Core.dll
 0002:00000340       __imp_?qt_metacall@TaskSignalMapper@U2@@UAEHW4Call@QMetaObject@@HPAPAX@Z 10015340     U2Core:U2Core.dll
 0002:00000344       __imp_?qt_metacall@FailTask@U2@@UAEHW4Call@QMetaObject@@HPAPAX@Z 10015344     U2Core:U2Core.dll
 0002:00000348       __imp_?metaObject@TaskSignalMapper@U2@@UBEPBUQMetaObject@@XZ 10015348     U2Core:U2Core.dll
 0002:0000034c       __imp_?metaObject@FailTask@U2@@UBEPBUQMetaObject@@XZ 1001534c     U2Core:U2Core.dll
 0002:00000350       __imp_?runScript@ScriptTask@U2@@SA?AVQScriptValue@@PAVQScriptEngine@@ABV?$QMap@VQString@@VQScriptValue@@@@ABVQString@@AAVTaskStateInfo@2@@Z 10015350     U2Core:U2Core.dll
 0002:00000354       __imp_?addListeners@ExternalToolSupportTask@U2@@QAEXABV?$QList@PAVExternalToolListener@U2@@@@@Z 10015354     U2Core:U2Core.dll
 0002:00000358       __imp_??1U2OpStatus2Log@U2@@UAE@XZ 10015358     U2Core:U2Core.dll
 0002:0000035c       __imp_??0U2OpStatus2Log@U2@@QAE@W4LogLevel@1@@Z 1001535c     U2Core:U2Core.dll
 0002:00000360       __imp_?getError@U2OpStatusImpl@U2@@UBE?AVQString@@XZ 10015360     U2Core:U2Core.dll
 0002:00000364       __imp_??0TaskSignalMapper@U2@@QAE@PAVTask@1@@Z 10015364     U2Core:U2Core.dll
 0002:00000368       __imp_?createDirectory@GUrlUtils@U2@@SA?AVQString@@ABV3@0AAVU2OpStatus@2@@Z 10015368     U2Core:U2Core.dll
 0002:0000036c       __imp_?createWorkingDir@FileAndDirectoryUtils@U2@@SA?AVQString@@ABV3@H00@Z 1001536c     U2Core:U2Core.dll
 0002:00000370       __imp_??1FailTask@U2@@UAE@XZ 10015370     U2Core:U2Core.dll
 0002:00000374       __imp_??0FailTask@U2@@QAE@ABVQString@@@Z 10015374     U2Core:U2Core.dll
 0002:00000378       __imp_?hasError@Task@U2@@QBE_NXZ 10015378     U2Core:U2Core.dll
 0002:0000037c       __imp_?isReportingEnabled@Task@U2@@UBE_NXZ 1001537c     U2Core:U2Core.dll
 0002:00000380       __imp_??1TaskStateInfo@U2@@UAE@XZ 10015380     U2Core:U2Core.dll
 0002:00000384       __imp_?setError@TaskStateInfo@U2@@UAEXABVQString@@@Z 10015384     U2Core:U2Core.dll
 0002:00000388       __imp_?getError@TaskStateInfo@U2@@UBE?AVQString@@XZ 10015388     U2Core:U2Core.dll
 0002:0000038c       __imp_??0TaskStateInfo@U2@@QAE@XZ 1001538c     U2Core:U2Core.dll
 0002:00000390       __imp_?error@Logger@U2@@QAEXABVQString@@@Z 10015390     U2Core:U2Core.dll
 0002:00000394       __imp_?setListenerForTask@ExternalToolSupportTask@U2@@MAEXPAVExternalToolRunTask@2@H@Z 10015394     U2Core:U2Core.dll
 0002:00000398       __imp_?setListenerForHelper@ExternalToolSupportTask@U2@@MAEXPAVExternalToolRunTaskHelper@2@H@Z 10015398     U2Core:U2Core.dll
 0002:0000039c       __imp_?setLastError@ExternalToolLogParser@U2@@MAEXABVQString@@@Z 1001539c     U2Core:U2Core.dll
 0002:000003a0       __imp_?run@ExternalToolRunTask@U2@@UAEXXZ 100153a0     U2Core:U2Core.dll
 0002:000003a4       __imp_?report@Task@U2@@UAE?AW4ReportResult@12@XZ 100153a4     U2Core:U2Core.dll
 0002:000003a8       __imp_?qt_metacast@ExternalToolRunTask@U2@@UAEPAXPBD@Z 100153a8     U2Core:U2Core.dll
 0002:000003ac       __imp_?qt_metacast@ExternalToolLogParser@U2@@UAEPAXPBD@Z 100153ac     U2Core:U2Core.dll
 0002:000003b0       __imp_?qt_metacall@ExternalToolRunTask@U2@@UAEHW4Call@QMetaObject@@HPAPAX@Z 100153b0     U2Core:U2Core.dll
 0002:000003b4       __imp_?qt_metacall@ExternalToolLogParser@U2@@UAEHW4Call@QMetaObject@@HPAPAX@Z 100153b4     U2Core:U2Core.dll
 0002:000003b8       __imp_?processLine@ExternalToolLogParser@U2@@MAEXABVQString@@@Z 100153b8     U2Core:U2Core.dll
 0002:000003bc       __imp_?processErrLine@ExternalToolLogParser@U2@@MAEXABVQString@@@Z 100153bc     U2Core:U2Core.dll
 0002:000003c0       __imp_?parseOutput@ExternalToolLogParser@U2@@UAEXABVQString@@@Z 100153c0     U2Core:U2Core.dll
 0002:000003c4       __imp_?parseErrOutput@ExternalToolLogParser@U2@@UAEXABVQString@@@Z 100153c4     U2Core:U2Core.dll
 0002:000003c8       __imp_?metaObject@ExternalToolRunTask@U2@@UBEPBUQMetaObject@@XZ 100153c8     U2Core:U2Core.dll
 0002:000003cc       __imp_?metaObject@ExternalToolLogParser@U2@@UBEPBUQMetaObject@@XZ 100153cc     U2Core:U2Core.dll
 0002:000003d0       __imp_?getDataPathRegistry@AppContext@U2@@SAPAVU2DataPathRegistry@2@XZ 100153d0     U2Core:U2Core.dll
 0002:000003d4       __imp_?isError@ExternalToolLogParser@U2@@MBE_NABVQString@@@Z 100153d4     U2Core:U2Core.dll
 0002:000003d8       __imp_?getProgress@ExternalToolLogParser@U2@@UAEHXZ 100153d8     U2Core:U2Core.dll
 0002:000003dc       __imp_??1ExternalToolLogParser@U2@@UAE@XZ 100153dc     U2Core:U2Core.dll
 0002:000003e0       __imp_??0ExternalToolLogParser@U2@@QAE@XZ 100153e0     U2Core:U2Core.dll
 0002:000003e4       __imp_??1ExternalToolSupportTask@U2@@UAE@XZ 100153e4     U2Core:U2Core.dll
 0002:000003e8       __imp_??0ExternalToolSupportTask@U2@@QAE@ABVQString@@V?$QFlags@W4TaskFlag@U2@@@@@Z 100153e8     U2Core:U2Core.dll
 0002:000003ec       __imp_??1ExternalToolRunTask@U2@@UAE@XZ 100153ec     U2Core:U2Core.dll
 0002:000003f0       __imp_??0ExternalToolRunTask@U2@@QAE@ABVQString@@ABVQStringList@@PAVExternalToolLogParser@1@010_N@Z 100153f0     U2Core:U2Core.dll
 0002:000003f4       __imp_?addSubTask@Task@U2@@QAEXPAV12@@Z 100153f4     U2Core:U2Core.dll
 0002:000003f8       __imp_?open@IOAdapterUtils@U2@@SAPAVIOAdapter@2@ABVGUrl@2@AAVU2OpStatus@2@W4IOAdapterMode@2@PAVIOAdapterFactory@2@@Z 100153f8     U2Core:U2Core.dll
 0002:000003fc       __imp_??1Plugin@U2@@UAE@XZ 100153fc     U2Core:U2Core.dll
 0002:00000400       __imp_??0Plugin@U2@@QAE@ABVQString@@0_NW4PluginState@1@@Z 10015400     U2Core:U2Core.dll
 0002:00000404       __imp_?unregisterEntry@ExternalToolRegistry@U2@@QAEXABVQString@@@Z 10015404     U2Core:U2Core.dll
 0002:00000408       __imp_?registerEntry@ExternalToolRegistry@U2@@QAE_NPAVExternalTool@2@@Z 10015408     U2Core:U2Core.dll
 0002:0000040c       __imp_?getExternalToolRegistry@AppContext@U2@@SAPAVExternalToolRegistry@2@XZ 1001540c     U2Core:U2Core.dll
 0002:00000410       __imp_?qt_metacast@ExternalTool@U2@@UAEPAXPBD@Z 10015410     U2Core:U2Core.dll
 0002:00000414       __imp_?qt_metacall@ExternalTool@U2@@UAEHW4Call@QMetaObject@@HPAPAX@Z 10015414     U2Core:U2Core.dll
 0002:00000418       __imp_?performAdditionalChecks@ExternalTool@U2@@UAEXABVQString@@@Z 10015418     U2Core:U2Core.dll
 0002:0000041c       __imp_?metaObject@ExternalTool@U2@@UBEPBUQMetaObject@@XZ 1001541c     U2Core:U2Core.dll
 0002:00000420       __imp_?getToolRunnerAdditionalOptions@ExternalTool@U2@@UAE?BVQStringList@@XZ 10015420     U2Core:U2Core.dll
 0002:00000424       __imp_?getAdditionalPaths@ExternalTool@U2@@UBE?AVQStringList@@XZ 10015424     U2Core:U2Core.dll
 0002:00000428       __imp_?getAdditionalParameters@ExternalTool@U2@@UAEXABVQString@@@Z 10015428     U2Core:U2Core.dll
 0002:0000042c       __imp_??1ExternalTool@U2@@UAE@XZ 1001542c     U2Core:U2Core.dll
 0002:00000430       __imp_??0ExternalTool@U2@@QAE@VQString@@0@Z 10015430     U2Core:U2Core.dll
 0002:00000434       __imp_?tr@ExternalTool@U2@@SA?AVQString@@PBD0H@Z 10015434     U2Core:U2Core.dll
 0002:00000438       __imp_?CUSTOM_FILE_TO_FILE@StorageRoles@U2@@2VQString@@B 10015438     U2Core:U2Core.dll
 0002:0000043c       __imp_?setReportingSupported@Task@U2@@UAEX_N@Z 1001543c     U2Core:U2Core.dll
 0002:00000440       __imp_?setReportingEnabled@Task@U2@@UAEX_N@Z 10015440     U2Core:U2Core.dll
 0002:00000444       __imp_?setNotificationReport@Task@U2@@UAEX_N@Z 10015444     U2Core:U2Core.dll
 0002:00000448       __imp_?setNoAutoDelete@Task@U2@@UAEX_N@Z 10015448     U2Core:U2Core.dll
 0002:0000044c       __imp_?setCollectChildrensWarningsFlag@Task@U2@@UAEX_N@Z 1001544c     U2Core:U2Core.dll
 0002:00000450       __imp_?qt_metacast@Task@U2@@UAEPAXPBD@Z 10015450     U2Core:U2Core.dll
 0002:00000454       __imp_?qt_metacall@Task@U2@@UAEHW4Call@QMetaObject@@HPAPAX@Z 10015454     U2Core:U2Core.dll
 0002:00000458       __imp_?propagateSubtaskError@Task@U2@@UAE_NXZ 10015458     U2Core:U2Core.dll
 0002:0000045c       __imp_?prepare@Task@U2@@UAEXXZ 1001545c     U2Core:U2Core.dll
 0002:00000460       __imp_?onSubTaskFinished@Task@U2@@MAE?AV?$QList@PAVTask@U2@@@@PAV12@@Z 10015460     U2Core:U2Core.dll
 0002:00000464       __imp_?metaObject@Task@U2@@UBEPBUQMetaObject@@XZ 10015464     U2Core:U2Core.dll
 0002:00000468       __imp_?isTopLevelTask@Task@U2@@UBE_NXZ 10015468     U2Core:U2Core.dll
 0002:0000046c       __imp_?isReportingSupported@Task@U2@@UBE_NXZ 1001546c     U2Core:U2Core.dll
 0002:00000470       \177U2Core_NULL_THUNK_DATA 10015470     U2Core:U2Core.dll
 0002:00000474       __imp_?setModelData@SpinBoxDelegate@U2@@UBEXPAVQWidget@@PAVQAbstractItemModel@@ABVQModelIndex@@@Z 10015474     U2Designer:U2Designer.dll
 0002:00000478       __imp_?setModelData@URLDelegate@U2@@UBEXPAVQWidget@@PAVQAbstractItemModel@@ABVQModelIndex@@@Z 10015478     U2Designer:U2Designer.dll
 0002:0000047c       __imp_?type@URLDelegate@U2@@UBE?AW4Type@PropertyDelegate@2@XZ 1001547c     U2Designer:U2Designer.dll
 0002:00000480       __imp_?updateDelegate@DelegateEditor@U2@@UAEXABVQString@@@Z 10015480     U2Designer:U2Designer.dll
 0002:00000484       __imp_?updateDelegates@DelegateEditor@U2@@UAEXXZ 10015484     U2Designer:U2Designer.dll
 0002:00000488       __imp_?setEditorData@URLDelegate@U2@@UBEXPAVQWidget@@ABVQModelIndex@@@Z 10015488     U2Designer:U2Designer.dll
 0002:0000048c       __imp_?setEditorData@SpinBoxDelegate@U2@@UBEXPAVQWidget@@ABVQModelIndex@@@Z 1001548c     U2Designer:U2Designer.dll
 0002:00000490       __imp_?removeDelegate@DelegateEditor@U2@@UAEPAVPropertyDelegate@2@ABVQString@@@Z 10015490     U2Designer:U2Designer.dll
 0002:00000494       __imp_?qt_metacast@URLDelegate@U2@@UAEPAXPBD@Z 10015494     U2Designer:U2Designer.dll
 0002:00000498       __imp_?qt_metacast@SpinBoxDelegate@U2@@UAEPAXPBD@Z 10015498     U2Designer:U2Designer.dll
 0002:0000049c       __imp_?qt_metacast@DelegateEditor@U2@@UAEPAXPBD@Z 1001549c     U2Designer:U2Designer.dll
 0002:000004a0       __imp_?qt_metacall@URLDelegate@U2@@UAEHW4Call@QMetaObject@@HPAPAX@Z 100154a0     U2Designer:U2Designer.dll
 0002:000004a4       __imp_?qt_metacall@SpinBoxDelegate@U2@@UAEHW4Call@QMetaObject@@HPAPAX@Z 100154a4     U2Designer:U2Designer.dll
 0002:000004a8       __imp_?qt_metacall@DelegateEditor@U2@@UAEHW4Call@QMetaObject@@HPAPAX@Z 100154a8     U2Designer:U2Designer.dll
 0002:000004ac       __imp_?metaObject@URLDelegate@U2@@UBEPBUQMetaObject@@XZ 100154ac     U2Designer:U2Designer.dll
 0002:000004b0       __imp_?metaObject@SpinBoxDelegate@U2@@UBEPBUQMetaObject@@XZ 100154b0     U2Designer:U2Designer.dll
 0002:000004b4       __imp_?metaObject@DelegateEditor@U2@@UBEPBUQMetaObject@@XZ 100154b4     U2Designer:U2Designer.dll
 0002:000004b8       __imp_?getItems@SpinBoxDelegate@U2@@UBEXAAV?$QMap@VQString@@VQVariant@@@@@Z 100154b8     U2Designer:U2Designer.dll
 0002:000004bc       __imp_?getDisplayValue@URLDelegate@U2@@UBE?AVQVariant@@ABV3@@Z 100154bc     U2Designer:U2Designer.dll
 0002:000004c0       __imp_?getDisplayValue@SpinBoxDelegate@U2@@UBE?AVQVariant@@ABV3@@Z 100154c0     U2Designer:U2Designer.dll
 0002:000004c4       __imp_?getDelegate@DelegateEditor@U2@@UAEPAVPropertyDelegate@2@ABVQString@@@Z 100154c4     U2Designer:U2Designer.dll
 0002:000004c8       __imp_?createWizardWidget@URLDelegate@U2@@UBEPAVPropertyWidget@2@AAVU2OpStatus@2@PAVQWidget@@@Z 100154c8     U2Designer:U2Designer.dll
 0002:000004cc       __imp_?createWizardWidget@SpinBoxDelegate@U2@@UBEPAVPropertyWidget@2@AAVU2OpStatus@2@PAVQWidget@@@Z 100154cc     U2Designer:U2Designer.dll
 0002:000004d0       __imp_?createEditor@URLDelegate@U2@@UBEPAVQWidget@@PAV3@ABVQStyleOptionViewItem@@ABVQModelIndex@@@Z 100154d0     U2Designer:U2Designer.dll
 0002:000004d4       __imp_?createEditor@SpinBoxDelegate@U2@@UBEPAVQWidget@@PAV3@ABVQStyleOptionViewItem@@ABVQModelIndex@@@Z 100154d4     U2Designer:U2Designer.dll
 0002:000004d8       __imp_?commit@DelegateEditor@U2@@UAEXXZ 100154d8     U2Designer:U2Designer.dll
 0002:000004dc       __imp_?clone@URLDelegate@U2@@UAEPAVPropertyDelegate@2@XZ 100154dc     U2Designer:U2Designer.dll
 0002:000004e0       __imp_?clone@SpinBoxDelegate@U2@@UAEPAVPropertyDelegate@2@XZ 100154e0     U2Designer:U2Designer.dll
 0002:000004e4       __imp_?clone@DelegateEditor@U2@@UAEPAVConfigurationEditor@2@XZ 100154e4     U2Designer:U2Designer.dll
 0002:000004e8       __imp_?addDelegate@DelegateEditor@U2@@UAEXPAVPropertyDelegate@2@ABVQString@@@Z 100154e8     U2Designer:U2Designer.dll
 0002:000004ec       __imp_??1SpinBoxDelegate@U2@@UAE@XZ 100154ec     U2Designer:U2Designer.dll
 0002:000004f0       __imp_??0SpinBoxDelegate@U2@@QAE@ABV?$QMap@VQString@@VQVariant@@@@PAVQObject@@@Z 100154f0     U2Designer:U2Designer.dll
 0002:000004f4       __imp_??1URLDelegate@U2@@UAE@XZ 100154f4     U2Designer:U2Designer.dll
 0002:000004f8       __imp_??0URLDelegate@U2@@QAE@ABVDelegateTags@1@ABVQString@@_N22PAVQObject@@2@Z 100154f8     U2Designer:U2Designer.dll
 0002:000004fc       __imp_??1DelegateEditor@U2@@UAE@XZ 100154fc     U2Designer:U2Designer.dll
 0002:00000500       __imp_??0DelegateEditor@U2@@QAE@ABV?$QMap@VQString@@PAVPropertyDelegate@U2@@@@@Z 10015500     U2Designer:U2Designer.dll
 0002:00000504       \177U2Designer_NULL_THUNK_DATA 10015504     U2Designer:U2Designer.dll
 0002:00000508       __imp_?hasNextLine@TabulatedFormatReader@U2@@QBE_NXZ 10015508     U2Formats:U2Formats.dll
 0002:0000050c       __imp_?getNextLine@TabulatedFormatReader@U2@@QAE?AVQStringList@@XZ 1001550c     U2Formats:U2Formats.dll
 0002:00000510       __imp_??1TabulatedFormatReader@U2@@UAE@XZ 10015510     U2Formats:U2Formats.dll
 0002:00000514       __imp_??0TabulatedFormatReader@U2@@QAE@AAVU2OpStatus@1@PAVIOAdapter@1@@Z 10015514     U2Formats:U2Formats.dll
 0002:00000518       \177U2Formats_NULL_THUNK_DATA 10015518     U2Formats:U2Formats.dll
 0002:0000051c       __imp_?prepareDocumentsFileFilter@DialogUtils@U2@@SA?AVQString@@ABV3@_NABVQStringList@@@Z 1001551c     U2Gui:U2Gui.dll
 0002:00000520       \177U2Gui_NULL_THUNK_DATA  10015520     U2Gui:U2Gui.dll
 0002:00000524       __imp_??_7ConfigurationValidator@U2@@6B@ 10015524     U2Lang:U2Lang.dll
 0002:00000528       __imp_?PLACEHOLDER_TEXT@DelegateTags@U2@@2VQString@@B 10015528     U2Lang:U2Lang.dll
 0002:0000052c       __imp_?validate@Attribute@U2@@UAE_NAAV?$QList@VWorkflowNotification@U2@@@@@Z 1001552c     U2Lang:U2Lang.dll
 0002:00000530       __imp_?validate@ActorValidator@Workflow@U2@@UBE_NPBVConfiguration@3@AAV?$QList@VWorkflowNotification@U2@@@@@Z 10015530     U2Lang:U2Lang.dll
 0002:00000534       __imp_?updateActorIds@Attribute@U2@@UAEXABV?$QMap@VQString@@V1@@@@Z 10015534     U2Lang:U2Lang.dll
 0002:00000538       __imp_?update@PropertyDelegate@U2@@UAEXXZ 10015538     U2Lang:U2Lang.dll
 0002:0000053c       __imp_?unregisterEntry@?$IdRegistry@VDomainFactory@Workflow@U2@@@U2@@UAEPAVDomainFactory@Workflow@2@ABVQString@@@Z 1001553c     U2Lang:U2Lang.dll
 0002:00000540       __imp_?type@PropertyDelegate@U2@@UBE?AW4Type@12@XZ 10015540     U2Lang:U2Lang.dll
 0002:00000544       __imp_?setVisibleSlot@PortDescriptor@Workflow@U2@@UAEXABVQString@@_N@Z 10015544     U2Lang:U2Lang.dll
 0002:00000548       __imp_?setAttributeValue@Attribute@U2@@UAEXABVQVariant@@@Z 10015548     U2Lang:U2Lang.dll
 0002:0000054c       __imp_?registerEntry@?$IdRegistry@VDomainFactory@Workflow@U2@@@U2@@UAE_NPAVDomainFactory@Workflow@2@@Z 1001554c     U2Lang:U2Lang.dll
 0002:00000550       __imp_?kind@MapDataType@U2@@UBE?AW4Kind@DataType@2@XZ 10015550     U2Lang:U2Lang.dll
 0002:00000554       __imp_?isEmpty@ConfigurationEditor@U2@@UBE_NXZ 10015554     U2Lang:U2Lang.dll
 0002:00000558       __imp_?isEmpty@Attribute@U2@@UBE_NXZ 10015558     U2Lang:U2Lang.dll
 0002:0000055c       __imp_?isDefaultValue@Attribute@U2@@UBE_NXZ 1001555c     U2Lang:U2Lang.dll
 0002:00000560       __imp_?isAcceptableDrop@ActorPrototype@Workflow@U2@@UBE_NPBVQMimeData@@PAV?$QMap@VQString@@VQVariant@@@@@Z 10015560     U2Lang:U2Lang.dll
 0002:00000564       __imp_?getWidget@ConfigurationEditor@U2@@UAEPAVQWidget@@XZ 10015564     U2Lang:U2Lang.dll
 0002:00000568       __imp_?getType@PortDescriptor@Workflow@U2@@UBE?AV?$QExplicitlySharedDataPointer@VDataType@U2@@@@XZ 10015568     U2Lang:U2Lang.dll
 0002:0000056c       __imp_?getItems@PropertyDelegate@U2@@UBEXAAV?$QMap@VQString@@VQVariant@@@@@Z 1001556c     U2Lang:U2Lang.dll
 0002:00000570       __imp_?getGroup@Attribute@U2@@UAE?AW4AttributeGroup@2@XZ 10015570     U2Lang:U2Lang.dll
 0002:00000574       __imp_?getDefaultPureValue@Attribute@U2@@UBEABVQVariant@@XZ 10015574     U2Lang:U2Lang.dll
 0002:00000578       __imp_?getDatatypeByDescriptor@MapDataType@U2@@UBE?AV?$QExplicitlySharedDataPointer@VDataType@U2@@@@ABVDescriptor@2@@Z 10015578     U2Lang:U2Lang.dll
 0002:0000057c       __imp_?getById@?$IdRegistry@VDomainFactory@Workflow@U2@@@U2@@UAEPAVDomainFactory@Workflow@2@ABVQString@@@Z 1001557c     U2Lang:U2Lang.dll
 0002:00000580       __imp_?getAttributePureValue@Attribute@U2@@UBEABVQVariant@@XZ 10015580     U2Lang:U2Lang.dll
 0002:00000584       __imp_?getAllIds@?$IdRegistry@VDomainFactory@Workflow@U2@@@U2@@UBE?AV?$QList@VQString@@@@XZ 10015584     U2Lang:U2Lang.dll
 0002:00000588       __imp_?getAllEntries@?$IdRegistry@VDomainFactory@Workflow@U2@@@U2@@UBE?AV?$QList@PAVDomainFactory@Workflow@U2@@@@XZ 10015588     U2Lang:U2Lang.dll
 0002:0000058c       __imp_?getAllDescriptors@MapDataType@U2@@UBE?AV?$QList@VDescriptor@U2@@@@XZ 1001558c     U2Lang:U2Lang.dll
 0002:00000590       __imp_?destroy@DomainFactory@Workflow@U2@@UAEXPAVScheduler@23@PAVSchema@23@@Z 10015590     U2Lang:U2Lang.dll
 0002:00000594       __imp_?createScheduler@DomainFactory@Workflow@U2@@UAEPAVScheduler@23@PAVSchema@23@@Z 10015594     U2Lang:U2Lang.dll
 0002:00000598       __imp_?createPort@IntegralBusActorPrototype@Workflow@U2@@UAEPAVPort@23@ABVPortDescriptor@23@PAVActor@23@@Z 10015598     U2Lang:U2Lang.dll
 0002:0000059c       __imp_?createInstance@ActorPrototype@Workflow@U2@@UAEPAVActor@23@ABVQString@@PAVAttributeScript@3@ABV?$QMap@VQString@@VQVariant@@@@@Z 1001559c     U2Lang:U2Lang.dll
 0002:000005a0       __imp_?createConnection@DomainFactory@Workflow@U2@@UAEPAVCommunicationChannel@23@PAVLink@23@@Z 100155a0     U2Lang:U2Lang.dll
 0002:000005a4       __imp_?clone@Attribute@U2@@UAEPAV12@XZ 100155a4     U2Lang:U2Lang.dll
 0002:000005a8       __imp_??1DomainFactory@Workflow@U2@@UAE@XZ 100155a8     U2Lang:U2Lang.dll
 0002:000005ac       __imp_??0DomainFactory@Workflow@U2@@QAE@ABVQString@@@Z 100155ac     U2Lang:U2Lang.dll
 0002:000005b0       __imp_?getInstance@WorkflowEnv@Workflow@U2@@KAPAV123@XZ 100155b0     U2Lang:U2Lang.dll
 0002:000005b4       __imp_?NUM_TYPE@BaseTypes@U2@@SA?AV?$QExplicitlySharedDataPointer@VDataType@U2@@@@XZ 100155b4     U2Lang:U2Lang.dll
 0002:000005b8       __imp_?staticMetaObject@PrompterBaseImpl@U2@@2UQMetaObject@@B 100155b8     U2Lang:U2Lang.dll
 0002:000005bc       __imp_?unregisterProto@ActorPrototypeRegistry@Workflow@U2@@QAEPAVActorPrototype@23@ABVQString@@@Z 100155bc     U2Lang:U2Lang.dll
 0002:000005c0       __imp_?registerProto@ActorPrototypeRegistry@Workflow@U2@@QAEXABVDescriptor@3@PAVActorPrototype@23@@Z 100155c0     U2Lang:U2Lang.dll
 0002:000005c4       __imp_?addExternalTool@ActorPrototype@Workflow@U2@@QAEXABVQString@@0@Z 100155c4     U2Lang:U2Lang.dll
 0002:000005c8       __imp_?setPrompter@ActorPrototype@Workflow@U2@@QAEXPAVPrompter@23@@Z 100155c8     U2Lang:U2Lang.dll
 0002:000005cc       __imp_?setValidator@ActorPrototype@Workflow@U2@@QAEXPAVConfigurationValidator@3@@Z 100155cc     U2Lang:U2Lang.dll
 0002:000005d0       __imp_?setEditor@ActorPrototype@Workflow@U2@@QAEXPAVConfigurationEditor@3@@Z 100155d0     U2Lang:U2Lang.dll
 0002:000005d4       __imp_??1ActorPrototype@Workflow@U2@@UAE@XZ 100155d4     U2Lang:U2Lang.dll
 0002:000005d8       __imp_??0ActorPrototype@Workflow@U2@@QAE@ABVDescriptor@2@ABV?$QList@PAVPortDescriptor@Workflow@U2@@@@ABV?$QList@PAVAttribute@U2@@@@@Z 100155d8     U2Lang:U2Lang.dll
 0002:000005dc       __imp_??1PortDescriptor@Workflow@U2@@UAE@XZ 100155dc     U2Lang:U2Lang.dll
 0002:000005e0       __imp_??0PortDescriptor@Workflow@U2@@QAE@ABVDescriptor@2@V?$QExplicitlySharedDataPointer@VDataType@U2@@@@_N2I@Z 100155e0     U2Lang:U2Lang.dll
 0002:000005e4       __imp_??1DelegateTags@U2@@UAE@XZ 100155e4     U2Lang:U2Lang.dll
 0002:000005e8       __imp_?set@DelegateTags@U2@@QAEXABVQString@@ABVQVariant@@@Z 100155e8     U2Lang:U2Lang.dll
 0002:000005ec       __imp_??0DelegateTags@U2@@QAE@PAVQObject@@@Z 100155ec     U2Lang:U2Lang.dll
 0002:000005f0       __imp_??1Attribute@U2@@UAE@XZ 100155f0     U2Lang:U2Lang.dll
 0002:000005f4       __imp_??0Attribute@U2@@QAE@ABVDescriptor@1@V?$QExplicitlySharedDataPointer@VDataType@U2@@@@_NABVQVariant@@@Z 100155f4     U2Lang:U2Lang.dll
 0002:000005f8       __imp_??0Attribute@U2@@QAE@ABVDescriptor@1@V?$QExplicitlySharedDataPointer@VDataType@U2@@@@V?$QFlags@W4Flag@Attribute@U2@@@@ABVQVariant@@@Z 100155f8     U2Lang:U2Lang.dll
 0002:000005fc       __imp_??1MapDataType@U2@@UAE@XZ 100155fc     U2Lang:U2Lang.dll
 0002:00000600       __imp_??_7ActorValidator@Workflow@U2@@6B@ 10015600     U2Lang:U2Lang.dll
 0002:00000604       __imp_??0Descriptor@U2@@QAE@ABVQString@@@Z 10015604     U2Lang:U2Lang.dll
 0002:00000608       __imp_??0Descriptor@U2@@QAE@ABVQString@@00@Z 10015608     U2Lang:U2Lang.dll
 0002:0000060c       __imp_?U2_INFO@WorkflowNotification@U2@@2VQString@@B 1001560c     U2Lang:U2Lang.dll
 0002:00000610       __imp_?setDone@BaseWorker@LocalWorkflow@U2@@UAEXXZ 10015610     U2Lang:U2Lang.dll
 0002:00000614       __imp_?isReady@BaseWorker@LocalWorkflow@U2@@UBE_NXZ 10015614     U2Lang:U2Lang.dll
 0002:00000618       __imp_?isDone@BaseWorker@LocalWorkflow@U2@@UBE_NXZ 10015618     U2Lang:U2Lang.dll
 0002:0000061c       __imp_?getOutputFiles@BaseWorker@LocalWorkflow@U2@@UAE?AVQStringList@@XZ 1001561c     U2Lang:U2Lang.dll
 0002:00000620       __imp_?getMessageAndSetupScriptValues@BaseWorker@LocalWorkflow@U2@@UAE?AVMessage@Workflow@3@PAVCommunicationChannel@53@@Z 10015620     U2Lang:U2Lang.dll
 0002:00000624       __imp_?getCommunication@BaseWorker@LocalWorkflow@U2@@UAEPAVCommunicationChannel@Workflow@3@ABVQString@@@Z 10015624     U2Lang:U2Lang.dll
 0002:00000628       __imp_?getActorId@BaseWorker@LocalWorkflow@U2@@UBE?AVQString@@XZ 10015628     U2Lang:U2Lang.dll
 0002:0000062c       __imp_?canTaskBeCanceled@BaseWorker@LocalWorkflow@U2@@MBE_NPAVTask@3@@Z 1001562c     U2Lang:U2Lang.dll
 0002:00000630       __imp_?addCommunication@BaseWorker@LocalWorkflow@U2@@UAE_NABVQString@@PAVCommunicationChannel@Workflow@3@@Z 10015630     U2Lang:U2Lang.dll
 0002:00000634       __imp_?createLogListeners@BaseWorker@LocalWorkflow@U2@@QAE?AV?$QList@PAVExternalToolListener@U2@@@@H@Z 10015634     U2Lang:U2Lang.dll
 0002:00000638       __imp_??1BaseWorker@LocalWorkflow@U2@@UAE@XZ 10015638     U2Lang:U2Lang.dll
 0002:0000063c       __imp_??0BaseWorker@LocalWorkflow@U2@@QAE@PAVActor@Workflow@2@_N@Z 1001563c     U2Lang:U2Lang.dll
 0002:00000640       __imp_?getBusType@IntegralBus@Workflow@U2@@QBE?AV?$QExplicitlySharedDataPointer@VDataType@U2@@@@XZ 10015640     U2Lang:U2Lang.dll
 0002:00000644       __imp_?isOutUrlAttribute@RFSUtils@U2@@SA_NPAVAttribute@2@PAVActor@Workflow@2@AA_N@Z 10015644     U2Lang:U2Lang.dll
 0002:00000648       __imp_?addInfo@WorkflowMonitor@Workflow@U2@@QAEXABVQString@@00@Z 10015648     U2Lang:U2Lang.dll
 0002:0000064c       __imp_?addOutputFile@WorkflowMonitor@Workflow@U2@@QAEXABVQString@@0_N@Z 1001564c     U2Lang:U2Lang.dll
 0002:00000650       __imp_??1Message@Workflow@U2@@QAE@XZ 10015650     U2Lang:U2Lang.dll
 0002:00000654       __imp_?getMetadataId@Message@Workflow@U2@@QBEHXZ 10015654     U2Lang:U2Lang.dll
 0002:00000658       __imp_?getData@Message@Workflow@U2@@QBE?AVQVariant@@XZ 10015658     U2Lang:U2Lang.dll
 0002:0000065c       __imp_??0Message@Workflow@U2@@QAE@V?$QExplicitlySharedDataPointer@VDataType@U2@@@@ABVQVariant@@H@Z 1001565c     U2Lang:U2Lang.dll
 0002:00000660       __imp_?getScriptVars@AttributeScript@U2@@QBEABV?$QMap@VDescriptor@U2@@VQVariant@@@@XZ 10015660     U2Lang:U2Lang.dll
 0002:00000664       __imp_?getScriptText@AttributeScript@U2@@QBEABVQString@@XZ 10015664     U2Lang:U2Lang.dll
 0002:00000668       __imp_?isEmpty@AttributeScript@U2@@QBE_NXZ 10015668     U2Lang:U2Lang.dll
 0002:0000066c       __imp_??1WorkflowScriptEngine@U2@@UAE@XZ 1001566c     U2Lang:U2Lang.dll
 0002:00000670       __imp_??0WorkflowScriptEngine@U2@@QAE@PAVWorkflowContext@Workflow@1@@Z 10015670     U2Lang:U2Lang.dll
 0002:00000674       __imp_?getMetadataStorage@WorkflowContext@Workflow@U2@@QAEAAVMessageMetadataStorage@3@XZ 10015674     U2Lang:U2Lang.dll
 0002:00000678       __imp_?absolutePath@WorkflowContext@Workflow@U2@@QBE?AVQString@@ABV4@@Z 10015678     U2Lang:U2Lang.dll
 0002:0000067c       __imp_?workingDir@WorkflowContext@Workflow@U2@@QBE?AVQString@@XZ 1001567c     U2Lang:U2Lang.dll
 0002:00000680       __imp_?getWorkflowProcess@WorkflowContext@Workflow@U2@@QAEAAVWorkflowProcess@FileStorage@3@XZ 10015680     U2Lang:U2Lang.dll
 0002:00000684       __imp_?getMonitor@WorkflowContext@Workflow@U2@@QAEPAVWorkflowMonitor@23@XZ 10015684     U2Lang:U2Lang.dll
 0002:00000688       __imp_?get@MessageMetadataStorage@U2@@QBE?AVMessageMetadata@2@H@Z 10015688     U2Lang:U2Lang.dll
 0002:0000068c       __imp_??1MessageMetadata@U2@@QAE@XZ 1001568c     U2Lang:U2Lang.dll
 0002:00000690       __imp_?getFileUrl@MessageMetadata@U2@@QBEABVQString@@XZ 10015690     U2Lang:U2Lang.dll
 0002:00000694       __imp_?initEngine@WorkflowScriptLibrary@U2@@SAXPAVWorkflowScriptEngine@2@@Z 10015694     U2Lang:U2Lang.dll
 0002:00000698       __imp_?URL_SLOT@BaseSlots@Workflow@U2@@SA?BVDescriptor@3@XZ 10015698     U2Lang:U2Lang.dll
 0002:0000069c       __imp_??0Descriptor@U2@@QAE@ABV01@@Z 1001569c     U2Lang:U2Lang.dll
 0002:000006a0       __imp_?getId@Descriptor@U2@@QBE?AVQString@@XZ 100156a0     U2Lang:U2Lang.dll
 0002:000006a4       __imp_??1Descriptor@U2@@UAE@XZ 100156a4     U2Lang:U2Lang.dll
 0002:000006a8       __imp_?U2_ERROR@WorkflowNotification@U2@@2VQString@@B 100156a8     U2Lang:U2Lang.dll
 0002:000006ac       __imp_?getId@Actor@Workflow@U2@@QBE?AVQString@@XZ 100156ac     U2Lang:U2Lang.dll
 0002:000006b0       __imp_??0WorkflowNotification@U2@@QAE@ABV01@@Z 100156b0     U2Lang:U2Lang.dll
 0002:000006b4       __imp_??1WorkflowNotification@U2@@QAE@XZ 100156b4     U2Lang:U2Lang.dll
 0002:000006b8       __imp_??0WorkflowNotification@U2@@QAE@ABVQString@@00@Z 100156b8     U2Lang:U2Lang.dll
 0002:000006bc       __imp_?update@PrompterBaseImpl@U2@@UAEXABV?$QMap@VQString@@VQVariant@@@@@Z 100156bc     U2Lang:U2Lang.dll
 0002:000006c0       __imp_?sl_actorModified@PrompterBaseImpl@U2@@MAEXXZ 100156c0     U2Lang:U2Lang.dll
 0002:000006c4       __imp_?qt_metacast@PrompterBaseImpl@U2@@UAEPAXPBD@Z 100156c4     U2Lang:U2Lang.dll
 0002:000006c8       __imp_?qt_metacall@PrompterBaseImpl@U2@@UAEHW4Call@QMetaObject@@HPAPAX@Z 100156c8     U2Lang:U2Lang.dll
 0002:000006cc       __imp_?metaObject@PrompterBaseImpl@U2@@UBEPBUQMetaObject@@XZ 100156cc     U2Lang:U2Lang.dll
 0002:000006d0       __imp_??1PrompterBaseImpl@U2@@UAE@XZ 100156d0     U2Lang:U2Lang.dll
 0002:000006d4       __imp_??0PrompterBaseImpl@U2@@QAE@PAVActor@Workflow@1@@Z 100156d4     U2Lang:U2Lang.dll
 0002:000006d8       __imp_?getOutputPorts@Actor@Workflow@U2@@QBE?AV?$QList@PAVPort@Workflow@U2@@@@XZ 100156d8     U2Lang:U2Lang.dll
 0002:000006dc       __imp_?getInputPorts@Actor@Workflow@U2@@QBE?AV?$QList@PAVPort@Workflow@U2@@@@XZ 100156dc     U2Lang:U2Lang.dll
 0002:000006e0       __imp_??0MapDataType@U2@@QAE@ABVDescriptor@1@ABV?$QMap@VDescriptor@U2@@V?$QExplicitlySharedDataPointer@VDataType@U2@@@@@@@Z 100156e0     U2Lang:U2Lang.dll
 0002:000006e4       __imp_?ID@LocalDomainFactory@LocalWorkflow@U2@@2VQString@@B 100156e4     U2Lang:U2Lang.dll
 0002:000006e8       __imp_?qt_metacast@BaseWorker@LocalWorkflow@U2@@UAEPAXPBD@Z 100156e8     U2Lang:U2Lang.dll
 0002:000006ec       __imp_?qt_metacall@BaseWorker@LocalWorkflow@U2@@UAEHW4Call@QMetaObject@@HPAPAX@Z 100156ec     U2Lang:U2Lang.dll
 0002:000006f0       __imp_?staticMetaObject@BaseWorker@LocalWorkflow@U2@@2UQMetaObject@@B 100156f0     U2Lang:U2Lang.dll
 0002:000006f4       __imp_?STRING_TYPE@BaseTypes@U2@@SA?AV?$QExplicitlySharedDataPointer@VDataType@U2@@@@XZ 100156f4     U2Lang:U2Lang.dll
 0002:000006f8       __imp_?FILTER@DelegateTags@U2@@2VQString@@B 100156f8     U2Lang:U2Lang.dll
 0002:000006fc       __imp_?getDatatypesMap@MapDataType@U2@@UBE?AV?$QMap@VDescriptor@U2@@V?$QExplicitlySharedDataPointer@VDataType@U2@@@@@@XZ 100156fc     U2Lang:U2Lang.dll
 0002:00000700       \177U2Lang_NULL_THUNK_DATA 10015700     U2Lang:U2Lang.dll
 0002:00000704       __imp_?WORKFLOW_CLASSIFY_TOOL_ID@NgsReadsClassificationPlugin@U2@@2VQString@@B 10015704     ngs_reads_classification:ngs_reads_classification.dll
 0002:00000708       __imp_?WORKFLOW_ELEMENTS_GROUP@NgsReadsClassificationPlugin@U2@@2VQString@@B 10015708     ngs_reads_classification:ngs_reads_classification.dll
 0002:0000070c       __imp_?TAXONOMY_CLASSIFICATION_TYPE@TaxonomySupport@LocalWorkflow@U2@@SA?AV?$QExplicitlySharedDataPointer@VDataType@U2@@@@XZ 1001570c     ngs_reads_classification:ngs_reads_classification.dll
 0002:00000710       __imp_?TAXONOMY_CLASSIFICATION_SLOT@TaxonomySupport@LocalWorkflow@U2@@SA?BVDescriptor@3@XZ 10015710     ngs_reads_classification:ngs_reads_classification.dll
 0002:00000714       __imp_?TAXONOMY_CLASSIFICATION_SLOT_ID@TaxonomySupport@LocalWorkflow@U2@@2VQString@@B 10015714     ngs_reads_classification:ngs_reads_classification.dll
 0002:00000718       __imp_?countClassified@NgsReadsClassificationUtils@U2@@SAHABV?$QMap@VQString@@I@@@Z 10015718     ngs_reads_classification:ngs_reads_classification.dll
 0002:0000071c       __imp_?TAXON_NAMES_ITEM_ID@NgsReadsClassificationPlugin@U2@@2VQString@@B 1001571c     ngs_reads_classification:ngs_reads_classification.dll
 0002:00000720       __imp_?TAXON_NODES_ITEM_ID@NgsReadsClassificationPlugin@U2@@2VQString@@B 10015720     ngs_reads_classification:ngs_reads_classification.dll
 0002:00000724       __imp_?TAXONOMY_DATA_ID@NgsReadsClassificationPlugin@U2@@2VQString@@B 10015724     ngs_reads_classification:ngs_reads_classification.dll
 0002:00000728       \177ngs_reads_classification_NULL_THUNK_DATA 10015728     ngs_reads_classification:ngs_reads_classification.dll
 0002:0000072c       ___xc_a                    1001572c     MSVCRT:cinitexe.obj
 0002:000008fc       ___xc_z                    100158fc     MSVCRT:cinitexe.obj
 0002:00000900       ___xi_a                    10015900     MSVCRT:cinitexe.obj
 0002:0000090c       ___xi_z                    1001590c     MSVCRT:cinitexe.obj
 0002:00000948       ?BUFFER_SIZE@PrepareWevoteTaxonomyDataTask@U2@@0_JB 10015948     PrepareWevoteTaxonomyDataTask.obj
 0002:00000954       ??_7error_category@std@@6B@ 10015954     PrepareWevoteTaxonomyDataTask.obj
 0002:00000970       ??_7_Generic_error_category@std@@6B@ 10015970     PrepareWevoteTaxonomyDataTask.obj
 0002:00000988       ??_C@_07DCLBNMLN@generic?$AA@ 10015988     PrepareWevoteTaxonomyDataTask.obj
 0002:00000990       ??_C@_0O@BFJCFAAK@unknown?5error?$AA@ 10015990     PrepareWevoteTaxonomyDataTask.obj
 0002:000009a4       ??_7_Iostream_error_category@std@@6B@ 100159a4     PrepareWevoteTaxonomyDataTask.obj
 0002:000009bc       ??_C@_08LLGCOLLL@iostream?$AA@ 100159bc     PrepareWevoteTaxonomyDataTask.obj
 0002:000009c8       ??_C@_0BG@PADBLCHM@iostream?5stream?5error?$AA@ 100159c8     PrepareWevoteTaxonomyDataTask.obj
 0002:000009e4       ??_7_System_error_category@std@@6B@ 100159e4     PrepareWevoteTaxonomyDataTask.obj
 0002:000009fc       ??_C@_06FHFOAHML@system?$AA@ 100159fc     PrepareWevoteTaxonomyDataTask.obj
 0002:00000a04       ??_C@_0L@JLHNEGIN@Algorithms?$AA@ 10015a04     PrepareWevoteTaxonomyDataTask.obj
 0002:00000a10       ??_C@_07PGLPGHFC@Console?$AA@ 10015a10     PrepareWevoteTaxonomyDataTask.obj
 0002:00000a18       ??_C@_0O@BOFHOPCF@Core?5Services?$AA@ 10015a18     PrepareWevoteTaxonomyDataTask.obj
 0002:00000a28       ??_C@_0N@PPADAKBM@Input?1Output?$AA@ 10015a28     PrepareWevoteTaxonomyDataTask.obj
 0002:00000a38       ??_C@_0M@KPPBKPKK@Performance?$AA@ 10015a38     PrepareWevoteTaxonomyDataTask.obj
 0002:00000a44       ??_C@_07BFDHHBBI@Scripts?$AA@ 10015a44     PrepareWevoteTaxonomyDataTask.obj
 0002:00000a4c       ??_C@_05EEGKELMG@Tasks?$AA@ 10015a4c     PrepareWevoteTaxonomyDataTask.obj
 0002:00000a54       ??_C@_0P@NIIOBHGA@User?5Interface?$AA@ 10015a54     PrepareWevoteTaxonomyDataTask.obj
 0002:00000a64       ??_C@_0N@JINCGGMN@User?5Actions?$AA@ 10015a64     PrepareWevoteTaxonomyDataTask.obj
 0002:00000a78       ??_7PrepareWevoteTaxonomyDataTask@U2@@6B@ 10015a78     PrepareWevoteTaxonomyDataTask.obj
 0002:00000b04       ??_C@_0BA@FJACALII@wevote_taxonomy?$AA@ 10015b04     PrepareWevoteTaxonomyDataTask.obj
 0002:00000b14       ??_C@_0BB@LFKJGFPN@nodes_wevote?4dmp?$AA@ 10015b14     PrepareWevoteTaxonomyDataTask.obj
 0002:00000b28       ??_C@_0BB@ODFJIEDJ@names_wevote?4dmp?$AA@ 10015b28     PrepareWevoteTaxonomyDataTask.obj
 0002:00000b3c       ??_C@_0BA@HPNCAFBN@scientific_name?$AA@ 10015b3c     PrepareWevoteTaxonomyDataTask.obj
 0002:00000b4c       ??_C@_0CB@DOOLNHNJ@Prepare?5taxonomy?5data?5for?5WEVOTE@ 10015b4c     PrepareWevoteTaxonomyDataTask.obj
 0002:00000b70       ??_C@_0BL@PLINAGHB@U2DataPathRegistry?5is?5NULL?$AA@ 10015b70     PrepareWevoteTaxonomyDataTask.obj
 0002:00000b8c       ??_C@_0CF@OJBLMLIA@Taxonomy?5data?5path?5is?5not?5regist@ 10015b8c     PrepareWevoteTaxonomyDataTask.obj
 0002:00000bb4       ??_C@_0BJ@IAIMAPKP@Taxonomy?5data?5are?5missed?$AA@ 10015bb4     PrepareWevoteTaxonomyDataTask.obj
 0002:00000bd0       ??_C@_0CB@KKHCKIIB@Taxonomy?5file?5?8?$CF1?8?5is?5not?5found?4@ 10015bd0     PrepareWevoteTaxonomyDataTask.obj
 0002:00000bf4       ??_C@_01KMDKNFGN@?1?$AA@   10015bf4     PrepareWevoteTaxonomyDataTask.obj
 0002:00000bf8       ??_C@_0CO@CADDANN@WEVOTE?5taxonomy?5is?5out?5of?5date?0?5@ 10015bf8     PrepareWevoteTaxonomyDataTask.obj
 0002:00000c28       ??_C@_0CE@PDGMMBOP@WEVOTE?5taxonomy?5is?5up?5to?5date?0?5s@ 10015c28     PrepareWevoteTaxonomyDataTask.obj
 0002:00000c4c       ??_C@_0BA@JFNIOLAK@string?5too?5long?$AA@ 10015c4c     PrepareWevoteTaxonomyDataTask.obj
 0002:00000c5c       ??_C@_0BI@CFPLBAOH@invalid?5string?5position?$AA@ 10015c5c     PrepareWevoteTaxonomyDataTask.obj
 0002:00000c78       ??_7?$PrompterBase@VWevotePrompter@LocalWorkflow@U2@@@U2@@6BActorDocument@Workflow@1@@ 10015c78     WevotePrompter.obj
 0002:00000cc0       ??_7?$PrompterBase@VWevotePrompter@LocalWorkflow@U2@@@U2@@6BPrompter@Workflow@1@@ 10015cc0     WevotePrompter.obj
 0002:00000ccc       ??_7WevotePrompter@LocalWorkflow@U2@@6BActorDocument@Workflow@2@@ 10015ccc     WevotePrompter.obj
 0002:00000d14       ??_7WevotePrompter@LocalWorkflow@U2@@6BPrompter@Workflow@2@@ 10015d14     WevotePrompter.obj
 0002:00000d1c       ??_C@_0DH@DNIPLCEA@Ensemble?5classification?5data?0?5pr@ 10015d1c     WevotePrompter.obj
 0002:00000d54       ??_C@_0BE@LGBLLFOL@1sl_actorModified?$CI?$CJ?$AA@ 10015d54     WevotePrompter.obj
 0002:00000d68       ??_C@_0BD@FGIDJNMI@2si_labelChanged?$CI?$CJ?$AA@ 10015d68     WevotePrompter.obj
 0002:00000d7c       ??_C@_0P@DIBOLHGA@2si_modified?$CI?$CJ?$AA@ 10015d7c     WevotePrompter.obj
 0002:00000d8c       ??_C@_0BC@HBGBGNIM@2bindingChanged?$CI?$CJ?$AA@ 10015d8c     WevotePrompter.obj
 0002:00000d9e       ??_C@_00CNPNBAHC@?$AA@     10015d9e     WevoteSupport.obj
 0002:00000da4       ??_7WevoteSupport@U2@@6B@  10015da4     WevoteSupport.obj
 0002:00000de0       ??_C@_06EJOLCDEL@WEVOTE?$AA@ 10015de0     WevoteSupport.obj
 0002:00000de8       ??_C@_0DB@GGOGAIJG@less?5than?5the?5required?5minimum?5n@ 10015de8     WevoteSupport.obj
 0002:00000e20       ??_C@_0OF@ONBNCCP@WEVOTE?5?$CIWEighted?5VOting?5Taxonomi@ 10015e20     WevoteSupport.obj
 0002:00000f0c       ??_7WevoteSupportPlugin@U2@@6B@ 10015f0c     WevoteSupportPlugin.obj
 0002:00000f38       ??_C@_0BN@IJKOJBDC@WEVOTE?5external?5tool?5support?$AA@ 10015f38     WevoteSupportPlugin.obj
 0002:00000f58       ??_C@_0LI@PBEHHIDD@The?5plugin?5supports?5WEVOTE?5?$CIWEig@ 10015f58     WevoteSupportPlugin.obj
 0002:00001014       ??_SExternalToolRunTask@U2@@6B@ 10016014     WevoteTask.obj
 0002:000010a4       ??_SExternalToolLogParser@U2@@6B@ 100160a4     WevoteTask.obj
 0002:000010f0       ??_7WevoteTask@U2@@6B@     100160f0     WevoteTask.obj
 0002:00001184       ??_C@_0BE@JCHPLFGM@_WEVOTE_Details?4txt?$AA@ 10016184     WevoteTask.obj
 0002:00001198       ??_C@_0CD@KLPEDMB@Improve?5classification?5with?5WEVO@ 10016198     WevoteTask.obj
 0002:000011bc       ??_C@_0BN@HEGKFALG@Wevote?5output?5file?5not?5found?$AA@ 100161bc     WevoteTask.obj
 0002:000011dc       ??_C@_0BO@OJHFJEMB@Penalty?5is?5less?5or?5equal?5zero?$AA@ 100161dc     WevoteTask.obj
 0002:000011fc       ??_C@_0CJ@BIMJOOED@Number?5of?5agreed?5tools?5is?5less?5t@ 100161fc     WevoteTask.obj
 0002:00001228       ??_C@_0CC@PBJDDAMD@Score?5threshold?5is?5less?5than?5zer@ 10016228     WevoteTask.obj
 0002:0000124c       ??_C@_0CI@IAMHNDCE@Number?5of?5threads?5is?5less?5or?5equ@ 1001624c     WevoteTask.obj
 0002:00001274       ??_C@_0BI@EGEGNHIN@Input?5file?5URL?5is?5empty?$AA@ 10016274     WevoteTask.obj
 0002:0000128c       ??_C@_0BJ@IDNFNCOB@Output?5file?5URL?5is?5empty?$AA@ 1001628c     WevoteTask.obj
 0002:000012a8       ??_C@_02EJEOCNCO@?9v?$AA@  100162a8     WevoteTask.obj
 0002:000012ac       ??_C@_02IEBECDLA@?9i?$AA@  100162ac     WevoteTask.obj
 0002:000012b0       ??_C@_02BPBEIKKI@?9p?$AA@  100162b0     WevoteTask.obj
 0002:000012b4       ??_C@_0BM@KJBJPMBF@prepareTaxonomyTask?5is?5NULL?$AA@ 100162b4     WevoteTask.obj
 0002:000012d0       ??_C@_0CI@FEGHGDKD@Can?8t?5find?5prepared?5taxonomy?5for@ 100162d0     WevoteTask.obj
 0002:000012f8       ??_C@_02DBLKFNPN@?9d?$AA@  100162f8     WevoteTask.obj
 0002:000012fc       ??_C@_02DEDJNJGL@?9s?$AA@  100162fc     WevoteTask.obj
 0002:00001300       ??_C@_02MLFFLFHH@?9n?$AA@  10016300     WevoteTask.obj
 0002:00001304       ??_C@_02LGCCEBDC@?9k?$AA@  10016304     WevoteTask.obj
 0002:00001308       ??_C@_02EMMNKJLI@?9a?$AA@  10016308     WevoteTask.obj
 0002:0000130c       ??_C@_0BO@JILOKKKC@Can?8t?5overwrite?5the?5file?5?$CC?$CF1?$CC?$AA@ 1001630c     WevoteTask.obj
 0002:0000132c       ??_C@_0CE@CAAPBGLM@Too?5few?5columns?5in?5the?5result?5fi@ 1001632c     WevoteTask.obj
 0002:00001350       ??_C@_0BM@DPIFFBP@Can?8t?5parse?5the?5taxID?3?5?$CC?$CF1?$CC?$AA@ 10016350     WevoteTask.obj
 0002:0000136c       ??_C@_0BA@IBCMGEID@WevoteValidator?$AA@ 1001636c     WevoteValidator.obj
 0002:0000137c       ??_C@_0DK@FGLPPHNF@Taxonomy?5classification?5data?5fro@ 1001637c     WevoteValidator.obj
 0002:000013b8       ??_C@_0EL@ENMJCHGK@Taxonomy?5classification?5data?5fro@ 100163b8     WevoteValidator.obj
 0002:00001404       ??_C@_0CM@ICPJCNAJ@QtMetaTypePrivate?3?3QAssociativeI@ 10016404     WevoteWorker.obj
 0002:00001434       ??_SFailTask@U2@@6B@       10016434     WevoteWorker.obj
 0002:000014c4       ??_STaskSignalMapper@U2@@6B@ 100164c4     WevoteWorker.obj
 0002:000014f4       ??_SDescriptor@U2@@6B@     100164f4     WevoteWorker.obj
 0002:000014f8       ??_C@_0BF@COKBMJP@Script?5task?5canceled?$AA@ 100164f8     WevoteWorker.obj
 0002:00001510       ??_C@_0DA@ENPGIFBJ@U2?3?3LocalWorkflow?3?3TaxonomyClass@ 10016510     WevoteWorker.obj
 0002:00001544       ??_7WevoteWorker@LocalWorkflow@U2@@6BQObject@@@ 10016544     WevoteWorker.obj
 0002:00001588       ??_7WevoteWorker@LocalWorkflow@U2@@6BWorker@Workflow@2@@ 10016588     WevoteWorker.obj
 0002:000015a4       ??_7WevoteWorker@LocalWorkflow@U2@@6BCommunicationSubject@Workflow@2@@ 100165a4     WevoteWorker.obj
 0002:000015b0       ??_C@_06ENMAPNJJ@wevote?$AA@ 100165b0     WevoteWorker.obj
 0002:000015b8       ??_C@_0CK@IGBIANDN@Trying?5to?5recover?5from?5error?3?5?$CF1@ 100165b8     WevoteWorker.obj
 0002:000015e4       ??_C@_0BK@LMMJOEHE@Port?5with?5id?5?8?$CF1?8?5is?5NULL?$AA@ 100165e4     WevoteWorker.obj
 0002:00001600       ??_C@_0BF@CEJCJJJL@src?2WevoteWorker?4cpp?$AA@ 10016600     WevoteWorker.obj
 0002:00001618       ??_C@_0BJ@JJNIMNNJ@1sl_taskFinished?$CITask?5?$CK?$CJ?$AA@ 10016618     WevoteWorker.obj
 0002:00001634       ??_C@_0BJ@DHBKDAMN@2si_taskFinished?$CITask?5?$CK?$CJ?$AA@ 10016634     WevoteWorker.obj
 0002:00001650       ??_C@_0DF@GPCBDEIK@There?5were?5?$CF1?5input?5reads?0?5?$CF2?5re@ 10016650     WevoteWorker.obj
 0002:00001688       ??_C@_0CE@KJFNIPFG@Empty?5input?5file?5URL?5in?5the?5mess@ 10016688     WevoteWorker.obj
 0002:000016ac       ??_C@_01IDAFKMJL@_?$AA@    100166ac     WevoteWorker.obj
 0002:000016b4       ??_SMapDataType@U2@@6B@    100166b4     WevoteWorkerFactory.obj
 0002:000016cc       ??_SAttribute@U2@@6B@      100166cc     WevoteWorkerFactory.obj
 0002:000016fc       ??_SDelegateEditor@U2@@6B@ 100166fc     WevoteWorkerFactory.obj
 0002:00001754       ??_SURLDelegate@U2@@6B@    10016754     WevoteWorkerFactory.obj
 0002:000017d4       ??_SSpinBoxDelegate@U2@@6B@ 100167d4     WevoteWorkerFactory.obj
 0002:00001854       ??_SPortDescriptor@Workflow@U2@@6B@ 10016854     WevoteWorkerFactory.obj
 0002:00001864       ??_SIntegralBusActorPrototype@Workflow@U2@@6B@ 10016864     WevoteWorkerFactory.obj
 0002:00001878       ??_7WevoteValidator@Workflow@U2@@6B@ 10016878     WevoteWorkerFactory.obj
 0002:00001888       ??_7WevoteWorkerFactory@LocalWorkflow@U2@@6B?$IdRegistry@VDomainFactory@Workflow@U2@@@2@@ 10016888     WevoteWorkerFactory.obj
 0002:000018b4       ??_7WevoteWorkerFactory@LocalWorkflow@U2@@6BDescriptor@2@@ 100168b4     WevoteWorkerFactory.obj
 0002:000018b8       ??_C@_0BA@MPAGJMLH@wevote?9classify?$AA@ 100168b8     WevoteWorkerFactory.obj
 0002:000018c8       ??_C@_02LMMGJAGL@in?$AA@   100168c8     WevoteWorkerFactory.obj
 0002:000018cc       ??_C@_03KEJHNBPP@out?$AA@  100168cc     WevoteWorkerFactory.obj
 0002:000018d0       ??_C@_07KFFKKIBL@penalty?$AA@ 100168d0     WevoteWorkerFactory.obj
 0002:000018d8       ??_C@_0BH@LOJDFJGI@number?9of?9agreed?9tools?$AA@ 100168d8     WevoteWorkerFactory.obj
 0002:000018f0       ??_C@_0BA@GDLOHMKD@score?9threshold?$AA@ 100168f0     WevoteWorkerFactory.obj
 0002:00001900       ??_C@_07NFPADACG@threads?$AA@ 10016900     WevoteWorkerFactory.obj
 0002:00001908       ??_C@_0L@JDEFPCKN@output?9url?$AA@ 10016908     WevoteWorkerFactory.obj
 0002:00001914       ??_C@_0L@BOLLAKIP@Input?5URL?4?$AA@ 10016914     WevoteWorkerFactory.obj
 0002:00001920       ??_C@_09GGCOOKFN@Input?5URL?$AA@ 10016920     WevoteWorkerFactory.obj
 0002:00001930       ??_C@_0IA@HFCJFPBD@Input?5a?5CSV?5file?5in?5the?5followin@ 10016930     WevoteWorkerFactory.obj
 0002:000019b0       ??_C@_0BO@FDCLPIAJ@Input?5classification?5CSV?5file?$AA@ 100169b0     WevoteWorkerFactory.obj
 0002:000019d0       ??_C@_0DK@BEDFJFHJ@A?5map?5of?5sequence?5names?5with?5the@ 100169d0     WevoteWorkerFactory.obj
 0002:00001a0c       ??_C@_0BG@IKCAIPGK@WEVOTE?5Classification?$AA@ 10016a0c     WevoteWorkerFactory.obj
 0002:00001a24       ??_C@_03DAJLOBIG@?9in?$AA@ 10016a24     WevoteWorkerFactory.obj
 0002:00001a28       ??_C@_04HKKABCEL@?9out?$AA@ 10016a28     WevoteWorkerFactory.obj
 0002:00001a30       ??_C@_0CF@FBBOPKLM@Score?5penalty?5for?5disagreements?5@ 10016a30     WevoteWorkerFactory.obj
 0002:00001a58       ??_C@_07FMCMMKEN@Penalty?$AA@ 10016a58     WevoteWorkerFactory.obj
 0002:00001a60       ??_C@_0EE@JPEGDLGA@Specify?5the?5minimum?5number?5of?5to@ 10016a60     WevoteWorkerFactory.obj
 0002:00001aa4       ??_C@_0BH@HIOFOHHJ@Number?5of?5agreed?5tools?$AA@ 10016aa4     WevoteWorkerFactory.obj
 0002:00001abc       ??_C@_0BF@LPEICJGP@Score?5threshold?5?$CI?9s?$CJ?$AA@ 10016abc     WevoteWorkerFactory.obj
 0002:00001ad4       ??_C@_0BA@LPBFEKNJ@Score?5threshold?$AA@ 10016ad4     WevoteWorkerFactory.obj
 0002:00001ae4       ??_C@_0BL@LPCPNDGI@Use?5multiple?5threads?5?$CI?9n?$CJ?4?$AA@ 10016ae4     WevoteWorkerFactory.obj
 0002:00001b00       ??_C@_0BC@GJADDMKB@Number?5of?5threads?$AA@ 10016b00     WevoteWorkerFactory.obj
 0002:00001b14       ??_C@_0CD@JJEBAIHM@Specify?5the?5output?5text?5file?5nam@ 10016b14     WevoteWorkerFactory.obj
 0002:00001b38       ??_C@_0M@LEIJPAKP@Output?5file?$AA@ 10016b38     WevoteWorkerFactory.obj
 0002:00001b44       ??_C@_0CA@BBFPBJKD@Classify?5tool?4?5Hidden?5attribute?$AA@ 10016b44     WevoteWorkerFactory.obj
 0002:00001b64       ??_C@_07CCOEHHFD@minimum?$AA@ 10016b64     WevoteWorkerFactory.obj
 0002:00001b6c       ??_C@_07MEIENILC@maximum?$AA@ 10016b6c     WevoteWorkerFactory.obj
 0002:00001b74       ??_C@_04LBDCJOFB@Auto?$AA@ 10016b74     WevoteWorkerFactory.obj
 0002:00001b7c       ??_C@_03GBOLEDH@?4gz?$AA@  10016b7c     WevoteWorkerFactory.obj
 0002:00001b80       ??_C@_0BD@KCKLELAE@wevote?1output_file?$AA@ 10016b80     WevoteWorkerFactory.obj
 0002:00001b98       ??_C@_0LH@CPMLMFPD@WEVOTE?5?$CIWEighted?5VOting?5Taxonomi@ 10016b98     WevoteWorkerFactory.obj
 0002:00001c50       ??_C@_0CD@LGFGBFGL@Improve?5Classification?5with?5WEVO@ 10016c50     WevoteWorkerFactory.obj
 0002:00001e94       ?value@?$integral_constant@_N$0A@@std@@2_NB 10016e94     MSVCRT:ti_inst.obj
 0002:00001e95       ?value@?$integral_constant@_N$00@std@@2_NB 10016e95     MSVCRT:ti_inst.obj
 0002:00001e9c       ??_7type_info@@6B@         10016e9c     MSVCRT:ti_inst.obj
 0002:00001ea0       __pDefaultRawDllMain       10016ea0     MSVCRT:crtdll.obj
 0002:00001ea0       __pRawDllMain              10016ea0     MSVCRT:crtdll.obj
 0002:00001eac       ?ProcessDetach@NativeDll@<CrtImplementationDetails>@@0IB 10016eac     MSVCRT:initsect.obj
 0002:00001eb0       ?ProcessAttach@NativeDll@<CrtImplementationDetails>@@0IB 10016eb0     MSVCRT:initsect.obj
 0002:00001eb4       ?ThreadAttach@NativeDll@<CrtImplementationDetails>@@0IB 10016eb4     MSVCRT:initsect.obj
 0002:00001eb8       ?ThreadDetach@NativeDll@<CrtImplementationDetails>@@0IB 10016eb8     MSVCRT:initsect.obj
 0002:00001ebc       ?ProcessVerifier@NativeDll@<CrtImplementationDetails>@@0IB 10016ebc     MSVCRT:initsect.obj
 0002:00001ec0       __load_config_used         10016ec0     MSVCRT:loadcfg.obj
 0002:00001f7c       ??_R4error_category@std@@6B@ 10016f7c     PrepareWevoteTaxonomyDataTask.obj
 0002:00001f90       ??_R3error_category@std@@8 10016f90     PrepareWevoteTaxonomyDataTask.obj
 0002:00001fa0       ??_R2error_category@std@@8 10016fa0     PrepareWevoteTaxonomyDataTask.obj
 0002:00001fa8       ??_R1A@?0A@EA@error_category@std@@8 10016fa8     PrepareWevoteTaxonomyDataTask.obj
 0002:00001fc4       ??_R4_Generic_error_category@std@@6B@ 10016fc4     PrepareWevoteTaxonomyDataTask.obj
 0002:00001fd8       ??_R3_Generic_error_category@std@@8 10016fd8     PrepareWevoteTaxonomyDataTask.obj
 0002:00001fe8       ??_R2_Generic_error_category@std@@8 10016fe8     PrepareWevoteTaxonomyDataTask.obj
 0002:00001ff4       ??_R1A@?0A@EA@_Generic_error_category@std@@8 10016ff4     PrepareWevoteTaxonomyDataTask.obj
 0002:00002010       ??_R4_Iostream_error_category@std@@6B@ 10017010     PrepareWevoteTaxonomyDataTask.obj
 0002:00002024       ??_R3_Iostream_error_category@std@@8 10017024     PrepareWevoteTaxonomyDataTask.obj
 0002:00002034       ??_R2_Iostream_error_category@std@@8 10017034     PrepareWevoteTaxonomyDataTask.obj
 0002:00002044       ??_R1A@?0A@EA@_Iostream_error_category@std@@8 10017044     PrepareWevoteTaxonomyDataTask.obj
 0002:00002060       ??_R4_System_error_category@std@@6B@ 10017060     PrepareWevoteTaxonomyDataTask.obj
 0002:00002074       ??_R3_System_error_category@std@@8 10017074     PrepareWevoteTaxonomyDataTask.obj
 0002:00002084       ??_R2_System_error_category@std@@8 10017084     PrepareWevoteTaxonomyDataTask.obj
 0002:00002094       ??_R1A@?0A@EA@_System_error_category@std@@8 10017094     PrepareWevoteTaxonomyDataTask.obj
 0002:000020b0       ??_R4PrepareWevoteTaxonomyDataTask@U2@@6B@ 100170b0     PrepareWevoteTaxonomyDataTask.obj
 0002:000020c4       ??_R3PrepareWevoteTaxonomyDataTask@U2@@8 100170c4     PrepareWevoteTaxonomyDataTask.obj
 0002:000020d4       ??_R2PrepareWevoteTaxonomyDataTask@U2@@8 100170d4     PrepareWevoteTaxonomyDataTask.obj
 0002:000020e4       ??_R1A@?0A@EA@PrepareWevoteTaxonomyDataTask@U2@@8 100170e4     PrepareWevoteTaxonomyDataTask.obj
 0002:00002100       ??_R1A@?0A@EA@Task@U2@@8   10017100     PrepareWevoteTaxonomyDataTask.obj
 0002:0000211c       ??_R3Task@U2@@8            1001711c     PrepareWevoteTaxonomyDataTask.obj
 0002:0000212c       ??_R2Task@U2@@8            1001712c     PrepareWevoteTaxonomyDataTask.obj
 0002:00002138       ??_R1A@?0A@EA@QObject@@8   10017138     PrepareWevoteTaxonomyDataTask.obj
 0002:00002154       ??_R3QObject@@8            10017154     PrepareWevoteTaxonomyDataTask.obj
 0002:00002164       ??_R2QObject@@8            10017164     PrepareWevoteTaxonomyDataTask.obj
 0002:0000216c       ??_R4WevotePrompter@LocalWorkflow@U2@@6BActorDocument@Workflow@2@@ 1001716c     WevotePrompter.obj
 0002:00002180       ??_R3WevotePrompter@LocalWorkflow@U2@@8 10017180     WevotePrompter.obj
 0002:00002190       ??_R2WevotePrompter@LocalWorkflow@U2@@8 10017190     WevotePrompter.obj
 0002:000021b0       ??_R1A@?0A@EA@WevotePrompter@LocalWorkflow@U2@@8 100171b0     WevotePrompter.obj
 0002:000021cc       ??_R1A@?0A@EA@?$PrompterBase@VWevotePrompter@LocalWorkflow@U2@@@U2@@8 100171cc     WevotePrompter.obj
 0002:000021e8       ??_R3?$PrompterBase@VWevotePrompter@LocalWorkflow@U2@@@U2@@8 100171e8     WevotePrompter.obj
 0002:000021f8       ??_R2?$PrompterBase@VWevotePrompter@LocalWorkflow@U2@@@U2@@8 100171f8     WevotePrompter.obj
 0002:00002214       ??_R1A@?0A@EA@PrompterBaseImpl@U2@@8 10017214     WevotePrompter.obj
 0002:00002230       ??_R3PrompterBaseImpl@U2@@8 10017230     WevotePrompter.obj
 0002:00002240       ??_R2PrompterBaseImpl@U2@@8 10017240     WevotePrompter.obj
 0002:00002258       ??_R1A@?0A@EA@ActorDocument@Workflow@U2@@8 10017258     WevotePrompter.obj
 0002:00002274       ??_R3ActorDocument@Workflow@U2@@8 10017274     WevotePrompter.obj
 0002:00002284       ??_R2ActorDocument@Workflow@U2@@8 10017284     WevotePrompter.obj
 0002:00002294       ??_R1A@?0A@EA@QTextDocument@@8 10017294     WevotePrompter.obj
 0002:000022b0       ??_R3QTextDocument@@8      100172b0     WevotePrompter.obj
 0002:000022c0       ??_R2QTextDocument@@8      100172c0     WevotePrompter.obj
 0002:000022cc       ??_R1M@?0A@EA@Prompter@Workflow@U2@@8 100172cc     WevotePrompter.obj
 0002:000022e8       ??_R3Prompter@Workflow@U2@@8 100172e8     WevotePrompter.obj
 0002:000022f8       ??_R2Prompter@Workflow@U2@@8 100172f8     WevotePrompter.obj
 0002:00002300       ??_R1A@?0A@EA@Prompter@Workflow@U2@@8 10017300     WevotePrompter.obj
 0002:0000231c       ??_R4WevotePrompter@LocalWorkflow@U2@@6BPrompter@Workflow@2@@ 1001731c     WevotePrompter.obj
 0002:00002330       ??_R4?$PrompterBase@VWevotePrompter@LocalWorkflow@U2@@@U2@@6BActorDocument@Workflow@1@@ 10017330     WevotePrompter.obj
 0002:00002344       ??_R4?$PrompterBase@VWevotePrompter@LocalWorkflow@U2@@@U2@@6BPrompter@Workflow@1@@ 10017344     WevotePrompter.obj
 0002:00002358       ??_R4WevoteSupport@U2@@6B@ 10017358     WevoteSupport.obj
 0002:0000236c       ??_R3WevoteSupport@U2@@8   1001736c     WevoteSupport.obj
 0002:0000237c       ??_R2WevoteSupport@U2@@8   1001737c     WevoteSupport.obj
 0002:0000238c       ??_R1A@?0A@EA@WevoteSupport@U2@@8 1001738c     WevoteSupport.obj
 0002:000023a8       ??_R1A@?0A@EA@ExternalTool@U2@@8 100173a8     WevoteSupport.obj
 0002:000023c4       ??_R3ExternalTool@U2@@8    100173c4     WevoteSupport.obj
 0002:000023d4       ??_R2ExternalTool@U2@@8    100173d4     WevoteSupport.obj
 0002:000023e0       ??_R4WevoteSupportPlugin@U2@@6B@ 100173e0     WevoteSupportPlugin.obj
 0002:000023f4       ??_R3WevoteSupportPlugin@U2@@8 100173f4     WevoteSupportPlugin.obj
 0002:00002404       ??_R2WevoteSupportPlugin@U2@@8 10017404     WevoteSupportPlugin.obj
 0002:00002414       ??_R1A@?0A@EA@WevoteSupportPlugin@U2@@8 10017414     WevoteSupportPlugin.obj
 0002:00002430       ??_R1A@?0A@EA@Plugin@U2@@8 10017430     WevoteSupportPlugin.obj
 0002:0000244c       ??_R3Plugin@U2@@8          1001744c     WevoteSupportPlugin.obj
 0002:0000245c       ??_R2Plugin@U2@@8          1001745c     WevoteSupportPlugin.obj
 0002:00002468       ??_R4ExternalToolLogParser@U2@@6B@ 10017468     WevoteTask.obj
 0002:0000247c       ??_R3ExternalToolLogParser@U2@@8 1001747c     WevoteTask.obj
 0002:0000248c       ??_R2ExternalToolLogParser@U2@@8 1001748c     WevoteTask.obj
 0002:00002498       ??_R1A@?0A@EA@ExternalToolLogParser@U2@@8 10017498     WevoteTask.obj
 0002:000024b4       ??_R4ExternalToolRunTask@U2@@6B@ 100174b4     WevoteTask.obj
 0002:000024c8       ??_R3ExternalToolRunTask@U2@@8 100174c8     WevoteTask.obj
 0002:000024d8       ??_R2ExternalToolRunTask@U2@@8 100174d8     WevoteTask.obj
 0002:000024e8       ??_R1A@?0A@EA@ExternalToolRunTask@U2@@8 100174e8     WevoteTask.obj
 0002:00002504       ??_R4WevoteTask@U2@@6B@    10017504     WevoteTask.obj
 0002:00002518       ??_R3WevoteTask@U2@@8      10017518     WevoteTask.obj
 0002:00002528       ??_R2WevoteTask@U2@@8      10017528     WevoteTask.obj
 0002:0000253c       ??_R1A@?0A@EA@WevoteTask@U2@@8 1001753c     WevoteTask.obj
 0002:00002558       ??_R1A@?0A@EA@ExternalToolSupportTask@U2@@8 10017558     WevoteTask.obj
 0002:00002574       ??_R3ExternalToolSupportTask@U2@@8 10017574     WevoteTask.obj
 0002:00002584       ??_R2ExternalToolSupportTask@U2@@8 10017584     WevoteTask.obj
 0002:00002594       ??_R4FailTask@U2@@6B@      10017594     WevoteWorker.obj
 0002:000025a8       ??_R3FailTask@U2@@8        100175a8     WevoteWorker.obj
 0002:000025b8       ??_R2FailTask@U2@@8        100175b8     WevoteWorker.obj
 0002:000025c8       ??_R1A@?0A@EA@FailTask@U2@@8 100175c8     WevoteWorker.obj
 0002:000025e4       ??_R4TaskSignalMapper@U2@@6B@ 100175e4     WevoteWorker.obj
 0002:000025f8       ??_R3TaskSignalMapper@U2@@8 100175f8     WevoteWorker.obj
 0002:00002608       ??_R2TaskSignalMapper@U2@@8 10017608     WevoteWorker.obj
 0002:00002614       ??_R1A@?0A@EA@TaskSignalMapper@U2@@8 10017614     WevoteWorker.obj
 0002:00002630       ??_R4Descriptor@U2@@6B@    10017630     WevoteWorker.obj
 0002:00002644       ??_R3Descriptor@U2@@8      10017644     WevoteWorker.obj
 0002:00002654       ??_R2Descriptor@U2@@8      10017654     WevoteWorker.obj
 0002:0000265c       ??_R1A@?0A@EA@Descriptor@U2@@8 1001765c     WevoteWorker.obj
 0002:00002678       ??_R4WevoteWorker@LocalWorkflow@U2@@6BQObject@@@ 10017678     WevoteWorker.obj
 0002:0000268c       ??_R3WevoteWorker@LocalWorkflow@U2@@8 1001768c     WevoteWorker.obj
 0002:0000269c       ??_R2WevoteWorker@LocalWorkflow@U2@@8 1001769c     WevoteWorker.obj
 0002:000026b4       ??_R1A@?0A@EA@WevoteWorker@LocalWorkflow@U2@@8 100176b4     WevoteWorker.obj
 0002:000026d0       ??_R1A@?0A@EA@BaseWorker@LocalWorkflow@U2@@8 100176d0     WevoteWorker.obj
 0002:000026ec       ??_R3BaseWorker@LocalWorkflow@U2@@8 100176ec     WevoteWorker.obj
 0002:000026fc       ??_R2BaseWorker@LocalWorkflow@U2@@8 100176fc     WevoteWorker.obj
 0002:00002710       ??_R17?0A@EA@Worker@Workflow@U2@@8 10017710     WevoteWorker.obj
 0002:0000272c       ??_R3Worker@Workflow@U2@@8 1001772c     WevoteWorker.obj
 0002:0000273c       ??_R2Worker@Workflow@U2@@8 1001773c     WevoteWorker.obj
 0002:00002744       ??_R1A@?0A@EA@Worker@Workflow@U2@@8 10017744     WevoteWorker.obj
 0002:00002760       ??_R1BA@?0A@EA@CommunicationSubject@Workflow@U2@@8 10017760     WevoteWorker.obj
 0002:0000277c       ??_R3CommunicationSubject@Workflow@U2@@8 1001777c     WevoteWorker.obj
 0002:0000278c       ??_R2CommunicationSubject@Workflow@U2@@8 1001778c     WevoteWorker.obj
 0002:00002794       ??_R1A@?0A@EA@CommunicationSubject@Workflow@U2@@8 10017794     WevoteWorker.obj
 0002:000027b0       ??_R4WevoteWorker@LocalWorkflow@U2@@6BWorker@Workflow@2@@ 100177b0     WevoteWorker.obj
 0002:000027c4       ??_R4WevoteWorker@LocalWorkflow@U2@@6BCommunicationSubject@Workflow@2@@ 100177c4     WevoteWorker.obj
 0002:000027d8       ??_R4MapDataType@U2@@6B@   100177d8     WevoteWorkerFactory.obj
 0002:000027ec       ??_R3MapDataType@U2@@8     100177ec     WevoteWorkerFactory.obj
 0002:000027fc       ??_R2MapDataType@U2@@8     100177fc     WevoteWorkerFactory.obj
 0002:00002810       ??_R1A@?0A@EA@MapDataType@U2@@8 10017810     WevoteWorkerFactory.obj
 0002:0000282c       ??_R1A@?0A@EA@DataType@U2@@8 1001782c     WevoteWorkerFactory.obj
 0002:00002848       ??_R3DataType@U2@@8        10017848     WevoteWorkerFactory.obj
 0002:00002858       ??_R2DataType@U2@@8        10017858     WevoteWorkerFactory.obj
 0002:00002868       ??_R1BA@?0A@EA@QSharedData@@8 10017868     WevoteWorkerFactory.obj
 0002:00002884       ??_R3QSharedData@@8        10017884     WevoteWorkerFactory.obj
 0002:00002894       ??_R2QSharedData@@8        10017894     WevoteWorkerFactory.obj
 0002:0000289c       ??_R1A@?0A@EA@QSharedData@@8 1001789c     WevoteWorkerFactory.obj
 0002:000028b8       ??_R4Attribute@U2@@6B@     100178b8     WevoteWorkerFactory.obj
 0002:000028cc       ??_R3Attribute@U2@@8       100178cc     WevoteWorkerFactory.obj
 0002:000028dc       ??_R2Attribute@U2@@8       100178dc     WevoteWorkerFactory.obj
 0002:000028e8       ??_R1A@?0A@EA@Attribute@U2@@8 100178e8     WevoteWorkerFactory.obj
 0002:00002904       ??_R3ConfigurationEditor@U2@@8 10017904     WevoteWorkerFactory.obj
 0002:00002914       ??_R2ConfigurationEditor@U2@@8 10017914     WevoteWorkerFactory.obj
 0002:00002920       ??_R1A@?0A@EA@ConfigurationEditor@U2@@8 10017920     WevoteWorkerFactory.obj
 0002:0000293c       ??_R4DelegateEditor@U2@@6B@ 1001793c     WevoteWorkerFactory.obj
 0002:00002950       ??_R3DelegateEditor@U2@@8  10017950     WevoteWorkerFactory.obj
 0002:00002960       ??_R2DelegateEditor@U2@@8  10017960     WevoteWorkerFactory.obj
 0002:00002970       ??_R1A@?0A@EA@DelegateEditor@U2@@8 10017970     WevoteWorkerFactory.obj
 0002:0000298c       ??_R4URLDelegate@U2@@6B@   1001798c     WevoteWorkerFactory.obj
 0002:000029a0       ??_R3URLDelegate@U2@@8     100179a0     WevoteWorkerFactory.obj
 0002:000029b0       ??_R2URLDelegate@U2@@8     100179b0     WevoteWorkerFactory.obj
 0002:000029c8       ??_R1A@?0A@EA@URLDelegate@U2@@8 100179c8     WevoteWorkerFactory.obj
 0002:000029e4       ??_R1A@?0A@EA@PropertyDelegate@U2@@8 100179e4     WevoteWorkerFactory.obj
 0002:00002a00       ??_R3PropertyDelegate@U2@@8 10017a00     WevoteWorkerFactory.obj
 0002:00002a10       ??_R2PropertyDelegate@U2@@8 10017a10     WevoteWorkerFactory.obj
 0002:00002a24       ??_R1A@?0A@EA@QItemDelegate@@8 10017a24     WevoteWorkerFactory.obj
 0002:00002a40       ??_R3QItemDelegate@@8      10017a40     WevoteWorkerFactory.obj
 0002:00002a50       ??_R2QItemDelegate@@8      10017a50     WevoteWorkerFactory.obj
 0002:00002a60       ??_R1A@?0A@EA@QAbstractItemDelegate@@8 10017a60     WevoteWorkerFactory.obj
 0002:00002a7c       ??_R3QAbstractItemDelegate@@8 10017a7c     WevoteWorkerFactory.obj
 0002:00002a8c       ??_R2QAbstractItemDelegate@@8 10017a8c     WevoteWorkerFactory.obj
 0002:00002a98       ??_R4SpinBoxDelegate@U2@@6B@ 10017a98     WevoteWorkerFactory.obj
 0002:00002aac       ??_R3SpinBoxDelegate@U2@@8 10017aac     WevoteWorkerFactory.obj
 0002:00002abc       ??_R2SpinBoxDelegate@U2@@8 10017abc     WevoteWorkerFactory.obj
 0002:00002ad4       ??_R1A@?0A@EA@SpinBoxDelegate@U2@@8 10017ad4     WevoteWorkerFactory.obj
 0002:00002af0       ??_R4PortDescriptor@Workflow@U2@@6B@ 10017af0     WevoteWorkerFactory.obj
 0002:00002b04       ??_R3PortDescriptor@Workflow@U2@@8 10017b04     WevoteWorkerFactory.obj
 0002:00002b14       ??_R2PortDescriptor@Workflow@U2@@8 10017b14     WevoteWorkerFactory.obj
 0002:00002b20       ??_R1A@?0A@EA@PortDescriptor@Workflow@U2@@8 10017b20     WevoteWorkerFactory.obj
 0002:00002b3c       ??_R17?0A@EA@Descriptor@U2@@8 10017b3c     WevoteWorkerFactory.obj
 0002:00002b58       ??_R4IntegralBusActorPrototype@Workflow@U2@@6B@ 10017b58     WevoteWorkerFactory.obj
 0002:00002b6c       ??_R3IntegralBusActorPrototype@Workflow@U2@@8 10017b6c     WevoteWorkerFactory.obj
 0002:00002b7c       ??_R2IntegralBusActorPrototype@Workflow@U2@@8 10017b7c     WevoteWorkerFactory.obj
 0002:00002b90       ??_R1A@?0A@EA@IntegralBusActorPrototype@Workflow@U2@@8 10017b90     WevoteWorkerFactory.obj
 0002:00002bac       ??_R1A@?0A@EA@ActorPrototype@Workflow@U2@@8 10017bac     WevoteWorkerFactory.obj
 0002:00002bc8       ??_R3ActorPrototype@Workflow@U2@@8 10017bc8     WevoteWorkerFactory.obj
 0002:00002bd8       ??_R2ActorPrototype@Workflow@U2@@8 10017bd8     WevoteWorkerFactory.obj
 0002:00002be8       ??_R1A@?0A@EA@VisualDescriptor@U2@@8 10017be8     WevoteWorkerFactory.obj
 0002:00002c04       ??_R3VisualDescriptor@U2@@8 10017c04     WevoteWorkerFactory.obj
 0002:00002c14       ??_R2VisualDescriptor@U2@@8 10017c14     WevoteWorkerFactory.obj
 0002:00002c20       ??_R4WevoteValidator@Workflow@U2@@6B@ 10017c20     WevoteWorkerFactory.obj
 0002:00002c34       ??_R3WevoteValidator@Workflow@U2@@8 10017c34     WevoteWorkerFactory.obj
 0002:00002c44       ??_R2WevoteValidator@Workflow@U2@@8 10017c44     WevoteWorkerFactory.obj
 0002:00002c54       ??_R1A@?0A@EA@WevoteValidator@Workflow@U2@@8 10017c54     WevoteWorkerFactory.obj
 0002:00002c70       ??_R1A@?0A@EA@ActorValidator@Workflow@U2@@8 10017c70     WevoteWorkerFactory.obj
 0002:00002c8c       ??_R3ActorValidator@Workflow@U2@@8 10017c8c     WevoteWorkerFactory.obj
 0002:00002c9c       ??_R2ActorValidator@Workflow@U2@@8 10017c9c     WevoteWorkerFactory.obj
 0002:00002ca8       ??_R1A@?0A@EA@ConfigurationValidator@U2@@8 10017ca8     WevoteWorkerFactory.obj
 0002:00002cc4       ??_R3ConfigurationValidator@U2@@8 10017cc4     WevoteWorkerFactory.obj
 0002:00002cd4       ??_R2ConfigurationValidator@U2@@8 10017cd4     WevoteWorkerFactory.obj
 0002:00002cdc       ??_R4WevoteWorkerFactory@LocalWorkflow@U2@@6B?$IdRegistry@VDomainFactory@Workflow@U2@@@2@@ 10017cdc     WevoteWorkerFactory.obj
 0002:00002cf0       ??_R3WevoteWorkerFactory@LocalWorkflow@U2@@8 10017cf0     WevoteWorkerFactory.obj
 0002:00002d00       ??_R2WevoteWorkerFactory@LocalWorkflow@U2@@8 10017d00     WevoteWorkerFactory.obj
 0002:00002d14       ??_R1A@?0A@EA@WevoteWorkerFactory@LocalWorkflow@U2@@8 10017d14     WevoteWorkerFactory.obj
 0002:00002d30       ??_R1A@?0A@EA@DomainFactory@Workflow@U2@@8 10017d30     WevoteWorkerFactory.obj
 0002:00002d4c       ??_R3DomainFactory@Workflow@U2@@8 10017d4c     WevoteWorkerFactory.obj
 0002:00002d5c       ??_R2DomainFactory@Workflow@U2@@8 10017d5c     WevoteWorkerFactory.obj
 0002:00002d6c       ??_R1A@?0A@EA@?$IdRegistry@VDomainFactory@Workflow@U2@@@U2@@8 10017d6c     WevoteWorkerFactory.obj
 0002:00002d88       ??_R3?$IdRegistry@VDomainFactory@Workflow@U2@@@U2@@8 10017d88     WevoteWorkerFactory.obj
 0002:00002d98       ??_R2?$IdRegistry@VDomainFactory@Workflow@U2@@@U2@@8 10017d98     WevoteWorkerFactory.obj
 0002:00002da0       ??_R4WevoteWorkerFactory@LocalWorkflow@U2@@6BDescriptor@2@@ 10017da0     WevoteWorkerFactory.obj
 0002:00002db4       ??_R4type_info@@6B@        10017db4     MSVCRT:ti_inst.obj
 0002:00002dc8       ??_R3type_info@@8          10017dc8     MSVCRT:ti_inst.obj
 0002:00002dd8       ??_R2type_info@@8          10017dd8     MSVCRT:ti_inst.obj
 0002:00002de0       ??_R1A@?0A@EA@type_info@@8 10017de0     MSVCRT:ti_inst.obj
 0002:00002e00       ___safe_se_handler_table   10017e00     <linker-defined>
 0002:000030a4       ___rtc_iaa                 100180a4     MSVCRT:initsect.obj
 0002:000030a8       ___rtc_izz                 100180a8     MSVCRT:initsect.obj
 0002:000030ac       ___rtc_taa                 100180ac     MSVCRT:initsect.obj
 0002:000030b0       ___rtc_tzz                 100180b0     MSVCRT:initsect.obj
 0002:00006308       __IMPORT_DESCRIPTOR_ngs_reads_classification 1001b308     ngs_reads_classification:ngs_reads_classification.dll
 0002:0000631c       __IMPORT_DESCRIPTOR_U2Core 1001b31c     U2Core:U2Core.dll
 0002:00006330       __IMPORT_DESCRIPTOR_U2Formats 1001b330     U2Formats:U2Formats.dll
 0002:00006344       __IMPORT_DESCRIPTOR_U2Gui  1001b344     U2Gui:U2Gui.dll
 0002:00006358       __IMPORT_DESCRIPTOR_U2Lang 1001b358     U2Lang:U2Lang.dll
 0002:0000636c       __IMPORT_DESCRIPTOR_U2Designer 1001b36c     U2Designer:U2Designer.dll
 0002:00006380       __IMPORT_DESCRIPTOR_Qt5Widgets 1001b380     Qt5Widgets:Qt5Widgets.dll
 0002:00006394       __IMPORT_DESCRIPTOR_Qt5Gui 1001b394     Qt5Gui:Qt5Gui.dll
 0002:000063a8       __IMPORT_DESCRIPTOR_Qt5Script 1001b3a8     Qt5Script:Qt5Script.dll
 0002:000063bc       __IMPORT_DESCRIPTOR_Qt5Core 1001b3bc     Qt5Core:Qt5Core.dll
 0002:000063d0       __IMPORT_DESCRIPTOR_MSVCP120 1001b3d0     msvcprt:MSVCP120.dll
 0002:000063e4       __IMPORT_DESCRIPTOR_MSVCR120 1001b3e4     MSVCRT:MSVCR120.dll
 0002:000063f8       __IMPORT_DESCRIPTOR_KERNEL32 1001b3f8     kernel32:KERNEL32.dll
 0002:0000640c       __NULL_IMPORT_DESCRIPTOR   1001b40c     ngs_reads_classification:ngs_reads_classification.dll
 0003:00000000       ?_Generic_object@?$_Error_objects@H@std@@2V_Generic_error_category@2@A 10022000     PrepareWevoteTaxonomyDataTask.obj
 0003:00000004       ?_Iostream_object@?$_Error_objects@H@std@@2V_Iostream_error_category@2@A 10022004     PrepareWevoteTaxonomyDataTask.obj
 0003:00000008       ?_System_object@?$_Error_objects@H@std@@2V_System_error_category@2@A 10022008     PrepareWevoteTaxonomyDataTask.obj
 0003:0000000c       ?staticMetaObject@WevotePrompter@LocalWorkflow@U2@@2UQMetaObject@@B 1002200c     moc_WevotePrompter.obj
 0003:00000024       ?staticMetaObject@WevoteSupportPlugin@U2@@2UQMetaObject@@B 10022024     moc_WevoteSupportPlugin.obj
 0003:0000003c       ?staticMetaObject@WevoteTask@U2@@2UQMetaObject@@B 1002203c     moc_WevoteTask.obj
 0003:00000054       ?staticMetaObject@WevoteWorker@LocalWorkflow@U2@@2UQMetaObject@@B 10022054     moc_WevoteWorker.obj
 0003:0000006c       ___security_cookie         1002206c     MSVCRT:gs_cookie.obj
 0003:00000070       ___security_cookie_complement 10022070     MSVCRT:gs_cookie.obj
 0003:00000080       ___native_dllmain_reason   10022080     MSVCRT:natstart.obj
 0003:00000088       ??_R0?AVerror_category@std@@@8 10022088     PrepareWevoteTaxonomyDataTask.obj
 0003:000000ac       ??_R0?AV_Generic_error_category@std@@@8 100220ac     PrepareWevoteTaxonomyDataTask.obj
 0003:000000d8       ??_R0?AV_Iostream_error_category@std@@@8 100220d8     PrepareWevoteTaxonomyDataTask.obj
 0003:00000104       ??_R0?AV_System_error_category@std@@@8 10022104     PrepareWevoteTaxonomyDataTask.obj
 0003:00000130       ??_R0?AVPrepareWevoteTaxonomyDataTask@U2@@@8 10022130     PrepareWevoteTaxonomyDataTask.obj
 0003:00000160       ??_R0?AVTask@U2@@@8        10022160     PrepareWevoteTaxonomyDataTask.obj
 0003:00000178       ??_R0?AVQObject@@@8        10022178     PrepareWevoteTaxonomyDataTask.obj
 0003:00000190       ??_R0?AVWevotePrompter@LocalWorkflow@U2@@@8 10022190     WevotePrompter.obj
 0003:000001c0       ??_R0?AV?$PrompterBase@VWevotePrompter@LocalWorkflow@U2@@@U2@@@8 100221c0     WevotePrompter.obj
 0003:00000204       ??_R0?AVPrompterBaseImpl@U2@@@8 10022204     WevotePrompter.obj
 0003:00000228       ??_R0?AVActorDocument@Workflow@U2@@@8 10022228     WevotePrompter.obj
 0003:00000250       ??_R0?AVQTextDocument@@@8  10022250     WevotePrompter.obj
 0003:0000026c       ??_R0?AVPrompter@Workflow@U2@@@8 1002226c     WevotePrompter.obj
 0003:00000290       ??_R0?AVWevoteSupport@U2@@@8 10022290     WevoteSupport.obj
 0003:000002b0       ??_R0?AVExternalTool@U2@@@8 100222b0     WevoteSupport.obj
 0003:000002d0       ??_R0?AVWevoteSupportPlugin@U2@@@8 100222d0     WevoteSupportPlugin.obj
 0003:000002f8       ??_R0?AVPlugin@U2@@@8      100222f8     WevoteSupportPlugin.obj
 0003:00000310       ??_R0?AVExternalToolLogParser@U2@@@8 10022310     WevoteTask.obj
 0003:00000338       ??_R0?AVExternalToolRunTask@U2@@@8 10022338     WevoteTask.obj
 0003:00000360       ??_R0?AVWevoteTask@U2@@@8  10022360     WevoteTask.obj
 0003:0000037c       ??_R0?AVExternalToolSupportTask@U2@@@8 1002237c     WevoteTask.obj
 0003:000003a8       ??_R0?AVFailTask@U2@@@8    100223a8     WevoteWorker.obj
 0003:000003c4       ??_R0?AVTaskSignalMapper@U2@@@8 100223c4     WevoteWorker.obj
 0003:000003e8       ??_R0?AVDescriptor@U2@@@8  100223e8     WevoteWorker.obj
 0003:00000404       ??_R0?AVWevoteWorker@LocalWorkflow@U2@@@8 10022404     WevoteWorker.obj
 0003:00000430       ??_R0?AVBaseWorker@LocalWorkflow@U2@@@8 10022430     WevoteWorker.obj
 0003:0000045c       ??_R0?AVWorker@Workflow@U2@@@8 1002245c     WevoteWorker.obj
 0003:00000480       ??_R0?AVCommunicationSubject@Workflow@U2@@@8 10022480     WevoteWorker.obj
 0003:000004b0       ??_R0?AVMapDataType@U2@@@8 100224b0     WevoteWorkerFactory.obj
 0003:000004d0       ??_R0?AVDataType@U2@@@8    100224d0     WevoteWorkerFactory.obj
 0003:000004ec       ??_R0?AVQSharedData@@@8    100224ec     WevoteWorkerFactory.obj
 0003:00000508       ??_R0?AVAttribute@U2@@@8   10022508     WevoteWorkerFactory.obj
 0003:00000524       ??_R0?AVConfigurationEditor@U2@@@8 10022524     WevoteWorkerFactory.obj
 0003:0000054c       ??_R0?AVDelegateEditor@U2@@@8 1002254c     WevoteWorkerFactory.obj
 0003:0000056c       ??_R0?AVURLDelegate@U2@@@8 1002256c     WevoteWorkerFactory.obj
 0003:0000058c       ??_R0?AVPropertyDelegate@U2@@@8 1002258c     WevoteWorkerFactory.obj
 0003:000005b0       ??_R0?AVQItemDelegate@@@8  100225b0     WevoteWorkerFactory.obj
 0003:000005cc       ??_R0?AVQAbstractItemDelegate@@@8 100225cc     WevoteWorkerFactory.obj
 0003:000005f0       ??_R0?AVSpinBoxDelegate@U2@@@8 100225f0     WevoteWorkerFactory.obj
 0003:00000614       ??_R0?AVPortDescriptor@Workflow@U2@@@8 10022614     WevoteWorkerFactory.obj
 0003:00000640       ??_R0?AVIntegralBusActorPrototype@Workflow@U2@@@8 10022640     WevoteWorkerFactory.obj
 0003:00000674       ??_R0?AVActorPrototype@Workflow@U2@@@8 10022674     WevoteWorkerFactory.obj
 0003:000006a0       ??_R0?AVVisualDescriptor@U2@@@8 100226a0     WevoteWorkerFactory.obj
 0003:000006c4       ??_R0?AVWevoteValidator@Workflow@U2@@@8 100226c4     WevoteWorkerFactory.obj
 0003:000006f0       ??_R0?AVActorValidator@Workflow@U2@@@8 100226f0     WevoteWorkerFactory.obj
 0003:0000071c       ??_R0?AVConfigurationValidator@U2@@@8 1002271c     WevoteWorkerFactory.obj
 0003:00000744       ??_R0?AVWevoteWorkerFactory@LocalWorkflow@U2@@@8 10022744     WevoteWorkerFactory.obj
 0003:00000778       ??_R0?AVDomainFactory@Workflow@U2@@@8 10022778     WevoteWorkerFactory.obj
 0003:000007a0       ??_R0?AV?$IdRegistry@VDomainFactory@Workflow@U2@@@U2@@@8 100227a0     WevoteWorkerFactory.obj
 0003:000007dc       ??_R0?AVtype_info@@@8      100227dc     MSVCRT:ti_inst.obj
 0003:0000080c       ?SCIENTIFIC_NAME@PrepareWevoteTaxonomyDataTask@U2@@0VQString@@B 1002280c     PrepareWevoteTaxonomyDataTask.obj
 0003:00000820       ?WEVOTE_DIR@PrepareWevoteTaxonomyDataTask@U2@@0VQString@@B 10022820     PrepareWevoteTaxonomyDataTask.obj
 0003:00000824       ?WEVOTE_NODES@PrepareWevoteTaxonomyDataTask@U2@@0VQString@@B 10022824     PrepareWevoteTaxonomyDataTask.obj
 0003:00000830       ?WEVOTE_NAMES@PrepareWevoteTaxonomyDataTask@U2@@0VQString@@B 10022830     PrepareWevoteTaxonomyDataTask.obj
 0003:00000854       ?id@?$num_put@DV?$back_insert_iterator@V?$basic_string@DU?$char_traits@D@std@@V?$allocator@D@2@@std@@@std@@@std@@2V0locale@2@A 10022854     PrepareWevoteTaxonomyDataTask.obj
 0003:00000858       ?id@?$num_put@_WV?$back_insert_iterator@V?$basic_string@_WU?$char_traits@_W@std@@V?$allocator@_W@2@@std@@@std@@@std@@2V0locale@2@A 10022858     PrepareWevoteTaxonomyDataTask.obj
 0003:000008ac       ?TOOL_NAME@WevoteSupport@U2@@2VQString@@B 100228ac     WevoteSupport.obj
 0003:000008c4       ?PLUGIN_DESCRIPRION@WevoteSupportPlugin@U2@@2VQString@@B 100228c4     WevoteSupportPlugin.obj
 0003:000008c8       ?PLUGIN_NAME@WevoteSupportPlugin@U2@@2VQString@@B 100228c8     WevoteSupportPlugin.obj
 0003:00000950       ?SUFFIX@WevoteTask@U2@@2VQString@@B 10022950     WevoteTask.obj
 0003:000009cc       ?WEVOTE_DIR@WevoteWorker@LocalWorkflow@U2@@0VQString@@B 100229cc     WevoteWorker.obj
 0003:000009f0       ?metatype_id@?1??qt_metatype_id@?$QMetaTypeId@VQAssociativeIterableImpl@QtMetaTypePrivate@@@@SAHXZ@4V?$QBasicAtomicInteger@H@@A 100229f0     WevoteWorker.obj
 0003:000009f4       ?metatype_id@?1??qt_metatype_id@?$QMetaTypeId@V?$QMap@VQString@@I@@@@SAHXZ@4V?$QBasicAtomicInteger@H@@A 100229f4     WevoteWorker.obj
 0003:000009f8       ?f@?4??registerConverter@?$AssociativeValueTypeIsMetaType@V?$QMap@VQString@@I@@$00@QtPrivate@@SA_NH@Z@4U?$ConverterFunctor@V?$QMap@VQString@@I@@VQAssociativeIterableImpl@QtMetaTypePrivate@@U?$QAssociativeIterableConvertFunctor@V?$QMap@VQString@@I@@@3@@3@B 100229f8     WevoteWorker.obj
 0003:00000a00       ??_B?4??registerConverter@?$AssociativeValueTypeIsMetaType@V?$QMap@VQString@@I@@$00@QtPrivate@@SA_NH@Z@54 10022a00     WevoteWorker.obj
 0003:00000a08       ?OUTPUT_PORT_ID@WevoteWorkerFactory@LocalWorkflow@U2@@2VQString@@B 10022a08     WevoteWorkerFactory.obj
 0003:00000a0c       ?NUMBER_OF_AGREED_TOOLS_ATTR_ID@WevoteWorkerFactory@LocalWorkflow@U2@@2VQString@@B 10022a0c     WevoteWorkerFactory.obj
 0003:00000a38       ?PENALTY_ATTR_ID@WevoteWorkerFactory@LocalWorkflow@U2@@2VQString@@B 10022a38     WevoteWorkerFactory.obj
 0003:00000a3c       ?NUMBER_OF_THREADS_ATTR_ID@WevoteWorkerFactory@LocalWorkflow@U2@@2VQString@@B 10022a3c     WevoteWorkerFactory.obj
 0003:00000a50       ?ACTOR_ID@WevoteWorkerFactory@LocalWorkflow@U2@@2VQString@@B 10022a50     WevoteWorkerFactory.obj
 0003:00000a64       ?SCORE_THRESHOLD_ATTR_ID@WevoteWorkerFactory@LocalWorkflow@U2@@2VQString@@B 10022a64     WevoteWorkerFactory.obj
 0003:00000a68       ?WORKFLOW_CLASSIFY_TOOL_WEVOTE@WevoteWorkerFactory@LocalWorkflow@U2@@2VQString@@B 10022a68     WevoteWorkerFactory.obj
 0003:00000a6c       ?OUTPUT_FILE_ATTR_ID@WevoteWorkerFactory@LocalWorkflow@U2@@2VQString@@B 10022a6c     WevoteWorkerFactory.obj
 0003:00000a70       ?INPUT_PORT_ID@WevoteWorkerFactory@LocalWorkflow@U2@@2VQString@@B 10022a70     WevoteWorkerFactory.obj
 0003:00000b5c       ?metatype_id@?1??qt_metatype_id@?$QMetaTypeIdQObject@PAVTask@U2@@$00@@SAHXZ@4V?$QBasicAtomicInteger@H@@A 10022b5c     moc_WevoteWorker.obj
 0003:00000e88       ?__type_info_root_node@@3U__type_info_node@@A 10022e88     MSVCRT:tncleanup.obj
 0003:00000e90       ___native_startup_lock     10022e90     <common>
 0003:00000e94       ___native_startup_state    10022e94     <common>
 0003:00000e98       ___dyn_tls_init_callback   10022e98     <common>
 0003:00000e9c       ___onexitend               10022e9c     <common>
 0003:00000ea0       ___onexitbegin             10022ea0     <common>

 entry point at        0001:0000fc45

 Static symbols

 0000:fffd9000       .debug$S                   10000000     MSVCRT:MSVCR120.dll
 0000:fffd9000       .debug$S                   10000000     MSVCRT:MSVCR120.dll
 0000:fffd9000       .debug$S                   10000000     MSVCRT:MSVCR120.dll
 0000:fffd9000       .debug$S                   10000000     MSVCRT:MSVCR120.dll
 0000:fffd9000       .debug$S                   10000000     MSVCRT:MSVCR120.dll
 0000:fffd9000       .debug$S                   10000000     MSVCRT:MSVCR120.dll
 0000:fffd9000       .debug$S                   10000000     MSVCRT:MSVCR120.dll
 0000:fffd9000       .debug$S                   10000000     MSVCRT:MSVCR120.dll
 0000:fffd9000       .debug$S                   10000000     MSVCRT:MSVCR120.dll
 0002:fffeb000       ?_System_object$initializer$@?$_Error_objects@H@std@@2P6AXXZA 10000000     WevoteWorker.obj
 0000:fffd9000       .debug$S                   10000000     MSVCRT:MSVCR120.dll
 0002:fffeb000       ?_Iostream_object$initializer$@?$_Error_objects@H@std@@2P6AXXZA 10000000     WevoteWorker.obj
 0000:fffd9000       .debug$S                   10000000     MSVCRT:MSVCR120.dll
 0002:fffeb000       ?_Generic_object$initializer$@?$_Error_objects@H@std@@2P6AXXZA 10000000     WevoteWorker.obj
 0000:fffd9000       .debug$S                   10000000     MSVCRT:MSVCR120.dll
 0001:fffff000       __ehhandler$?_Copy@?$basic_string@DU?$char_traits@D@std@@V?$allocator@D@2@@std@@QAEXII@Z 10000000 f   WevoteValidator.obj
 0000:fffd9000       .debug$S                   10000000     MSVCRT:MSVCR120.dll
 0002:fffeb000       __catchsym$?_Copy@?$basic_string@DU?$char_traits@D@std@@V?$allocator@D@2@@std@@QAEXII@Z$5 10000000     WevoteValidator.obj
 0000:fffd9000       .debug$S                   10000000     MSVCRT:MSVCR120.dll
 0002:fffeb000       ?_Generic_object$initializer$@?$_Error_objects@H@std@@2P6AXXZA 10000000     WevoteValidator.obj
 0000:fffd9000       .debug$S                   10000000     MSVCRT:MSVCR120.dll
 0002:fffeb000       ?_Iostream_object$initializer$@?$_Error_objects@H@std@@2P6AXXZA 10000000     WevoteValidator.obj
 0000:fffd9000       .debug$S                   10000000     MSVCRT:MSVCR120.dll
 0002:fffeb000       ?_System_object$initializer$@?$_Error_objects@H@std@@2P6AXXZA 10000000     WevoteValidator.obj
 0000:fffd9000       .debug$S                   10000000     MSVCRT:MSVCR120.dll
 0002:fffeb000       __catchsym$?createNode@?$QMapData@VQString@@I@@QAEPAU?$QMapNode@VQString@@I@@ABVQString@@ABIPAU2@_N@Z$5 10000000     WevoteWorker.obj
 0000:fffd9000       .debug$S                   10000000     MSVCRT:MSVCR120.dll
 0001:fffff000       __ehhandler$?_Copy@?$basic_string@DU?$char_traits@D@std@@V?$allocator@D@2@@std@@QAEXII@Z 10000000 f   WevoteTask.obj
 0001:fffff000       __unwindfunclet$??H@YA?BVQString@@ABV0@0@Z$0 10000000 f   WevoteTask.obj
 0000:fffd9000       .debug$S                   10000000     MSVCRT:MSVCR120.dll
 0001:fffff000       __unwindfunclet$??H@YA?BVQString@@ABV0@PBD@Z$0 10000000 f   WevoteTask.obj
 0000:fffd9000       .debug$S                   10000000     MSVCRT:MSVCR120.dll
 0002:fffeb000       __unwindtable$??0WevoteTaskSettings@U2@@QAE@ABU01@@Z 10000000     WevoteWorker.obj
 0000:fffd9000       .debug$S                   10000000     MSVCRT:MSVCR120.dll
 0001:fffff000       __ehhandler$?_Copy@?$basic_string@DU?$char_traits@D@std@@V?$allocator@D@2@@std@@QAEXII@Z 10000000 f   moc_WevoteWorker.obj
 0002:fffeb000       __unwindtable$??1WevoteTaskSettings@U2@@QAE@XZ 10000000     WevoteWorker.obj
 0002:fffeb000       __catchsym$?_Copy@?$basic_string@DU?$char_traits@D@std@@V?$allocator@D@2@@std@@QAEXII@Z$5 10000000     WevoteTask.obj
 0000:fffd9000       .debug$S                   10000000     MSVCRT:MSVCR120.dll
 0000:fffd9000       .debug$S                   10000000     MSVCRT:MSVCR120.dll
 0000:fffd9000       .debug$S                   10000000     MSVCRT:MSVCR120.dll
 0000:fffd9000       .debug$S                   10000000     MSVCRT:MSVCR120.dll
 0000:fffd9000       .debug$S                   10000000     MSVCRT:MSVCR120.dll
 0002:fffeb000       __unwindtable$??H@YA?BVQString@@ABV0@0@Z 10000000     WevoteTask.obj
 0002:fffeb000       __unwindtable$??H@YA?BVQString@@ABV0@PBD@Z 10000000     WevoteTask.obj
 0002:fffeb000       ?_Generic_object$initializer$@?$_Error_objects@H@std@@2P6AXXZA 10000000     WevoteTask.obj
 0002:fffeb000       ?_Iostream_object$initializer$@?$_Error_objects@H@std@@2P6AXXZA 10000000     WevoteTask.obj
 0002:fffeb000       ?_System_object$initializer$@?$_Error_objects@H@std@@2P6AXXZA 10000000     WevoteTask.obj
 0000:fffd9000       .debug$S                   10000000     msvcprt:MSVCP120.dll
 0000:fffd9000       .debug$S                   10000000     msvcprt:MSVCP120.dll
 0000:fffd9000       .debug$S                   10000000     msvcprt:MSVCP120.dll
 0000:fffd9000       .debug$S                   10000000     msvcprt:MSVCP120.dll
 0000:fffd9000       .debug$S                   10000000     msvcprt:MSVCP120.dll
 0000:fffd9000       .debug$S                   10000000     kernel32:KERNEL32.dll
 0000:fffd9000       .debug$S                   10000000     kernel32:KERNEL32.dll
 0000:fffd9000       .debug$S                   10000000     kernel32:KERNEL32.dll
 0000:fffd9000       .debug$S                   10000000     kernel32:KERNEL32.dll
 0000:fffd9000       .debug$S                   10000000     kernel32:KERNEL32.dll
 0001:fffff000       __ehhandler$?_Copy@?$basic_string@DU?$char_traits@D@std@@V?$allocator@D@2@@std@@QAEXII@Z 10000000 f   WevoteSupportPlugin.obj
 0002:fffeb000       __unwindtable$??H@YA?BVQString@@ABV0@PBD@Z 10000000     WevoteWorker.obj
 0002:fffeb000       __unwindtable$??H@YA?BVQString@@ABV0@0@Z 10000000     WevoteWorker.obj
 0002:fffeb000       __catchsym$?_Copy@?$basic_string@DU?$char_traits@D@std@@V?$allocator@D@2@@std@@QAEXII@Z$5 10000000     WevoteWorker.obj
 0002:fffeb000       __catchsym$?_Copy@?$basic_string@DU?$char_traits@D@std@@V?$allocator@D@2@@std@@QAEXII@Z$5 10000000     moc_WevoteWorker.obj
 0000:fffd9000       .debug$S                   10000000     kernel32:KERNEL32.dll
 0000:fffd9000       .debug$S                   10000000     kernel32:KERNEL32.dll
 0000:fffd9000       .debug$S                   10000000     kernel32:KERNEL32.dll
 0000:fffd9000       .debug$S                   10000000     kernel32:KERNEL32.dll
 0000:fffd9000       .debug$S                   10000000     Qt5Core:Qt5Core.dll
 0000:fffd9000       .debug$S                   10000000     Qt5Core:Qt5Core.dll
 0000:fffd9000       .debug$S                   10000000     Qt5Core:Qt5Core.dll
 0000:fffd9000       .debug$S                   10000000     Qt5Core:Qt5Core.dll
 0000:fffd9000       .debug$S                   10000000     Qt5Core:Qt5Core.dll
 0000:fffd9000       .debug$S                   10000000     Qt5Core:Qt5Core.dll
 0000:fffd9000       .debug$S                   10000000     Qt5Core:Qt5Core.dll
 0000:fffd9000       .debug$S                   10000000     Qt5Core:Qt5Core.dll
 0000:fffd9000       .debug$S                   10000000     Qt5Core:Qt5Core.dll
 0000:fffd9000       .debug$S                   10000000     Qt5Core:Qt5Core.dll
 0000:fffd9000       .debug$S                   10000000     Qt5Core:Qt5Core.dll
 0000:fffd9000       .debug$S                   10000000     Qt5Core:Qt5Core.dll
 0000:fffd9000       .debug$S                   10000000     Qt5Core:Qt5Core.dll
 0000:fffd9000       .debug$S                   10000000     Qt5Core:Qt5Core.dll
 0000:fffd9000       .debug$S                   10000000     Qt5Core:Qt5Core.dll
 0000:fffd9000       .debug$S                   10000000     Qt5Core:Qt5Core.dll
 0000:fffd9000       .debug$S                   10000000     Qt5Core:Qt5Core.dll
 0000:fffd9000       .debug$S                   10000000     Qt5Core:Qt5Core.dll
 0000:fffd9000       .debug$S                   10000000     Qt5Core:Qt5Core.dll
 0000:fffd9000       .debug$S                   10000000     Qt5Core:Qt5Core.dll
 0000:fffd9000       .debug$S                   10000000     Qt5Core:Qt5Core.dll
 0000:fffd9000       .debug$S                   10000000     Qt5Core:Qt5Core.dll
 0000:fffd9000       .debug$S                   10000000     Qt5Core:Qt5Core.dll
 0000:fffd9000       .debug$S                   10000000     Qt5Core:Qt5Core.dll
 0000:fffd9000       .debug$S                   10000000     Qt5Core:Qt5Core.dll
 0000:fffd9000       .debug$S                   10000000     Qt5Core:Qt5Core.dll
 0000:fffd9000       .debug$S                   10000000     Qt5Core:Qt5Core.dll
 0000:fffd9000       .debug$S                   10000000     Qt5Core:Qt5Core.dll
 0000:fffd9000       .debug$S                   10000000     Qt5Core:Qt5Core.dll
 0000:fffd9000       .debug$S                   10000000     Qt5Core:Qt5Core.dll
 0000:fffd9000       .debug$S                   10000000     Qt5Core:Qt5Core.dll
 0000:fffd9000       .debug$S                   10000000     Qt5Core:Qt5Core.dll
 0000:fffd9000       .debug$S                   10000000     Qt5Core:Qt5Core.dll
 0000:fffd9000       .debug$S                   10000000     Qt5Core:Qt5Core.dll
 0000:fffd9000       .debug$S                   10000000     Qt5Core:Qt5Core.dll
 0000:fffd9000       .debug$S                   10000000     Qt5Core:Qt5Core.dll
 0000:fffd9000       .debug$S                   10000000     Qt5Core:Qt5Core.dll
 0000:fffd9000       .debug$S                   10000000     Qt5Core:Qt5Core.dll
 0000:fffd9000       .debug$S                   10000000     Qt5Core:Qt5Core.dll
 0002:fffeb000       ?_Generic_object$initializer$@?$_Error_objects@H@std@@2P6AXXZA 10000000     moc_WevoteWorker.obj
 0002:fffeb000       ?_Iostream_object$initializer$@?$_Error_objects@H@std@@2P6AXXZA 10000000     moc_WevoteWorker.obj
 0002:fffeb000       ?_System_object$initializer$@?$_Error_objects@H@std@@2P6AXXZA 10000000     moc_WevoteWorker.obj
 0000:fffd9000       .debug$S                   10000000     Qt5Core:Qt5Core.dll
 0000:fffd9000       .debug$S                   10000000     Qt5Core:Qt5Core.dll
 0002:fffeb000       __catchsym$?_Copy@?$basic_string@DU?$char_traits@D@std@@V?$allocator@D@2@@std@@QAEXII@Z$5 10000000     WevoteSupportPlugin.obj
 0000:fffd9000       .debug$S                   10000000     Qt5Core:Qt5Core.dll
 0002:fffeb000       ?_Generic_object$initializer$@?$_Error_objects@H@std@@2P6AXXZA 10000000     WevoteSupportPlugin.obj
 0000:fffd9000       .debug$S                   10000000     Qt5Core:Qt5Core.dll
 0002:fffeb000       ?_Iostream_object$initializer$@?$_Error_objects@H@std@@2P6AXXZA 10000000     WevoteSupportPlugin.obj
 0000:fffd9000       .debug$S                   10000000     Qt5Core:Qt5Core.dll
 0001:fffff000       __unwindfunclet$?createNode@?$QMapData@VQString@@I@@QAEPAU?$QMapNode@VQString@@I@@ABVQString@@ABIPAU2@_N@Z$4 10000000 f   WevoteWorker.obj
 0000:fffd9000       .debug$S                   10000000     Qt5Core:Qt5Core.dll
 0002:fffeb000       ?_System_object$initializer$@?$_Error_objects@H@std@@2P6AXXZA 10000000     WevoteSupportPlugin.obj
 0000:fffd9000       .debug$S                   10000000     Qt5Core:Qt5Core.dll
 0001:fffff000       __ehhandler$?_Copy@?$basic_string@DU?$char_traits@D@std@@V?$allocator@D@2@@std@@QAEXII@Z 10000000 f   WevoteSupport.obj
 0000:fffd9000       .debug$S                   10000000     Qt5Core:Qt5Core.dll
 0002:fffeb000       __catchsym$?_Copy@?$basic_string@DU?$char_traits@D@std@@V?$allocator@D@2@@std@@QAEXII@Z$5 10000000     WevoteSupport.obj
 0000:fffd9000       .debug$S                   10000000     Qt5Core:Qt5Core.dll
 0002:fffeb000       ?_Generic_object$initializer$@?$_Error_objects@H@std@@2P6AXXZA 10000000     WevoteSupport.obj
 0000:fffd9000       .debug$S                   10000000     Qt5Core:Qt5Core.dll
 0002:fffeb000       ?_Iostream_object$initializer$@?$_Error_objects@H@std@@2P6AXXZA 10000000     WevoteSupport.obj
 0000:fffd9000       .debug$S                   10000000     Qt5Core:Qt5Core.dll
 0002:fffeb000       ?_System_object$initializer$@?$_Error_objects@H@std@@2P6AXXZA 10000000     WevoteSupport.obj
 0001:fffff000       __ehhandler$?_Copy@?$basic_string@DU?$char_traits@D@std@@V?$allocator@D@2@@std@@QAEXII@Z 10000000 f   WevotePrompter.obj
 0000:fffd9000       .debug$S                   10000000     Qt5Core:Qt5Core.dll
 0002:fffeb000       __catchsym$?_Copy@?$basic_string@DU?$char_traits@D@std@@V?$allocator@D@2@@std@@QAEXII@Z$5 10000000     WevotePrompter.obj
 0000:fffd9000       .debug$S                   10000000     Qt5Core:Qt5Core.dll
 0002:fffeb000       ?_Generic_object$initializer$@?$_Error_objects@H@std@@2P6AXXZA 10000000     WevotePrompter.obj
 0000:fffd9000       .debug$S                   10000000     Qt5Core:Qt5Core.dll
 0001:fffff000       __ehhandler$?_Copy@?$basic_string@DU?$char_traits@D@std@@V?$allocator@D@2@@std@@QAEXII@Z 10000000 f   moc_WevoteTask.obj
 0002:fffeb000       ?_Iostream_object$initializer$@?$_Error_objects@H@std@@2P6AXXZA 10000000     WevotePrompter.obj
 0002:fffeb000       ?_System_object$initializer$@?$_Error_objects@H@std@@2P6AXXZA 10000000     WevotePrompter.obj
 0000:fffd9000       .debug$S                   10000000     Qt5Core:Qt5Core.dll
 0000:fffd9000       .debug$S                   10000000     Qt5Core:Qt5Core.dll
 0000:fffd9000       .debug$S                   10000000     Qt5Core:Qt5Core.dll
 0000:fffd9000       .debug$S                   10000000     Qt5Core:Qt5Core.dll
 0000:fffd9000       .debug$S                   10000000     Qt5Core:Qt5Core.dll
 0000:fffd9000       .debug$S                   10000000     Qt5Core:Qt5Core.dll
 0000:fffd9000       .debug$S                   10000000     Qt5Core:Qt5Core.dll
 0000:fffd9000       .debug$S                   10000000     Qt5Core:Qt5Core.dll
 0000:fffd9000       .debug$S                   10000000     Qt5Core:Qt5Core.dll
 0000:fffd9000       .debug$S                   10000000     Qt5Core:Qt5Core.dll
 0000:fffd9000       .debug$S                   10000000     Qt5Core:Qt5Core.dll
 0000:fffd9000       .debug$S                   10000000     Qt5Core:Qt5Core.dll
 0000:fffd9000       .debug$S                   10000000     Qt5Core:Qt5Core.dll
 0000:fffd9000       .debug$S                   10000000     Qt5Core:Qt5Core.dll
 0000:fffd9000       .debug$S                   10000000     Qt5Core:Qt5Core.dll
 0000:fffd9000       .debug$S                   10000000     Qt5Core:Qt5Core.dll
 0000:fffd9000       .debug$S                   10000000     Qt5Core:Qt5Core.dll
 0000:fffd9000       .debug$S                   10000000     Qt5Core:Qt5Core.dll
 0001:fffff000       __unwindfunclet$??0WevoteTaskSettings@U2@@QAE@ABU01@@Z$0 10000000 f   WevoteWorker.obj
 0001:fffff000       __unwindfunclet$??1WevoteTaskSettings@U2@@QAE@XZ$0 10000000 f   WevoteWorker.obj
 0001:fffff000       __unwindfunclet$??H@YA?BVQString@@ABV0@PBD@Z$0 10000000 f   WevoteWorker.obj
 0001:fffff000       __unwindfunclet$??H@YA?BVQString@@ABV0@0@Z$0 10000000 f   WevoteWorker.obj
 0002:fffeb000       __catchsym$?_Copy@?$basic_string@DU?$char_traits@D@std@@V?$allocator@D@2@@std@@QAEXII@Z$5 10000000     moc_WevoteTask.obj
 0000:fffd9000       .debug$S                   10000000     Qt5Core:Qt5Core.dll
 0000:fffd9000       .debug$S                   10000000     Qt5Core:Qt5Core.dll
 0000:fffd9000       .debug$S                   10000000     Qt5Core:Qt5Core.dll
 0000:fffd9000       .debug$S                   10000000     Qt5Core:Qt5Core.dll
 0000:fffd9000       .debug$S                   10000000     Qt5Core:Qt5Core.dll
 0000:fffd9000       .debug$S                   10000000     Qt5Core:Qt5Core.dll
 0000:fffd9000       .debug$S                   10000000     Qt5Core:Qt5Core.dll
 0000:fffd9000       .debug$S                   10000000     Qt5Core:Qt5Core.dll
 0000:fffd9000       .debug$S                   10000000     Qt5Core:Qt5Core.dll
 0000:fffd9000       .debug$S                   10000000     Qt5Core:Qt5Core.dll
 0000:fffd9000       .debug$S                   10000000     Qt5Core:Qt5Core.dll
 0000:fffd9000       .debug$S                   10000000     Qt5Core:Qt5Core.dll
 0000:fffd9000       .debug$S                   10000000     Qt5Core:Qt5Core.dll
 0000:fffd9000       .debug$S                   10000000     Qt5Core:Qt5Core.dll
 0000:fffd9000       .debug$S                   10000000     Qt5Core:Qt5Core.dll
 0000:fffd9000       .debug$S                   10000000     Qt5Core:Qt5Core.dll
 0000:fffd9000       .debug$S                   10000000     Qt5Core:Qt5Core.dll
 0000:fffd9000       .debug$S                   10000000     Qt5Core:Qt5Core.dll
 0000:fffd9000       .debug$S                   10000000     Qt5Core:Qt5Core.dll
 0000:fffd9000       .debug$S                   10000000     Qt5Core:Qt5Core.dll
 0000:fffd9000       .debug$S                   10000000     Qt5Core:Qt5Core.dll
 0000:fffd9000       .debug$S                   10000000     Qt5Core:Qt5Core.dll
 0000:fffd9000       .debug$S                   10000000     Qt5Core:Qt5Core.dll
 0000:fffd9000       .debug$S                   10000000     Qt5Core:Qt5Core.dll
 0000:fffd9000       .debug$S                   10000000     Qt5Core:Qt5Core.dll
 0000:fffd9000       .debug$S                   10000000     Qt5Script:Qt5Script.dll
 0000:fffd9000       .debug$S                   10000000     Qt5Script:Qt5Script.dll
 0000:fffd9000       .debug$S                   10000000     Qt5Script:Qt5Script.dll
 0000:fffd9000       .debug$S                   10000000     Qt5Script:Qt5Script.dll
 0000:fffd9000       .debug$S                   10000000     Qt5Script:Qt5Script.dll
 0000:fffd9000       .debug$S                   10000000     Qt5Script:Qt5Script.dll
 0000:fffd9000       .debug$S                   10000000     Qt5Script:Qt5Script.dll
 0000:fffd9000       .debug$S                   10000000     Qt5Script:Qt5Script.dll
 0000:fffd9000       .debug$S                   10000000     Qt5Script:Qt5Script.dll
 0000:fffd9000       .debug$S                   10000000     Qt5Script:Qt5Script.dll
 0000:fffd9000       .debug$S                   10000000     Qt5Gui:Qt5Gui.dll
 0000:fffd9000       .debug$S                   10000000     Qt5Gui:Qt5Gui.dll
 0000:fffd9000       .debug$S                   10000000     Qt5Gui:Qt5Gui.dll
 0000:fffd9000       .debug$S                   10000000     Qt5Widgets:Qt5Widgets.dll
 0000:fffd9000       .debug$S                   10000000     Qt5Widgets:Qt5Widgets.dll
 0000:fffd9000       .debug$S                   10000000     Qt5Widgets:Qt5Widgets.dll
 0002:fffeb000       ?_Generic_object$initializer$@?$_Error_objects@H@std@@2P6AXXZA 10000000     moc_WevoteTask.obj
 0002:fffeb000       ?_Iostream_object$initializer$@?$_Error_objects@H@std@@2P6AXXZA 10000000     moc_WevoteTask.obj
 0002:fffeb000       ?_System_object$initializer$@?$_Error_objects@H@std@@2P6AXXZA 10000000     moc_WevoteTask.obj
 0000:fffd9000       .debug$S                   10000000     Qt5Widgets:Qt5Widgets.dll
 0000:fffd9000       .debug$S                   10000000     Qt5Widgets:Qt5Widgets.dll
 0001:fffff000       __ehhandler$?_Copy@?$basic_string@DU?$char_traits@D@std@@V?$allocator@D@2@@std@@QAEXII@Z 10000000 f   WevoteWorker.obj
 0002:fffeb000       ?_System_object$initializer$@?$_Error_objects@H@std@@2P6AXXZA 10000000     WevoteWorkerFactory.obj
 0000:fffd9000       .debug$S                   10000000     Qt5Widgets:Qt5Widgets.dll
 0002:fffeb000       ?_Iostream_object$initializer$@?$_Error_objects@H@std@@2P6AXXZA 10000000     WevoteWorkerFactory.obj
 0000:fffd9000       .debug$S                   10000000     Qt5Widgets:Qt5Widgets.dll
 0002:fffeb000       ?_Generic_object$initializer$@?$_Error_objects@H@std@@2P6AXXZA 10000000     WevoteWorkerFactory.obj
 0000:fffd9000       .debug$S                   10000000     Qt5Widgets:Qt5Widgets.dll
 0001:fffff000       __ehhandler$?_Copy@?$basic_string@DU?$char_traits@D@std@@V?$allocator@D@2@@std@@QAEXII@Z 10000000 f   moc_WevoteSupportPlugin.obj
 0000:fffd9000       .debug$S                   10000000     ngs_reads_classification:ngs_reads_classification.dll
 0000:fffd9000       .debug$S                   10000000     ngs_reads_classification:ngs_reads_classification.dll
 0000:fffd9000       .debug$S                   10000000     ngs_reads_classification:ngs_reads_classification.dll
 0000:fffd9000       .debug$S                   10000000     ngs_reads_classification:ngs_reads_classification.dll
 0000:fffd9000       .debug$S                   10000000     ngs_reads_classification:ngs_reads_classification.dll
 0000:fffd9000       .debug$S                   10000000     ngs_reads_classification:ngs_reads_classification.dll
 0002:fffeb000       __catchsym$?_Copy@?$basic_string@DU?$char_traits@D@std@@V?$allocator@D@2@@std@@QAEXII@Z$5 10000000     moc_WevoteSupportPlugin.obj
 0000:fffd9000       .debug$S                   10000000     Qt5Widgets:Qt5Widgets.dll
 0000:fffd9000       .debug$S                   10000000     Qt5Widgets:Qt5Widgets.dll
 0000:fffd9000       .debug$S                   10000000     Qt5Widgets:Qt5Widgets.dll
 0000:fffd9000       .debug$S                   10000000     Qt5Widgets:Qt5Widgets.dll
 0000:fffd9000       .debug$S                   10000000     U2Designer:U2Designer.dll
 0002:fffeb000       ?_Generic_object$initializer$@?$_Error_objects@H@std@@2P6AXXZA 10000000     moc_WevoteSupportPlugin.obj
 0002:fffeb000       ?_Iostream_object$initializer$@?$_Error_objects@H@std@@2P6AXXZA 10000000     moc_WevoteSupportPlugin.obj
 0002:fffeb000       ?_System_object$initializer$@?$_Error_objects@H@std@@2P6AXXZA 10000000     moc_WevoteSupportPlugin.obj
 0000:fffd9000       .debug$S                   10000000     U2Designer:U2Designer.dll
 0000:fffd9000       .debug$S                   10000000     U2Designer:U2Designer.dll
 0000:fffd9000       .debug$S                   10000000     ngs_reads_classification:ngs_reads_classification.dll
 0000:fffd9000       .debug$S                   10000000     U2Designer:U2Designer.dll
 0000:fffd9000       .debug$S                   10000000     ngs_reads_classification:ngs_reads_classification.dll
 0000:fffd9000       .debug$S                   10000000     U2Designer:U2Designer.dll
 0000:fffd9000       .debug$S                   10000000     ngs_reads_classification:ngs_reads_classification.dll
 0000:fffd9000       .debug$S                   10000000     U2Designer:U2Designer.dll
 0000:fffd9000       .debug$S                   10000000     U2Core:U2Core.dll
 0000:fffd9000       .debug$S                   10000000     U2Designer:U2Designer.dll
 0000:fffd9000       .debug$S                   10000000     U2Core:U2Core.dll
 0000:fffd9000       .debug$S                   10000000     U2Designer:U2Designer.dll
 0000:fffd9000       .debug$S                   10000000     U2Core:U2Core.dll
 0000:fffd9000       .debug$S                   10000000     U2Designer:U2Designer.dll
 0000:fffd9000       .debug$S                   10000000     U2Core:U2Core.dll
 0000:fffd9000       .debug$S                   10000000     U2Designer:U2Designer.dll
 0000:fffd9000       .debug$S                   10000000     U2Core:U2Core.dll
 0000:fffd9000       .debug$S                   10000000     U2Designer:U2Designer.dll
 0002:fffeb000       __catchsym$?createNode@?$QMapData@VQString@@VQVariant@@@@QAEPAU?$QMapNode@VQString@@VQVariant@@@@ABVQString@@ABVQVariant@@PAU2@_N@Z$7 10000000     WevoteWorkerFactory.obj
 0000:fffd9000       .debug$S                   10000000     U2Designer:U2Designer.dll
 0000:fffd9000       .debug$S                   10000000     U2Core:U2Core.dll
 0000:fffd9000       .debug$S                   10000000     U2Core:U2Core.dll
 0000:fffd9000       .debug$S                   10000000     U2Designer:U2Designer.dll
 0000:fffd9000       .debug$S                   10000000     U2Core:U2Core.dll
 0000:fffd9000       .debug$S                   10000000     U2Designer:U2Designer.dll
 0000:fffd9000       .debug$S                   10000000     U2Core:U2Core.dll
 0000:fffd9000       .debug$S                   10000000     U2Designer:U2Designer.dll
 0001:fffff000       __ehhandler$?_Copy@?$basic_string@DU?$char_traits@D@std@@V?$allocator@D@2@@std@@QAEXII@Z 10000000 f   moc_WevotePrompter.obj
 0000:fffd9000       .debug$S                   10000000     U2Core:U2Core.dll
 0000:fffd9000       .debug$S                   10000000     U2Core:U2Core.dll
 0000:fffd9000       .debug$S                   10000000     U2Designer:U2Designer.dll
 0000:fffd9000       .debug$S                   10000000     U2Designer:U2Designer.dll
 0000:fffd9000       .debug$S                   10000000     U2Designer:U2Designer.dll
 0000:fffd9000       .debug$S                   10000000     U2Designer:U2Designer.dll
 0000:fffd9000       .debug$S                   10000000     U2Designer:U2Designer.dll
 0000:fffd9000       .debug$S                   10000000     U2Designer:U2Designer.dll
 0000:fffd9000       .debug$S                   10000000     U2Designer:U2Designer.dll
 0000:fffd9000       .debug$S                   10000000     U2Designer:U2Designer.dll
 0000:fffd9000       .debug$S                   10000000     U2Designer:U2Designer.dll
 0000:fffd9000       .debug$S                   10000000     U2Designer:U2Designer.dll
 0000:fffd9000       .debug$S                   10000000     U2Designer:U2Designer.dll
 0000:fffd9000       .debug$S                   10000000     U2Designer:U2Designer.dll
 0000:fffd9000       .debug$S                   10000000     U2Designer:U2Designer.dll
 0000:fffd9000       .debug$S                   10000000     U2Designer:U2Designer.dll
 0000:fffd9000       .debug$S                   10000000     U2Designer:U2Designer.dll
 0000:fffd9000       .debug$S                   10000000     U2Designer:U2Designer.dll
 0000:fffd9000       .debug$S                   10000000     U2Designer:U2Designer.dll
 0000:fffd9000       .debug$S                   10000000     U2Designer:U2Designer.dll
 0000:fffd9000       .debug$S                   10000000     U2Core:U2Core.dll
 0000:fffd9000       .debug$S                   10000000     U2Core:U2Core.dll
 0000:fffd9000       .debug$S                   10000000     U2Core:U2Core.dll
 0000:fffd9000       .debug$S                   10000000     U2Core:U2Core.dll
 0002:fffeb000       __catchsym$?_Copy@?$basic_string@DU?$char_traits@D@std@@V?$allocator@D@2@@std@@QAEXII@Z$5 10000000     moc_WevotePrompter.obj
 0000:fffd9000       .debug$S                   10000000     U2Designer:U2Designer.dll
 0000:fffd9000       .debug$S                   10000000     U2Designer:U2Designer.dll
 0000:fffd9000       .debug$S                   10000000     U2Designer:U2Designer.dll
 0000:fffd9000       .debug$S                   10000000     U2Lang:U2Lang.dll
 0000:fffd9000       .debug$S                   10000000     U2Lang:U2Lang.dll
 0000:fffd9000       .debug$S                   10000000     U2Lang:U2Lang.dll
 0000:fffd9000       .debug$S                   10000000     U2Lang:U2Lang.dll
 0000:fffd9000       .debug$S                   10000000     U2Lang:U2Lang.dll
 0000:fffd9000       .debug$S                   10000000     U2Lang:U2Lang.dll
 0000:fffd9000       .debug$S                   10000000     U2Lang:U2Lang.dll
 0000:fffd9000       .debug$S                   10000000     U2Lang:U2Lang.dll
 0000:fffd9000       .debug$S                   10000000     U2Lang:U2Lang.dll
 0000:fffd9000       .debug$S                   10000000     U2Lang:U2Lang.dll
 0000:fffd9000       .debug$S                   10000000     U2Lang:U2Lang.dll
 0000:fffd9000       .debug$S                   10000000     U2Lang:U2Lang.dll
 0000:fffd9000       .debug$S                   10000000     U2Lang:U2Lang.dll
 0000:fffd9000       .debug$S                   10000000     U2Lang:U2Lang.dll
 0000:fffd9000       .debug$S                   10000000     U2Lang:U2Lang.dll
 0000:fffd9000       .debug$S                   10000000     U2Lang:U2Lang.dll
 0000:fffd9000       .debug$S                   10000000     U2Lang:U2Lang.dll
 0000:fffd9000       .debug$S                   10000000     U2Lang:U2Lang.dll
 0000:fffd9000       .debug$S                   10000000     U2Lang:U2Lang.dll
 0000:fffd9000       .debug$S                   10000000     U2Lang:U2Lang.dll
 0000:fffd9000       .debug$S                   10000000     U2Lang:U2Lang.dll
 0000:fffd9000       .debug$S                   10000000     U2Lang:U2Lang.dll
 0000:fffd9000       .debug$S                   10000000     U2Lang:U2Lang.dll
 0000:fffd9000       .debug$S                   10000000     U2Lang:U2Lang.dll
 0000:fffd9000       .debug$S                   10000000     U2Lang:U2Lang.dll
 0000:fffd9000       .debug$S                   10000000     U2Lang:U2Lang.dll
 0000:fffd9000       .debug$S                   10000000     U2Lang:U2Lang.dll
 0000:fffd9000       .debug$S                   10000000     U2Lang:U2Lang.dll
 0000:fffd9000       .debug$S                   10000000     U2Lang:U2Lang.dll
 0000:fffd9000       .debug$S                   10000000     U2Lang:U2Lang.dll
 0000:fffd9000       .debug$S                   10000000     U2Lang:U2Lang.dll
 0000:fffd9000       .debug$S                   10000000     U2Lang:U2Lang.dll
 0000:fffd9000       .debug$S                   10000000     U2Lang:U2Lang.dll
 0000:fffd9000       .debug$S                   10000000     U2Lang:U2Lang.dll
 0000:fffd9000       .debug$S                   10000000     U2Lang:U2Lang.dll
 0000:fffd9000       .debug$S                   10000000     U2Lang:U2Lang.dll
 0000:fffd9000       .debug$S                   10000000     U2Lang:U2Lang.dll
 0000:fffd9000       .debug$S                   10000000     U2Lang:U2Lang.dll
 0002:fffeb000       ?_Generic_object$initializer$@?$_Error_objects@H@std@@2P6AXXZA 10000000     moc_WevotePrompter.obj
 0002:fffeb000       ?_Iostream_object$initializer$@?$_Error_objects@H@std@@2P6AXXZA 10000000     moc_WevotePrompter.obj
 0002:fffeb000       ?_System_object$initializer$@?$_Error_objects@H@std@@2P6AXXZA 10000000     moc_WevotePrompter.obj
 0000:fffd9000       .debug$S                   10000000     U2Core:U2Core.dll
 0000:fffd9000       .debug$S                   10000000     U2Lang:U2Lang.dll
 0000:fffd9000       .debug$S                   10000000     U2Core:U2Core.dll
 0000:fffd9000       .debug$S                   10000000     U2Lang:U2Lang.dll
 0000:fffd9000       .debug$S                   10000000     U2Core:U2Core.dll
 0000:fffd9000       .debug$S                   10000000     U2Lang:U2Lang.dll
 0000:fffd9000       .debug$S                   10000000     U2Core:U2Core.dll
 0000:fffd9000       .debug$S                   10000000     U2Lang:U2Lang.dll
 0000:fffd9000       .debug$S                   10000000     U2Core:U2Core.dll
 0000:fffd9000       .debug$S                   10000000     U2Lang:U2Lang.dll
 0000:fffd9000       .debug$S                   10000000     U2Core:U2Core.dll
 0000:fffd9000       .debug$S                   10000000     U2Lang:U2Lang.dll
 0000:fffd9000       .debug$S                   10000000     U2Core:U2Core.dll
 0000:fffd9000       .debug$S                   10000000     U2Lang:U2Lang.dll
 0000:fffd9000       .debug$S                   10000000     U2Core:U2Core.dll
 0000:fffd9000       .debug$S                   10000000     U2Lang:U2Lang.dll
 0000:fffd9000       .debug$S                   10000000     U2Core:U2Core.dll
 0000:fffd9000       .debug$S                   10000000     U2Lang:U2Lang.dll
 0000:fffd9000       .debug$S                   10000000     U2Core:U2Core.dll
 0000:fffd9000       .debug$S                   10000000     U2Lang:U2Lang.dll
 0000:fffd9000       .debug$S                   10000000     U2Core:U2Core.dll
 0000:fffd9000       .debug$S                   10000000     U2Lang:U2Lang.dll
 0000:fffd9000       .debug$S                   10000000     U2Core:U2Core.dll
 0000:fffd9000       .debug$S                   10000000     U2Lang:U2Lang.dll
 0000:fffd9000       .debug$S                   10000000     U2Core:U2Core.dll
 0000:fffd9000       .debug$S                   10000000     U2Lang:U2Lang.dll
 0000:fffd9000       .debug$S                   10000000     U2Core:U2Core.dll
 0000:fffd9000       .debug$S                   10000000     U2Lang:U2Lang.dll
 0000:fffd9000       .debug$S                   10000000     U2Core:U2Core.dll
 0000:fffd9000       .debug$S                   10000000     U2Lang:U2Lang.dll
 0000:fffd9000       .debug$S                   10000000     U2Core:U2Core.dll
 0000:fffd9000       .debug$S                   10000000     U2Lang:U2Lang.dll
 0000:fffd9000       .debug$S                   10000000     U2Core:U2Core.dll
 0000:fffd9000       .debug$S                   10000000     U2Lang:U2Lang.dll
 0000:fffd9000       .debug$S                   10000000     U2Core:U2Core.dll
 0000:fffd9000       .debug$S                   10000000     U2Lang:U2Lang.dll
 0000:fffd9000       .debug$S                   10000000     U2Core:U2Core.dll
 0000:fffd9000       .debug$S                   10000000     U2Lang:U2Lang.dll
 0000:fffd9000       .debug$S                   10000000     U2Core:U2Core.dll
 0000:fffd9000       .debug$S                   10000000     U2Lang:U2Lang.dll
 0000:fffd9000       .debug$S                   10000000     U2Core:U2Core.dll
 0000:fffd9000       .debug$S                   10000000     U2Lang:U2Lang.dll
 0001:fffff000       __ehhandler$?_Copy@?$basic_string@DU?$char_traits@D@std@@V?$allocator@D@2@@std@@QAEXII@Z 10000000 f   WevoteWorkerFactory.obj
 0000:fffd9000       .debug$S                   10000000     U2Core:U2Core.dll
 0000:fffd9000       .debug$S                   10000000     U2Core:U2Core.dll
 0000:fffd9000       .debug$S                   10000000     U2Core:U2Core.dll
 0001:fffff000       __unwindfunclet$??H@YA?BVQString@@ABV0@PBD@Z$0 10000000 f   WevoteWorkerFactory.obj
 0000:fffd9000       .debug$S                   10000000     U2Core:U2Core.dll
 0000:fffd9000       .debug$S                   10000000     U2Core:U2Core.dll
 0000:fffd9000       .debug$S                   10000000     U2Core:U2Core.dll
 0000:fffd9000       .debug$S                   10000000     U2Core:U2Core.dll
 0001:fffff000       __unwindfunclet$?append@?$QList@VQString@@@@QAEXABVQString@@@Z$7 10000000 f   WevoteWorkerFactory.obj
 0000:fffd9000       .debug$S                   10000000     U2Core:U2Core.dll
 0001:fffff000       __ehhandler$?detach_helper_grow@?$QList@VQString@@@@AAEPAUNode@1@HH@Z 10000000 f   WevoteWorkerFactory.obj
 0000:fffd9000       .debug$S                   10000000     U2Core:U2Core.dll
 0000:fffd9000       .debug$S                   10000000     U2Core:U2Core.dll
 0000:fffd9000       .debug$S                   10000000     U2Core:U2Core.dll
 0001:fffff000       __unwindfunclet$?node_construct@?$QList@VQString@@@@AAEXPAUNode@1@ABVQString@@@Z$1 10000000 f   WevoteWorkerFactory.obj
 0002:fffeb000       __unwindtable$??A?$QMap@VQString@@VQVariant@@@@QAEAAVQVariant@@ABVQString@@@Z 10000000     WevoteWorkerFactory.obj
 0000:fffd9000       .debug$S                   10000000     U2Core:U2Core.dll
 0001:fffff000       __unwindfunclet$?node_copy@?$QList@VQString@@@@AAEXPAUNode@1@00@Z$5 10000000 f   WevoteWorkerFactory.obj
 0000:fffd9000       .debug$S                   10000000     U2Lang:U2Lang.dll
 0000:fffd9000       .debug$S                   10000000     U2Lang:U2Lang.dll
 0000:fffd9000       .debug$S                   10000000     U2Core:U2Core.dll
 0001:fffff000       __unwindfunclet$??A?$QMap@VQString@@VQVariant@@@@QAEAAVQVariant@@ABVQString@@@Z$0 10000000 f   WevoteWorkerFactory.obj
 0000:fffd9000       .debug$S                   10000000     U2Lang:U2Lang.dll
 0000:fffd9000       .debug$S                   10000000     U2Lang:U2Lang.dll
 0000:fffd9000       .debug$S                   10000000     U2Lang:U2Lang.dll
 0000:fffd9000       .debug$S                   10000000     U2Lang:U2Lang.dll
 0000:fffd9000       .debug$S                   10000000     U2Lang:U2Lang.dll
 0000:fffd9000       .debug$S                   10000000     U2Lang:U2Lang.dll
 0000:fffd9000       .debug$S                   10000000     U2Lang:U2Lang.dll
 0000:fffd9000       .debug$S                   10000000     U2Lang:U2Lang.dll
 0000:fffd9000       .debug$S                   10000000     U2Lang:U2Lang.dll
 0000:fffd9000       .debug$S                   10000000     U2Lang:U2Lang.dll
 0000:fffd9000       .debug$S                   10000000     U2Lang:U2Lang.dll
 0000:fffd9000       .debug$S                   10000000     U2Lang:U2Lang.dll
 0000:fffd9000       .debug$S                   10000000     U2Lang:U2Lang.dll
 0000:fffd9000       .debug$S                   10000000     U2Lang:U2Lang.dll
 0000:fffd9000       .debug$S                   10000000     U2Lang:U2Lang.dll
 0000:fffd9000       .debug$S                   10000000     U2Lang:U2Lang.dll
 0000:fffd9000       .debug$S                   10000000     U2Lang:U2Lang.dll
 0000:fffd9000       .debug$S                   10000000     U2Lang:U2Lang.dll
 0000:fffd9000       .debug$S                   10000000     U2Lang:U2Lang.dll
 0000:fffd9000       .debug$S                   10000000     U2Lang:U2Lang.dll
 0000:fffd9000       .debug$S                   10000000     U2Lang:U2Lang.dll
 0002:fffeb000       __catchsym$?node_copy@?$QList@VQString@@@@AAEXPAUNode@1@00@Z$6 10000000     WevoteWorkerFactory.obj
 0000:fffd9000       .debug$S                   10000000     U2Lang:U2Lang.dll
 0002:fffeb000       __unwindtable$?node_construct@?$QList@VQString@@@@AAEXPAUNode@1@ABVQString@@@Z 10000000     WevoteWorkerFactory.obj
 0002:fffeb000       __catchsym$?detach_helper_grow@?$QList@VQString@@@@AAEPAUNode@1@HH@Z$5 10000000     WevoteWorkerFactory.obj
 0000:fffd9000       .debug$S                   10000000     U2Lang:U2Lang.dll
 0002:fffeb000       __catchsym$?append@?$QList@VQString@@@@QAEXABVQString@@@Z$13 10000000     WevoteWorkerFactory.obj
 0000:fffd9000       .debug$S                   10000000     U2Lang:U2Lang.dll
 0002:fffeb000       __unwindtable$??H@YA?BVQString@@ABV0@PBD@Z 10000000     WevoteWorkerFactory.obj
 0002:fffeb000       __catchsym$?_Copy@?$basic_string@DU?$char_traits@D@std@@V?$allocator@D@2@@std@@QAEXII@Z$5 10000000     WevoteWorkerFactory.obj
 0000:fffd9000       .debug$S                   10000000     U2Lang:U2Lang.dll
 0000:fffd9000       .debug$S                   10000000     U2Lang:U2Lang.dll
 0000:fffd9000       .debug$S                   10000000     U2Lang:U2Lang.dll
 0000:fffd9000       .debug$S                   10000000     U2Lang:U2Lang.dll
 0000:fffd9000       .debug$S                   10000000     U2Lang:U2Lang.dll
 0000:fffd9000       .debug$S                   10000000     U2Lang:U2Lang.dll
 0000:fffd9000       .debug$S                   10000000     U2Lang:U2Lang.dll
 0000:fffd9000       .debug$S                   10000000     U2Lang:U2Lang.dll
 0000:fffd9000       .debug$S                   10000000     U2Lang:U2Lang.dll
 0000:fffd9000       .debug$S                   10000000     U2Lang:U2Lang.dll
 0000:fffd9000       .debug$S                   10000000     U2Lang:U2Lang.dll
 0000:fffd9000       .debug$S                   10000000     U2Lang:U2Lang.dll
 0000:fffd9000       .debug$S                   10000000     U2Lang:U2Lang.dll
 0000:fffd9000       .debug$S                   10000000     U2Lang:U2Lang.dll
 0000:fffd9000       .debug$S                   10000000     U2Lang:U2Lang.dll
 0000:fffd9000       .debug$S                   10000000     U2Lang:U2Lang.dll
 0000:fffd9000       .debug$S                   10000000     U2Lang:U2Lang.dll
 0000:fffd9000       .debug$S                   10000000     U2Lang:U2Lang.dll
 0000:fffd9000       .debug$S                   10000000     U2Lang:U2Lang.dll
 0000:fffd9000       .debug$S                   10000000     U2Lang:U2Lang.dll
 0000:fffd9000       .debug$S                   10000000     U2Lang:U2Lang.dll
 0000:fffd9000       .debug$S                   10000000     U2Lang:U2Lang.dll
 0000:fffd9000       .debug$S                   10000000     U2Lang:U2Lang.dll
 0000:fffd9000       .debug$S                   10000000     U2Lang:U2Lang.dll
 0000:fffd9000       .debug$S                   10000000     U2Lang:U2Lang.dll
 0000:fffd9000       .debug$S                   10000000     U2Lang:U2Lang.dll
 0000:fffd9000       .debug$S                   10000000     U2Lang:U2Lang.dll
 0000:fffd9000       .debug$S                   10000000     U2Lang:U2Lang.dll
 0000:fffd9000       .debug$S                   10000000     U2Lang:U2Lang.dll
 0000:fffd9000       .debug$S                   10000000     U2Lang:U2Lang.dll
 0000:fffd9000       .debug$S                   10000000     U2Lang:U2Lang.dll
 0000:fffd9000       .debug$S                   10000000     U2Lang:U2Lang.dll
 0000:fffd9000       .debug$S                   10000000     U2Lang:U2Lang.dll
 0000:fffd9000       .debug$S                   10000000     U2Lang:U2Lang.dll
 0000:fffd9000       .debug$S                   10000000     U2Gui:U2Gui.dll
 0000:fffd9000       .debug$S                   10000000     U2Formats:U2Formats.dll
 0000:fffd9000       .debug$S                   10000000     U2Formats:U2Formats.dll
 0000:fffd9000       .debug$S                   10000000     U2Formats:U2Formats.dll
 0000:fffd9000       .debug$S                   10000000     U2Formats:U2Formats.dll
 0000:fffd9000       .debug$S                   10000000     U2Core:U2Core.dll
 0000:fffd9000       .debug$S                   10000000     U2Core:U2Core.dll
 0000:fffd9000       .debug$S                   10000000     U2Core:U2Core.dll
 0000:fffd9000       .debug$S                   10000000     U2Core:U2Core.dll
 0000:fffd9000       .debug$S                   10000000     U2Core:U2Core.dll
 0000:fffd9000       .debug$S                   10000000     U2Core:U2Core.dll
 0000:fffd9000       .debug$S                   10000000     U2Core:U2Core.dll
 0000:fffd9000       .debug$S                   10000000     U2Core:U2Core.dll
 0000:fffd9000       .debug$S                   10000000     U2Core:U2Core.dll
 0000:fffd9000       .debug$S                   10000000     U2Core:U2Core.dll
 0000:fffd9000       .debug$S                   10000000     U2Core:U2Core.dll
 0000:fffd9000       .debug$S                   10000000     U2Core:U2Core.dll
 0000:fffd9000       .debug$S                   10000000     U2Core:U2Core.dll
 0000:fffd9000       .debug$S                   10000000     U2Core:U2Core.dll
 0000:fffd9000       .debug$S                   10000000     U2Core:U2Core.dll
 0000:fffd9000       .debug$S                   10000000     U2Core:U2Core.dll
 0000:fffd9000       .debug$S                   10000000     U2Core:U2Core.dll
 0000:fffd9000       .debug$S                   10000000     U2Core:U2Core.dll
 0000:fffd9000       .debug$S                   10000000     U2Core:U2Core.dll
 0000:fffd9000       .debug$S                   10000000     U2Core:U2Core.dll
 0000:fffd9000       .debug$S                   10000000     U2Core:U2Core.dll
 0000:fffd9000       .debug$S                   10000000     U2Core:U2Core.dll
 0000:fffd9000       .debug$S                   10000000     U2Core:U2Core.dll
 0000:fffd9000       .debug$S                   10000000     U2Core:U2Core.dll
 0000:fffd9000       .debug$S                   10000000     U2Core:U2Core.dll
 0000:fffd9000       .debug$S                   10000000     U2Core:U2Core.dll
 0000:fffd9000       .debug$S                   10000000     U2Core:U2Core.dll
 0000:fffd9000       .debug$S                   10000000     U2Core:U2Core.dll
 0000:fffd9000       .debug$S                   10000000     U2Core:U2Core.dll
 0000:fffd9000       .debug$S                   10000000     U2Core:U2Core.dll
 0000:fffd9000       .debug$S                   10000000     U2Core:U2Core.dll
 0000:fffd9000       .debug$S                   10000000     U2Core:U2Core.dll
 0000:fffd9000       .debug$S                   10000000     U2Core:U2Core.dll
 0000:fffd9000       .debug$S                   10000000     U2Core:U2Core.dll
 0000:fffd9000       .debug$S                   10000000     U2Core:U2Core.dll
 0000:fffd9000       .debug$S                   10000000     U2Core:U2Core.dll
 0000:fffd9000       .debug$S                   10000000     U2Core:U2Core.dll
 0000:fffd9000       .debug$S                   10000000     U2Core:U2Core.dll
 0000:fffd9000       .debug$S                   10000000     U2Core:U2Core.dll
 0000:fffd9000       .debug$S                   10000000     U2Core:U2Core.dll
 0000:fffd9000       .debug$S                   10000000     U2Core:U2Core.dll
 0000:fffd9000       .debug$S                   10000000     U2Core:U2Core.dll
 0000:fffd9000       .debug$S                   10000000     U2Core:U2Core.dll
 0000:fffd9000       .debug$S                   10000000     U2Core:U2Core.dll
 0000:fffd9000       .debug$S                   10000000     U2Core:U2Core.dll
 0000:fffd9000       .debug$S                   10000000     U2Core:U2Core.dll
 0000:fffd9000       .debug$S                   10000000     U2Core:U2Core.dll
 0000:fffd9000       .debug$S                   10000000     U2Core:U2Core.dll
 0000:fffd9000       .debug$S                   10000000     U2Core:U2Core.dll
 0000:fffd9000       .debug$S                   10000000     U2Core:U2Core.dll
 0000:fffd9000       .debug$S                   10000000     U2Core:U2Core.dll
 0000:fffd9000       .debug$S                   10000000     U2Core:U2Core.dll
 0000:fffd9000       .debug$S                   10000000     U2Core:U2Core.dll
 0000:fffd9000       .debug$S                   10000000     U2Core:U2Core.dll
 0000:fffd9000       .debug$S                   10000000     U2Core:U2Core.dll
 0000:fffd9000       .debug$S                   10000000     U2Core:U2Core.dll
 0000:fffd9000       .debug$S                   10000000     U2Core:U2Core.dll
 0000:fffd9000       .debug$S                   10000000     U2Core:U2Core.dll
 0000:fffd9000       .debug$S                   10000000     U2Core:U2Core.dll
 0000:fffd9000       .debug$S                   10000000     U2Core:U2Core.dll
 0000:fffd9000       .debug$S                   10000000     U2Core:U2Core.dll
 0000:fffd9000       .debug$S                   10000000     U2Core:U2Core.dll
 0000:fffd9000       .debug$S                   10000000     U2Core:U2Core.dll
 0000:fffd9000       .debug$S                   10000000     U2Core:U2Core.dll
 0000:fffd9000       .debug$S                   10000000     U2Core:U2Core.dll
 0000:fffd9000       .debug$S                   10000000     U2Core:U2Core.dll
 0001:fffff000       __unwindfunclet$?createNode@?$QMapData@VQString@@VQVariant@@@@QAEPAU?$QMapNode@VQString@@VQVariant@@@@ABVQString@@ABVQVariant@@PAU2@_N@Z$4 10000000 f   WevoteWorkerFactory.obj
 0000:fffd9000       .debug$S                   10000000     U2Core:U2Core.dll
 0002:fffeb008       __ehfuncinfo$??H@YA?BVQString@@ABV0@0@Z 10000008     WevoteTask.obj
 0002:fffeb008       __ehfuncinfo$??A?$QMap@VQString@@VQVariant@@@@QAEAAVQVariant@@ABVQString@@@Z 10000008     WevoteWorkerFactory.obj
 0002:fffeb008       __ehfuncinfo$??H@YA?BVQString@@ABV0@0@Z 10000008     WevoteWorker.obj
 0001:fffff009       __ehhandler$??A?$QMap@VQString@@VQVariant@@@@QAEAAVQVariant@@ABVQString@@@Z 10000009 f   WevoteWorkerFactory.obj
 0001:fffff00c       __unwindfunclet$??0WevoteTaskSettings@U2@@QAE@ABU01@@Z$1 1000000c f   WevoteWorker.obj
 0001:fffff00c       __unwindfunclet$??1WevoteTaskSettings@U2@@QAE@XZ$1 1000000c f   WevoteWorker.obj
 0002:fffeb010       __catchsym$?_Copy@?$basic_string@DU?$char_traits@D@std@@V?$allocator@D@2@@std@@QAEXII@Z$4 10000010     moc_WevoteSupportPlugin.obj
 0002:fffeb010       __catchsym$?_Copy@?$basic_string@DU?$char_traits@D@std@@V?$allocator@D@2@@std@@QAEXII@Z$4 10000010     WevoteSupportPlugin.obj
 0002:fffeb010       __catchsym$?createNode@?$QMapData@VQString@@VQVariant@@@@QAEPAU?$QMapNode@VQString@@VQVariant@@@@ABVQString@@ABVQVariant@@PAU2@_N@Z$6 10000010     WevoteWorkerFactory.obj
 0002:fffeb010       __catchsym$?_Copy@?$basic_string@DU?$char_traits@D@std@@V?$allocator@D@2@@std@@QAEXII@Z$4 10000010     WevoteWorkerFactory.obj
 0002:fffeb010       __catchsym$?_Copy@?$basic_string@DU?$char_traits@D@std@@V?$allocator@D@2@@std@@QAEXII@Z$4 10000010     WevoteWorker.obj
 0002:fffeb010       __ehfuncinfo$??H@YA?BVQString@@ABV0@PBD@Z 10000010     WevoteWorkerFactory.obj
 0002:fffeb010       __catchsym$?_Copy@?$basic_string@DU?$char_traits@D@std@@V?$allocator@D@2@@std@@QAEXII@Z$4 10000010     moc_WevoteWorker.obj
 0002:fffeb010       __catchsym$?_Copy@?$basic_string@DU?$char_traits@D@std@@V?$allocator@D@2@@std@@QAEXII@Z$4 10000010     WevoteSupport.obj
 0002:fffeb010       __catchsym$?_Copy@?$basic_string@DU?$char_traits@D@std@@V?$allocator@D@2@@std@@QAEXII@Z$4 10000010     moc_WevotePrompter.obj
 0002:fffeb010       __ehfuncinfo$??H@YA?BVQString@@ABV0@PBD@Z 10000010     WevoteWorker.obj
 0002:fffeb010       __catchsym$?append@?$QList@VQString@@@@QAEXABVQString@@@Z$12 10000010     WevoteWorkerFactory.obj
 0002:fffeb010       __ehfuncinfo$??H@YA?BVQString@@ABV0@PBD@Z 10000010     WevoteTask.obj
 0002:fffeb010       __catchsym$?_Copy@?$basic_string@DU?$char_traits@D@std@@V?$allocator@D@2@@std@@QAEXII@Z$4 10000010     WevotePrompter.obj
 0002:fffeb010       __catchsym$?_Copy@?$basic_string@DU?$char_traits@D@std@@V?$allocator@D@2@@std@@QAEXII@Z$4 10000010     moc_WevoteTask.obj
 0002:fffeb010       __catchsym$?_Copy@?$basic_string@DU?$char_traits@D@std@@V?$allocator@D@2@@std@@QAEXII@Z$4 10000010     WevoteTask.obj
 0002:fffeb010       __catchsym$?detach_helper_grow@?$QList@VQString@@@@AAEPAUNode@1@HH@Z$4 10000010     WevoteWorkerFactory.obj
 0002:fffeb010       __catchsym$?_Copy@?$basic_string@DU?$char_traits@D@std@@V?$allocator@D@2@@std@@QAEXII@Z$4 10000010     WevoteValidator.obj
 0002:fffeb010       __ehfuncinfo$?node_construct@?$QList@VQString@@@@AAEXPAUNode@1@ABVQString@@@Z 10000010     WevoteWorkerFactory.obj
 0002:fffeb010       __tryblocktable$?createNode@?$QMapData@VQString@@I@@QAEPAU?$QMapNode@VQString@@I@@ABVQString@@ABIPAU2@_N@Z 10000010     WevoteWorker.obj
 0002:fffeb010       __ehfuncinfo$??1WevoteTaskSettings@U2@@QAE@XZ 10000010     WevoteWorker.obj
 0002:fffeb010       __ehfuncinfo$??0WevoteTaskSettings@U2@@QAE@ABU01@@Z 10000010     WevoteWorker.obj
 0002:fffeb010       __tryblocktable$?node_copy@?$QList@VQString@@@@AAEXPAUNode@1@00@Z 10000010     WevoteWorkerFactory.obj
 0001:fffff011       __ehhandler$?node_copy@?$QList@VQString@@@@AAEXPAUNode@1@00@Z 10000011 f   WevoteWorkerFactory.obj
 0001:fffff011       __ehhandler$?node_construct@?$QList@VQString@@@@AAEXPAUNode@1@ABVQString@@@Z 10000011 f   WevoteWorkerFactory.obj
 0001:fffff011       __unwindfunclet$?append@?$QList@VQString@@@@QAEXABVQString@@@Z$11 10000011 f   WevoteWorkerFactory.obj
 0001:fffff014       __ehhandler$?createNode@?$QMapData@VQString@@I@@QAEPAU?$QMapNode@VQString@@I@@ABVQString@@ABIPAU2@_N@Z 10000014 f   WevoteWorker.obj
 0001:fffff014       __unwindfunclet$?createNode@?$QMapData@VQString@@VQVariant@@@@QAEPAU?$QMapNode@VQString@@VQVariant@@@@ABVQString@@ABVQVariant@@PAU2@_N@Z$5 10000014 f   WevoteWorkerFactory.obj
 0001:fffff018       __ehhandler$??0WevoteTaskSettings@U2@@QAE@ABU01@@Z 10000018 f   WevoteWorker.obj
 0001:fffff018       __ehhandler$??1WevoteTaskSettings@U2@@QAE@XZ 10000018 f   WevoteWorker.obj
 0001:fffff01a       __ehhandler$??H@YA?BVQString@@ABV0@0@Z 1000001a f   WevoteWorker.obj
 0001:fffff01a       __unwindfunclet$??H@YA?BVQString@@ABV0@PBD@Z$1 1000001a f   WevoteTask.obj
 0001:fffff01a       __unwindfunclet$??H@YA?BVQString@@ABV0@PBD@Z$1 1000001a f   WevoteWorker.obj
 0001:fffff01a       __unwindfunclet$??H@YA?BVQString@@ABV0@PBD@Z$1 1000001a f   WevoteWorkerFactory.obj
 0001:fffff01a       __ehhandler$??H@YA?BVQString@@ABV0@0@Z 1000001a f   WevoteTask.obj
 0002:fffeb020       __unwindtable$?_Copy@?$basic_string@DU?$char_traits@D@std@@V?$allocator@D@2@@std@@QAEXII@Z 10000020     WevoteSupportPlugin.obj
 0002:fffeb020       __unwindtable$?_Copy@?$basic_string@DU?$char_traits@D@std@@V?$allocator@D@2@@std@@QAEXII@Z 10000020     moc_WevoteWorker.obj
 0002:fffeb020       __unwindtable$?_Copy@?$basic_string@DU?$char_traits@D@std@@V?$allocator@D@2@@std@@QAEXII@Z 10000020     WevoteWorker.obj
 0002:fffeb020       __unwindtable$?_Copy@?$basic_string@DU?$char_traits@D@std@@V?$allocator@D@2@@std@@QAEXII@Z 10000020     WevotePrompter.obj
 0002:fffeb020       __unwindtable$?_Copy@?$basic_string@DU?$char_traits@D@std@@V?$allocator@D@2@@std@@QAEXII@Z 10000020     moc_WevotePrompter.obj
 0002:fffeb020       __unwindtable$?_Copy@?$basic_string@DU?$char_traits@D@std@@V?$allocator@D@2@@std@@QAEXII@Z 10000020     WevoteSupport.obj
 0002:fffeb020       __unwindtable$?_Copy@?$basic_string@DU?$char_traits@D@std@@V?$allocator@D@2@@std@@QAEXII@Z 10000020     moc_WevoteTask.obj
 0002:fffeb020       __unwindtable$?_Copy@?$basic_string@DU?$char_traits@D@std@@V?$allocator@D@2@@std@@QAEXII@Z 10000020     WevoteWorkerFactory.obj
 0002:fffeb020       __unwindtable$?detach_helper_grow@?$QList@VQString@@@@AAEPAUNode@1@HH@Z 10000020     WevoteWorkerFactory.obj
 0002:fffeb020       __ehfuncinfo$?append@?$QList@VQString@@@@QAEXABVQString@@@Z 10000020     WevoteWorkerFactory.obj
 0002:fffeb020       __ehfuncinfo$?createNode@?$QMapData@VQString@@VQVariant@@@@QAEPAU?$QMapNode@VQString@@VQVariant@@@@ABVQString@@ABVQVariant@@PAU2@_N@Z 10000020     WevoteWorkerFactory.obj
 0002:fffeb020       __unwindtable$?_Copy@?$basic_string@DU?$char_traits@D@std@@V?$allocator@D@2@@std@@QAEXII@Z 10000020     WevoteValidator.obj
 0002:fffeb020       __unwindtable$?_Copy@?$basic_string@DU?$char_traits@D@std@@V?$allocator@D@2@@std@@QAEXII@Z 10000020     moc_WevoteSupportPlugin.obj
 0002:fffeb020       __unwindtable$?_Copy@?$basic_string@DU?$char_traits@D@std@@V?$allocator@D@2@@std@@QAEXII@Z 10000020     WevoteTask.obj
 0001:fffff022       __ehhandler$?append@?$QList@VQString@@@@QAEXABVQString@@@Z 10000022 f   WevoteWorkerFactory.obj
 0001:fffff023       __ehhandler$??H@YA?BVQString@@ABV0@PBD@Z 10000023 f   WevoteWorkerFactory.obj
 0001:fffff023       __ehhandler$??H@YA?BVQString@@ABV0@PBD@Z 10000023 f   WevoteTask.obj
 0001:fffff023       __ehhandler$??H@YA?BVQString@@ABV0@PBD@Z 10000023 f   WevoteWorker.obj
 0002:fffeb024       __ehfuncinfo$?node_copy@?$QList@VQString@@@@AAEXPAUNode@1@00@Z 10000024     WevoteWorkerFactory.obj
 0002:fffeb024       __ehfuncinfo$?createNode@?$QMapData@VQString@@I@@QAEPAU?$QMapNode@VQString@@I@@ABVQString@@ABIPAU2@_N@Z 10000024     WevoteWorker.obj
 0001:fffff028       __ehhandler$?createNode@?$QMapData@VQString@@VQVariant@@@@QAEPAU?$QMapNode@VQString@@VQVariant@@@@ABVQString@@ABVQVariant@@PAU2@_N@Z 10000028 f   WevoteWorkerFactory.obj
 0002:fffeb040       __ehfuncinfo$?_Copy@?$basic_string@DU?$char_traits@D@std@@V?$allocator@D@2@@std@@QAEXII@Z 10000040     WevoteTask.obj
 0002:fffeb040       __ehfuncinfo$?detach_helper_grow@?$QList@VQString@@@@AAEPAUNode@1@HH@Z 10000040     WevoteWorkerFactory.obj
 0002:fffeb040       __ehfuncinfo$?_Copy@?$basic_string@DU?$char_traits@D@std@@V?$allocator@D@2@@std@@QAEXII@Z 10000040     WevoteValidator.obj
 0002:fffeb040       __ehfuncinfo$?_Copy@?$basic_string@DU?$char_traits@D@std@@V?$allocator@D@2@@std@@QAEXII@Z 10000040     moc_WevoteSupportPlugin.obj
 0002:fffeb040       __ehfuncinfo$?_Copy@?$basic_string@DU?$char_traits@D@std@@V?$allocator@D@2@@std@@QAEXII@Z 10000040     WevotePrompter.obj
 0002:fffeb040       __ehfuncinfo$?_Copy@?$basic_string@DU?$char_traits@D@std@@V?$allocator@D@2@@std@@QAEXII@Z 10000040     WevoteWorkerFactory.obj
 0002:fffeb040       __ehfuncinfo$?_Copy@?$basic_string@DU?$char_traits@D@std@@V?$allocator@D@2@@std@@QAEXII@Z 10000040     moc_WevoteWorker.obj
 0002:fffeb040       __ehfuncinfo$?_Copy@?$basic_string@DU?$char_traits@D@std@@V?$allocator@D@2@@std@@QAEXII@Z 10000040     moc_WevotePrompter.obj
 0002:fffeb040       __ehfuncinfo$?_Copy@?$basic_string@DU?$char_traits@D@std@@V?$allocator@D@2@@std@@QAEXII@Z 10000040     WevoteSupport.obj
 0002:fffeb040       __ehfuncinfo$?_Copy@?$basic_string@DU?$char_traits@D@std@@V?$allocator@D@2@@std@@QAEXII@Z 10000040     WevoteSupportPlugin.obj
 0002:fffeb040       __ehfuncinfo$?_Copy@?$basic_string@DU?$char_traits@D@std@@V?$allocator@D@2@@std@@QAEXII@Z 10000040     WevoteWorker.obj
 0002:fffeb040       __ehfuncinfo$?_Copy@?$basic_string@DU?$char_traits@D@std@@V?$allocator@D@2@@std@@QAEXII@Z 10000040     moc_WevoteTask.obj
 0002:fffeb044       __tryblocktable$?append@?$QList@VQString@@@@QAEXABVQString@@@Z 10000044     WevoteWorkerFactory.obj
 0002:fffeb044       __tryblocktable$?createNode@?$QMapData@VQString@@VQVariant@@@@QAEPAU?$QMapNode@VQString@@VQVariant@@@@ABVQString@@ABVQVariant@@PAU2@_N@Z 10000044     WevoteWorkerFactory.obj
 0002:fffeb048       __unwindtable$?createNode@?$QMapData@VQString@@I@@QAEPAU?$QMapNode@VQString@@I@@ABVQString@@ABIPAU2@_N@Z 10000048     WevoteWorker.obj
 0002:fffeb048       __unwindtable$?node_copy@?$QList@VQString@@@@AAEXPAUNode@1@00@Z 10000048     WevoteWorkerFactory.obj
 0001:fffff062       __catch$?node_copy@?$QList@VQString@@@@AAEXPAUNode@1@00@Z$2 10000062 f   WevoteWorkerFactory.obj
 0002:fffeb064       __tryblocktable$?_Copy@?$basic_string@DU?$char_traits@D@std@@V?$allocator@D@2@@std@@QAEXII@Z 10000064     WevoteWorkerFactory.obj
 0002:fffeb064       __tryblocktable$?_Copy@?$basic_string@DU?$char_traits@D@std@@V?$allocator@D@2@@std@@QAEXII@Z 10000064     WevoteWorker.obj
 0002:fffeb064       __tryblocktable$?_Copy@?$basic_string@DU?$char_traits@D@std@@V?$allocator@D@2@@std@@QAEXII@Z 10000064     moc_WevoteTask.obj
 0002:fffeb064       __tryblocktable$?_Copy@?$basic_string@DU?$char_traits@D@std@@V?$allocator@D@2@@std@@QAEXII@Z 10000064     moc_WevoteWorker.obj
 0002:fffeb064       __tryblocktable$?_Copy@?$basic_string@DU?$char_traits@D@std@@V?$allocator@D@2@@std@@QAEXII@Z 10000064     WevoteSupport.obj
 0002:fffeb064       __tryblocktable$?_Copy@?$basic_string@DU?$char_traits@D@std@@V?$allocator@D@2@@std@@QAEXII@Z 10000064     moc_WevotePrompter.obj
 0002:fffeb064       __tryblocktable$?_Copy@?$basic_string@DU?$char_traits@D@std@@V?$allocator@D@2@@std@@QAEXII@Z 10000064     WevoteSupportPlugin.obj
 0002:fffeb064       __tryblocktable$?_Copy@?$basic_string@DU?$char_traits@D@std@@V?$allocator@D@2@@std@@QAEXII@Z 10000064     WevoteTask.obj
 0002:fffeb064       __tryblocktable$?detach_helper_grow@?$QList@VQString@@@@AAEPAUNode@1@HH@Z 10000064     WevoteWorkerFactory.obj
 0002:fffeb064       __tryblocktable$?_Copy@?$basic_string@DU?$char_traits@D@std@@V?$allocator@D@2@@std@@QAEXII@Z 10000064     moc_WevoteSupportPlugin.obj
 0002:fffeb064       __tryblocktable$?_Copy@?$basic_string@DU?$char_traits@D@std@@V?$allocator@D@2@@std@@QAEXII@Z 10000064     WevoteValidator.obj
 0002:fffeb064       __tryblocktable$?_Copy@?$basic_string@DU?$char_traits@D@std@@V?$allocator@D@2@@std@@QAEXII@Z 10000064     WevotePrompter.obj
 0002:fffeb06c       __unwindtable$?createNode@?$QMapData@VQString@@VQVariant@@@@QAEPAU?$QMapNode@VQString@@VQVariant@@@@ABVQString@@ABVQVariant@@PAU2@_N@Z 1000006c     WevoteWorkerFactory.obj
 0002:fffeb06c       __unwindtable$?append@?$QList@VQString@@@@QAEXABVQString@@@Z 1000006c     WevoteWorkerFactory.obj
 0001:fffff07d       __catch$?append@?$QList@VQString@@@@QAEXABVQString@@@Z$0 1000007d f   WevoteWorkerFactory.obj
 0001:fffff085       __catch$?createNode@?$QMapData@VQString@@I@@QAEPAU?$QMapNode@VQString@@I@@ABVQString@@ABIPAU2@_N@Z$2 10000085 f   WevoteWorker.obj
 0001:fffff08e       __catch$?createNode@?$QMapData@VQString@@VQVariant@@@@QAEPAU?$QMapNode@VQString@@VQVariant@@@@ABVQString@@ABVQVariant@@PAU2@_N@Z$0 1000008e f   WevoteWorkerFactory.obj
 0001:fffff096       __catch$?_Copy@?$basic_string@DU?$char_traits@D@std@@V?$allocator@D@2@@std@@QAEXII@Z$0 10000096 f   WevoteSupport.obj
 0001:fffff096       __catch$?_Copy@?$basic_string@DU?$char_traits@D@std@@V?$allocator@D@2@@std@@QAEXII@Z$0 10000096 f   moc_WevoteSupportPlugin.obj
 0001:fffff096       __catch$?_Copy@?$basic_string@DU?$char_traits@D@std@@V?$allocator@D@2@@std@@QAEXII@Z$0 10000096 f   moc_WevotePrompter.obj
 0001:fffff096       __catch$?_Copy@?$basic_string@DU?$char_traits@D@std@@V?$allocator@D@2@@std@@QAEXII@Z$0 10000096 f   WevoteWorkerFactory.obj
 0001:fffff096       __catch$?_Copy@?$basic_string@DU?$char_traits@D@std@@V?$allocator@D@2@@std@@QAEXII@Z$0 10000096 f   WevotePrompter.obj
 0001:fffff096       __catch$?_Copy@?$basic_string@DU?$char_traits@D@std@@V?$allocator@D@2@@std@@QAEXII@Z$0 10000096 f   WevoteValidator.obj
 0001:fffff096       __catch$?_Copy@?$basic_string@DU?$char_traits@D@std@@V?$allocator@D@2@@std@@QAEXII@Z$0 10000096 f   WevoteTask.obj
 0001:fffff096       __catch$?_Copy@?$basic_string@DU?$char_traits@D@std@@V?$allocator@D@2@@std@@QAEXII@Z$0 10000096 f   moc_WevoteTask.obj
 0001:fffff096       __catch$?_Copy@?$basic_string@DU?$char_traits@D@std@@V?$allocator@D@2@@std@@QAEXII@Z$0 10000096 f   moc_WevoteWorker.obj
 0001:fffff096       __catch$?_Copy@?$basic_string@DU?$char_traits@D@std@@V?$allocator@D@2@@std@@QAEXII@Z$0 10000096 f   WevoteSupportPlugin.obj
 0001:fffff096       __catch$?_Copy@?$basic_string@DU?$char_traits@D@std@@V?$allocator@D@2@@std@@QAEXII@Z$0 10000096 f   WevoteWorker.obj
 0001:fffff0a3       __catch$?createNode@?$QMapData@VQString@@VQVariant@@@@QAEPAU?$QMapNode@VQString@@VQVariant@@@@ABVQString@@ABVQVariant@@PAU2@_N@Z$2 100000a3 f   WevoteWorkerFactory.obj
 0001:fffff0ce       __catch$?append@?$QList@VQString@@@@QAEXABVQString@@@Z$4 100000ce f   WevoteWorkerFactory.obj
 0001:fffff0d3       __catch$?_Copy@?$basic_string@DU?$char_traits@D@std@@V?$allocator@D@2@@std@@QAEXII@Z$1 100000d3 f   moc_WevoteSupportPlugin.obj
 0001:fffff0d3       __catch$?_Copy@?$basic_string@DU?$char_traits@D@std@@V?$allocator@D@2@@std@@QAEXII@Z$1 100000d3 f   moc_WevotePrompter.obj
 0001:fffff0d3       __catch$?_Copy@?$basic_string@DU?$char_traits@D@std@@V?$allocator@D@2@@std@@QAEXII@Z$1 100000d3 f   WevoteSupportPlugin.obj
 0001:fffff0d3       __catch$?_Copy@?$basic_string@DU?$char_traits@D@std@@V?$allocator@D@2@@std@@QAEXII@Z$1 100000d3 f   WevoteSupport.obj
 0001:fffff0d3       __catch$?_Copy@?$basic_string@DU?$char_traits@D@std@@V?$allocator@D@2@@std@@QAEXII@Z$1 100000d3 f   WevoteTask.obj
 0001:fffff0d3       __catch$?_Copy@?$basic_string@DU?$char_traits@D@std@@V?$allocator@D@2@@std@@QAEXII@Z$1 100000d3 f   WevoteWorkerFactory.obj
 0001:fffff0d3       __catch$?_Copy@?$basic_string@DU?$char_traits@D@std@@V?$allocator@D@2@@std@@QAEXII@Z$1 100000d3 f   WevotePrompter.obj
 0001:fffff0d3       __catch$?_Copy@?$basic_string@DU?$char_traits@D@std@@V?$allocator@D@2@@std@@QAEXII@Z$1 100000d3 f   WevoteWorker.obj
 0001:fffff0d3       __catch$?_Copy@?$basic_string@DU?$char_traits@D@std@@V?$allocator@D@2@@std@@QAEXII@Z$1 100000d3 f   moc_WevoteTask.obj
 0001:fffff0d3       __catch$?_Copy@?$basic_string@DU?$char_traits@D@std@@V?$allocator@D@2@@std@@QAEXII@Z$1 100000d3 f   moc_WevoteWorker.obj
 0001:fffff0d3       __catch$?_Copy@?$basic_string@DU?$char_traits@D@std@@V?$allocator@D@2@@std@@QAEXII@Z$1 100000d3 f   WevoteValidator.obj
 0001:fffff11e       __catch$?detach_helper_grow@?$QList@VQString@@@@AAEPAUNode@1@HH@Z$2 1000011e f   WevoteWorkerFactory.obj
 0001:fffff159       __catch$?detach_helper_grow@?$QList@VQString@@@@AAEPAUNode@1@HH@Z$0 10000159 f   WevoteWorkerFactory.obj
 0001:00000000       ??__E?SCIENTIFIC_NAME@PrepareWevoteTaxonomyDataTask@U2@@0VQString@@B@@YAXXZ 10001000 f   PrepareWevoteTaxonomyDataTask.obj
 0001:00000020       ??__E?WEVOTE_DIR@PrepareWevoteTaxonomyDataTask@U2@@0VQString@@B@@YAXXZ 10001020 f   PrepareWevoteTaxonomyDataTask.obj
 0001:00000040       ??__E?WEVOTE_NAMES@PrepareWevoteTaxonomyDataTask@U2@@0VQString@@B@@YAXXZ 10001040 f   PrepareWevoteTaxonomyDataTask.obj
 0001:00000060       ??__E?WEVOTE_NODES@PrepareWevoteTaxonomyDataTask@U2@@0VQString@@B@@YAXXZ 10001060 f   PrepareWevoteTaxonomyDataTask.obj
 0001:00000080       ??__E?_Generic_object@?$_Error_objects@H@std@@2V_Generic_error_category@2@A@@YAXXZ 10001080 f   PrepareWevoteTaxonomyDataTask.obj
 0001:00000090       ??__E?_Iostream_object@?$_Error_objects@H@std@@2V_Iostream_error_category@2@A@@YAXXZ 10001090 f   PrepareWevoteTaxonomyDataTask.obj
 0001:000000a0       ??__E?_System_object@?$_Error_objects@H@std@@2V_System_error_category@2@A@@YAXXZ 100010a0 f   PrepareWevoteTaxonomyDataTask.obj
 0001:000000b0       ??__EalgoLog@U2@@YAXXZ     100010b0 f   PrepareWevoteTaxonomyDataTask.obj
 0001:00000130       ??__EcmdLog@U2@@YAXXZ      10001130 f   PrepareWevoteTaxonomyDataTask.obj
 0001:000001b0       ??__EcoreLog@U2@@YAXXZ     100011b0 f   PrepareWevoteTaxonomyDataTask.obj
 0001:00000230       ??__EioLog@U2@@YAXXZ       10001230 f   PrepareWevoteTaxonomyDataTask.obj
 0001:000002b0       ??__EperfLog@U2@@YAXXZ     100012b0 f   PrepareWevoteTaxonomyDataTask.obj
 0001:00000330       ??__EscriptLog@U2@@YAXXZ   10001330 f   PrepareWevoteTaxonomyDataTask.obj
 0001:000003b0       ??__EtaskLog@U2@@YAXXZ     100013b0 f   PrepareWevoteTaxonomyDataTask.obj
 0001:00000430       ??__EuiLog@U2@@YAXXZ       10001430 f   PrepareWevoteTaxonomyDataTask.obj
 0001:000004b0       ??__EuserActLog@U2@@YAXXZ  100014b0 f   PrepareWevoteTaxonomyDataTask.obj
 0001:00000530       ??__E?_Generic_object@?$_Error_objects@H@std@@2V_Generic_error_category@2@A@@YAXXZ 10001530 f   WevotePrompter.obj
 0001:00000540       ??__E?_Iostream_object@?$_Error_objects@H@std@@2V_Iostream_error_category@2@A@@YAXXZ 10001540 f   WevotePrompter.obj
 0001:00000550       ??__E?_System_object@?$_Error_objects@H@std@@2V_System_error_category@2@A@@YAXXZ 10001550 f   WevotePrompter.obj
 0001:00000560       ??__EalgoLog@U2@@YAXXZ     10001560 f   WevotePrompter.obj
 0001:000005e0       ??__EcmdLog@U2@@YAXXZ      100015e0 f   WevotePrompter.obj
 0001:00000660       ??__EcoreLog@U2@@YAXXZ     10001660 f   WevotePrompter.obj
 0001:000006e0       ??__EioLog@U2@@YAXXZ       100016e0 f   WevotePrompter.obj
 0001:00000760       ??__EperfLog@U2@@YAXXZ     10001760 f   WevotePrompter.obj
 0001:000007e0       ??__EscriptLog@U2@@YAXXZ   100017e0 f   WevotePrompter.obj
 0001:00000860       ??__EtaskLog@U2@@YAXXZ     10001860 f   WevotePrompter.obj
 0001:000008e0       ??__EuiLog@U2@@YAXXZ       100018e0 f   WevotePrompter.obj
 0001:00000960       ??__EuserActLog@U2@@YAXXZ  10001960 f   WevotePrompter.obj
 0001:000009e0       ??__E?TOOL_NAME@WevoteSupport@U2@@2VQString@@B@@YAXXZ 100019e0 f   WevoteSupport.obj
 0001:00000a00       ??__E?_Generic_object@?$_Error_objects@H@std@@2V_Generic_error_category@2@A@@YAXXZ 10001a00 f   WevoteSupport.obj
 0001:00000a10       ??__E?_Iostream_object@?$_Error_objects@H@std@@2V_Iostream_error_category@2@A@@YAXXZ 10001a10 f   WevoteSupport.obj
 0001:00000a20       ??__E?_System_object@?$_Error_objects@H@std@@2V_System_error_category@2@A@@YAXXZ 10001a20 f   WevoteSupport.obj
 0001:00000a30       ??__E?PLUGIN_DESCRIPRION@WevoteSupportPlugin@U2@@2VQString@@B@@YAXXZ 10001a30 f   WevoteSupportPlugin.obj
 0001:00000a60       ??__E?PLUGIN_NAME@WevoteSupportPlugin@U2@@2VQString@@B@@YAXXZ 10001a60 f   WevoteSupportPlugin.obj
 0001:00000a90       ??__E?_Generic_object@?$_Error_objects@H@std@@2V_Generic_error_category@2@A@@YAXXZ 10001a90 f   WevoteSupportPlugin.obj
 0001:00000aa0       ??__E?_Iostream_object@?$_Error_objects@H@std@@2V_Iostream_error_category@2@A@@YAXXZ 10001aa0 f   WevoteSupportPlugin.obj
 0001:00000ab0       ??__E?_System_object@?$_Error_objects@H@std@@2V_System_error_category@2@A@@YAXXZ 10001ab0 f   WevoteSupportPlugin.obj
 0001:00000ac0       ??__EalgoLog@U2@@YAXXZ     10001ac0 f   WevoteSupportPlugin.obj
 0001:00000b40       ??__EcmdLog@U2@@YAXXZ      10001b40 f   WevoteSupportPlugin.obj
 0001:00000bc0       ??__EcoreLog@U2@@YAXXZ     10001bc0 f   WevoteSupportPlugin.obj
 0001:00000c40       ??__EioLog@U2@@YAXXZ       10001c40 f   WevoteSupportPlugin.obj
 0001:00000cc0       ??__EperfLog@U2@@YAXXZ     10001cc0 f   WevoteSupportPlugin.obj
 0001:00000d40       ??__EscriptLog@U2@@YAXXZ   10001d40 f   WevoteSupportPlugin.obj
 0001:00000dc0       ??__EtaskLog@U2@@YAXXZ     10001dc0 f   WevoteSupportPlugin.obj
 0001:00000e40       ??__EuiLog@U2@@YAXXZ       10001e40 f   WevoteSupportPlugin.obj
 0001:00000ec0       ??__EuserActLog@U2@@YAXXZ  10001ec0 f   WevoteSupportPlugin.obj
 0001:00000f40       ??__E?SUFFIX@WevoteTask@U2@@2VQString@@B@@YAXXZ 10001f40 f   WevoteTask.obj
 0001:00000f60       ??__E?_Generic_object@?$_Error_objects@H@std@@2V_Generic_error_category@2@A@@YAXXZ 10001f60 f   WevoteTask.obj
 0001:00000f70       ??__E?_Iostream_object@?$_Error_objects@H@std@@2V_Iostream_error_category@2@A@@YAXXZ 10001f70 f   WevoteTask.obj
 0001:00000f80       ??__E?_System_object@?$_Error_objects@H@std@@2V_System_error_category@2@A@@YAXXZ 10001f80 f   WevoteTask.obj
 0001:00000f90       ??__EalgoLog@U2@@YAXXZ     10001f90 f   WevoteTask.obj
 0001:00001010       ??__EcmdLog@U2@@YAXXZ      10002010 f   WevoteTask.obj
 0001:00001090       ??__EcoreLog@U2@@YAXXZ     10002090 f   WevoteTask.obj
 0001:00001110       ??__EioLog@U2@@YAXXZ       10002110 f   WevoteTask.obj
 0001:00001190       ??__EperfLog@U2@@YAXXZ     10002190 f   WevoteTask.obj
 0001:00001210       ??__EscriptLog@U2@@YAXXZ   10002210 f   WevoteTask.obj
 0001:00001290       ??__EtaskLog@U2@@YAXXZ     10002290 f   WevoteTask.obj
 0001:00001310       ??__EuiLog@U2@@YAXXZ       10002310 f   WevoteTask.obj
 0001:00001390       ??__EuserActLog@U2@@YAXXZ  10002390 f   WevoteTask.obj
 0001:00001410       ??__E?_Generic_object@?$_Error_objects@H@std@@2V_Generic_error_category@2@A@@YAXXZ 10002410 f   WevoteValidator.obj
 0001:00001420       ??__E?_Iostream_object@?$_Error_objects@H@std@@2V_Iostream_error_category@2@A@@YAXXZ 10002420 f   WevoteValidator.obj
 0001:00001430       ??__E?_System_object@?$_Error_objects@H@std@@2V_System_error_category@2@A@@YAXXZ 10002430 f   WevoteValidator.obj
 0001:00001440       ??__EalgoLog@U2@@YAXXZ     10002440 f   WevoteValidator.obj
 0001:000014c0       ??__EcmdLog@U2@@YAXXZ      100024c0 f   WevoteValidator.obj
 0001:00001540       ??__EcoreLog@U2@@YAXXZ     10002540 f   WevoteValidator.obj
 0001:000015c0       ??__EioLog@U2@@YAXXZ       100025c0 f   WevoteValidator.obj
 0001:00001640       ??__EperfLog@U2@@YAXXZ     10002640 f   WevoteValidator.obj
 0001:000016c0       ??__EscriptLog@U2@@YAXXZ   100026c0 f   WevoteValidator.obj
 0001:00001740       ??__EtaskLog@U2@@YAXXZ     10002740 f   WevoteValidator.obj
 0001:000017c0       ??__EuiLog@U2@@YAXXZ       100027c0 f   WevoteValidator.obj
 0001:00001840       ??__EuserActLog@U2@@YAXXZ  10002840 f   WevoteValidator.obj
 0001:000018c0       ??__E?WEVOTE_DIR@WevoteWorker@LocalWorkflow@U2@@0VQString@@B@@YAXXZ 100028c0 f   WevoteWorker.obj
 0001:000018e0       ??__E?_Generic_object@?$_Error_objects@H@std@@2V_Generic_error_category@2@A@@YAXXZ 100028e0 f   WevoteWorker.obj
 0001:000018f0       ??__E?_Iostream_object@?$_Error_objects@H@std@@2V_Iostream_error_category@2@A@@YAXXZ 100028f0 f   WevoteWorker.obj
 0001:00001900       ??__E?_System_object@?$_Error_objects@H@std@@2V_System_error_category@2@A@@YAXXZ 10002900 f   WevoteWorker.obj
 0001:00001910       ??__EalgoLog@U2@@YAXXZ     10002910 f   WevoteWorker.obj
 0001:00001990       ??__EcmdLog@U2@@YAXXZ      10002990 f   WevoteWorker.obj
 0001:00001a10       ??__EcoreLog@U2@@YAXXZ     10002a10 f   WevoteWorker.obj
 0001:00001a90       ??__EioLog@U2@@YAXXZ       10002a90 f   WevoteWorker.obj
 0001:00001b10       ??__EperfLog@U2@@YAXXZ     10002b10 f   WevoteWorker.obj
 0001:00001b90       ??__EscriptLog@U2@@YAXXZ   10002b90 f   WevoteWorker.obj
 0001:00001c10       ??__EtaskLog@U2@@YAXXZ     10002c10 f   WevoteWorker.obj
 0001:00001c90       ??__EuiLog@U2@@YAXXZ       10002c90 f   WevoteWorker.obj
 0001:00001d10       ??__EuserActLog@U2@@YAXXZ  10002d10 f   WevoteWorker.obj
 0001:00001d90       ??__E?ACTOR_ID@WevoteWorkerFactory@LocalWorkflow@U2@@2VQString@@B@@YAXXZ 10002d90 f   WevoteWorkerFactory.obj
 0001:00001db0       ??__E?INPUT_PORT_ID@WevoteWorkerFactory@LocalWorkflow@U2@@2VQString@@B@@YAXXZ 10002db0 f   WevoteWorkerFactory.obj
 0001:00001dd0       ??__E?NUMBER_OF_AGREED_TOOLS_ATTR_ID@WevoteWorkerFactory@LocalWorkflow@U2@@2VQString@@B@@YAXXZ 10002dd0 f   WevoteWorkerFactory.obj
 0001:00001df0       ??__E?NUMBER_OF_THREADS_ATTR_ID@WevoteWorkerFactory@LocalWorkflow@U2@@2VQString@@B@@YAXXZ 10002df0 f   WevoteWorkerFactory.obj
 0001:00001e10       ??__E?OUTPUT_FILE_ATTR_ID@WevoteWorkerFactory@LocalWorkflow@U2@@2VQString@@B@@YAXXZ 10002e10 f   WevoteWorkerFactory.obj
 0001:00001e30       ??__E?OUTPUT_PORT_ID@WevoteWorkerFactory@LocalWorkflow@U2@@2VQString@@B@@YAXXZ 10002e30 f   WevoteWorkerFactory.obj
 0001:00001e50       ??__E?PENALTY_ATTR_ID@WevoteWorkerFactory@LocalWorkflow@U2@@2VQString@@B@@YAXXZ 10002e50 f   WevoteWorkerFactory.obj
 0001:00001e70       ??__E?SCORE_THRESHOLD_ATTR_ID@WevoteWorkerFactory@LocalWorkflow@U2@@2VQString@@B@@YAXXZ 10002e70 f   WevoteWorkerFactory.obj
 0001:00001e90       ??__E?WORKFLOW_CLASSIFY_TOOL_WEVOTE@WevoteWorkerFactory@LocalWorkflow@U2@@2VQString@@B@@YAXXZ 10002e90 f   WevoteWorkerFactory.obj
 0001:00001eb0       ??__E?_Generic_object@?$_Error_objects@H@std@@2V_Generic_error_category@2@A@@YAXXZ 10002eb0 f   WevoteWorkerFactory.obj
 0001:00001ec0       ??__E?_Iostream_object@?$_Error_objects@H@std@@2V_Iostream_error_category@2@A@@YAXXZ 10002ec0 f   WevoteWorkerFactory.obj
 0001:00001ed0       ??__E?_System_object@?$_Error_objects@H@std@@2V_System_error_category@2@A@@YAXXZ 10002ed0 f   WevoteWorkerFactory.obj
 0001:00001ee0       ??__EalgoLog@U2@@YAXXZ     10002ee0 f   WevoteWorkerFactory.obj
 0001:00001f60       ??__EcmdLog@U2@@YAXXZ      10002f60 f   WevoteWorkerFactory.obj
 0001:00001fe0       ??__EcoreLog@U2@@YAXXZ     10002fe0 f   WevoteWorkerFactory.obj
 0001:00002060       ??__EioLog@U2@@YAXXZ       10003060 f   WevoteWorkerFactory.obj
 0001:000020e0       ??__EperfLog@U2@@YAXXZ     100030e0 f   WevoteWorkerFactory.obj
 0001:00002160       ??__EscriptLog@U2@@YAXXZ   10003160 f   WevoteWorkerFactory.obj
 0001:000021e0       ??__EtaskLog@U2@@YAXXZ     100031e0 f   WevoteWorkerFactory.obj
 0001:00002260       ??__EuiLog@U2@@YAXXZ       10003260 f   WevoteWorkerFactory.obj
 0001:000022e0       ??__EuserActLog@U2@@YAXXZ  100032e0 f   WevoteWorkerFactory.obj
 0001:00002360       ??__E?_Generic_object@?$_Error_objects@H@std@@2V_Generic_error_category@2@A@@YAXXZ 10003360 f   moc_WevotePrompter.obj
 0001:00002370       ??__E?_Iostream_object@?$_Error_objects@H@std@@2V_Iostream_error_category@2@A@@YAXXZ 10003370 f   moc_WevotePrompter.obj
 0001:00002380       ??__E?_System_object@?$_Error_objects@H@std@@2V_System_error_category@2@A@@YAXXZ 10003380 f   moc_WevotePrompter.obj
 0001:00002390       ??__E?staticMetaObject@WevotePrompter@LocalWorkflow@U2@@2UQMetaObject@@B@@YAXXZ 10003390 f   moc_WevotePrompter.obj
 0001:000023a0       ??__EalgoLog@U2@@YAXXZ     100033a0 f   moc_WevotePrompter.obj
 0001:00002420       ??__EcmdLog@U2@@YAXXZ      10003420 f   moc_WevotePrompter.obj
 0001:000024a0       ??__EcoreLog@U2@@YAXXZ     100034a0 f   moc_WevotePrompter.obj
 0001:00002520       ??__EioLog@U2@@YAXXZ       10003520 f   moc_WevotePrompter.obj
 0001:000025a0       ??__EperfLog@U2@@YAXXZ     100035a0 f   moc_WevotePrompter.obj
 0001:00002620       ??__EscriptLog@U2@@YAXXZ   10003620 f   moc_WevotePrompter.obj
 0001:000026a0       ??__EtaskLog@U2@@YAXXZ     100036a0 f   moc_WevotePrompter.obj
 0001:00002720       ??__EuiLog@U2@@YAXXZ       10003720 f   moc_WevotePrompter.obj
 0001:000027a0       ??__EuserActLog@U2@@YAXXZ  100037a0 f   moc_WevotePrompter.obj
 0001:00002820       ??__E?_Generic_object@?$_Error_objects@H@std@@2V_Generic_error_category@2@A@@YAXXZ 10003820 f   moc_WevoteSupportPlugin.obj
 0001:00002830       ??__E?_Iostream_object@?$_Error_objects@H@std@@2V_Iostream_error_category@2@A@@YAXXZ 10003830 f   moc_WevoteSupportPlugin.obj
 0001:00002840       ??__E?_System_object@?$_Error_objects@H@std@@2V_System_error_category@2@A@@YAXXZ 10003840 f   moc_WevoteSupportPlugin.obj
 0001:00002850       ??__E?staticMetaObject@WevoteSupportPlugin@U2@@2UQMetaObject@@B@@YAXXZ 10003850 f   moc_WevoteSupportPlugin.obj
 0001:00002860       ??__E?_Generic_object@?$_Error_objects@H@std@@2V_Generic_error_category@2@A@@YAXXZ 10003860 f   moc_WevoteTask.obj
 0001:00002870       ??__E?_Iostream_object@?$_Error_objects@H@std@@2V_Iostream_error_category@2@A@@YAXXZ 10003870 f   moc_WevoteTask.obj
 0001:00002880       ??__E?_System_object@?$_Error_objects@H@std@@2V_System_error_category@2@A@@YAXXZ 10003880 f   moc_WevoteTask.obj
 0001:00002890       ??__E?staticMetaObject@WevoteTask@U2@@2UQMetaObject@@B@@YAXXZ 10003890 f   moc_WevoteTask.obj
 0001:000028a0       ??__EalgoLog@U2@@YAXXZ     100038a0 f   moc_WevoteTask.obj
 0001:00002920       ??__EcmdLog@U2@@YAXXZ      10003920 f   moc_WevoteTask.obj
 0001:000029a0       ??__EcoreLog@U2@@YAXXZ     100039a0 f   moc_WevoteTask.obj
 0001:00002a20       ??__EioLog@U2@@YAXXZ       10003a20 f   moc_WevoteTask.obj
 0001:00002aa0       ??__EperfLog@U2@@YAXXZ     10003aa0 f   moc_WevoteTask.obj
 0001:00002b20       ??__EscriptLog@U2@@YAXXZ   10003b20 f   moc_WevoteTask.obj
 0001:00002ba0       ??__EtaskLog@U2@@YAXXZ     10003ba0 f   moc_WevoteTask.obj
 0001:00002c20       ??__EuiLog@U2@@YAXXZ       10003c20 f   moc_WevoteTask.obj
 0001:00002ca0       ??__EuserActLog@U2@@YAXXZ  10003ca0 f   moc_WevoteTask.obj
 0001:00002d20       ??__E?_Generic_object@?$_Error_objects@H@std@@2V_Generic_error_category@2@A@@YAXXZ 10003d20 f   moc_WevoteWorker.obj
 0001:00002d30       ??__E?_Iostream_object@?$_Error_objects@H@std@@2V_Iostream_error_category@2@A@@YAXXZ 10003d30 f   moc_WevoteWorker.obj
 0001:00002d40       ??__E?_System_object@?$_Error_objects@H@std@@2V_System_error_category@2@A@@YAXXZ 10003d40 f   moc_WevoteWorker.obj
 0001:00002d50       ??__E?staticMetaObject@WevoteWorker@LocalWorkflow@U2@@2UQMetaObject@@B@@YAXXZ 10003d50 f   moc_WevoteWorker.obj
 0001:00002d60       ??__EalgoLog@U2@@YAXXZ     10003d60 f   moc_WevoteWorker.obj
 0001:00002de0       ??__EcmdLog@U2@@YAXXZ      10003de0 f   moc_WevoteWorker.obj
 0001:00002e60       ??__EcoreLog@U2@@YAXXZ     10003e60 f   moc_WevoteWorker.obj
 0001:00002ee0       ??__EioLog@U2@@YAXXZ       10003ee0 f   moc_WevoteWorker.obj
 0001:00002f60       ??__EperfLog@U2@@YAXXZ     10003f60 f   moc_WevoteWorker.obj
 0001:00002fe0       ??__EscriptLog@U2@@YAXXZ   10003fe0 f   moc_WevoteWorker.obj
 0001:00003060       ??__EtaskLog@U2@@YAXXZ     10004060 f   moc_WevoteWorker.obj
 0001:000030e0       ??__EuiLog@U2@@YAXXZ       100040e0 f   moc_WevoteWorker.obj
 0001:00003160       ??__EuserActLog@U2@@YAXXZ  10004160 f   moc_WevoteWorker.obj
 0001:00003bb6       __catch$?_Copy@?$basic_string@DU?$char_traits@D@std@@V?$allocator@D@2@@std@@QAEXII@Z$0 10004bb6 f i PrepareWevoteTaxonomyDataTask.obj
 0001:00003bf3       __catch$?_Copy@?$basic_string@DU?$char_traits@D@std@@V?$allocator@D@2@@std@@QAEXII@Z$1 10004bf3 f i PrepareWevoteTaxonomyDataTask.obj
 0001:0000500e       __catch$??0?$QList@PAVPort@Workflow@U2@@@@QAE@ABV0@@Z$0 1000600e f i WevotePrompter.obj
 0001:0000598e       __catch$??0?$QList@VQString@@@@QAE@ABV0@@Z$0 1000698e f i WevoteTask.obj
 0001:000060c5       __catch$?append@?$QList@PAVTask@U2@@@@QAEXABQAVTask@U2@@@Z$4 100070c5 f i WevoteTask.obj
 0001:0000614d       __catch$?append@?$QList@VQString@@@@QAEXABVQString@@@Z$0 1000714d f i WevoteTask.obj
 0001:0000619e       __catch$?append@?$QList@VQString@@@@QAEXABVQString@@@Z$4 1000719e f i WevoteTask.obj
 0001:000064c5       __catch$?createNode@?$QMapData@VQString@@I@@QAEPAU?$QMapNode@VQString@@I@@ABVQString@@ABIPAU2@_N@Z$2 100074c5 f i WevoteTask.obj
 0001:00006791       __catch$?detach_helper_grow@?$QList@PAVTask@U2@@@@AAEPAUNode@1@HH@Z$2 10007791 f i WevoteTask.obj
 0001:00006791       __catch$?detach_helper_grow@?$QList@PAVTask@U2@@@@AAEPAUNode@1@HH@Z$0 10007791 f i WevoteTask.obj
 0001:000068ce       __catch$?detach_helper_grow@?$QList@VQString@@@@AAEPAUNode@1@HH@Z$2 100078ce f i WevoteTask.obj
 0001:00006909       __catch$?detach_helper_grow@?$QList@VQString@@@@AAEPAUNode@1@HH@Z$0 10007909 f i WevoteTask.obj
 0001:00007012       __catch$?node_copy@?$QList@VQString@@@@AAEXPAUNode@1@00@Z$2 10008012 f i WevoteTask.obj
 0001:000078d0       __catch$?append@?$QList@VWorkflowNotification@U2@@@@QAEXABVWorkflowNotification@U2@@@Z$2 100088d0 f i WevoteValidator.obj
 0001:000078d0       __catch$?append@?$QList@VWorkflowNotification@U2@@@@QAEXABVWorkflowNotification@U2@@@Z$0 100088d0 f i WevoteValidator.obj
 0001:00007a5f       __catch$?detach_helper_grow@?$QList@VWorkflowNotification@U2@@@@AAEPAUNode@1@HH@Z$2 10008a5f f i WevoteValidator.obj
 0001:00007a9a       __catch$?detach_helper_grow@?$QList@VWorkflowNotification@U2@@@@AAEPAUNode@1@HH@Z$0 10008a9a f i WevoteValidator.obj
 0001:00007bbe       __catch$?node_copy@?$QList@VWorkflowNotification@U2@@@@AAEXPAUNode@1@00@Z$0 10008bbe f i WevoteValidator.obj
 0001:000090ce       __catch$??0?$QList@VDescriptor@U2@@@@QAE@ABV0@@Z$0 1000a0ce f i WevoteWorker.obj
 0001:00009b8c       __catch$?append@?$QList@VDescriptor@U2@@@@QAEXABVDescriptor@U2@@@Z$0 1000ab8c f i WevoteWorker.obj
 0001:00009b8c       __catch$?append@?$QList@VDescriptor@U2@@@@QAEXABVDescriptor@U2@@@Z$2 1000ab8c f i WevoteWorker.obj
 0001:00009f2e       __catch$?createNode@?$QMapData@VQString@@VQScriptValue@@@@QAEPAU?$QMapNode@VQString@@VQScriptValue@@@@ABVQString@@ABVQScriptValue@@PAU2@_N@Z$0 1000af2e f i WevoteWorker.obj
 0001:00009f43       __catch$?createNode@?$QMapData@VQString@@VQScriptValue@@@@QAEPAU?$QMapNode@VQString@@VQScriptValue@@@@ABVQString@@ABVQScriptValue@@PAU2@_N@Z$2 1000af43 f i WevoteWorker.obj
 0001:00009fee       __catch$?createNode@?$QMapData@VQString@@VQVariant@@@@QAEPAU?$QMapNode@VQString@@VQVariant@@@@ABVQString@@ABVQVariant@@PAU2@_N@Z$0 1000afee f i WevoteWorker.obj
 0001:0000a003       __catch$?createNode@?$QMapData@VQString@@VQVariant@@@@QAEPAU?$QMapNode@VQString@@VQVariant@@@@ABVQString@@ABVQVariant@@PAU2@_N@Z$2 1000b003 f i WevoteWorker.obj
 0001:0000a28a       __catch$?detach_helper@?$QList@VDescriptor@U2@@@@AAEXH@Z$0 1000b28a f i WevoteWorker.obj
 0001:0000a49f       __catch$?detach_helper_grow@?$QList@VDescriptor@U2@@@@AAEPAUNode@1@HH@Z$2 1000b49f f i WevoteWorker.obj
 0001:0000a4da       __catch$?detach_helper_grow@?$QList@VDescriptor@U2@@@@AAEPAUNode@1@HH@Z$0 1000b4da f i WevoteWorker.obj
 0001:0000b5d5       __catch$?node_copy@?$QList@VDescriptor@U2@@@@AAEXPAUNode@1@00@Z$0 1000c5d5 f i WevoteWorker.obj
 0001:0000c8c5       __catch$?append@?$QList@PAVAttribute@U2@@@@QAEXABQAVAttribute@U2@@@Z$4 1000d8c5 f i WevoteWorkerFactory.obj
 0001:0000c955       __catch$?append@?$QList@PAVPortDescriptor@Workflow@U2@@@@QAEXABQAVPortDescriptor@Workflow@U2@@@Z$4 1000d955 f i WevoteWorkerFactory.obj
 0001:0000cb8d       __catch$?createNode@?$QMapData@VDescriptor@U2@@V?$QExplicitlySharedDataPointer@VDataType@U2@@@@@@QAEPAU?$QMapNode@VDescriptor@U2@@V?$QExplicitlySharedDataPointer@VDataType@U2@@@@@@ABVDescriptor@U2@@ABV?$QExplicitlySharedDataPointer@VDataType@U2@@@@PAU2@_N@Z$2 1000db8d f i WevoteWorkerFactory.obj
 0001:0000cc35       __catch$?createNode@?$QMapData@VQString@@PAVPropertyDelegate@U2@@@@QAEPAU?$QMapNode@VQString@@PAVPropertyDelegate@U2@@@@ABVQString@@ABQAVPropertyDelegate@U2@@PAU2@_N@Z$2 1000dc35 f i WevoteWorkerFactory.obj
 0001:0000d061       __catch$?detach_helper_grow@?$QList@PAVAttribute@U2@@@@AAEPAUNode@1@HH@Z$0 1000e061 f i WevoteWorkerFactory.obj
 0001:0000d061       __catch$?detach_helper_grow@?$QList@PAVAttribute@U2@@@@AAEPAUNode@1@HH@Z$2 1000e061 f i WevoteWorkerFactory.obj
 0001:0000d171       __catch$?detach_helper_grow@?$QList@PAVPortDescriptor@Workflow@U2@@@@AAEPAUNode@1@HH@Z$0 1000e171 f i WevoteWorkerFactory.obj
 0001:0000d171       __catch$?detach_helper_grow@?$QList@PAVPortDescriptor@Workflow@U2@@@@AAEPAUNode@1@HH@Z$2 1000e171 f i WevoteWorkerFactory.obj
 0001:0000f9d0       $$000000                   100109d0     MSVCRT:chkstk.obj
 0001:0000f9fb       _pre_c_init                100109fb f   MSVCRT:crtdll.obj
 0001:0000fc68       ___DllMainCRTStartup       10010c68 f   MSVCRT:crtdll.obj
 0001:0000fdc0       $$000000                   10010dc0     MSVCRT:sehprolg4.obj
 0001:000101d5       ?ArrayUnwindFilter@@YAHPAU_EXCEPTION_POINTERS@@@Z 100111d5 f   MSVCRT:ehvecdtr.obj
 0001:00010520       __unwindfunclet$??0PrepareWevoteTaxonomyDataTask@U2@@QAE@AAVWorkflowProcess@FileStorage@1@@Z$0 10011520 f   PrepareWevoteTaxonomyDataTask.obj
 0001:00010529       __unwindfunclet$??0PrepareWevoteTaxonomyDataTask@U2@@QAE@AAVWorkflowProcess@FileStorage@1@@Z$1 10011529 f   PrepareWevoteTaxonomyDataTask.obj
 0001:00010532       __unwindfunclet$??0PrepareWevoteTaxonomyDataTask@U2@@QAE@AAVWorkflowProcess@FileStorage@1@@Z$2 10011532 f   PrepareWevoteTaxonomyDataTask.obj
 0001:00010541       __unwindfunclet$??0PrepareWevoteTaxonomyDataTask@U2@@QAE@AAVWorkflowProcess@FileStorage@1@@Z$3 10011541 f   PrepareWevoteTaxonomyDataTask.obj
 0001:00010550       __unwindfunclet$??0PrepareWevoteTaxonomyDataTask@U2@@QAE@AAVWorkflowProcess@FileStorage@1@@Z$4 10011550 f   PrepareWevoteTaxonomyDataTask.obj
 0001:0001055f       __unwindfunclet$??0PrepareWevoteTaxonomyDataTask@U2@@QAE@AAVWorkflowProcess@FileStorage@1@@Z$5 1001155f f   PrepareWevoteTaxonomyDataTask.obj
 0001:00010568       __unwindfunclet$??0PrepareWevoteTaxonomyDataTask@U2@@QAE@AAVWorkflowProcess@FileStorage@1@@Z$6 10011568 f   PrepareWevoteTaxonomyDataTask.obj
 0001:00010571       __unwindfunclet$??0PrepareWevoteTaxonomyDataTask@U2@@QAE@AAVWorkflowProcess@FileStorage@1@@Z$7 10011571 f   PrepareWevoteTaxonomyDataTask.obj
 0001:0001057a       __unwindfunclet$??0PrepareWevoteTaxonomyDataTask@U2@@QAE@AAVWorkflowProcess@FileStorage@1@@Z$8 1001157a f   PrepareWevoteTaxonomyDataTask.obj
 0001:00010583       __unwindfunclet$??0PrepareWevoteTaxonomyDataTask@U2@@QAE@AAVWorkflowProcess@FileStorage@1@@Z$9 10011583 f   PrepareWevoteTaxonomyDataTask.obj
 0001:0001058c       __unwindfunclet$??0PrepareWevoteTaxonomyDataTask@U2@@QAE@AAVWorkflowProcess@FileStorage@1@@Z$10 1001158c f   PrepareWevoteTaxonomyDataTask.obj
 0001:00010595       __unwindfunclet$??0PrepareWevoteTaxonomyDataTask@U2@@QAE@AAVWorkflowProcess@FileStorage@1@@Z$11 10011595 f   PrepareWevoteTaxonomyDataTask.obj
 0001:0001059e       __unwindfunclet$??0PrepareWevoteTaxonomyDataTask@U2@@QAE@AAVWorkflowProcess@FileStorage@1@@Z$12 1001159e f   PrepareWevoteTaxonomyDataTask.obj
 0001:000105a7       __unwindfunclet$??0PrepareWevoteTaxonomyDataTask@U2@@QAE@AAVWorkflowProcess@FileStorage@1@@Z$13 100115a7 f   PrepareWevoteTaxonomyDataTask.obj
 0001:000105b0       __unwindfunclet$??0PrepareWevoteTaxonomyDataTask@U2@@QAE@AAVWorkflowProcess@FileStorage@1@@Z$14 100115b0 f   PrepareWevoteTaxonomyDataTask.obj
 0001:000105b9       __unwindfunclet$??0PrepareWevoteTaxonomyDataTask@U2@@QAE@AAVWorkflowProcess@FileStorage@1@@Z$15 100115b9 f   PrepareWevoteTaxonomyDataTask.obj
 0001:000105c2       __unwindfunclet$??0PrepareWevoteTaxonomyDataTask@U2@@QAE@AAVWorkflowProcess@FileStorage@1@@Z$16 100115c2 f   PrepareWevoteTaxonomyDataTask.obj
 0001:000105cb       __unwindfunclet$??0PrepareWevoteTaxonomyDataTask@U2@@QAE@AAVWorkflowProcess@FileStorage@1@@Z$17 100115cb f   PrepareWevoteTaxonomyDataTask.obj
 0001:000105d4       __unwindfunclet$??0PrepareWevoteTaxonomyDataTask@U2@@QAE@AAVWorkflowProcess@FileStorage@1@@Z$18 100115d4 f   PrepareWevoteTaxonomyDataTask.obj
 0001:000105dd       __ehhandler$??0PrepareWevoteTaxonomyDataTask@U2@@QAE@AAVWorkflowProcess@FileStorage@1@@Z 100115dd f   PrepareWevoteTaxonomyDataTask.obj
 0001:00010600       __unwindfunclet$??1PrepareWevoteTaxonomyDataTask@U2@@UAE@XZ$0 10011600 f   PrepareWevoteTaxonomyDataTask.obj
 0001:00010609       __unwindfunclet$??1PrepareWevoteTaxonomyDataTask@U2@@UAE@XZ$1 10011609 f   PrepareWevoteTaxonomyDataTask.obj
 0001:00010618       __unwindfunclet$??1PrepareWevoteTaxonomyDataTask@U2@@UAE@XZ$2 10011618 f   PrepareWevoteTaxonomyDataTask.obj
 0001:00010627       __ehhandler$??1PrepareWevoteTaxonomyDataTask@U2@@UAE@XZ 10011627 f   PrepareWevoteTaxonomyDataTask.obj
 0001:00010650       __unwindfunclet$??H@YA?BVQString@@ABV0@0@Z$0 10011650 f   PrepareWevoteTaxonomyDataTask.obj
 0001:0001066a       __ehhandler$??H@YA?BVQString@@ABV0@0@Z 1001166a f   PrepareWevoteTaxonomyDataTask.obj
 0001:00010690       __unwindfunclet$??H@YA?BVQString@@ABV0@PBD@Z$0 10011690 f   PrepareWevoteTaxonomyDataTask.obj
 0001:000106aa       __unwindfunclet$??H@YA?BVQString@@ABV0@PBD@Z$1 100116aa f   PrepareWevoteTaxonomyDataTask.obj
 0001:000106b3       __ehhandler$??H@YA?BVQString@@ABV0@PBD@Z 100116b3 f   PrepareWevoteTaxonomyDataTask.obj
 0001:000106d0       __unwindfunclet$??_GPrepareWevoteTaxonomyDataTask@U2@@UAEPAXI@Z$0 100116d0 f   PrepareWevoteTaxonomyDataTask.obj
 0001:000106d9       __unwindfunclet$??_GPrepareWevoteTaxonomyDataTask@U2@@UAEPAXI@Z$1 100116d9 f   PrepareWevoteTaxonomyDataTask.obj
 0001:000106e8       __unwindfunclet$??_GPrepareWevoteTaxonomyDataTask@U2@@UAEPAXI@Z$2 100116e8 f   PrepareWevoteTaxonomyDataTask.obj
 0001:000106f7       __ehhandler$??_GPrepareWevoteTaxonomyDataTask@U2@@UAEPAXI@Z 100116f7 f   PrepareWevoteTaxonomyDataTask.obj
 0001:00010720       __unwindfunclet$??__EalgoLog@U2@@YAXXZ$0 10011720 f   PrepareWevoteTaxonomyDataTask.obj
 0001:00010729       __ehhandler$??__EalgoLog@U2@@YAXXZ 10011729 f   PrepareWevoteTaxonomyDataTask.obj
 0001:00010750       __unwindfunclet$??__EcmdLog@U2@@YAXXZ$0 10011750 f   PrepareWevoteTaxonomyDataTask.obj
 0001:00010759       __ehhandler$??__EcmdLog@U2@@YAXXZ 10011759 f   PrepareWevoteTaxonomyDataTask.obj
 0001:00010780       __unwindfunclet$??__EcoreLog@U2@@YAXXZ$0 10011780 f   PrepareWevoteTaxonomyDataTask.obj
 0001:00010789       __ehhandler$??__EcoreLog@U2@@YAXXZ 10011789 f   PrepareWevoteTaxonomyDataTask.obj
 0001:000107b0       __unwindfunclet$??__EioLog@U2@@YAXXZ$0 100117b0 f   PrepareWevoteTaxonomyDataTask.obj
 0001:000107b9       __ehhandler$??__EioLog@U2@@YAXXZ 100117b9 f   PrepareWevoteTaxonomyDataTask.obj
 0001:000107e0       __unwindfunclet$??__EperfLog@U2@@YAXXZ$0 100117e0 f   PrepareWevoteTaxonomyDataTask.obj
 0001:000107e9       __ehhandler$??__EperfLog@U2@@YAXXZ 100117e9 f   PrepareWevoteTaxonomyDataTask.obj
 0001:00010810       __unwindfunclet$??__EscriptLog@U2@@YAXXZ$0 10011810 f   PrepareWevoteTaxonomyDataTask.obj
 0001:00010819       __ehhandler$??__EscriptLog@U2@@YAXXZ 10011819 f   PrepareWevoteTaxonomyDataTask.obj
 0001:00010840       __unwindfunclet$??__EtaskLog@U2@@YAXXZ$0 10011840 f   PrepareWevoteTaxonomyDataTask.obj
 0001:00010849       __ehhandler$??__EtaskLog@U2@@YAXXZ 10011849 f   PrepareWevoteTaxonomyDataTask.obj
 0001:00010870       __unwindfunclet$??__EuiLog@U2@@YAXXZ$0 10011870 f   PrepareWevoteTaxonomyDataTask.obj
 0001:00010879       __ehhandler$??__EuiLog@U2@@YAXXZ 10011879 f   PrepareWevoteTaxonomyDataTask.obj
 0001:000108a0       __unwindfunclet$??__EuserActLog@U2@@YAXXZ$0 100118a0 f   PrepareWevoteTaxonomyDataTask.obj
 0001:000108a9       __ehhandler$??__EuserActLog@U2@@YAXXZ 100118a9 f   PrepareWevoteTaxonomyDataTask.obj
 0001:000108d0       __ehhandler$?_Copy@?$basic_string@DU?$char_traits@D@std@@V?$allocator@D@2@@std@@QAEXII@Z 100118d0 f   PrepareWevoteTaxonomyDataTask.obj
 0001:000108f0       __unwindfunclet$?isActual@PrepareWevoteTaxonomyDataTask@U2@@ABE_NXZ$0 100118f0 f   PrepareWevoteTaxonomyDataTask.obj
 0001:000108f9       __ehhandler$?isActual@PrepareWevoteTaxonomyDataTask@U2@@ABE_NXZ 100118f9 f   PrepareWevoteTaxonomyDataTask.obj
 0001:00010920       __unwindfunclet$?prepareNamesFile@PrepareWevoteTaxonomyDataTask@U2@@AAEXXZ$0 10011920 f   PrepareWevoteTaxonomyDataTask.obj
 0001:00010929       __unwindfunclet$?prepareNamesFile@PrepareWevoteTaxonomyDataTask@U2@@AAEXXZ$1 10011929 f   PrepareWevoteTaxonomyDataTask.obj
 0001:00010932       __unwindfunclet$?prepareNamesFile@PrepareWevoteTaxonomyDataTask@U2@@AAEXXZ$2 10011932 f   PrepareWevoteTaxonomyDataTask.obj
 0001:0001093b       __unwindfunclet$?prepareNamesFile@PrepareWevoteTaxonomyDataTask@U2@@AAEXXZ$3 1001193b f   PrepareWevoteTaxonomyDataTask.obj
 0001:00010944       __unwindfunclet$?prepareNamesFile@PrepareWevoteTaxonomyDataTask@U2@@AAEXXZ$4 10011944 f   PrepareWevoteTaxonomyDataTask.obj
 0001:0001094d       __unwindfunclet$?prepareNamesFile@PrepareWevoteTaxonomyDataTask@U2@@AAEXXZ$5 1001194d f   PrepareWevoteTaxonomyDataTask.obj
 0001:00010956       __unwindfunclet$?prepareNamesFile@PrepareWevoteTaxonomyDataTask@U2@@AAEXXZ$6 10011956 f   PrepareWevoteTaxonomyDataTask.obj
 0001:0001095f       __unwindfunclet$?prepareNamesFile@PrepareWevoteTaxonomyDataTask@U2@@AAEXXZ$7 1001195f f   PrepareWevoteTaxonomyDataTask.obj
 0001:00010968       __unwindfunclet$?prepareNamesFile@PrepareWevoteTaxonomyDataTask@U2@@AAEXXZ$8 10011968 f   PrepareWevoteTaxonomyDataTask.obj
 0001:00010971       __unwindfunclet$?prepareNamesFile@PrepareWevoteTaxonomyDataTask@U2@@AAEXXZ$9 10011971 f   PrepareWevoteTaxonomyDataTask.obj
 0001:0001097a       __unwindfunclet$?prepareNamesFile@PrepareWevoteTaxonomyDataTask@U2@@AAEXXZ$10 1001197a f   PrepareWevoteTaxonomyDataTask.obj
 0001:00010983       __unwindfunclet$?prepareNamesFile@PrepareWevoteTaxonomyDataTask@U2@@AAEXXZ$11 10011983 f   PrepareWevoteTaxonomyDataTask.obj
 0001:0001098c       __unwindfunclet$?prepareNamesFile@PrepareWevoteTaxonomyDataTask@U2@@AAEXXZ$12 1001198c f   PrepareWevoteTaxonomyDataTask.obj
 0001:00010995       __unwindfunclet$?prepareNamesFile@PrepareWevoteTaxonomyDataTask@U2@@AAEXXZ$13 10011995 f   PrepareWevoteTaxonomyDataTask.obj
 0001:0001099e       __unwindfunclet$?prepareNamesFile@PrepareWevoteTaxonomyDataTask@U2@@AAEXXZ$14 1001199e f   PrepareWevoteTaxonomyDataTask.obj
 0001:000109a7       __unwindfunclet$?prepareNamesFile@PrepareWevoteTaxonomyDataTask@U2@@AAEXXZ$15 100119a7 f   PrepareWevoteTaxonomyDataTask.obj
 0001:000109b0       __unwindfunclet$?prepareNamesFile@PrepareWevoteTaxonomyDataTask@U2@@AAEXXZ$16 100119b0 f   PrepareWevoteTaxonomyDataTask.obj
 0001:000109b9       __ehhandler$?prepareNamesFile@PrepareWevoteTaxonomyDataTask@U2@@AAEXXZ 100119b9 f   PrepareWevoteTaxonomyDataTask.obj
 0001:000109e0       __unwindfunclet$?prepareNodesFile@PrepareWevoteTaxonomyDataTask@U2@@AAEXXZ$0 100119e0 f   PrepareWevoteTaxonomyDataTask.obj
 0001:000109e9       __unwindfunclet$?prepareNodesFile@PrepareWevoteTaxonomyDataTask@U2@@AAEXXZ$1 100119e9 f   PrepareWevoteTaxonomyDataTask.obj
 0001:000109f2       __unwindfunclet$?prepareNodesFile@PrepareWevoteTaxonomyDataTask@U2@@AAEXXZ$2 100119f2 f   PrepareWevoteTaxonomyDataTask.obj
 0001:000109fb       __unwindfunclet$?prepareNodesFile@PrepareWevoteTaxonomyDataTask@U2@@AAEXXZ$3 100119fb f   PrepareWevoteTaxonomyDataTask.obj
 0001:00010a04       __unwindfunclet$?prepareNodesFile@PrepareWevoteTaxonomyDataTask@U2@@AAEXXZ$4 10011a04 f   PrepareWevoteTaxonomyDataTask.obj
 0001:00010a0d       __unwindfunclet$?prepareNodesFile@PrepareWevoteTaxonomyDataTask@U2@@AAEXXZ$5 10011a0d f   PrepareWevoteTaxonomyDataTask.obj
 0001:00010a16       __unwindfunclet$?prepareNodesFile@PrepareWevoteTaxonomyDataTask@U2@@AAEXXZ$6 10011a16 f   PrepareWevoteTaxonomyDataTask.obj
 0001:00010a1f       __unwindfunclet$?prepareNodesFile@PrepareWevoteTaxonomyDataTask@U2@@AAEXXZ$7 10011a1f f   PrepareWevoteTaxonomyDataTask.obj
 0001:00010a28       __unwindfunclet$?prepareNodesFile@PrepareWevoteTaxonomyDataTask@U2@@AAEXXZ$8 10011a28 f   PrepareWevoteTaxonomyDataTask.obj
 0001:00010a31       __unwindfunclet$?prepareNodesFile@PrepareWevoteTaxonomyDataTask@U2@@AAEXXZ$9 10011a31 f   PrepareWevoteTaxonomyDataTask.obj
 0001:00010a3a       __unwindfunclet$?prepareNodesFile@PrepareWevoteTaxonomyDataTask@U2@@AAEXXZ$10 10011a3a f   PrepareWevoteTaxonomyDataTask.obj
 0001:00010a43       __unwindfunclet$?prepareNodesFile@PrepareWevoteTaxonomyDataTask@U2@@AAEXXZ$11 10011a43 f   PrepareWevoteTaxonomyDataTask.obj
 0001:00010a4c       __unwindfunclet$?prepareNodesFile@PrepareWevoteTaxonomyDataTask@U2@@AAEXXZ$12 10011a4c f   PrepareWevoteTaxonomyDataTask.obj
 0001:00010a55       __unwindfunclet$?prepareNodesFile@PrepareWevoteTaxonomyDataTask@U2@@AAEXXZ$13 10011a55 f   PrepareWevoteTaxonomyDataTask.obj
 0001:00010a5e       __unwindfunclet$?prepareNodesFile@PrepareWevoteTaxonomyDataTask@U2@@AAEXXZ$14 10011a5e f   PrepareWevoteTaxonomyDataTask.obj
 0001:00010a67       __unwindfunclet$?prepareNodesFile@PrepareWevoteTaxonomyDataTask@U2@@AAEXXZ$15 10011a67 f   PrepareWevoteTaxonomyDataTask.obj
 0001:00010a70       __ehhandler$?prepareNodesFile@PrepareWevoteTaxonomyDataTask@U2@@AAEXXZ 10011a70 f   PrepareWevoteTaxonomyDataTask.obj
 0001:00010a90       __unwindfunclet$?report@PrepareWevoteTaxonomyDataTask@U2@@EAE?AW4ReportResult@Task@2@XZ$0 10011a90 f   PrepareWevoteTaxonomyDataTask.obj
 0001:00010a99       __unwindfunclet$?report@PrepareWevoteTaxonomyDataTask@U2@@EAE?AW4ReportResult@Task@2@XZ$1 10011a99 f   PrepareWevoteTaxonomyDataTask.obj
 0001:00010aa2       __unwindfunclet$?report@PrepareWevoteTaxonomyDataTask@U2@@EAE?AW4ReportResult@Task@2@XZ$2 10011aa2 f   PrepareWevoteTaxonomyDataTask.obj
 0001:00010aab       __unwindfunclet$?report@PrepareWevoteTaxonomyDataTask@U2@@EAE?AW4ReportResult@Task@2@XZ$3 10011aab f   PrepareWevoteTaxonomyDataTask.obj
 0001:00010ab4       __unwindfunclet$?report@PrepareWevoteTaxonomyDataTask@U2@@EAE?AW4ReportResult@Task@2@XZ$4 10011ab4 f   PrepareWevoteTaxonomyDataTask.obj
 0001:00010abd       __unwindfunclet$?report@PrepareWevoteTaxonomyDataTask@U2@@EAE?AW4ReportResult@Task@2@XZ$5 10011abd f   PrepareWevoteTaxonomyDataTask.obj
 0001:00010ac6       __ehhandler$?report@PrepareWevoteTaxonomyDataTask@U2@@EAE?AW4ReportResult@Task@2@XZ 10011ac6 f   PrepareWevoteTaxonomyDataTask.obj
 0001:00010af0       __unwindfunclet$?run@PrepareWevoteTaxonomyDataTask@U2@@EAEXXZ$0 10011af0 f   PrepareWevoteTaxonomyDataTask.obj
 0001:00010af9       __unwindfunclet$?run@PrepareWevoteTaxonomyDataTask@U2@@EAEXXZ$1 10011af9 f   PrepareWevoteTaxonomyDataTask.obj
 0001:00010b02       __ehhandler$?run@PrepareWevoteTaxonomyDataTask@U2@@EAEXXZ 10011b02 f   PrepareWevoteTaxonomyDataTask.obj
 0001:00010b20       __ehhandler$??0?$QList@PAVPort@Workflow@U2@@@@QAE@ABV0@@Z 10011b20 f   WevotePrompter.obj
 0001:00010b40       __unwindfunclet$??__EalgoLog@U2@@YAXXZ$0 10011b40 f   WevotePrompter.obj
 0001:00010b49       __ehhandler$??__EalgoLog@U2@@YAXXZ 10011b49 f   WevotePrompter.obj
 0001:00010b70       __unwindfunclet$??__EcmdLog@U2@@YAXXZ$0 10011b70 f   WevotePrompter.obj
 0001:00010b79       __ehhandler$??__EcmdLog@U2@@YAXXZ 10011b79 f   WevotePrompter.obj
 0001:00010ba0       __unwindfunclet$??__EcoreLog@U2@@YAXXZ$0 10011ba0 f   WevotePrompter.obj
 0001:00010ba9       __ehhandler$??__EcoreLog@U2@@YAXXZ 10011ba9 f   WevotePrompter.obj
 0001:00010bd0       __unwindfunclet$??__EioLog@U2@@YAXXZ$0 10011bd0 f   WevotePrompter.obj
 0001:00010bd9       __ehhandler$??__EioLog@U2@@YAXXZ 10011bd9 f   WevotePrompter.obj
 0001:00010c00       __unwindfunclet$??__EperfLog@U2@@YAXXZ$0 10011c00 f   WevotePrompter.obj
 0001:00010c09       __ehhandler$??__EperfLog@U2@@YAXXZ 10011c09 f   WevotePrompter.obj
 0001:00010c30       __unwindfunclet$??__EscriptLog@U2@@YAXXZ$0 10011c30 f   WevotePrompter.obj
 0001:00010c39       __ehhandler$??__EscriptLog@U2@@YAXXZ 10011c39 f   WevotePrompter.obj
 0001:00010c60       __unwindfunclet$??__EtaskLog@U2@@YAXXZ$0 10011c60 f   WevotePrompter.obj
 0001:00010c69       __ehhandler$??__EtaskLog@U2@@YAXXZ 10011c69 f   WevotePrompter.obj
 0001:00010c90       __unwindfunclet$??__EuiLog@U2@@YAXXZ$0 10011c90 f   WevotePrompter.obj
 0001:00010c99       __ehhandler$??__EuiLog@U2@@YAXXZ 10011c99 f   WevotePrompter.obj
 0001:00010cc0       __unwindfunclet$??__EuserActLog@U2@@YAXXZ$0 10011cc0 f   WevotePrompter.obj
 0001:00010cc9       __ehhandler$??__EuserActLog@U2@@YAXXZ 10011cc9 f   WevotePrompter.obj
 0001:00010cf0       __unwindfunclet$?createDescription@?$PrompterBase@VWevotePrompter@LocalWorkflow@U2@@@U2@@UAEPAVActorDocument@Workflow@2@PAVActor@42@@Z$0 10011cf0 f   WevotePrompter.obj
 0001:00010cfb       __unwindfunclet$?createDescription@?$PrompterBase@VWevotePrompter@LocalWorkflow@U2@@@U2@@UAEPAVActorDocument@Workflow@2@PAVActor@42@@Z$3 10011cfb f   WevotePrompter.obj
 0001:00010d03       __unwindfunclet$?createDescription@?$PrompterBase@VWevotePrompter@LocalWorkflow@U2@@@U2@@UAEPAVActorDocument@Workflow@2@PAVActor@42@@Z$4 10011d03 f   WevotePrompter.obj
 0001:00010d0b       __unwindfunclet$?createDescription@?$PrompterBase@VWevotePrompter@LocalWorkflow@U2@@@U2@@UAEPAVActorDocument@Workflow@2@PAVActor@42@@Z$6 10011d0b f   WevotePrompter.obj
 0001:00010d13       __unwindfunclet$?createDescription@?$PrompterBase@VWevotePrompter@LocalWorkflow@U2@@@U2@@UAEPAVActorDocument@Workflow@2@PAVActor@42@@Z$7 10011d13 f   WevotePrompter.obj
 0001:00010d1b       __ehhandler$?createDescription@?$PrompterBase@VWevotePrompter@LocalWorkflow@U2@@@U2@@UAEPAVActorDocument@Workflow@2@PAVActor@42@@Z 10011d1b f   WevotePrompter.obj
 0001:00010d40       __unwindfunclet$??0WevoteSupport@U2@@QAE@XZ$0 10011d40 f   WevoteSupport.obj
 0001:00010d49       __unwindfunclet$??0WevoteSupport@U2@@QAE@XZ$2 10011d49 f   WevoteSupport.obj
 0001:00010d52       __unwindfunclet$??0WevoteSupport@U2@@QAE@XZ$3 10011d52 f   WevoteSupport.obj
 0001:00010d5b       __ehhandler$??0WevoteSupport@U2@@QAE@XZ 10011d5b f   WevoteSupport.obj
 0001:00010d80       __unwindfunclet$??0WevoteSupportPlugin@U2@@QAE@XZ$0 10011d80 f   WevoteSupportPlugin.obj
 0001:00010d89       __unwindfunclet$??0WevoteSupportPlugin@U2@@QAE@XZ$1 10011d89 f   WevoteSupportPlugin.obj
 0001:00010d94       __ehhandler$??0WevoteSupportPlugin@U2@@QAE@XZ 10011d94 f   WevoteSupportPlugin.obj
 0001:00010db0       __unwindfunclet$??1WevoteSupportPlugin@U2@@UAE@XZ$0 10011db0 f   WevoteSupportPlugin.obj
 0001:00010db9       __ehhandler$??1WevoteSupportPlugin@U2@@UAE@XZ 10011db9 f   WevoteSupportPlugin.obj
 0001:00010de0       __unwindfunclet$??_GWevoteSupportPlugin@U2@@UAEPAXI@Z$0 10011de0 f   WevoteSupportPlugin.obj
 0001:00010de9       __ehhandler$??_GWevoteSupportPlugin@U2@@UAEPAXI@Z 10011de9 f   WevoteSupportPlugin.obj
 0001:00010e10       __unwindfunclet$??__EalgoLog@U2@@YAXXZ$0 10011e10 f   WevoteSupportPlugin.obj
 0001:00010e19       __ehhandler$??__EalgoLog@U2@@YAXXZ 10011e19 f   WevoteSupportPlugin.obj
 0001:00010e40       __unwindfunclet$??__EcmdLog@U2@@YAXXZ$0 10011e40 f   WevoteSupportPlugin.obj
 0001:00010e49       __ehhandler$??__EcmdLog@U2@@YAXXZ 10011e49 f   WevoteSupportPlugin.obj
 0001:00010e70       __unwindfunclet$??__EcoreLog@U2@@YAXXZ$0 10011e70 f   WevoteSupportPlugin.obj
 0001:00010e79       __ehhandler$??__EcoreLog@U2@@YAXXZ 10011e79 f   WevoteSupportPlugin.obj
 0001:00010ea0       __unwindfunclet$??__EioLog@U2@@YAXXZ$0 10011ea0 f   WevoteSupportPlugin.obj
 0001:00010ea9       __ehhandler$??__EioLog@U2@@YAXXZ 10011ea9 f   WevoteSupportPlugin.obj
 0001:00010ed0       __unwindfunclet$??__EperfLog@U2@@YAXXZ$0 10011ed0 f   WevoteSupportPlugin.obj
 0001:00010ed9       __ehhandler$??__EperfLog@U2@@YAXXZ 10011ed9 f   WevoteSupportPlugin.obj
 0001:00010f00       __unwindfunclet$??__EscriptLog@U2@@YAXXZ$0 10011f00 f   WevoteSupportPlugin.obj
 0001:00010f09       __ehhandler$??__EscriptLog@U2@@YAXXZ 10011f09 f   WevoteSupportPlugin.obj
 0001:00010f30       __unwindfunclet$??__EtaskLog@U2@@YAXXZ$0 10011f30 f   WevoteSupportPlugin.obj
 0001:00010f39       __ehhandler$??__EtaskLog@U2@@YAXXZ 10011f39 f   WevoteSupportPlugin.obj
 0001:00010f60       __unwindfunclet$??__EuiLog@U2@@YAXXZ$0 10011f60 f   WevoteSupportPlugin.obj
 0001:00010f69       __ehhandler$??__EuiLog@U2@@YAXXZ 10011f69 f   WevoteSupportPlugin.obj
 0001:00010f90       __unwindfunclet$??__EuserActLog@U2@@YAXXZ$0 10011f90 f   WevoteSupportPlugin.obj
 0001:00010f99       __ehhandler$??__EuserActLog@U2@@YAXXZ 10011f99 f   WevoteSupportPlugin.obj
 0001:00010fc0       __ehhandler$??0?$QList@VQString@@@@QAE@ABV0@@Z 10011fc0 f   WevoteTask.obj
 0001:00010fe0       __unwindfunclet$??0WevoteTask@U2@@QAE@ABUWevoteTaskSettings@1@AAVWorkflowProcess@FileStorage@1@@Z$0 10011fe0 f   WevoteTask.obj
 0001:00010fe9       __unwindfunclet$??0WevoteTask@U2@@QAE@ABUWevoteTaskSettings@1@AAVWorkflowProcess@FileStorage@1@@Z$1 10011fe9 f   WevoteTask.obj
 0001:00010ff2       __unwindfunclet$??0WevoteTask@U2@@QAE@ABUWevoteTaskSettings@1@AAVWorkflowProcess@FileStorage@1@@Z$8 10011ff2 f   WevoteTask.obj
 0001:00010ffe       __unwindfunclet$??0WevoteTask@U2@@QAE@ABUWevoteTaskSettings@1@AAVWorkflowProcess@FileStorage@1@@Z$9 10011ffe f   WevoteTask.obj
 0001:0001100a       __unwindfunclet$??0WevoteTask@U2@@QAE@ABUWevoteTaskSettings@1@AAVWorkflowProcess@FileStorage@1@@Z$2 1001200a f   WevoteTask.obj
 0001:00011018       __unwindfunclet$??0WevoteTask@U2@@QAE@ABUWevoteTaskSettings@1@AAVWorkflowProcess@FileStorage@1@@Z$3 10012018 f   WevoteTask.obj
 0001:00011021       __unwindfunclet$??0WevoteTask@U2@@QAE@ABUWevoteTaskSettings@1@AAVWorkflowProcess@FileStorage@1@@Z$4 10012021 f   WevoteTask.obj
 0001:0001102a       __unwindfunclet$??0WevoteTask@U2@@QAE@ABUWevoteTaskSettings@1@AAVWorkflowProcess@FileStorage@1@@Z$5 1001202a f   WevoteTask.obj
 0001:00011033       __unwindfunclet$??0WevoteTask@U2@@QAE@ABUWevoteTaskSettings@1@AAVWorkflowProcess@FileStorage@1@@Z$6 10012033 f   WevoteTask.obj
 0001:00011042       __unwindfunclet$??0WevoteTask@U2@@QAE@ABUWevoteTaskSettings@1@AAVWorkflowProcess@FileStorage@1@@Z$7 10012042 f   WevoteTask.obj
 0001:00011050       __ehhandler$??0WevoteTask@U2@@QAE@ABUWevoteTaskSettings@1@AAVWorkflowProcess@FileStorage@1@@Z 10012050 f   WevoteTask.obj
 0001:00011070       __unwindfunclet$??0WevoteTaskSettings@U2@@QAE@ABU01@@Z$0 10012070 f   WevoteTask.obj
 0001:0001107c       __unwindfunclet$??0WevoteTaskSettings@U2@@QAE@ABU01@@Z$1 1001207c f   WevoteTask.obj
 0001:00011088       __ehhandler$??0WevoteTaskSettings@U2@@QAE@ABU01@@Z 10012088 f   WevoteTask.obj
 0001:000110b0       __unwindfunclet$??0WevoteTaskSettings@U2@@QAE@XZ$0 100120b0 f   WevoteTask.obj
 0001:000110bc       __unwindfunclet$??0WevoteTaskSettings@U2@@QAE@XZ$1 100120bc f   WevoteTask.obj
 0001:000110c8       __ehhandler$??0WevoteTaskSettings@U2@@QAE@XZ 100120c8 f   WevoteTask.obj
 0001:000110f0       __unwindfunclet$??1WevoteTask@U2@@UAE@XZ$0 100120f0 f   WevoteTask.obj
 0001:000110f9       __unwindfunclet$??1WevoteTask@U2@@UAE@XZ$1 100120f9 f   WevoteTask.obj
 0001:00011107       __unwindfunclet$??1WevoteTask@U2@@UAE@XZ$2 10012107 f   WevoteTask.obj
 0001:00011116       __unwindfunclet$??1WevoteTask@U2@@UAE@XZ$4 10012116 f   WevoteTask.obj
 0001:00011122       __unwindfunclet$??1WevoteTask@U2@@UAE@XZ$5 10012122 f   WevoteTask.obj
 0001:0001112e       __ehhandler$??1WevoteTask@U2@@UAE@XZ 1001212e f   WevoteTask.obj
 0001:00011150       __unwindfunclet$??1WevoteTaskSettings@U2@@QAE@XZ$0 10012150 f   WevoteTask.obj
 0001:0001115c       __unwindfunclet$??1WevoteTaskSettings@U2@@QAE@XZ$1 1001215c f   WevoteTask.obj
 0001:00011168       __ehhandler$??1WevoteTaskSettings@U2@@QAE@XZ 10012168 f   WevoteTask.obj
 0001:00011190       __unwindfunclet$??__EalgoLog@U2@@YAXXZ$0 10012190 f   WevoteTask.obj
 0001:00011199       __ehhandler$??__EalgoLog@U2@@YAXXZ 10012199 f   WevoteTask.obj
 0001:000111c0       __unwindfunclet$??__EcmdLog@U2@@YAXXZ$0 100121c0 f   WevoteTask.obj
 0001:000111c9       __ehhandler$??__EcmdLog@U2@@YAXXZ 100121c9 f   WevoteTask.obj
 0001:000111f0       __unwindfunclet$??__EcoreLog@U2@@YAXXZ$0 100121f0 f   WevoteTask.obj
 0001:000111f9       __ehhandler$??__EcoreLog@U2@@YAXXZ 100121f9 f   WevoteTask.obj
 0001:00011220       __unwindfunclet$??__EioLog@U2@@YAXXZ$0 10012220 f   WevoteTask.obj
 0001:00011229       __ehhandler$??__EioLog@U2@@YAXXZ 10012229 f   WevoteTask.obj
 0001:00011250       __unwindfunclet$??__EperfLog@U2@@YAXXZ$0 10012250 f   WevoteTask.obj
 0001:00011259       __ehhandler$??__EperfLog@U2@@YAXXZ 10012259 f   WevoteTask.obj
 0001:00011280       __unwindfunclet$??__EscriptLog@U2@@YAXXZ$0 10012280 f   WevoteTask.obj
 0001:00011289       __ehhandler$??__EscriptLog@U2@@YAXXZ 10012289 f   WevoteTask.obj
 0001:000112b0       __unwindfunclet$??__EtaskLog@U2@@YAXXZ$0 100122b0 f   WevoteTask.obj
 0001:000112b9       __ehhandler$??__EtaskLog@U2@@YAXXZ 100122b9 f   WevoteTask.obj
 0001:000112e0       __unwindfunclet$??__EuiLog@U2@@YAXXZ$0 100122e0 f   WevoteTask.obj
 0001:000112e9       __ehhandler$??__EuiLog@U2@@YAXXZ 100122e9 f   WevoteTask.obj
 0001:00011310       __unwindfunclet$??__EuserActLog@U2@@YAXXZ$0 10012310 f   WevoteTask.obj
 0001:00011319       __ehhandler$??__EuserActLog@U2@@YAXXZ 10012319 f   WevoteTask.obj
 0001:00011340       __ehhandler$?append@?$QList@PAVTask@U2@@@@QAEXABQAVTask@U2@@@Z 10012340 f   WevoteTask.obj
 0001:00011360       __unwindfunclet$?append@?$QList@VQString@@@@QAEXABVQString@@@Z$7 10012360 f   WevoteTask.obj
 0001:00011371       __unwindfunclet$?append@?$QList@VQString@@@@QAEXABVQString@@@Z$11 10012371 f   WevoteTask.obj
 0001:00011382       __ehhandler$?append@?$QList@VQString@@@@QAEXABVQString@@@Z 10012382 f   WevoteTask.obj
 0001:000113a0       __unwindfunclet$?checkSettings@WevoteTask@U2@@AAEXXZ$0 100123a0 f   WevoteTask.obj
 0001:000113a9       __unwindfunclet$?checkSettings@WevoteTask@U2@@AAEXXZ$1 100123a9 f   WevoteTask.obj
 0001:000113b2       __unwindfunclet$?checkSettings@WevoteTask@U2@@AAEXXZ$2 100123b2 f   WevoteTask.obj
 0001:000113bb       __unwindfunclet$?checkSettings@WevoteTask@U2@@AAEXXZ$3 100123bb f   WevoteTask.obj
 0001:000113c4       __unwindfunclet$?checkSettings@WevoteTask@U2@@AAEXXZ$4 100123c4 f   WevoteTask.obj
 0001:000113cd       __unwindfunclet$?checkSettings@WevoteTask@U2@@AAEXXZ$5 100123cd f   WevoteTask.obj
 0001:000113d6       __ehhandler$?checkSettings@WevoteTask@U2@@AAEXXZ 100123d6 f   WevoteTask.obj
 0001:00011400       __unwindfunclet$?createNode@?$QMapData@VQString@@I@@QAEPAU?$QMapNode@VQString@@I@@ABVQString@@ABIPAU2@_N@Z$4 10012400 f   WevoteTask.obj
 0001:00011414       __ehhandler$?createNode@?$QMapData@VQString@@I@@QAEPAU?$QMapNode@VQString@@I@@ABVQString@@ABIPAU2@_N@Z 10012414 f   WevoteTask.obj
 0001:00011430       __ehhandler$?detach_helper_grow@?$QList@PAVTask@U2@@@@AAEPAUNode@1@HH@Z 10012430 f   WevoteTask.obj
 0001:00011450       __ehhandler$?detach_helper_grow@?$QList@VQString@@@@AAEPAUNode@1@HH@Z 10012450 f   WevoteTask.obj
 0001:00011470       __unwindfunclet$?getArguments@WevoteTask@U2@@AAE?AVQStringList@@XZ$0 10012470 f   WevoteTask.obj
 0001:00011478       __unwindfunclet$?getArguments@WevoteTask@U2@@AAE?AVQStringList@@XZ$1 10012478 f   WevoteTask.obj
 0001:00011481       __unwindfunclet$?getArguments@WevoteTask@U2@@AAE?AVQStringList@@XZ$2 10012481 f   WevoteTask.obj
 0001:0001148a       __unwindfunclet$?getArguments@WevoteTask@U2@@AAE?AVQStringList@@XZ$3 1001248a f   WevoteTask.obj
 0001:00011493       __unwindfunclet$?getArguments@WevoteTask@U2@@AAE?AVQStringList@@XZ$4 10012493 f   WevoteTask.obj
 0001:0001149c       __unwindfunclet$?getArguments@WevoteTask@U2@@AAE?AVQStringList@@XZ$5 1001249c f   WevoteTask.obj
 0001:000114b5       __unwindfunclet$?getArguments@WevoteTask@U2@@AAE?AVQStringList@@XZ$6 100124b5 f   WevoteTask.obj
 0001:000114be       __unwindfunclet$?getArguments@WevoteTask@U2@@AAE?AVQStringList@@XZ$7 100124be f   WevoteTask.obj
 0001:000114c7       __unwindfunclet$?getArguments@WevoteTask@U2@@AAE?AVQStringList@@XZ$8 100124c7 f   WevoteTask.obj
 0001:000114d0       __unwindfunclet$?getArguments@WevoteTask@U2@@AAE?AVQStringList@@XZ$9 100124d0 f   WevoteTask.obj
 0001:000114d9       __unwindfunclet$?getArguments@WevoteTask@U2@@AAE?AVQStringList@@XZ$10 100124d9 f   WevoteTask.obj
 0001:000114e2       __unwindfunclet$?getArguments@WevoteTask@U2@@AAE?AVQStringList@@XZ$11 100124e2 f   WevoteTask.obj
 0001:000114eb       __unwindfunclet$?getArguments@WevoteTask@U2@@AAE?AVQStringList@@XZ$12 100124eb f   WevoteTask.obj
 0001:000114f4       __unwindfunclet$?getArguments@WevoteTask@U2@@AAE?AVQStringList@@XZ$13 100124f4 f   WevoteTask.obj
 0001:000114fd       __unwindfunclet$?getArguments@WevoteTask@U2@@AAE?AVQStringList@@XZ$14 100124fd f   WevoteTask.obj
 0001:00011506       __unwindfunclet$?getArguments@WevoteTask@U2@@AAE?AVQStringList@@XZ$15 10012506 f   WevoteTask.obj
 0001:0001150f       __unwindfunclet$?getArguments@WevoteTask@U2@@AAE?AVQStringList@@XZ$16 1001250f f   WevoteTask.obj
 0001:00011518       __ehhandler$?getArguments@WevoteTask@U2@@AAE?AVQStringList@@XZ 10012518 f   WevoteTask.obj
 0001:00011540       __unwindfunclet$?moveFile@WevoteTask@U2@@AAEXXZ$0 10012540 f   WevoteTask.obj
 0001:00011549       __unwindfunclet$?moveFile@WevoteTask@U2@@AAEXXZ$1 10012549 f   WevoteTask.obj
 0001:00011552       __unwindfunclet$?moveFile@WevoteTask@U2@@AAEXXZ$2 10012552 f   WevoteTask.obj
 0001:0001155b       __unwindfunclet$?moveFile@WevoteTask@U2@@AAEXXZ$3 1001255b f   WevoteTask.obj
 0001:00011564       __ehhandler$?moveFile@WevoteTask@U2@@AAEXXZ 10012564 f   WevoteTask.obj
 0001:00011580       __unwindfunclet$?node_construct@?$QList@VQString@@@@AAEXPAUNode@1@ABVQString@@@Z$1 10012580 f   WevoteTask.obj
 0001:00011591       __ehhandler$?node_construct@?$QList@VQString@@@@AAEXPAUNode@1@ABVQString@@@Z 10012591 f   WevoteTask.obj
 0001:000115b0       __unwindfunclet$?node_copy@?$QList@VQString@@@@AAEXPAUNode@1@00@Z$5 100125b0 f   WevoteTask.obj
 0001:000115c1       __ehhandler$?node_copy@?$QList@VQString@@@@AAEXPAUNode@1@00@Z 100125c1 f   WevoteTask.obj
 0001:000115e0       __unwindfunclet$?onSubTaskFinished@WevoteTask@U2@@EAE?AV?$QList@PAVTask@U2@@@@PAVTask@2@@Z$0 100125e0 f   WevoteTask.obj
 0001:000115e8       __unwindfunclet$?onSubTaskFinished@WevoteTask@U2@@EAE?AV?$QList@PAVTask@U2@@@@PAVTask@2@@Z$1 100125e8 f   WevoteTask.obj
 0001:00011601       __unwindfunclet$?onSubTaskFinished@WevoteTask@U2@@EAE?AV?$QList@PAVTask@U2@@@@PAVTask@2@@Z$2 10012601 f   WevoteTask.obj
 0001:00011609       __unwindfunclet$?onSubTaskFinished@WevoteTask@U2@@EAE?AV?$QList@PAVTask@U2@@@@PAVTask@2@@Z$3 10012609 f   WevoteTask.obj
 0001:00011614       __unwindfunclet$?onSubTaskFinished@WevoteTask@U2@@EAE?AV?$QList@PAVTask@U2@@@@PAVTask@2@@Z$4 10012614 f   WevoteTask.obj
 0001:0001162e       __unwindfunclet$?onSubTaskFinished@WevoteTask@U2@@EAE?AV?$QList@PAVTask@U2@@@@PAVTask@2@@Z$5 1001262e f   WevoteTask.obj
 0001:00011639       __unwindfunclet$?onSubTaskFinished@WevoteTask@U2@@EAE?AV?$QList@PAVTask@U2@@@@PAVTask@2@@Z$6 10012639 f   WevoteTask.obj
 0001:00011653       __unwindfunclet$?onSubTaskFinished@WevoteTask@U2@@EAE?AV?$QList@PAVTask@U2@@@@PAVTask@2@@Z$7 10012653 f   WevoteTask.obj
 0001:0001166c       __ehhandler$?onSubTaskFinished@WevoteTask@U2@@EAE?AV?$QList@PAVTask@U2@@@@PAVTask@2@@Z 1001266c f   WevoteTask.obj
 0001:00011690       __unwindfunclet$?parseClassification@WevoteTask@U2@@AAEXXZ$0 10012690 f   WevoteTask.obj
 0001:0001169c       __unwindfunclet$?parseClassification@WevoteTask@U2@@AAEXXZ$1 1001269c f   WevoteTask.obj
 0001:000116a7       __unwindfunclet$?parseClassification@WevoteTask@U2@@AAEXXZ$2 100126a7 f   WevoteTask.obj
 0001:000116b3       __unwindfunclet$?parseClassification@WevoteTask@U2@@AAEXXZ$3 100126b3 f   WevoteTask.obj
 0001:000116be       __unwindfunclet$?parseClassification@WevoteTask@U2@@AAEXXZ$5 100126be f   WevoteTask.obj
 0001:000116ca       __unwindfunclet$?parseClassification@WevoteTask@U2@@AAEXXZ$6 100126ca f   WevoteTask.obj
 0001:000116d6       __unwindfunclet$?parseClassification@WevoteTask@U2@@AAEXXZ$4 100126d6 f   WevoteTask.obj
 0001:000116e2       __ehhandler$?parseClassification@WevoteTask@U2@@AAEXXZ 100126e2 f   WevoteTask.obj
 0001:00011710       __unwindfunclet$?prepare@WevoteTask@U2@@EAEXXZ$0 10012710 f   WevoteTask.obj
 0001:0001171b       __ehhandler$?prepare@WevoteTask@U2@@EAEXXZ 1001271b f   WevoteTask.obj
 0001:00011740       __unwindfunclet$?run@WevoteTask@U2@@EAEXXZ$0 10012740 f   WevoteTask.obj
 0001:00011749       __unwindfunclet$?run@WevoteTask@U2@@EAEXXZ$1 10012749 f   WevoteTask.obj
 0001:00011752       __unwindfunclet$?run@WevoteTask@U2@@EAEXXZ$2 10012752 f   WevoteTask.obj
 0001:0001175b       __ehhandler$?run@WevoteTask@U2@@EAEXXZ 1001275b f   WevoteTask.obj
 0001:00011780       __unwindfunclet$??__EalgoLog@U2@@YAXXZ$0 10012780 f   WevoteValidator.obj
 0001:00011789       __ehhandler$??__EalgoLog@U2@@YAXXZ 10012789 f   WevoteValidator.obj
 0001:000117b0       __unwindfunclet$??__EcmdLog@U2@@YAXXZ$0 100127b0 f   WevoteValidator.obj
 0001:000117b9       __ehhandler$??__EcmdLog@U2@@YAXXZ 100127b9 f   WevoteValidator.obj
 0001:000117e0       __unwindfunclet$??__EcoreLog@U2@@YAXXZ$0 100127e0 f   WevoteValidator.obj
 0001:000117e9       __ehhandler$??__EcoreLog@U2@@YAXXZ 100127e9 f   WevoteValidator.obj
 0001:00011810       __unwindfunclet$??__EioLog@U2@@YAXXZ$0 10012810 f   WevoteValidator.obj
 0001:00011819       __ehhandler$??__EioLog@U2@@YAXXZ 10012819 f   WevoteValidator.obj
 0001:00011840       __unwindfunclet$??__EperfLog@U2@@YAXXZ$0 10012840 f   WevoteValidator.obj
 0001:00011849       __ehhandler$??__EperfLog@U2@@YAXXZ 10012849 f   WevoteValidator.obj
 0001:00011870       __unwindfunclet$??__EscriptLog@U2@@YAXXZ$0 10012870 f   WevoteValidator.obj
 0001:00011879       __ehhandler$??__EscriptLog@U2@@YAXXZ 10012879 f   WevoteValidator.obj
 0001:000118a0       __unwindfunclet$??__EtaskLog@U2@@YAXXZ$0 100128a0 f   WevoteValidator.obj
 0001:000118a9       __ehhandler$??__EtaskLog@U2@@YAXXZ 100128a9 f   WevoteValidator.obj
 0001:000118d0       __unwindfunclet$??__EuiLog@U2@@YAXXZ$0 100128d0 f   WevoteValidator.obj
 0001:000118d9       __ehhandler$??__EuiLog@U2@@YAXXZ 100128d9 f   WevoteValidator.obj
 0001:00011900       __unwindfunclet$??__EuserActLog@U2@@YAXXZ$0 10012900 f   WevoteValidator.obj
 0001:00011909       __ehhandler$??__EuserActLog@U2@@YAXXZ 10012909 f   WevoteValidator.obj
 0001:00011930       __unwindfunclet$?append@?$QList@VWorkflowNotification@U2@@@@QAEXABVWorkflowNotification@U2@@@Z$6 10012930 f   WevoteValidator.obj
 0001:0001193b       __ehhandler$?append@?$QList@VWorkflowNotification@U2@@@@QAEXABVWorkflowNotification@U2@@@Z 1001293b f   WevoteValidator.obj
 0001:00011960       __ehhandler$?detach_helper_grow@?$QList@VWorkflowNotification@U2@@@@AAEPAUNode@1@HH@Z 10012960 f   WevoteValidator.obj
 0001:00011980       __unwindfunclet$?node_construct@?$QList@VWorkflowNotification@U2@@@@AAEXPAUNode@1@ABVWorkflowNotification@U2@@@Z$0 10012980 f   WevoteValidator.obj
 0001:0001198b       __ehhandler$?node_construct@?$QList@VWorkflowNotification@U2@@@@AAEXPAUNode@1@ABVWorkflowNotification@U2@@@Z 1001298b f   WevoteValidator.obj
 0001:000119b0       __unwindfunclet$?node_copy@?$QList@VWorkflowNotification@U2@@@@AAEXPAUNode@1@00@Z$4 100129b0 f   WevoteValidator.obj
 0001:000119bb       __ehhandler$?node_copy@?$QList@VWorkflowNotification@U2@@@@AAEXPAUNode@1@00@Z 100129bb f   WevoteValidator.obj
 0001:000119e0       __unwindfunclet$?validateTaxonomy@WevoteValidator@Workflow@U2@@ABE_NPBVActor@23@AAV?$QList@VWorkflowNotification@U2@@@@@Z$0 100129e0 f   WevoteValidator.obj
 0001:000119e9       __unwindfunclet$?validateTaxonomy@WevoteValidator@Workflow@U2@@ABE_NPBVActor@23@AAV?$QList@VWorkflowNotification@U2@@@@@Z$1 100129e9 f   WevoteValidator.obj
 0001:000119f2       __unwindfunclet$?validateTaxonomy@WevoteValidator@Workflow@U2@@ABE_NPBVActor@23@AAV?$QList@VWorkflowNotification@U2@@@@@Z$2 100129f2 f   WevoteValidator.obj
 0001:000119fb       __unwindfunclet$?validateTaxonomy@WevoteValidator@Workflow@U2@@ABE_NPBVActor@23@AAV?$QList@VWorkflowNotification@U2@@@@@Z$6 100129fb f   WevoteValidator.obj
 0001:00011a04       __unwindfunclet$?validateTaxonomy@WevoteValidator@Workflow@U2@@ABE_NPBVActor@23@AAV?$QList@VWorkflowNotification@U2@@@@@Z$8 10012a04 f   WevoteValidator.obj
 0001:00011a0d       __unwindfunclet$?validateTaxonomy@WevoteValidator@Workflow@U2@@ABE_NPBVActor@23@AAV?$QList@VWorkflowNotification@U2@@@@@Z$9 10012a0d f   WevoteValidator.obj
 0001:00011a16       __unwindfunclet$?validateTaxonomy@WevoteValidator@Workflow@U2@@ABE_NPBVActor@23@AAV?$QList@VWorkflowNotification@U2@@@@@Z$10 10012a16 f   WevoteValidator.obj
 0001:00011a1f       __unwindfunclet$?validateTaxonomy@WevoteValidator@Workflow@U2@@ABE_NPBVActor@23@AAV?$QList@VWorkflowNotification@U2@@@@@Z$12 10012a1f f   WevoteValidator.obj
 0001:00011a28       __unwindfunclet$?validateTaxonomy@WevoteValidator@Workflow@U2@@ABE_NPBVActor@23@AAV?$QList@VWorkflowNotification@U2@@@@@Z$13 10012a28 f   WevoteValidator.obj
 0001:00011a31       __unwindfunclet$?validateTaxonomy@WevoteValidator@Workflow@U2@@ABE_NPBVActor@23@AAV?$QList@VWorkflowNotification@U2@@@@@Z$14 10012a31 f   WevoteValidator.obj
 0001:00011a3a       __unwindfunclet$?validateTaxonomy@WevoteValidator@Workflow@U2@@ABE_NPBVActor@23@AAV?$QList@VWorkflowNotification@U2@@@@@Z$3 10012a3a f   WevoteValidator.obj
 0001:00011a43       __unwindfunclet$?validateTaxonomy@WevoteValidator@Workflow@U2@@ABE_NPBVActor@23@AAV?$QList@VWorkflowNotification@U2@@@@@Z$4 10012a43 f   WevoteValidator.obj
 0001:00011a4c       __unwindfunclet$?validateTaxonomy@WevoteValidator@Workflow@U2@@ABE_NPBVActor@23@AAV?$QList@VWorkflowNotification@U2@@@@@Z$5 10012a4c f   WevoteValidator.obj
 0001:00011a55       __ehhandler$?validateTaxonomy@WevoteValidator@Workflow@U2@@ABE_NPBVActor@23@AAV?$QList@VWorkflowNotification@U2@@@@@Z 10012a55 f   WevoteValidator.obj
 0001:00011a70       __unwindfunclet$??$getAttributeValue@H@Attribute@U2@@QBEHPAVWorkflowContext@Workflow@1@@Z$0 10012a70 f   WevoteWorker.obj
 0001:00011a79       __unwindfunclet$??$getAttributeValue@H@Attribute@U2@@QBEHPAVWorkflowContext@Workflow@1@@Z$1 10012a79 f   WevoteWorker.obj
 0001:00011a81       __unwindfunclet$??$getAttributeValue@H@Attribute@U2@@QBEHPAVWorkflowContext@Workflow@1@@Z$2 10012a81 f   WevoteWorker.obj
 0001:00011a89       __unwindfunclet$??$getAttributeValue@H@Attribute@U2@@QBEHPAVWorkflowContext@Workflow@1@@Z$3 10012a89 f   WevoteWorker.obj
 0001:00011a91       __unwindfunclet$??$getAttributeValue@H@Attribute@U2@@QBEHPAVWorkflowContext@Workflow@1@@Z$4 10012a91 f   WevoteWorker.obj
 0001:00011a9a       __unwindfunclet$??$getAttributeValue@H@Attribute@U2@@QBEHPAVWorkflowContext@Workflow@1@@Z$5 10012a9a f   WevoteWorker.obj
 0001:00011aa3       __unwindfunclet$??$getAttributeValue@H@Attribute@U2@@QBEHPAVWorkflowContext@Workflow@1@@Z$6 10012aa3 f   WevoteWorker.obj
 0001:00011aac       __unwindfunclet$??$getAttributeValue@H@Attribute@U2@@QBEHPAVWorkflowContext@Workflow@1@@Z$7 10012aac f   WevoteWorker.obj
 0001:00011ab5       __unwindfunclet$??$getAttributeValue@H@Attribute@U2@@QBEHPAVWorkflowContext@Workflow@1@@Z$8 10012ab5 f   WevoteWorker.obj
 0001:00011abe       __unwindfunclet$??$getAttributeValue@H@Attribute@U2@@QBEHPAVWorkflowContext@Workflow@1@@Z$9 10012abe f   WevoteWorker.obj
 0001:00011ac7       __unwindfunclet$??$getAttributeValue@H@Attribute@U2@@QBEHPAVWorkflowContext@Workflow@1@@Z$10 10012ac7 f   WevoteWorker.obj
 0001:00011ad0       __unwindfunclet$??$getAttributeValue@H@Attribute@U2@@QBEHPAVWorkflowContext@Workflow@1@@Z$11 10012ad0 f   WevoteWorker.obj
 0001:00011ad9       __ehhandler$??$getAttributeValue@H@Attribute@U2@@QBEHPAVWorkflowContext@Workflow@1@@Z 10012ad9 f   WevoteWorker.obj
 0001:00011b00       __unwindfunclet$??$getAttributeValue@VQString@@@Attribute@U2@@QBE?AVQString@@PAVWorkflowContext@Workflow@1@@Z$0 10012b00 f   WevoteWorker.obj
 0001:00011b1a       __unwindfunclet$??$getAttributeValue@VQString@@@Attribute@U2@@QBE?AVQString@@PAVWorkflowContext@Workflow@1@@Z$1 10012b1a f   WevoteWorker.obj
 0001:00011b23       __unwindfunclet$??$getAttributeValue@VQString@@@Attribute@U2@@QBE?AVQString@@PAVWorkflowContext@Workflow@1@@Z$2 10012b23 f   WevoteWorker.obj
 0001:00011b2b       __unwindfunclet$??$getAttributeValue@VQString@@@Attribute@U2@@QBE?AVQString@@PAVWorkflowContext@Workflow@1@@Z$3 10012b2b f   WevoteWorker.obj
 0001:00011b33       __unwindfunclet$??$getAttributeValue@VQString@@@Attribute@U2@@QBE?AVQString@@PAVWorkflowContext@Workflow@1@@Z$4 10012b33 f   WevoteWorker.obj
 0001:00011b3b       __unwindfunclet$??$getAttributeValue@VQString@@@Attribute@U2@@QBE?AVQString@@PAVWorkflowContext@Workflow@1@@Z$5 10012b3b f   WevoteWorker.obj
 0001:00011b44       __unwindfunclet$??$getAttributeValue@VQString@@@Attribute@U2@@QBE?AVQString@@PAVWorkflowContext@Workflow@1@@Z$6 10012b44 f   WevoteWorker.obj
 0001:00011b4d       __unwindfunclet$??$getAttributeValue@VQString@@@Attribute@U2@@QBE?AVQString@@PAVWorkflowContext@Workflow@1@@Z$7 10012b4d f   WevoteWorker.obj
 0001:00011b56       __unwindfunclet$??$getAttributeValue@VQString@@@Attribute@U2@@QBE?AVQString@@PAVWorkflowContext@Workflow@1@@Z$8 10012b56 f   WevoteWorker.obj
 0001:00011b5f       __unwindfunclet$??$getAttributeValue@VQString@@@Attribute@U2@@QBE?AVQString@@PAVWorkflowContext@Workflow@1@@Z$9 10012b5f f   WevoteWorker.obj
 0001:00011b68       __unwindfunclet$??$getAttributeValue@VQString@@@Attribute@U2@@QBE?AVQString@@PAVWorkflowContext@Workflow@1@@Z$10 10012b68 f   WevoteWorker.obj
 0001:00011b71       __unwindfunclet$??$getAttributeValue@VQString@@@Attribute@U2@@QBE?AVQString@@PAVWorkflowContext@Workflow@1@@Z$11 10012b71 f   WevoteWorker.obj
 0001:00011b7a       __unwindfunclet$??$getAttributeValue@VQString@@@Attribute@U2@@QBE?AVQString@@PAVWorkflowContext@Workflow@1@@Z$12 10012b7a f   WevoteWorker.obj
 0001:00011b83       __ehhandler$??$getAttributeValue@VQString@@@Attribute@U2@@QBE?AVQString@@PAVWorkflowContext@Workflow@1@@Z 10012b83 f   WevoteWorker.obj
 0001:00011bb0       __unwindfunclet$??$getValue@VQString@@@BaseWorker@LocalWorkflow@U2@@IBE?AVQString@@ABV3@@Z$0 10012bb0 f   WevoteWorker.obj
 0001:00011bca       __unwindfunclet$??$getValue@VQString@@@BaseWorker@LocalWorkflow@U2@@IBE?AVQString@@ABV3@@Z$1 10012bca f   WevoteWorker.obj
 0001:00011bd3       __ehhandler$??$getValue@VQString@@@BaseWorker@LocalWorkflow@U2@@IBE?AVQString@@ABV3@@Z 10012bd3 f   WevoteWorker.obj
 0001:00011bf0       __unwindfunclet$??$qRegisterMetaType@V?$QMap@VQString@@I@@@@YAHPBDPAV?$QMap@VQString@@I@@W4DefinedType@?$MetaTypeDefinedHelper@V?$QMap@VQString@@I@@$00@QtPrivate@@@Z$0 10012bf0 f   WevoteWorker.obj
 0001:00011bf9       __ehhandler$??$qRegisterMetaType@V?$QMap@VQString@@I@@@@YAHPBDPAV?$QMap@VQString@@I@@W4DefinedType@?$MetaTypeDefinedHelper@V?$QMap@VQString@@I@@$00@QtPrivate@@@Z 10012bf9 f   WevoteWorker.obj
 0001:00011c20       __unwindfunclet$??$qRegisterMetaType@VQAssociativeIterableImpl@QtMetaTypePrivate@@@@YAHPBDPAVQAssociativeIterableImpl@QtMetaTypePrivate@@W4DefinedType@?$MetaTypeDefinedHelper@VQAssociativeIterableImpl@QtMetaTypePrivate@@$00@QtPrivate@@@Z$0 10012c20 f   WevoteWorker.obj
 0001:00011c29       __ehhandler$??$qRegisterMetaType@VQAssociativeIterableImpl@QtMetaTypePrivate@@@@YAHPBDPAVQAssociativeIterableImpl@QtMetaTypePrivate@@W4DefinedType@?$MetaTypeDefinedHelper@VQAssociativeIterableImpl@QtMetaTypePrivate@@$00@QtPrivate@@@Z 10012c29 f   WevoteWorker.obj
 0001:00011c50       __ehhandler$??0?$QList@VDescriptor@U2@@@@QAE@ABV0@@Z 10012c50 f   WevoteWorker.obj
 0001:00011c70       __unwindfunclet$??A?$QMap@VQString@@VQScriptValue@@@@QAEAAVQScriptValue@@ABVQString@@@Z$0 10012c70 f   WevoteWorker.obj
 0001:00011c79       __ehhandler$??A?$QMap@VQString@@VQScriptValue@@@@QAEAAVQScriptValue@@ABVQString@@@Z 10012c79 f   WevoteWorker.obj
 0001:00011ca0       __unwindfunclet$??A?$QMap@VQString@@VQVariant@@@@QAEAAVQVariant@@ABVQString@@@Z$0 10012ca0 f   WevoteWorker.obj
 0001:00011ca9       __ehhandler$??A?$QMap@VQString@@VQVariant@@@@QAEAAVQVariant@@ABVQString@@@Z 10012ca9 f   WevoteWorker.obj
 0001:00011cd0       __unwindfunclet$??__EalgoLog@U2@@YAXXZ$0 10012cd0 f   WevoteWorker.obj
 0001:00011cd9       __ehhandler$??__EalgoLog@U2@@YAXXZ 10012cd9 f   WevoteWorker.obj
 0001:00011d00       __unwindfunclet$??__EcmdLog@U2@@YAXXZ$0 10012d00 f   WevoteWorker.obj
 0001:00011d09       __ehhandler$??__EcmdLog@U2@@YAXXZ 10012d09 f   WevoteWorker.obj
 0001:00011d30       __unwindfunclet$??__EcoreLog@U2@@YAXXZ$0 10012d30 f   WevoteWorker.obj
 0001:00011d39       __ehhandler$??__EcoreLog@U2@@YAXXZ 10012d39 f   WevoteWorker.obj
 0001:00011d60       __unwindfunclet$??__EioLog@U2@@YAXXZ$0 10012d60 f   WevoteWorker.obj
 0001:00011d69       __ehhandler$??__EioLog@U2@@YAXXZ 10012d69 f   WevoteWorker.obj
 0001:00011d90       __unwindfunclet$??__EperfLog@U2@@YAXXZ$0 10012d90 f   WevoteWorker.obj
 0001:00011d99       __ehhandler$??__EperfLog@U2@@YAXXZ 10012d99 f   WevoteWorker.obj
 0001:00011dc0       __unwindfunclet$??__EscriptLog@U2@@YAXXZ$0 10012dc0 f   WevoteWorker.obj
 0001:00011dc9       __ehhandler$??__EscriptLog@U2@@YAXXZ 10012dc9 f   WevoteWorker.obj
 0001:00011df0       __unwindfunclet$??__EtaskLog@U2@@YAXXZ$0 10012df0 f   WevoteWorker.obj
 0001:00011df9       __ehhandler$??__EtaskLog@U2@@YAXXZ 10012df9 f   WevoteWorker.obj
 0001:00011e20       __unwindfunclet$??__EuiLog@U2@@YAXXZ$0 10012e20 f   WevoteWorker.obj
 0001:00011e29       __ehhandler$??__EuiLog@U2@@YAXXZ 10012e29 f   WevoteWorker.obj
 0001:00011e50       __unwindfunclet$??__EuserActLog@U2@@YAXXZ$0 10012e50 f   WevoteWorker.obj
 0001:00011e59       __ehhandler$??__EuserActLog@U2@@YAXXZ 10012e59 f   WevoteWorker.obj
 0001:00011e80       __unwindfunclet$?Construct@?$QMetaTypeFunctionHelper@V?$QMap@VQString@@I@@$00@QtMetaTypePrivate@@SAPAXPAXPBX@Z$0 10012e80 f   WevoteWorker.obj
 0001:00011e91       __ehhandler$?Construct@?$QMetaTypeFunctionHelper@V?$QMap@VQString@@I@@$00@QtMetaTypePrivate@@SAPAXPAXPBX@Z 10012e91 f   WevoteWorker.obj
 0001:00011eb0       __unwindfunclet$?Create@?$QMetaTypeFunctionHelper@V?$QMap@VQString@@I@@$00@QtMetaTypePrivate@@SAPAXPBX@Z$0 10012eb0 f   WevoteWorker.obj
 0001:00011ebb       __ehhandler$?Create@?$QMetaTypeFunctionHelper@V?$QMap@VQString@@I@@$00@QtMetaTypePrivate@@SAPAXPBX@Z 10012ebb f   WevoteWorker.obj
 0001:00011ee0       __unwindfunclet$?append@?$QList@VDescriptor@U2@@@@QAEXABVDescriptor@U2@@@Z$6 10012ee0 f   WevoteWorker.obj
 0001:00011eeb       __ehhandler$?append@?$QList@VDescriptor@U2@@@@QAEXABVDescriptor@U2@@@Z 10012eeb f   WevoteWorker.obj
 0001:00011f10       __unwindfunclet$?createNode@?$QMapData@VQString@@VQScriptValue@@@@QAEPAU?$QMapNode@VQString@@VQScriptValue@@@@ABVQString@@ABVQScriptValue@@PAU2@_N@Z$4 10012f10 f   WevoteWorker.obj
 0001:00011f24       __unwindfunclet$?createNode@?$QMapData@VQString@@VQScriptValue@@@@QAEPAU?$QMapNode@VQString@@VQScriptValue@@@@ABVQString@@ABVQScriptValue@@PAU2@_N@Z$5 10012f24 f   WevoteWorker.obj
 0001:00011f38       __ehhandler$?createNode@?$QMapData@VQString@@VQScriptValue@@@@QAEPAU?$QMapNode@VQString@@VQScriptValue@@@@ABVQString@@ABVQScriptValue@@PAU2@_N@Z 10012f38 f   WevoteWorker.obj
 0001:00011f60       __unwindfunclet$?createNode@?$QMapData@VQString@@VQVariant@@@@QAEPAU?$QMapNode@VQString@@VQVariant@@@@ABVQString@@ABVQVariant@@PAU2@_N@Z$4 10012f60 f   WevoteWorker.obj
 0001:00011f74       __unwindfunclet$?createNode@?$QMapData@VQString@@VQVariant@@@@QAEPAU?$QMapNode@VQString@@VQVariant@@@@ABVQString@@ABVQVariant@@PAU2@_N@Z$5 10012f74 f   WevoteWorker.obj
 0001:00011f88       __ehhandler$?createNode@?$QMapData@VQString@@VQVariant@@@@QAEPAU?$QMapNode@VQString@@VQVariant@@@@ABVQString@@ABVQVariant@@PAU2@_N@Z 10012f88 f   WevoteWorker.obj
 0001:00011fb0       __ehhandler$?detach_helper@?$QList@VDescriptor@U2@@@@AAEXH@Z 10012fb0 f   WevoteWorker.obj
 0001:00011fd0       __ehhandler$?detach_helper_grow@?$QList@VDescriptor@U2@@@@AAEPAUNode@1@HH@Z 10012fd0 f   WevoteWorker.obj
 0001:00011ff0       __unwindfunclet$?getSettings@WevoteWorker@LocalWorkflow@U2@@AAE?AUWevoteTaskSettings@3@AAVU2OpStatus@3@@Z$0 10012ff0 f   WevoteWorker.obj
 0001:00011ff8       __unwindfunclet$?getSettings@WevoteWorker@LocalWorkflow@U2@@AAE?AUWevoteTaskSettings@3@AAVU2OpStatus@3@@Z$1 10012ff8 f   WevoteWorker.obj
 0001:00012004       __unwindfunclet$?getSettings@WevoteWorker@LocalWorkflow@U2@@AAE?AUWevoteTaskSettings@3@AAVU2OpStatus@3@@Z$2 10013004 f   WevoteWorker.obj
 0001:0001200d       __unwindfunclet$?getSettings@WevoteWorker@LocalWorkflow@U2@@AAE?AUWevoteTaskSettings@3@AAVU2OpStatus@3@@Z$3 1001300d f   WevoteWorker.obj
 0001:00012016       __unwindfunclet$?getSettings@WevoteWorker@LocalWorkflow@U2@@AAE?AUWevoteTaskSettings@3@AAVU2OpStatus@3@@Z$4 10013016 f   WevoteWorker.obj
 0001:0001201f       __unwindfunclet$?getSettings@WevoteWorker@LocalWorkflow@U2@@AAE?AUWevoteTaskSettings@3@AAVU2OpStatus@3@@Z$5 1001301f f   WevoteWorker.obj
 0001:00012027       __unwindfunclet$?getSettings@WevoteWorker@LocalWorkflow@U2@@AAE?AUWevoteTaskSettings@3@AAVU2OpStatus@3@@Z$6 10013027 f   WevoteWorker.obj
 0001:00012030       __unwindfunclet$?getSettings@WevoteWorker@LocalWorkflow@U2@@AAE?AUWevoteTaskSettings@3@AAVU2OpStatus@3@@Z$7 10013030 f   WevoteWorker.obj
 0001:00012039       __unwindfunclet$?getSettings@WevoteWorker@LocalWorkflow@U2@@AAE?AUWevoteTaskSettings@3@AAVU2OpStatus@3@@Z$23 10013039 f   WevoteWorker.obj
 0001:00012045       __unwindfunclet$?getSettings@WevoteWorker@LocalWorkflow@U2@@AAE?AUWevoteTaskSettings@3@AAVU2OpStatus@3@@Z$24 10013045 f   WevoteWorker.obj
 0001:00012051       __unwindfunclet$?getSettings@WevoteWorker@LocalWorkflow@U2@@AAE?AUWevoteTaskSettings@3@AAVU2OpStatus@3@@Z$8 10013051 f   WevoteWorker.obj
 0001:0001206a       __unwindfunclet$?getSettings@WevoteWorker@LocalWorkflow@U2@@AAE?AUWevoteTaskSettings@3@AAVU2OpStatus@3@@Z$26 1001306a f   WevoteWorker.obj
 0001:00012073       __unwindfunclet$?getSettings@WevoteWorker@LocalWorkflow@U2@@AAE?AUWevoteTaskSettings@3@AAVU2OpStatus@3@@Z$27 10013073 f   WevoteWorker.obj
 0001:0001207c       __unwindfunclet$?getSettings@WevoteWorker@LocalWorkflow@U2@@AAE?AUWevoteTaskSettings@3@AAVU2OpStatus@3@@Z$9 1001307c f   WevoteWorker.obj
 0001:00012085       __unwindfunclet$?getSettings@WevoteWorker@LocalWorkflow@U2@@AAE?AUWevoteTaskSettings@3@AAVU2OpStatus@3@@Z$10 10013085 f   WevoteWorker.obj
 0001:0001208e       __unwindfunclet$?getSettings@WevoteWorker@LocalWorkflow@U2@@AAE?AUWevoteTaskSettings@3@AAVU2OpStatus@3@@Z$11 1001308e f   WevoteWorker.obj
 0001:00012097       __unwindfunclet$?getSettings@WevoteWorker@LocalWorkflow@U2@@AAE?AUWevoteTaskSettings@3@AAVU2OpStatus@3@@Z$12 10013097 f   WevoteWorker.obj
 0001:000120a0       __unwindfunclet$?getSettings@WevoteWorker@LocalWorkflow@U2@@AAE?AUWevoteTaskSettings@3@AAVU2OpStatus@3@@Z$13 100130a0 f   WevoteWorker.obj
 0001:000120a9       __unwindfunclet$?getSettings@WevoteWorker@LocalWorkflow@U2@@AAE?AUWevoteTaskSettings@3@AAVU2OpStatus@3@@Z$14 100130a9 f   WevoteWorker.obj
 0001:000120b2       __unwindfunclet$?getSettings@WevoteWorker@LocalWorkflow@U2@@AAE?AUWevoteTaskSettings@3@AAVU2OpStatus@3@@Z$15 100130b2 f   WevoteWorker.obj
 0001:000120bb       __unwindfunclet$?getSettings@WevoteWorker@LocalWorkflow@U2@@AAE?AUWevoteTaskSettings@3@AAVU2OpStatus@3@@Z$16 100130bb f   WevoteWorker.obj
 0001:000120c4       __unwindfunclet$?getSettings@WevoteWorker@LocalWorkflow@U2@@AAE?AUWevoteTaskSettings@3@AAVU2OpStatus@3@@Z$17 100130c4 f   WevoteWorker.obj
 0001:000120cd       __unwindfunclet$?getSettings@WevoteWorker@LocalWorkflow@U2@@AAE?AUWevoteTaskSettings@3@AAVU2OpStatus@3@@Z$18 100130cd f   WevoteWorker.obj
 0001:000120d6       __unwindfunclet$?getSettings@WevoteWorker@LocalWorkflow@U2@@AAE?AUWevoteTaskSettings@3@AAVU2OpStatus@3@@Z$19 100130d6 f   WevoteWorker.obj
 0001:000120df       __unwindfunclet$?getSettings@WevoteWorker@LocalWorkflow@U2@@AAE?AUWevoteTaskSettings@3@AAVU2OpStatus@3@@Z$20 100130df f   WevoteWorker.obj
 0001:000120e8       __unwindfunclet$?getSettings@WevoteWorker@LocalWorkflow@U2@@AAE?AUWevoteTaskSettings@3@AAVU2OpStatus@3@@Z$21 100130e8 f   WevoteWorker.obj
 0001:000120f1       __unwindfunclet$?getSettings@WevoteWorker@LocalWorkflow@U2@@AAE?AUWevoteTaskSettings@3@AAVU2OpStatus@3@@Z$22 100130f1 f   WevoteWorker.obj
 0001:000120fa       __unwindfunclet$?getSettings@WevoteWorker@LocalWorkflow@U2@@AAE?AUWevoteTaskSettings@3@AAVU2OpStatus@3@@Z$29 100130fa f   WevoteWorker.obj
 0001:00012106       __unwindfunclet$?getSettings@WevoteWorker@LocalWorkflow@U2@@AAE?AUWevoteTaskSettings@3@AAVU2OpStatus@3@@Z$30 10013106 f   WevoteWorker.obj
 0001:00012112       __unwindfunclet$?getSettings@WevoteWorker@LocalWorkflow@U2@@AAE?AUWevoteTaskSettings@3@AAVU2OpStatus@3@@Z$32 10013112 f   WevoteWorker.obj
 0001:0001211b       __unwindfunclet$?getSettings@WevoteWorker@LocalWorkflow@U2@@AAE?AUWevoteTaskSettings@3@AAVU2OpStatus@3@@Z$33 1001311b f   WevoteWorker.obj
 0001:00012124       __ehhandler$?getSettings@WevoteWorker@LocalWorkflow@U2@@AAE?AUWevoteTaskSettings@3@AAVU2OpStatus@3@@Z 10013124 f   WevoteWorker.obj
 0001:00012150       __unwindfunclet$?init@WevoteWorker@LocalWorkflow@U2@@UAEXXZ$0 10013150 f   WevoteWorker.obj
 0001:00012159       __unwindfunclet$?init@WevoteWorker@LocalWorkflow@U2@@UAEXXZ$1 10013159 f   WevoteWorker.obj
 0001:00012162       __unwindfunclet$?init@WevoteWorker@LocalWorkflow@U2@@UAEXXZ$2 10013162 f   WevoteWorker.obj
 0001:0001216b       __unwindfunclet$?init@WevoteWorker@LocalWorkflow@U2@@UAEXXZ$3 1001316b f   WevoteWorker.obj
 0001:00012174       __unwindfunclet$?init@WevoteWorker@LocalWorkflow@U2@@UAEXXZ$4 10013174 f   WevoteWorker.obj
 0001:0001217d       __unwindfunclet$?init@WevoteWorker@LocalWorkflow@U2@@UAEXXZ$5 1001317d f   WevoteWorker.obj
 0001:00012186       __unwindfunclet$?init@WevoteWorker@LocalWorkflow@U2@@UAEXXZ$6 10013186 f   WevoteWorker.obj
 0001:0001218f       __unwindfunclet$?init@WevoteWorker@LocalWorkflow@U2@@UAEXXZ$7 1001318f f   WevoteWorker.obj
 0001:00012198       __unwindfunclet$?init@WevoteWorker@LocalWorkflow@U2@@UAEXXZ$8 10013198 f   WevoteWorker.obj
 0001:000121a1       __unwindfunclet$?init@WevoteWorker@LocalWorkflow@U2@@UAEXXZ$9 100131a1 f   WevoteWorker.obj
 0001:000121aa       __unwindfunclet$?init@WevoteWorker@LocalWorkflow@U2@@UAEXXZ$10 100131aa f   WevoteWorker.obj
 0001:000121b3       __unwindfunclet$?init@WevoteWorker@LocalWorkflow@U2@@UAEXXZ$11 100131b3 f   WevoteWorker.obj
 0001:000121bc       __unwindfunclet$?init@WevoteWorker@LocalWorkflow@U2@@UAEXXZ$12 100131bc f   WevoteWorker.obj
 0001:000121c5       __unwindfunclet$?init@WevoteWorker@LocalWorkflow@U2@@UAEXXZ$13 100131c5 f   WevoteWorker.obj
 0001:000121ce       __ehhandler$?init@WevoteWorker@LocalWorkflow@U2@@UAEXXZ 100131ce f   WevoteWorker.obj
 0001:000121f0       __unwindfunclet$?metaType@?$QVariantValueHelper@VQString@@@QtPrivate@@SA?AVQString@@ABVQVariant@@@Z$0 100131f0 f   WevoteWorker.obj
 0001:0001220a       __unwindfunclet$?metaType@?$QVariantValueHelper@VQString@@@QtPrivate@@SA?AVQString@@ABVQVariant@@@Z$1 1001320a f   WevoteWorker.obj
 0001:00012213       __ehhandler$?metaType@?$QVariantValueHelper@VQString@@@QtPrivate@@SA?AVQString@@ABVQVariant@@@Z 10013213 f   WevoteWorker.obj
 0001:00012230       __unwindfunclet$?node_construct@?$QList@VDescriptor@U2@@@@AAEXPAUNode@1@ABVDescriptor@U2@@@Z$0 10013230 f   WevoteWorker.obj
 0001:0001223b       __ehhandler$?node_construct@?$QList@VDescriptor@U2@@@@AAEXPAUNode@1@ABVDescriptor@U2@@@Z 1001323b f   WevoteWorker.obj
 0001:00012260       __unwindfunclet$?node_copy@?$QList@VDescriptor@U2@@@@AAEXPAUNode@1@00@Z$4 10013260 f   WevoteWorker.obj
 0001:0001226b       __ehhandler$?node_copy@?$QList@VDescriptor@U2@@@@AAEXPAUNode@1@00@Z 1001326b f   WevoteWorker.obj
 0001:00012290       __unwindfunclet$?qt_metatype_id@?$QMetaTypeId@V?$QMap@VQString@@I@@@@SAHXZ$0 10013290 f   WevoteWorker.obj
 0001:00012299       __ehhandler$?qt_metatype_id@?$QMetaTypeId@V?$QMap@VQString@@I@@@@SAHXZ 10013299 f   WevoteWorker.obj
 0001:000122c0       __unwindfunclet$?qt_metatype_id@?$QMetaTypeId@VQAssociativeIterableImpl@QtMetaTypePrivate@@@@SAHXZ$0 100132c0 f   WevoteWorker.obj
 0001:000122c9       __ehhandler$?qt_metatype_id@?$QMetaTypeId@VQAssociativeIterableImpl@QtMetaTypePrivate@@@@SAHXZ 100132c9 f   WevoteWorker.obj
 0001:000122f0       __unwindfunclet$?sl_taskFinished@WevoteWorker@LocalWorkflow@U2@@AAEXPAVTask@3@@Z$0 100132f0 f   WevoteWorker.obj
 0001:000122f9       __unwindfunclet$?sl_taskFinished@WevoteWorker@LocalWorkflow@U2@@AAEXPAVTask@3@@Z$1 100132f9 f   WevoteWorker.obj
 0001:00012301       __unwindfunclet$?sl_taskFinished@WevoteWorker@LocalWorkflow@U2@@AAEXPAVTask@3@@Z$2 10013301 f   WevoteWorker.obj
 0001:00012309       __unwindfunclet$?sl_taskFinished@WevoteWorker@LocalWorkflow@U2@@AAEXPAVTask@3@@Z$3 10013309 f   WevoteWorker.obj
 0001:00012312       __unwindfunclet$?sl_taskFinished@WevoteWorker@LocalWorkflow@U2@@AAEXPAVTask@3@@Z$4 10013312 f   WevoteWorker.obj
 0001:0001231b       __unwindfunclet$?sl_taskFinished@WevoteWorker@LocalWorkflow@U2@@AAEXPAVTask@3@@Z$6 1001331b f   WevoteWorker.obj
 0001:00012324       __unwindfunclet$?sl_taskFinished@WevoteWorker@LocalWorkflow@U2@@AAEXPAVTask@3@@Z$7 10013324 f   WevoteWorker.obj
 0001:0001232d       __unwindfunclet$?sl_taskFinished@WevoteWorker@LocalWorkflow@U2@@AAEXPAVTask@3@@Z$8 1001332d f   WevoteWorker.obj
 0001:00012336       __unwindfunclet$?sl_taskFinished@WevoteWorker@LocalWorkflow@U2@@AAEXPAVTask@3@@Z$9 10013336 f   WevoteWorker.obj
 0001:0001233f       __unwindfunclet$?sl_taskFinished@WevoteWorker@LocalWorkflow@U2@@AAEXPAVTask@3@@Z$10 1001333f f   WevoteWorker.obj
 0001:00012348       __unwindfunclet$?sl_taskFinished@WevoteWorker@LocalWorkflow@U2@@AAEXPAVTask@3@@Z$11 10013348 f   WevoteWorker.obj
 0001:00012351       __unwindfunclet$?sl_taskFinished@WevoteWorker@LocalWorkflow@U2@@AAEXPAVTask@3@@Z$12 10013351 f   WevoteWorker.obj
 0001:0001235a       __unwindfunclet$?sl_taskFinished@WevoteWorker@LocalWorkflow@U2@@AAEXPAVTask@3@@Z$13 1001335a f   WevoteWorker.obj
 0001:00012363       __ehhandler$?sl_taskFinished@WevoteWorker@LocalWorkflow@U2@@AAEXPAVTask@3@@Z 10013363 f   WevoteWorker.obj
 0001:00012380       __unwindfunclet$?tick@WevoteWorker@LocalWorkflow@U2@@UAEPAVTask@3@XZ$0 10013380 f   WevoteWorker.obj
 0001:00012389       __unwindfunclet$?tick@WevoteWorker@LocalWorkflow@U2@@UAEPAVTask@3@XZ$1 10013389 f   WevoteWorker.obj
 0001:00012391       __unwindfunclet$?tick@WevoteWorker@LocalWorkflow@U2@@UAEPAVTask@3@XZ$2 10013391 f   WevoteWorker.obj
 0001:0001239c       __unwindfunclet$?tick@WevoteWorker@LocalWorkflow@U2@@UAEPAVTask@3@XZ$3 1001339c f   WevoteWorker.obj
 0001:000123b6       __unwindfunclet$?tick@WevoteWorker@LocalWorkflow@U2@@UAEPAVTask@3@XZ$4 100133b6 f   WevoteWorker.obj
 0001:000123c1       __unwindfunclet$?tick@WevoteWorker@LocalWorkflow@U2@@UAEPAVTask@3@XZ$5 100133c1 f   WevoteWorker.obj
 0001:000123c9       __unwindfunclet$?tick@WevoteWorker@LocalWorkflow@U2@@UAEPAVTask@3@XZ$6 100133c9 f   WevoteWorker.obj
 0001:000123d4       __unwindfunclet$?tick@WevoteWorker@LocalWorkflow@U2@@UAEPAVTask@3@XZ$8 100133d4 f   WevoteWorker.obj
 0001:000123dd       __unwindfunclet$?tick@WevoteWorker@LocalWorkflow@U2@@UAEPAVTask@3@XZ$9 100133dd f   WevoteWorker.obj
 0001:000123e6       __ehhandler$?tick@WevoteWorker@LocalWorkflow@U2@@UAEPAVTask@3@XZ 100133e6 f   WevoteWorker.obj
 0001:00012410       __unwindfunclet$?uniqueKeys@?$QMap@VDescriptor@U2@@VQVariant@@@@QBE?AV?$QList@VDescriptor@U2@@@@XZ$1 10013410 f   WevoteWorker.obj
 0001:00012429       __ehhandler$?uniqueKeys@?$QMap@VDescriptor@U2@@VQVariant@@@@QBE?AV?$QList@VDescriptor@U2@@@@XZ 10013429 f   WevoteWorker.obj
 0001:00012450       __unwindfunclet$??0QStringList@@QAE@ABVQString@@@Z$0 10013450 f   WevoteWorkerFactory.obj
 0001:00012458       __ehhandler$??0QStringList@@QAE@ABVQString@@@Z 10013458 f   WevoteWorkerFactory.obj
 0001:00012480       __unwindfunclet$??A?$QMap@VDescriptor@U2@@V?$QExplicitlySharedDataPointer@VDataType@U2@@@@@@QAEAAV?$QExplicitlySharedDataPointer@VDataType@U2@@@@ABVDescriptor@U2@@@Z$0 10013480 f   WevoteWorkerFactory.obj
 0001:00012488       __ehhandler$??A?$QMap@VDescriptor@U2@@V?$QExplicitlySharedDataPointer@VDataType@U2@@@@@@QAEAAV?$QExplicitlySharedDataPointer@VDataType@U2@@@@ABVDescriptor@U2@@@Z 10013488 f   WevoteWorkerFactory.obj
 0001:000124b0       __unwindfunclet$??__EalgoLog@U2@@YAXXZ$0 100134b0 f   WevoteWorkerFactory.obj
 0001:000124b9       __ehhandler$??__EalgoLog@U2@@YAXXZ 100134b9 f   WevoteWorkerFactory.obj
 0001:000124e0       __unwindfunclet$??__EcmdLog@U2@@YAXXZ$0 100134e0 f   WevoteWorkerFactory.obj
 0001:000124e9       __ehhandler$??__EcmdLog@U2@@YAXXZ 100134e9 f   WevoteWorkerFactory.obj
 0001:00012510       __unwindfunclet$??__EcoreLog@U2@@YAXXZ$0 10013510 f   WevoteWorkerFactory.obj
 0001:00012519       __ehhandler$??__EcoreLog@U2@@YAXXZ 10013519 f   WevoteWorkerFactory.obj
 0001:00012540       __unwindfunclet$??__EioLog@U2@@YAXXZ$0 10013540 f   WevoteWorkerFactory.obj
 0001:00012549       __ehhandler$??__EioLog@U2@@YAXXZ 10013549 f   WevoteWorkerFactory.obj
 0001:00012570       __unwindfunclet$??__EperfLog@U2@@YAXXZ$0 10013570 f   WevoteWorkerFactory.obj
 0001:00012579       __ehhandler$??__EperfLog@U2@@YAXXZ 10013579 f   WevoteWorkerFactory.obj
 0001:000125a0       __unwindfunclet$??__EscriptLog@U2@@YAXXZ$0 100135a0 f   WevoteWorkerFactory.obj
 0001:000125a9       __ehhandler$??__EscriptLog@U2@@YAXXZ 100135a9 f   WevoteWorkerFactory.obj
 0001:000125d0       __unwindfunclet$??__EtaskLog@U2@@YAXXZ$0 100135d0 f   WevoteWorkerFactory.obj
 0001:000125d9       __ehhandler$??__EtaskLog@U2@@YAXXZ 100135d9 f   WevoteWorkerFactory.obj
 0001:00012600       __unwindfunclet$??__EuiLog@U2@@YAXXZ$0 10013600 f   WevoteWorkerFactory.obj
 0001:00012609       __ehhandler$??__EuiLog@U2@@YAXXZ 10013609 f   WevoteWorkerFactory.obj
 0001:00012630       __unwindfunclet$??__EuserActLog@U2@@YAXXZ$0 10013630 f   WevoteWorkerFactory.obj
 0001:00012639       __ehhandler$??__EuserActLog@U2@@YAXXZ 10013639 f   WevoteWorkerFactory.obj
 0001:00012660       __ehhandler$?append@?$QList@PAVAttribute@U2@@@@QAEXABQAVAttribute@U2@@@Z 10013660 f   WevoteWorkerFactory.obj
 0001:00012680       __ehhandler$?append@?$QList@PAVPortDescriptor@Workflow@U2@@@@QAEXABQAVPortDescriptor@Workflow@U2@@@Z 10013680 f   WevoteWorkerFactory.obj
 0001:000126a0       __unwindfunclet$?createNode@?$QMapData@VDescriptor@U2@@V?$QExplicitlySharedDataPointer@VDataType@U2@@@@@@QAEPAU?$QMapNode@VDescriptor@U2@@V?$QExplicitlySharedDataPointer@VDataType@U2@@@@@@ABVDescriptor@U2@@ABV?$QExplicitlySharedDataPointer@VDataType@U2@@@@PAU2@_N@Z$4 100136a0 f   WevoteWorkerFactory.obj
 0001:000126b4       __ehhandler$?createNode@?$QMapData@VDescriptor@U2@@V?$QExplicitlySharedDataPointer@VDataType@U2@@@@@@QAEPAU?$QMapNode@VDescriptor@U2@@V?$QExplicitlySharedDataPointer@VDataType@U2@@@@@@ABVDescriptor@U2@@ABV?$QExplicitlySharedDataPointer@VDataType@U2@@@@PAU2@_N@Z 100136b4 f   WevoteWorkerFactory.obj
 0001:000126d0       __unwindfunclet$?createNode@?$QMapData@VQString@@PAVPropertyDelegate@U2@@@@QAEPAU?$QMapNode@VQString@@PAVPropertyDelegate@U2@@@@ABVQString@@ABQAVPropertyDelegate@U2@@PAU2@_N@Z$4 100136d0 f   WevoteWorkerFactory.obj
 0001:000126e4       __ehhandler$?createNode@?$QMapData@VQString@@PAVPropertyDelegate@U2@@@@QAEPAU?$QMapNode@VQString@@PAVPropertyDelegate@U2@@@@ABVQString@@ABQAVPropertyDelegate@U2@@PAU2@_N@Z 100136e4 f   WevoteWorkerFactory.obj
 0001:00012700       __unwindfunclet$?createWorker@WevoteWorkerFactory@LocalWorkflow@U2@@UAEPAVWorker@Workflow@3@PAVActor@53@@Z$0 10013700 f   WevoteWorkerFactory.obj
 0001:0001270b       __ehhandler$?createWorker@WevoteWorkerFactory@LocalWorkflow@U2@@UAEPAVWorker@Workflow@3@PAVActor@53@@Z 1001370b f   WevoteWorkerFactory.obj
 0001:00012730       __ehhandler$?detach_helper_grow@?$QList@PAVAttribute@U2@@@@AAEPAUNode@1@HH@Z 10013730 f   WevoteWorkerFactory.obj
 0001:00012750       __ehhandler$?detach_helper_grow@?$QList@PAVPortDescriptor@Workflow@U2@@@@AAEPAUNode@1@HH@Z 10013750 f   WevoteWorkerFactory.obj
 0001:00012770       __unwindfunclet$?init@WevoteWorkerFactory@LocalWorkflow@U2@@SAXXZ$0 10013770 f   WevoteWorkerFactory.obj
 0001:00012778       __unwindfunclet$?init@WevoteWorkerFactory@LocalWorkflow@U2@@SAXXZ$1 10013778 f   WevoteWorkerFactory.obj
 0001:00012781       __unwindfunclet$?init@WevoteWorkerFactory@LocalWorkflow@U2@@SAXXZ$2 10013781 f   WevoteWorkerFactory.obj
 0001:0001278a       __unwindfunclet$?init@WevoteWorkerFactory@LocalWorkflow@U2@@SAXXZ$3 1001378a f   WevoteWorkerFactory.obj
 0001:00012793       __unwindfunclet$?init@WevoteWorkerFactory@LocalWorkflow@U2@@SAXXZ$4 10013793 f   WevoteWorkerFactory.obj
 0001:0001279c       __unwindfunclet$?init@WevoteWorkerFactory@LocalWorkflow@U2@@SAXXZ$5 1001379c f   WevoteWorkerFactory.obj
 0001:000127a5       __unwindfunclet$?init@WevoteWorkerFactory@LocalWorkflow@U2@@SAXXZ$6 100137a5 f   WevoteWorkerFactory.obj
 0001:000127ad       __unwindfunclet$?init@WevoteWorkerFactory@LocalWorkflow@U2@@SAXXZ$7 100137ad f   WevoteWorkerFactory.obj
 0001:000127b5       __unwindfunclet$?init@WevoteWorkerFactory@LocalWorkflow@U2@@SAXXZ$8 100137b5 f   WevoteWorkerFactory.obj
 0001:000127bd       __unwindfunclet$?init@WevoteWorkerFactory@LocalWorkflow@U2@@SAXXZ$9 100137bd f   WevoteWorkerFactory.obj
 0001:000127c5       __unwindfunclet$?init@WevoteWorkerFactory@LocalWorkflow@U2@@SAXXZ$10 100137c5 f   WevoteWorkerFactory.obj
 0001:000127d1       __unwindfunclet$?init@WevoteWorkerFactory@LocalWorkflow@U2@@SAXXZ$11 100137d1 f   WevoteWorkerFactory.obj
 0001:000127da       __unwindfunclet$?init@WevoteWorkerFactory@LocalWorkflow@U2@@SAXXZ$12 100137da f   WevoteWorkerFactory.obj
 0001:000127e3       __unwindfunclet$?init@WevoteWorkerFactory@LocalWorkflow@U2@@SAXXZ$13 100137e3 f   WevoteWorkerFactory.obj
 0001:000127ef       __unwindfunclet$?init@WevoteWorkerFactory@LocalWorkflow@U2@@SAXXZ$14 100137ef f   WevoteWorkerFactory.obj
 0001:000127f8       __unwindfunclet$?init@WevoteWorkerFactory@LocalWorkflow@U2@@SAXXZ$15 100137f8 f   WevoteWorkerFactory.obj
 0001:00012801       __unwindfunclet$?init@WevoteWorkerFactory@LocalWorkflow@U2@@SAXXZ$16 10013801 f   WevoteWorkerFactory.obj
 0001:0001280d       __unwindfunclet$?init@WevoteWorkerFactory@LocalWorkflow@U2@@SAXXZ$17 1001380d f   WevoteWorkerFactory.obj
 0001:00012818       __unwindfunclet$?init@WevoteWorkerFactory@LocalWorkflow@U2@@SAXXZ$18 10013818 f   WevoteWorkerFactory.obj
 0001:00012823       __unwindfunclet$?init@WevoteWorkerFactory@LocalWorkflow@U2@@SAXXZ$19 10013823 f   WevoteWorkerFactory.obj
 0001:0001283d       __unwindfunclet$?init@WevoteWorkerFactory@LocalWorkflow@U2@@SAXXZ$20 1001383d f   WevoteWorkerFactory.obj
 0001:0001285a       __unwindfunclet$?init@WevoteWorkerFactory@LocalWorkflow@U2@@SAXXZ$22 1001385a f   WevoteWorkerFactory.obj
 0001:00012865       __unwindfunclet$?init@WevoteWorkerFactory@LocalWorkflow@U2@@SAXXZ$23 10013865 f   WevoteWorkerFactory.obj
 0001:00012870       __unwindfunclet$?init@WevoteWorkerFactory@LocalWorkflow@U2@@SAXXZ$24 10013870 f   WevoteWorkerFactory.obj
 0001:0001288a       __unwindfunclet$?init@WevoteWorkerFactory@LocalWorkflow@U2@@SAXXZ$25 1001388a f   WevoteWorkerFactory.obj
 0001:000128a7       __unwindfunclet$?init@WevoteWorkerFactory@LocalWorkflow@U2@@SAXXZ$27 100138a7 f   WevoteWorkerFactory.obj
 0001:000128af       __unwindfunclet$?init@WevoteWorkerFactory@LocalWorkflow@U2@@SAXXZ$28 100138af f   WevoteWorkerFactory.obj
 0001:000128b8       __unwindfunclet$?init@WevoteWorkerFactory@LocalWorkflow@U2@@SAXXZ$29 100138b8 f   WevoteWorkerFactory.obj
 0001:000128c1       __unwindfunclet$?init@WevoteWorkerFactory@LocalWorkflow@U2@@SAXXZ$30 100138c1 f   WevoteWorkerFactory.obj
 0001:000128ca       __unwindfunclet$?init@WevoteWorkerFactory@LocalWorkflow@U2@@SAXXZ$31 100138ca f   WevoteWorkerFactory.obj
 0001:000128d3       __unwindfunclet$?init@WevoteWorkerFactory@LocalWorkflow@U2@@SAXXZ$32 100138d3 f   WevoteWorkerFactory.obj
 0001:000128dc       __unwindfunclet$?init@WevoteWorkerFactory@LocalWorkflow@U2@@SAXXZ$33 100138dc f   WevoteWorkerFactory.obj
 0001:000128e8       __unwindfunclet$?init@WevoteWorkerFactory@LocalWorkflow@U2@@SAXXZ$34 100138e8 f   WevoteWorkerFactory.obj
 0001:000128f1       __unwindfunclet$?init@WevoteWorkerFactory@LocalWorkflow@U2@@SAXXZ$35 100138f1 f   WevoteWorkerFactory.obj
 0001:000128fa       __unwindfunclet$?init@WevoteWorkerFactory@LocalWorkflow@U2@@SAXXZ$36 100138fa f   WevoteWorkerFactory.obj
 0001:00012906       __unwindfunclet$?init@WevoteWorkerFactory@LocalWorkflow@U2@@SAXXZ$37 10013906 f   WevoteWorkerFactory.obj
 0001:0001290f       __unwindfunclet$?init@WevoteWorkerFactory@LocalWorkflow@U2@@SAXXZ$38 1001390f f   WevoteWorkerFactory.obj
 0001:00012918       __unwindfunclet$?init@WevoteWorkerFactory@LocalWorkflow@U2@@SAXXZ$39 10013918 f   WevoteWorkerFactory.obj
 0001:00012924       __unwindfunclet$?init@WevoteWorkerFactory@LocalWorkflow@U2@@SAXXZ$40 10013924 f   WevoteWorkerFactory.obj
 0001:00012930       __unwindfunclet$?init@WevoteWorkerFactory@LocalWorkflow@U2@@SAXXZ$41 10013930 f   WevoteWorkerFactory.obj
 0001:00012939       __unwindfunclet$?init@WevoteWorkerFactory@LocalWorkflow@U2@@SAXXZ$42 10013939 f   WevoteWorkerFactory.obj
 0001:00012945       __unwindfunclet$?init@WevoteWorkerFactory@LocalWorkflow@U2@@SAXXZ$43 10013945 f   WevoteWorkerFactory.obj
 0001:0001294e       __unwindfunclet$?init@WevoteWorkerFactory@LocalWorkflow@U2@@SAXXZ$44 1001394e f   WevoteWorkerFactory.obj
 0001:0001295a       __unwindfunclet$?init@WevoteWorkerFactory@LocalWorkflow@U2@@SAXXZ$45 1001395a f   WevoteWorkerFactory.obj
 0001:00012965       __unwindfunclet$?init@WevoteWorkerFactory@LocalWorkflow@U2@@SAXXZ$46 10013965 f   WevoteWorkerFactory.obj
 0001:0001297f       __unwindfunclet$?init@WevoteWorkerFactory@LocalWorkflow@U2@@SAXXZ$48 1001397f f   WevoteWorkerFactory.obj
 0001:0001298a       __unwindfunclet$?init@WevoteWorkerFactory@LocalWorkflow@U2@@SAXXZ$49 1001398a f   WevoteWorkerFactory.obj
 0001:000129a4       __unwindfunclet$?init@WevoteWorkerFactory@LocalWorkflow@U2@@SAXXZ$51 100139a4 f   WevoteWorkerFactory.obj
 0001:000129af       __unwindfunclet$?init@WevoteWorkerFactory@LocalWorkflow@U2@@SAXXZ$52 100139af f   WevoteWorkerFactory.obj
 0001:000129c9       __unwindfunclet$?init@WevoteWorkerFactory@LocalWorkflow@U2@@SAXXZ$54 100139c9 f   WevoteWorkerFactory.obj
 0001:000129d4       __unwindfunclet$?init@WevoteWorkerFactory@LocalWorkflow@U2@@SAXXZ$55 100139d4 f   WevoteWorkerFactory.obj
 0001:000129f3       __unwindfunclet$?init@WevoteWorkerFactory@LocalWorkflow@U2@@SAXXZ$57 100139f3 f   WevoteWorkerFactory.obj
 0001:000129fe       __unwindfunclet$?init@WevoteWorkerFactory@LocalWorkflow@U2@@SAXXZ$58 100139fe f   WevoteWorkerFactory.obj
 0001:00012a1d       __unwindfunclet$?init@WevoteWorkerFactory@LocalWorkflow@U2@@SAXXZ$60 10013a1d f   WevoteWorkerFactory.obj
 0001:00012a28       __unwindfunclet$?init@WevoteWorkerFactory@LocalWorkflow@U2@@SAXXZ$61 10013a28 f   WevoteWorkerFactory.obj
 0001:00012a47       __unwindfunclet$?init@WevoteWorkerFactory@LocalWorkflow@U2@@SAXXZ$63 10013a47 f   WevoteWorkerFactory.obj
 0001:00012a4f       __unwindfunclet$?init@WevoteWorkerFactory@LocalWorkflow@U2@@SAXXZ$64 10013a4f f   WevoteWorkerFactory.obj
 0001:00012a57       __unwindfunclet$?init@WevoteWorkerFactory@LocalWorkflow@U2@@SAXXZ$65 10013a57 f   WevoteWorkerFactory.obj
 0001:00012a60       __unwindfunclet$?init@WevoteWorkerFactory@LocalWorkflow@U2@@SAXXZ$66 10013a60 f   WevoteWorkerFactory.obj
 0001:00012a69       __unwindfunclet$?init@WevoteWorkerFactory@LocalWorkflow@U2@@SAXXZ$67 10013a69 f   WevoteWorkerFactory.obj
 0001:00012a72       __unwindfunclet$?init@WevoteWorkerFactory@LocalWorkflow@U2@@SAXXZ$68 10013a72 f   WevoteWorkerFactory.obj
 0001:00012a7b       __unwindfunclet$?init@WevoteWorkerFactory@LocalWorkflow@U2@@SAXXZ$69 10013a7b f   WevoteWorkerFactory.obj
 0001:00012a86       __unwindfunclet$?init@WevoteWorkerFactory@LocalWorkflow@U2@@SAXXZ$70 10013a86 f   WevoteWorkerFactory.obj
 0001:00012a8e       __unwindfunclet$?init@WevoteWorkerFactory@LocalWorkflow@U2@@SAXXZ$71 10013a8e f   WevoteWorkerFactory.obj
 0001:00012a97       __unwindfunclet$?init@WevoteWorkerFactory@LocalWorkflow@U2@@SAXXZ$72 10013a97 f   WevoteWorkerFactory.obj
 0001:00012aa0       __unwindfunclet$?init@WevoteWorkerFactory@LocalWorkflow@U2@@SAXXZ$73 10013aa0 f   WevoteWorkerFactory.obj
 0001:00012aa9       __unwindfunclet$?init@WevoteWorkerFactory@LocalWorkflow@U2@@SAXXZ$74 10013aa9 f   WevoteWorkerFactory.obj
 0001:00012ab2       __unwindfunclet$?init@WevoteWorkerFactory@LocalWorkflow@U2@@SAXXZ$75 10013ab2 f   WevoteWorkerFactory.obj
 0001:00012abd       __unwindfunclet$?init@WevoteWorkerFactory@LocalWorkflow@U2@@SAXXZ$76 10013abd f   WevoteWorkerFactory.obj
 0001:00012ac5       __unwindfunclet$?init@WevoteWorkerFactory@LocalWorkflow@U2@@SAXXZ$77 10013ac5 f   WevoteWorkerFactory.obj
 0001:00012ace       __unwindfunclet$?init@WevoteWorkerFactory@LocalWorkflow@U2@@SAXXZ$78 10013ace f   WevoteWorkerFactory.obj
 0001:00012ad7       __unwindfunclet$?init@WevoteWorkerFactory@LocalWorkflow@U2@@SAXXZ$79 10013ad7 f   WevoteWorkerFactory.obj
 0001:00012ae3       __unwindfunclet$?init@WevoteWorkerFactory@LocalWorkflow@U2@@SAXXZ$80 10013ae3 f   WevoteWorkerFactory.obj
 0001:00012aec       __unwindfunclet$?init@WevoteWorkerFactory@LocalWorkflow@U2@@SAXXZ$81 10013aec f   WevoteWorkerFactory.obj
 0001:00012af7       __unwindfunclet$?init@WevoteWorkerFactory@LocalWorkflow@U2@@SAXXZ$82 10013af7 f   WevoteWorkerFactory.obj
 0001:00012aff       __unwindfunclet$?init@WevoteWorkerFactory@LocalWorkflow@U2@@SAXXZ$83 10013aff f   WevoteWorkerFactory.obj
 0001:00012b08       __unwindfunclet$?init@WevoteWorkerFactory@LocalWorkflow@U2@@SAXXZ$84 10013b08 f   WevoteWorkerFactory.obj
 0001:00012b11       __unwindfunclet$?init@WevoteWorkerFactory@LocalWorkflow@U2@@SAXXZ$85 10013b11 f   WevoteWorkerFactory.obj
 0001:00012b1a       __unwindfunclet$?init@WevoteWorkerFactory@LocalWorkflow@U2@@SAXXZ$86 10013b1a f   WevoteWorkerFactory.obj
 0001:00012b23       __unwindfunclet$?init@WevoteWorkerFactory@LocalWorkflow@U2@@SAXXZ$87 10013b23 f   WevoteWorkerFactory.obj
 0001:00012b2e       __unwindfunclet$?init@WevoteWorkerFactory@LocalWorkflow@U2@@SAXXZ$88 10013b2e f   WevoteWorkerFactory.obj
 0001:00012b37       __unwindfunclet$?init@WevoteWorkerFactory@LocalWorkflow@U2@@SAXXZ$89 10013b37 f   WevoteWorkerFactory.obj
 0001:00012b40       __unwindfunclet$?init@WevoteWorkerFactory@LocalWorkflow@U2@@SAXXZ$90 10013b40 f   WevoteWorkerFactory.obj
 0001:00012b49       __unwindfunclet$?init@WevoteWorkerFactory@LocalWorkflow@U2@@SAXXZ$91 10013b49 f   WevoteWorkerFactory.obj
 0001:00012b52       __unwindfunclet$?init@WevoteWorkerFactory@LocalWorkflow@U2@@SAXXZ$106 10013b52 f   WevoteWorkerFactory.obj
 0001:00012b5a       __unwindfunclet$?init@WevoteWorkerFactory@LocalWorkflow@U2@@SAXXZ$92 10013b5a f   WevoteWorkerFactory.obj
 0001:00012b62       __unwindfunclet$?init@WevoteWorkerFactory@LocalWorkflow@U2@@SAXXZ$93 10013b62 f   WevoteWorkerFactory.obj
 0001:00012b6b       __unwindfunclet$?init@WevoteWorkerFactory@LocalWorkflow@U2@@SAXXZ$94 10013b6b f   WevoteWorkerFactory.obj
 0001:00012b74       __unwindfunclet$?init@WevoteWorkerFactory@LocalWorkflow@U2@@SAXXZ$95 10013b74 f   WevoteWorkerFactory.obj
 0001:00012b7f       __unwindfunclet$?init@WevoteWorkerFactory@LocalWorkflow@U2@@SAXXZ$96 10013b7f f   WevoteWorkerFactory.obj
 0001:00012b9e       __unwindfunclet$?init@WevoteWorkerFactory@LocalWorkflow@U2@@SAXXZ$97 10013b9e f   WevoteWorkerFactory.obj
 0001:00012ba7       __unwindfunclet$?init@WevoteWorkerFactory@LocalWorkflow@U2@@SAXXZ$98 10013ba7 f   WevoteWorkerFactory.obj
 0001:00012bb0       __unwindfunclet$?init@WevoteWorkerFactory@LocalWorkflow@U2@@SAXXZ$99 10013bb0 f   WevoteWorkerFactory.obj
 0001:00012bbc       __unwindfunclet$?init@WevoteWorkerFactory@LocalWorkflow@U2@@SAXXZ$100 10013bbc f   WevoteWorkerFactory.obj
 0001:00012bc7       __unwindfunclet$?init@WevoteWorkerFactory@LocalWorkflow@U2@@SAXXZ$101 10013bc7 f   WevoteWorkerFactory.obj
 0001:00012bd2       __unwindfunclet$?init@WevoteWorkerFactory@LocalWorkflow@U2@@SAXXZ$102 10013bd2 f   WevoteWorkerFactory.obj
 0001:00012bdd       __unwindfunclet$?init@WevoteWorkerFactory@LocalWorkflow@U2@@SAXXZ$103 10013bdd f   WevoteWorkerFactory.obj
 0001:00012be6       __unwindfunclet$?init@WevoteWorkerFactory@LocalWorkflow@U2@@SAXXZ$104 10013be6 f   WevoteWorkerFactory.obj
 0001:00012bef       __unwindfunclet$?init@WevoteWorkerFactory@LocalWorkflow@U2@@SAXXZ$105 10013bef f   WevoteWorkerFactory.obj
 0001:00012bfa       __ehhandler$?init@WevoteWorkerFactory@LocalWorkflow@U2@@SAXXZ 10013bfa f   WevoteWorkerFactory.obj
 0001:00012c20       __unwindfunclet$??__EalgoLog@U2@@YAXXZ$0 10013c20 f   moc_WevotePrompter.obj
 0001:00012c29       __ehhandler$??__EalgoLog@U2@@YAXXZ 10013c29 f   moc_WevotePrompter.obj
 0001:00012c50       __unwindfunclet$??__EcmdLog@U2@@YAXXZ$0 10013c50 f   moc_WevotePrompter.obj
 0001:00012c59       __ehhandler$??__EcmdLog@U2@@YAXXZ 10013c59 f   moc_WevotePrompter.obj
 0001:00012c80       __unwindfunclet$??__EcoreLog@U2@@YAXXZ$0 10013c80 f   moc_WevotePrompter.obj
 0001:00012c89       __ehhandler$??__EcoreLog@U2@@YAXXZ 10013c89 f   moc_WevotePrompter.obj
 0001:00012cb0       __unwindfunclet$??__EioLog@U2@@YAXXZ$0 10013cb0 f   moc_WevotePrompter.obj
 0001:00012cb9       __ehhandler$??__EioLog@U2@@YAXXZ 10013cb9 f   moc_WevotePrompter.obj
 0001:00012ce0       __unwindfunclet$??__EperfLog@U2@@YAXXZ$0 10013ce0 f   moc_WevotePrompter.obj
 0001:00012ce9       __ehhandler$??__EperfLog@U2@@YAXXZ 10013ce9 f   moc_WevotePrompter.obj
 0001:00012d10       __unwindfunclet$??__EscriptLog@U2@@YAXXZ$0 10013d10 f   moc_WevotePrompter.obj
 0001:00012d19       __ehhandler$??__EscriptLog@U2@@YAXXZ 10013d19 f   moc_WevotePrompter.obj
 0001:00012d40       __unwindfunclet$??__EtaskLog@U2@@YAXXZ$0 10013d40 f   moc_WevotePrompter.obj
 0001:00012d49       __ehhandler$??__EtaskLog@U2@@YAXXZ 10013d49 f   moc_WevotePrompter.obj
 0001:00012d70       __unwindfunclet$??__EuiLog@U2@@YAXXZ$0 10013d70 f   moc_WevotePrompter.obj
 0001:00012d79       __ehhandler$??__EuiLog@U2@@YAXXZ 10013d79 f   moc_WevotePrompter.obj
 0001:00012da0       __unwindfunclet$??__EuserActLog@U2@@YAXXZ$0 10013da0 f   moc_WevotePrompter.obj
 0001:00012da9       __ehhandler$??__EuserActLog@U2@@YAXXZ 10013da9 f   moc_WevotePrompter.obj
 0001:00012dd0       __unwindfunclet$??__EalgoLog@U2@@YAXXZ$0 10013dd0 f   moc_WevoteTask.obj
 0001:00012dd9       __ehhandler$??__EalgoLog@U2@@YAXXZ 10013dd9 f   moc_WevoteTask.obj
 0001:00012e00       __unwindfunclet$??__EcmdLog@U2@@YAXXZ$0 10013e00 f   moc_WevoteTask.obj
 0001:00012e09       __ehhandler$??__EcmdLog@U2@@YAXXZ 10013e09 f   moc_WevoteTask.obj
 0001:00012e30       __unwindfunclet$??__EcoreLog@U2@@YAXXZ$0 10013e30 f   moc_WevoteTask.obj
 0001:00012e39       __ehhandler$??__EcoreLog@U2@@YAXXZ 10013e39 f   moc_WevoteTask.obj
 0001:00012e60       __unwindfunclet$??__EioLog@U2@@YAXXZ$0 10013e60 f   moc_WevoteTask.obj
 0001:00012e69       __ehhandler$??__EioLog@U2@@YAXXZ 10013e69 f   moc_WevoteTask.obj
 0001:00012e90       __unwindfunclet$??__EperfLog@U2@@YAXXZ$0 10013e90 f   moc_WevoteTask.obj
 0001:00012e99       __ehhandler$??__EperfLog@U2@@YAXXZ 10013e99 f   moc_WevoteTask.obj
 0001:00012ec0       __unwindfunclet$??__EscriptLog@U2@@YAXXZ$0 10013ec0 f   moc_WevoteTask.obj
 0001:00012ec9       __ehhandler$??__EscriptLog@U2@@YAXXZ 10013ec9 f   moc_WevoteTask.obj
 0001:00012ef0       __unwindfunclet$??__EtaskLog@U2@@YAXXZ$0 10013ef0 f   moc_WevoteTask.obj
 0001:00012ef9       __ehhandler$??__EtaskLog@U2@@YAXXZ 10013ef9 f   moc_WevoteTask.obj
 0001:00012f20       __unwindfunclet$??__EuiLog@U2@@YAXXZ$0 10013f20 f   moc_WevoteTask.obj
 0001:00012f29       __ehhandler$??__EuiLog@U2@@YAXXZ 10013f29 f   moc_WevoteTask.obj
 0001:00012f50       __unwindfunclet$??__EuserActLog@U2@@YAXXZ$0 10013f50 f   moc_WevoteTask.obj
 0001:00012f59       __ehhandler$??__EuserActLog@U2@@YAXXZ 10013f59 f   moc_WevoteTask.obj
 0001:00012f80       __unwindfunclet$??__EalgoLog@U2@@YAXXZ$0 10013f80 f   moc_WevoteWorker.obj
 0001:00012f89       __ehhandler$??__EalgoLog@U2@@YAXXZ 10013f89 f   moc_WevoteWorker.obj
 0001:00012fb0       __unwindfunclet$??__EcmdLog@U2@@YAXXZ$0 10013fb0 f   moc_WevoteWorker.obj
 0001:00012fb9       __ehhandler$??__EcmdLog@U2@@YAXXZ 10013fb9 f   moc_WevoteWorker.obj
 0001:00012fe0       __unwindfunclet$??__EcoreLog@U2@@YAXXZ$0 10013fe0 f   moc_WevoteWorker.obj
 0001:00012fe9       __ehhandler$??__EcoreLog@U2@@YAXXZ 10013fe9 f   moc_WevoteWorker.obj
 0001:00013010       __unwindfunclet$??__EioLog@U2@@YAXXZ$0 10014010 f   moc_WevoteWorker.obj
 0001:00013019       __ehhandler$??__EioLog@U2@@YAXXZ 10014019 f   moc_WevoteWorker.obj
 0001:00013040       __unwindfunclet$??__EperfLog@U2@@YAXXZ$0 10014040 f   moc_WevoteWorker.obj
 0001:00013049       __ehhandler$??__EperfLog@U2@@YAXXZ 10014049 f   moc_WevoteWorker.obj
 0001:00013070       __unwindfunclet$??__EscriptLog@U2@@YAXXZ$0 10014070 f   moc_WevoteWorker.obj
 0001:00013079       __ehhandler$??__EscriptLog@U2@@YAXXZ 10014079 f   moc_WevoteWorker.obj
 0001:000130a0       __unwindfunclet$??__EtaskLog@U2@@YAXXZ$0 100140a0 f   moc_WevoteWorker.obj
 0001:000130a9       __ehhandler$??__EtaskLog@U2@@YAXXZ 100140a9 f   moc_WevoteWorker.obj
 0001:000130d0       __unwindfunclet$??__EuiLog@U2@@YAXXZ$0 100140d0 f   moc_WevoteWorker.obj
 0001:000130d9       __ehhandler$??__EuiLog@U2@@YAXXZ 100140d9 f   moc_WevoteWorker.obj
 0001:00013100       __unwindfunclet$??__EuserActLog@U2@@YAXXZ$0 10014100 f   moc_WevoteWorker.obj
 0001:00013109       __ehhandler$??__EuserActLog@U2@@YAXXZ 10014109 f   moc_WevoteWorker.obj
 0001:00013130       __unwindfunclet$?qt_metatype_id@?$QMetaTypeIdQObject@PAVTask@U2@@$00@@SAHXZ$0 10014130 f   moc_WevoteWorker.obj
 0001:00013139       __ehhandler$?qt_metatype_id@?$QMetaTypeIdQObject@PAVTask@U2@@$00@@SAHXZ 10014139 f   moc_WevoteWorker.obj
 0001:00013160       ??__F?SCIENTIFIC_NAME@PrepareWevoteTaxonomyDataTask@U2@@0VQString@@B@@YAXXZ 10014160 f   PrepareWevoteTaxonomyDataTask.obj
 0001:00013170       ??__F?WEVOTE_DIR@PrepareWevoteTaxonomyDataTask@U2@@0VQString@@B@@YAXXZ 10014170 f   PrepareWevoteTaxonomyDataTask.obj
 0001:00013180       ??__F?WEVOTE_NAMES@PrepareWevoteTaxonomyDataTask@U2@@0VQString@@B@@YAXXZ 10014180 f   PrepareWevoteTaxonomyDataTask.obj
 0001:00013190       ??__F?WEVOTE_NODES@PrepareWevoteTaxonomyDataTask@U2@@0VQString@@B@@YAXXZ 10014190 f   PrepareWevoteTaxonomyDataTask.obj
 0001:000131a0       ??__F?_Generic_object@?$_Error_objects@H@std@@2V_Generic_error_category@2@A@@YAXXZ 100141a0 f   PrepareWevoteTaxonomyDataTask.obj
 0001:000131b0       ??__F?_Iostream_object@?$_Error_objects@H@std@@2V_Iostream_error_category@2@A@@YAXXZ 100141b0 f   PrepareWevoteTaxonomyDataTask.obj
 0001:000131c0       ??__F?_System_object@?$_Error_objects@H@std@@2V_System_error_category@2@A@@YAXXZ 100141c0 f   PrepareWevoteTaxonomyDataTask.obj
 0001:000131d0       ??__FalgoLog@U2@@YAXXZ     100141d0 f   PrepareWevoteTaxonomyDataTask.obj
 0001:000131e0       ??__FcmdLog@U2@@YAXXZ      100141e0 f   PrepareWevoteTaxonomyDataTask.obj
 0001:000131f0       ??__FcoreLog@U2@@YAXXZ     100141f0 f   PrepareWevoteTaxonomyDataTask.obj
 0001:00013200       ??__FioLog@U2@@YAXXZ       10014200 f   PrepareWevoteTaxonomyDataTask.obj
 0001:00013210       ??__FperfLog@U2@@YAXXZ     10014210 f   PrepareWevoteTaxonomyDataTask.obj
 0001:00013220       ??__FscriptLog@U2@@YAXXZ   10014220 f   PrepareWevoteTaxonomyDataTask.obj
 0001:00013230       ??__FtaskLog@U2@@YAXXZ     10014230 f   PrepareWevoteTaxonomyDataTask.obj
 0001:00013240       ??__FuiLog@U2@@YAXXZ       10014240 f   PrepareWevoteTaxonomyDataTask.obj
 0001:00013250       ??__FuserActLog@U2@@YAXXZ  10014250 f   PrepareWevoteTaxonomyDataTask.obj
 0001:00013260       ??__F?_Generic_object@?$_Error_objects@H@std@@2V_Generic_error_category@2@A@@YAXXZ 10014260 f   WevotePrompter.obj
 0001:00013270       ??__F?_Iostream_object@?$_Error_objects@H@std@@2V_Iostream_error_category@2@A@@YAXXZ 10014270 f   WevotePrompter.obj
 0001:00013280       ??__F?_System_object@?$_Error_objects@H@std@@2V_System_error_category@2@A@@YAXXZ 10014280 f   WevotePrompter.obj
 0001:00013290       ??__FalgoLog@U2@@YAXXZ     10014290 f   WevotePrompter.obj
 0001:000132a0       ??__FcmdLog@U2@@YAXXZ      100142a0 f   WevotePrompter.obj
 0001:000132b0       ??__FcoreLog@U2@@YAXXZ     100142b0 f   WevotePrompter.obj
 0001:000132c0       ??__FioLog@U2@@YAXXZ       100142c0 f   WevotePrompter.obj
 0001:000132d0       ??__FperfLog@U2@@YAXXZ     100142d0 f   WevotePrompter.obj
 0001:000132e0       ??__FscriptLog@U2@@YAXXZ   100142e0 f   WevotePrompter.obj
 0001:000132f0       ??__FtaskLog@U2@@YAXXZ     100142f0 f   WevotePrompter.obj
 0001:00013300       ??__FuiLog@U2@@YAXXZ       10014300 f   WevotePrompter.obj
 0001:00013310       ??__FuserActLog@U2@@YAXXZ  10014310 f   WevotePrompter.obj
 0001:00013320       ??__F?TOOL_NAME@WevoteSupport@U2@@2VQString@@B@@YAXXZ 10014320 f   WevoteSupport.obj
 0001:00013330       ??__F?_Generic_object@?$_Error_objects@H@std@@2V_Generic_error_category@2@A@@YAXXZ 10014330 f   WevoteSupport.obj
 0001:00013340       ??__F?_Iostream_object@?$_Error_objects@H@std@@2V_Iostream_error_category@2@A@@YAXXZ 10014340 f   WevoteSupport.obj
 0001:00013350       ??__F?_System_object@?$_Error_objects@H@std@@2V_System_error_category@2@A@@YAXXZ 10014350 f   WevoteSupport.obj
 0001:00013360       ??__F?PLUGIN_DESCRIPRION@WevoteSupportPlugin@U2@@2VQString@@B@@YAXXZ 10014360 f   WevoteSupportPlugin.obj
 0001:00013370       ??__F?PLUGIN_NAME@WevoteSupportPlugin@U2@@2VQString@@B@@YAXXZ 10014370 f   WevoteSupportPlugin.obj
 0001:00013380       ??__F?_Generic_object@?$_Error_objects@H@std@@2V_Generic_error_category@2@A@@YAXXZ 10014380 f   WevoteSupportPlugin.obj
 0001:00013390       ??__F?_Iostream_object@?$_Error_objects@H@std@@2V_Iostream_error_category@2@A@@YAXXZ 10014390 f   WevoteSupportPlugin.obj
 0001:000133a0       ??__F?_System_object@?$_Error_objects@H@std@@2V_System_error_category@2@A@@YAXXZ 100143a0 f   WevoteSupportPlugin.obj
 0001:000133b0       ??__FalgoLog@U2@@YAXXZ     100143b0 f   WevoteSupportPlugin.obj
 0001:000133c0       ??__FcmdLog@U2@@YAXXZ      100143c0 f   WevoteSupportPlugin.obj
 0001:000133d0       ??__FcoreLog@U2@@YAXXZ     100143d0 f   WevoteSupportPlugin.obj
 0001:000133e0       ??__FioLog@U2@@YAXXZ       100143e0 f   WevoteSupportPlugin.obj
 0001:000133f0       ??__FperfLog@U2@@YAXXZ     100143f0 f   WevoteSupportPlugin.obj
 0001:00013400       ??__FscriptLog@U2@@YAXXZ   10014400 f   WevoteSupportPlugin.obj
 0001:00013410       ??__FtaskLog@U2@@YAXXZ     10014410 f   WevoteSupportPlugin.obj
 0001:00013420       ??__FuiLog@U2@@YAXXZ       10014420 f   WevoteSupportPlugin.obj
 0001:00013430       ??__FuserActLog@U2@@YAXXZ  10014430 f   WevoteSupportPlugin.obj
 0001:00013440       ??__F?SUFFIX@WevoteTask@U2@@2VQString@@B@@YAXXZ 10014440 f   WevoteTask.obj
 0001:00013450       ??__F?_Generic_object@?$_Error_objects@H@std@@2V_Generic_error_category@2@A@@YAXXZ 10014450 f   WevoteTask.obj
 0001:00013460       ??__F?_Iostream_object@?$_Error_objects@H@std@@2V_Iostream_error_category@2@A@@YAXXZ 10014460 f   WevoteTask.obj
 0001:00013470       ??__F?_System_object@?$_Error_objects@H@std@@2V_System_error_category@2@A@@YAXXZ 10014470 f   WevoteTask.obj
 0001:00013480       ??__FalgoLog@U2@@YAXXZ     10014480 f   WevoteTask.obj
 0001:00013490       ??__FcmdLog@U2@@YAXXZ      10014490 f   WevoteTask.obj
 0001:000134a0       ??__FcoreLog@U2@@YAXXZ     100144a0 f   WevoteTask.obj
 0001:000134b0       ??__FioLog@U2@@YAXXZ       100144b0 f   WevoteTask.obj
 0001:000134c0       ??__FperfLog@U2@@YAXXZ     100144c0 f   WevoteTask.obj
 0001:000134d0       ??__FscriptLog@U2@@YAXXZ   100144d0 f   WevoteTask.obj
 0001:000134e0       ??__FtaskLog@U2@@YAXXZ     100144e0 f   WevoteTask.obj
 0001:000134f0       ??__FuiLog@U2@@YAXXZ       100144f0 f   WevoteTask.obj
 0001:00013500       ??__FuserActLog@U2@@YAXXZ  10014500 f   WevoteTask.obj
 0001:00013510       ??__F?_Generic_object@?$_Error_objects@H@std@@2V_Generic_error_category@2@A@@YAXXZ 10014510 f   WevoteValidator.obj
 0001:00013520       ??__F?_Iostream_object@?$_Error_objects@H@std@@2V_Iostream_error_category@2@A@@YAXXZ 10014520 f   WevoteValidator.obj
 0001:00013530       ??__F?_System_object@?$_Error_objects@H@std@@2V_System_error_category@2@A@@YAXXZ 10014530 f   WevoteValidator.obj
 0001:00013540       ??__FalgoLog@U2@@YAXXZ     10014540 f   WevoteValidator.obj
 0001:00013550       ??__FcmdLog@U2@@YAXXZ      10014550 f   WevoteValidator.obj
 0001:00013560       ??__FcoreLog@U2@@YAXXZ     10014560 f   WevoteValidator.obj
 0001:00013570       ??__FioLog@U2@@YAXXZ       10014570 f   WevoteValidator.obj
 0001:00013580       ??__FperfLog@U2@@YAXXZ     10014580 f   WevoteValidator.obj
 0001:00013590       ??__FscriptLog@U2@@YAXXZ   10014590 f   WevoteValidator.obj
 0001:000135a0       ??__FtaskLog@U2@@YAXXZ     100145a0 f   WevoteValidator.obj
 0001:000135b0       ??__FuiLog@U2@@YAXXZ       100145b0 f   WevoteValidator.obj
 0001:000135c0       ??__FuserActLog@U2@@YAXXZ  100145c0 f   WevoteValidator.obj
 0001:000135d0       ??__F?WEVOTE_DIR@WevoteWorker@LocalWorkflow@U2@@0VQString@@B@@YAXXZ 100145d0 f   WevoteWorker.obj
 0001:000135e0       ??__F?_Generic_object@?$_Error_objects@H@std@@2V_Generic_error_category@2@A@@YAXXZ 100145e0 f   WevoteWorker.obj
 0001:000135f0       ??__F?_Iostream_object@?$_Error_objects@H@std@@2V_Iostream_error_category@2@A@@YAXXZ 100145f0 f   WevoteWorker.obj
 0001:00013600       ??__F?_System_object@?$_Error_objects@H@std@@2V_System_error_category@2@A@@YAXXZ 10014600 f   WevoteWorker.obj
 0001:00013610       ??__FalgoLog@U2@@YAXXZ     10014610 f   WevoteWorker.obj
 0001:00013620       ??__FcmdLog@U2@@YAXXZ      10014620 f   WevoteWorker.obj
 0001:00013630       ??__FcoreLog@U2@@YAXXZ     10014630 f   WevoteWorker.obj
 0001:00013660       ??__FioLog@U2@@YAXXZ       10014660 f   WevoteWorker.obj
 0001:00013670       ??__FperfLog@U2@@YAXXZ     10014670 f   WevoteWorker.obj
 0001:00013680       ??__FscriptLog@U2@@YAXXZ   10014680 f   WevoteWorker.obj
 0001:00013690       ??__FtaskLog@U2@@YAXXZ     10014690 f   WevoteWorker.obj
 0001:000136a0       ??__FuiLog@U2@@YAXXZ       100146a0 f   WevoteWorker.obj
 0001:000136b0       ??__FuserActLog@U2@@YAXXZ  100146b0 f   WevoteWorker.obj
 0001:000136c0       ??__F?ACTOR_ID@WevoteWorkerFactory@LocalWorkflow@U2@@2VQString@@B@@YAXXZ 100146c0 f   WevoteWorkerFactory.obj
 0001:000136d0       ??__F?INPUT_PORT_ID@WevoteWorkerFactory@LocalWorkflow@U2@@2VQString@@B@@YAXXZ 100146d0 f   WevoteWorkerFactory.obj
 0001:000136e0       ??__F?NUMBER_OF_AGREED_TOOLS_ATTR_ID@WevoteWorkerFactory@LocalWorkflow@U2@@2VQString@@B@@YAXXZ 100146e0 f   WevoteWorkerFactory.obj
 0001:000136f0       ??__F?NUMBER_OF_THREADS_ATTR_ID@WevoteWorkerFactory@LocalWorkflow@U2@@2VQString@@B@@YAXXZ 100146f0 f   WevoteWorkerFactory.obj
 0001:00013700       ??__F?OUTPUT_FILE_ATTR_ID@WevoteWorkerFactory@LocalWorkflow@U2@@2VQString@@B@@YAXXZ 10014700 f   WevoteWorkerFactory.obj
 0001:00013710       ??__F?OUTPUT_PORT_ID@WevoteWorkerFactory@LocalWorkflow@U2@@2VQString@@B@@YAXXZ 10014710 f   WevoteWorkerFactory.obj
 0001:00013720       ??__F?PENALTY_ATTR_ID@WevoteWorkerFactory@LocalWorkflow@U2@@2VQString@@B@@YAXXZ 10014720 f   WevoteWorkerFactory.obj
 0001:00013730       ??__F?SCORE_THRESHOLD_ATTR_ID@WevoteWorkerFactory@LocalWorkflow@U2@@2VQString@@B@@YAXXZ 10014730 f   WevoteWorkerFactory.obj
 0001:00013740       ??__F?WORKFLOW_CLASSIFY_TOOL_WEVOTE@WevoteWorkerFactory@LocalWorkflow@U2@@2VQString@@B@@YAXXZ 10014740 f   WevoteWorkerFactory.obj
 0001:00013750       ??__F?_Generic_object@?$_Error_objects@H@std@@2V_Generic_error_category@2@A@@YAXXZ 10014750 f   WevoteWorkerFactory.obj
 0001:00013760       ??__F?_Iostream_object@?$_Error_objects@H@std@@2V_Iostream_error_category@2@A@@YAXXZ 10014760 f   WevoteWorkerFactory.obj
 0001:00013770       ??__F?_System_object@?$_Error_objects@H@std@@2V_System_error_category@2@A@@YAXXZ 10014770 f   WevoteWorkerFactory.obj
 0001:00013780       ??__FalgoLog@U2@@YAXXZ     10014780 f   WevoteWorkerFactory.obj
 0001:00013790       ??__FcmdLog@U2@@YAXXZ      10014790 f   WevoteWorkerFactory.obj
 0001:000137a0       ??__FcoreLog@U2@@YAXXZ     100147a0 f   WevoteWorkerFactory.obj
 0001:000137b0       ??__FioLog@U2@@YAXXZ       100147b0 f   WevoteWorkerFactory.obj
 0001:000137c0       ??__FperfLog@U2@@YAXXZ     100147c0 f   WevoteWorkerFactory.obj
 0001:000137d0       ??__FscriptLog@U2@@YAXXZ   100147d0 f   WevoteWorkerFactory.obj
 0001:000137e0       ??__FtaskLog@U2@@YAXXZ     100147e0 f   WevoteWorkerFactory.obj
 0001:000137f0       ??__FuiLog@U2@@YAXXZ       100147f0 f   WevoteWorkerFactory.obj
 0001:00013800       ??__FuserActLog@U2@@YAXXZ  10014800 f   WevoteWorkerFactory.obj
 0001:00013810       ??__F?_Generic_object@?$_Error_objects@H@std@@2V_Generic_error_category@2@A@@YAXXZ 10014810 f   moc_WevotePrompter.obj
 0001:00013820       ??__F?_Iostream_object@?$_Error_objects@H@std@@2V_Iostream_error_category@2@A@@YAXXZ 10014820 f   moc_WevotePrompter.obj
 0001:00013830       ??__F?_System_object@?$_Error_objects@H@std@@2V_System_error_category@2@A@@YAXXZ 10014830 f   moc_WevotePrompter.obj
 0001:00013840       ??__FalgoLog@U2@@YAXXZ     10014840 f   moc_WevotePrompter.obj
 0001:00013850       ??__FcmdLog@U2@@YAXXZ      10014850 f   moc_WevotePrompter.obj
 0001:00013860       ??__FcoreLog@U2@@YAXXZ     10014860 f   moc_WevotePrompter.obj
 0001:00013870       ??__FioLog@U2@@YAXXZ       10014870 f   moc_WevotePrompter.obj
 0001:00013880       ??__FperfLog@U2@@YAXXZ     10014880 f   moc_WevotePrompter.obj
 0001:00013890       ??__FscriptLog@U2@@YAXXZ   10014890 f   moc_WevotePrompter.obj
 0001:000138a0       ??__FtaskLog@U2@@YAXXZ     100148a0 f   moc_WevotePrompter.obj
 0001:000138b0       ??__FuiLog@U2@@YAXXZ       100148b0 f   moc_WevotePrompter.obj
 0001:000138c0       ??__FuserActLog@U2@@YAXXZ  100148c0 f   moc_WevotePrompter.obj
 0001:000138d0       ??__F?_Generic_object@?$_Error_objects@H@std@@2V_Generic_error_category@2@A@@YAXXZ 100148d0 f   moc_WevoteSupportPlugin.obj
 0001:000138e0       ??__F?_Iostream_object@?$_Error_objects@H@std@@2V_Iostream_error_category@2@A@@YAXXZ 100148e0 f   moc_WevoteSupportPlugin.obj
 0001:000138f0       ??__F?_System_object@?$_Error_objects@H@std@@2V_System_error_category@2@A@@YAXXZ 100148f0 f   moc_WevoteSupportPlugin.obj
 0001:00013900       ??__F?_Generic_object@?$_Error_objects@H@std@@2V_Generic_error_category@2@A@@YAXXZ 10014900 f   moc_WevoteTask.obj
 0001:00013910       ??__F?_Iostream_object@?$_Error_objects@H@std@@2V_Iostream_error_category@2@A@@YAXXZ 10014910 f   moc_WevoteTask.obj
 0001:00013920       ??__F?_System_object@?$_Error_objects@H@std@@2V_System_error_category@2@A@@YAXXZ 10014920 f   moc_WevoteTask.obj
 0001:00013930       ??__FalgoLog@U2@@YAXXZ     10014930 f   moc_WevoteTask.obj
 0001:00013940       ??__FcmdLog@U2@@YAXXZ      10014940 f   moc_WevoteTask.obj
 0001:00013950       ??__FcoreLog@U2@@YAXXZ     10014950 f   moc_WevoteTask.obj
 0001:00013960       ??__FioLog@U2@@YAXXZ       10014960 f   moc_WevoteTask.obj
 0001:00013970       ??__FperfLog@U2@@YAXXZ     10014970 f   moc_WevoteTask.obj
 0001:00013980       ??__FscriptLog@U2@@YAXXZ   10014980 f   moc_WevoteTask.obj
 0001:00013990       ??__FtaskLog@U2@@YAXXZ     10014990 f   moc_WevoteTask.obj
 0001:000139a0       ??__FuiLog@U2@@YAXXZ       100149a0 f   moc_WevoteTask.obj
 0001:000139b0       ??__FuserActLog@U2@@YAXXZ  100149b0 f   moc_WevoteTask.obj
 0001:000139c0       ??__F?_Generic_object@?$_Error_objects@H@std@@2V_Generic_error_category@2@A@@YAXXZ 100149c0 f   moc_WevoteWorker.obj
 0001:000139d0       ??__F?_Iostream_object@?$_Error_objects@H@std@@2V_Iostream_error_category@2@A@@YAXXZ 100149d0 f   moc_WevoteWorker.obj
 0001:000139e0       ??__F?_System_object@?$_Error_objects@H@std@@2V_System_error_category@2@A@@YAXXZ 100149e0 f   moc_WevoteWorker.obj
 0001:000139f0       ??__FalgoLog@U2@@YAXXZ     100149f0 f   moc_WevoteWorker.obj
 0001:00013a00       ??__FcmdLog@U2@@YAXXZ      10014a00 f   moc_WevoteWorker.obj
 0001:00013a10       ??__FcoreLog@U2@@YAXXZ     10014a10 f   moc_WevoteWorker.obj
 0001:00013a20       ??__FioLog@U2@@YAXXZ       10014a20 f   moc_WevoteWorker.obj
 0001:00013a30       ??__FperfLog@U2@@YAXXZ     10014a30 f   moc_WevoteWorker.obj
 0001:00013a40       ??__FscriptLog@U2@@YAXXZ   10014a40 f   moc_WevoteWorker.obj
 0001:00013a50       ??__FtaskLog@U2@@YAXXZ     10014a50 f   moc_WevoteWorker.obj
 0001:00013a60       ??__FuiLog@U2@@YAXXZ       10014a60 f   moc_WevoteWorker.obj
 0001:00013a70       ??__FuserActLog@U2@@YAXXZ  10014a70 f   moc_WevoteWorker.obj
 0002:00000730       _algoLog$initializer$      10015730     PrepareWevoteTaxonomyDataTask.obj
 0002:00000734       _cmdLog$initializer$       10015734     PrepareWevoteTaxonomyDataTask.obj
 0002:00000738       _coreLog$initializer$      10015738     PrepareWevoteTaxonomyDataTask.obj
 0002:0000073c       _ioLog$initializer$        1001573c     PrepareWevoteTaxonomyDataTask.obj
 0002:00000740       _perfLog$initializer$      10015740     PrepareWevoteTaxonomyDataTask.obj
 0002:00000744       _scriptLog$initializer$    10015744     PrepareWevoteTaxonomyDataTask.obj
 0002:00000748       _taskLog$initializer$      10015748     PrepareWevoteTaxonomyDataTask.obj
 0002:0000074c       _uiLog$initializer$        1001574c     PrepareWevoteTaxonomyDataTask.obj
 0002:00000750       _userActLog$initializer$   10015750     PrepareWevoteTaxonomyDataTask.obj
 0002:00000754       ?WEVOTE_DIR$initializer$@PrepareWevoteTaxonomyDataTask@U2@@0P6AXXZA 10015754     PrepareWevoteTaxonomyDataTask.obj
 0002:00000758       ?WEVOTE_NODES$initializer$@PrepareWevoteTaxonomyDataTask@U2@@0P6AXXZA 10015758     PrepareWevoteTaxonomyDataTask.obj
 0002:0000075c       ?WEVOTE_NAMES$initializer$@PrepareWevoteTaxonomyDataTask@U2@@0P6AXXZA 1001575c     PrepareWevoteTaxonomyDataTask.obj
 0002:00000760       ?SCIENTIFIC_NAME$initializer$@PrepareWevoteTaxonomyDataTask@U2@@0P6AXXZA 10015760     PrepareWevoteTaxonomyDataTask.obj
 0002:00000764       ?_Generic_object$initializer$@?$_Error_objects@H@std@@2P6AXXZA 10015764     PrepareWevoteTaxonomyDataTask.obj
 0002:00000768       ?_Iostream_object$initializer$@?$_Error_objects@H@std@@2P6AXXZA 10015768     PrepareWevoteTaxonomyDataTask.obj
 0002:0000076c       ?_System_object$initializer$@?$_Error_objects@H@std@@2P6AXXZA 1001576c     PrepareWevoteTaxonomyDataTask.obj
 0002:00000770       _algoLog$initializer$      10015770     WevotePrompter.obj
 0002:00000774       _cmdLog$initializer$       10015774     WevotePrompter.obj
 0002:00000778       _coreLog$initializer$      10015778     WevotePrompter.obj
 0002:0000077c       _ioLog$initializer$        1001577c     WevotePrompter.obj
 0002:00000780       _perfLog$initializer$      10015780     WevotePrompter.obj
 0002:00000784       _scriptLog$initializer$    10015784     WevotePrompter.obj
 0002:00000788       _taskLog$initializer$      10015788     WevotePrompter.obj
 0002:0000078c       _uiLog$initializer$        1001578c     WevotePrompter.obj
 0002:00000790       _userActLog$initializer$   10015790     WevotePrompter.obj
 0002:00000794       ?TOOL_NAME$initializer$@WevoteSupport@U2@@2P6AXXZA 10015794     WevoteSupport.obj
 0002:00000798       _algoLog$initializer$      10015798     WevoteSupportPlugin.obj
 0002:0000079c       _cmdLog$initializer$       1001579c     WevoteSupportPlugin.obj
 0002:000007a0       _coreLog$initializer$      100157a0     WevoteSupportPlugin.obj
 0002:000007a4       _ioLog$initializer$        100157a4     WevoteSupportPlugin.obj
 0002:000007a8       _perfLog$initializer$      100157a8     WevoteSupportPlugin.obj
 0002:000007ac       _scriptLog$initializer$    100157ac     WevoteSupportPlugin.obj
 0002:000007b0       _taskLog$initializer$      100157b0     WevoteSupportPlugin.obj
 0002:000007b4       _uiLog$initializer$        100157b4     WevoteSupportPlugin.obj
 0002:000007b8       _userActLog$initializer$   100157b8     WevoteSupportPlugin.obj
 0002:000007bc       ?PLUGIN_NAME$initializer$@WevoteSupportPlugin@U2@@2P6AXXZA 100157bc     WevoteSupportPlugin.obj
 0002:000007c0       ?PLUGIN_DESCRIPRION$initializer$@WevoteSupportPlugin@U2@@2P6AXXZA 100157c0     WevoteSupportPlugin.obj
 0002:000007c4       _algoLog$initializer$      100157c4     WevoteTask.obj
 0002:000007c8       _cmdLog$initializer$       100157c8     WevoteTask.obj
 0002:000007cc       _coreLog$initializer$      100157cc     WevoteTask.obj
 0002:000007d0       _ioLog$initializer$        100157d0     WevoteTask.obj
 0002:000007d4       _perfLog$initializer$      100157d4     WevoteTask.obj
 0002:000007d8       _scriptLog$initializer$    100157d8     WevoteTask.obj
 0002:000007dc       _taskLog$initializer$      100157dc     WevoteTask.obj
 0002:000007e0       _uiLog$initializer$        100157e0     WevoteTask.obj
 0002:000007e4       _userActLog$initializer$   100157e4     WevoteTask.obj
 0002:000007e8       ?SUFFIX$initializer$@WevoteTask@U2@@2P6AXXZA 100157e8     WevoteTask.obj
 0002:000007ec       _algoLog$initializer$      100157ec     WevoteValidator.obj
 0002:000007f0       _cmdLog$initializer$       100157f0     WevoteValidator.obj
 0002:000007f4       _coreLog$initializer$      100157f4     WevoteValidator.obj
 0002:000007f8       _ioLog$initializer$        100157f8     WevoteValidator.obj
 0002:000007fc       _perfLog$initializer$      100157fc     WevoteValidator.obj
 0002:00000800       _scriptLog$initializer$    10015800     WevoteValidator.obj
 0002:00000804       _taskLog$initializer$      10015804     WevoteValidator.obj
 0002:00000808       _uiLog$initializer$        10015808     WevoteValidator.obj
 0002:0000080c       _userActLog$initializer$   1001580c     WevoteValidator.obj
 0002:00000810       _algoLog$initializer$      10015810     WevoteWorker.obj
 0002:00000814       _cmdLog$initializer$       10015814     WevoteWorker.obj
 0002:00000818       _coreLog$initializer$      10015818     WevoteWorker.obj
 0002:0000081c       _ioLog$initializer$        1001581c     WevoteWorker.obj
 0002:00000820       _perfLog$initializer$      10015820     WevoteWorker.obj
 0002:00000824       _scriptLog$initializer$    10015824     WevoteWorker.obj
 0002:00000828       _taskLog$initializer$      10015828     WevoteWorker.obj
 0002:0000082c       _uiLog$initializer$        1001582c     WevoteWorker.obj
 0002:00000830       _userActLog$initializer$   10015830     WevoteWorker.obj
 0002:00000834       ?WEVOTE_DIR$initializer$@WevoteWorker@LocalWorkflow@U2@@0P6AXXZA 10015834     WevoteWorker.obj
 0002:00000838       _algoLog$initializer$      10015838     WevoteWorkerFactory.obj
 0002:0000083c       _cmdLog$initializer$       1001583c     WevoteWorkerFactory.obj
 0002:00000840       _coreLog$initializer$      10015840     WevoteWorkerFactory.obj
 0002:00000844       _ioLog$initializer$        10015844     WevoteWorkerFactory.obj
 0002:00000848       _perfLog$initializer$      10015848     WevoteWorkerFactory.obj
 0002:0000084c       _scriptLog$initializer$    1001584c     WevoteWorkerFactory.obj
 0002:00000850       _taskLog$initializer$      10015850     WevoteWorkerFactory.obj
 0002:00000854       _uiLog$initializer$        10015854     WevoteWorkerFactory.obj
 0002:00000858       _userActLog$initializer$   10015858     WevoteWorkerFactory.obj
 0002:0000085c       ?ACTOR_ID$initializer$@WevoteWorkerFactory@LocalWorkflow@U2@@2P6AXXZA 1001585c     WevoteWorkerFactory.obj
 0002:00000860       ?INPUT_PORT_ID$initializer$@WevoteWorkerFactory@LocalWorkflow@U2@@2P6AXXZA 10015860     WevoteWorkerFactory.obj
 0002:00000864       ?OUTPUT_PORT_ID$initializer$@WevoteWorkerFactory@LocalWorkflow@U2@@2P6AXXZA 10015864     WevoteWorkerFactory.obj
 0002:00000868       ?PENALTY_ATTR_ID$initializer$@WevoteWorkerFactory@LocalWorkflow@U2@@2P6AXXZA 10015868     WevoteWorkerFactory.obj
 0002:0000086c       ?NUMBER_OF_AGREED_TOOLS_ATTR_ID$initializer$@WevoteWorkerFactory@LocalWorkflow@U2@@2P6AXXZA 1001586c     WevoteWorkerFactory.obj
 0002:00000870       ?SCORE_THRESHOLD_ATTR_ID$initializer$@WevoteWorkerFactory@LocalWorkflow@U2@@2P6AXXZA 10015870     WevoteWorkerFactory.obj
 0002:00000874       ?NUMBER_OF_THREADS_ATTR_ID$initializer$@WevoteWorkerFactory@LocalWorkflow@U2@@2P6AXXZA 10015874     WevoteWorkerFactory.obj
 0002:00000878       ?OUTPUT_FILE_ATTR_ID$initializer$@WevoteWorkerFactory@LocalWorkflow@U2@@2P6AXXZA 10015878     WevoteWorkerFactory.obj
 0002:0000087c       ?WORKFLOW_CLASSIFY_TOOL_WEVOTE$initializer$@WevoteWorkerFactory@LocalWorkflow@U2@@2P6AXXZA 1001587c     WevoteWorkerFactory.obj
 0002:00000880       _algoLog$initializer$      10015880     moc_WevotePrompter.obj
 0002:00000884       _cmdLog$initializer$       10015884     moc_WevotePrompter.obj
 0002:00000888       _coreLog$initializer$      10015888     moc_WevotePrompter.obj
 0002:0000088c       _ioLog$initializer$        1001588c     moc_WevotePrompter.obj
 0002:00000890       _perfLog$initializer$      10015890     moc_WevotePrompter.obj
 0002:00000894       _scriptLog$initializer$    10015894     moc_WevotePrompter.obj
 0002:00000898       _taskLog$initializer$      10015898     moc_WevotePrompter.obj
 0002:0000089c       _uiLog$initializer$        1001589c     moc_WevotePrompter.obj
 0002:000008a0       _userActLog$initializer$   100158a0     moc_WevotePrompter.obj
 0002:000008a4       ?staticMetaObject$initializer$@WevotePrompter@LocalWorkflow@U2@@2P6AXXZA 100158a4     moc_WevotePrompter.obj
 0002:000008a8       ?staticMetaObject$initializer$@WevoteSupportPlugin@U2@@2P6AXXZA 100158a8     moc_WevoteSupportPlugin.obj
 0002:000008ac       _algoLog$initializer$      100158ac     moc_WevoteTask.obj
 0002:000008b0       _cmdLog$initializer$       100158b0     moc_WevoteTask.obj
 0002:000008b4       _coreLog$initializer$      100158b4     moc_WevoteTask.obj
 0002:000008b8       _ioLog$initializer$        100158b8     moc_WevoteTask.obj
 0002:000008bc       _perfLog$initializer$      100158bc     moc_WevoteTask.obj
 0002:000008c0       _scriptLog$initializer$    100158c0     moc_WevoteTask.obj
 0002:000008c4       _taskLog$initializer$      100158c4     moc_WevoteTask.obj
 0002:000008c8       _uiLog$initializer$        100158c8     moc_WevoteTask.obj
 0002:000008cc       _userActLog$initializer$   100158cc     moc_WevoteTask.obj
 0002:000008d0       ?staticMetaObject$initializer$@WevoteTask@U2@@2P6AXXZA 100158d0     moc_WevoteTask.obj
 0002:000008d4       _algoLog$initializer$      100158d4     moc_WevoteWorker.obj
 0002:000008d8       _cmdLog$initializer$       100158d8     moc_WevoteWorker.obj
 0002:000008dc       _coreLog$initializer$      100158dc     moc_WevoteWorker.obj
 0002:000008e0       _ioLog$initializer$        100158e0     moc_WevoteWorker.obj
 0002:000008e4       _perfLog$initializer$      100158e4     moc_WevoteWorker.obj
 0002:000008e8       _scriptLog$initializer$    100158e8     moc_WevoteWorker.obj
 0002:000008ec       _taskLog$initializer$      100158ec     moc_WevoteWorker.obj
 0002:000008f0       _uiLog$initializer$        100158f0     moc_WevoteWorker.obj
 0002:000008f4       _userActLog$initializer$   100158f4     moc_WevoteWorker.obj
 0002:000008f8       ?staticMetaObject$initializer$@WevoteWorker@LocalWorkflow@U2@@2P6AXXZA 100158f8     moc_WevoteWorker.obj
 0002:00000904       _pcinit                    10015904     MSVCRT:crtdll.obj
 0002:00000908       _pinit                     10015908     MSVCRT:atonexit.obj
 0002:00001c74       _qt_meta_stringdata_U2__LocalWorkflow__WevotePrompter 10016c74     moc_WevotePrompter.obj
 0002:00001ca8       _qt_meta_data_U2__LocalWorkflow__WevotePrompter 10016ca8     moc_WevotePrompter.obj
 0002:00001ce4       _qt_meta_stringdata_U2__WevoteSupportPlugin 10016ce4     moc_WevoteSupportPlugin.obj
 0002:00001d0c       _qt_meta_data_U2__WevoteSupportPlugin 10016d0c     moc_WevoteSupportPlugin.obj
 0002:00001d48       _qt_meta_stringdata_U2__WevoteTask 10016d48     moc_WevoteTask.obj
 0002:00001d68       _qt_meta_data_U2__WevoteTask 10016d68     moc_WevoteTask.obj
 0002:00001da8       _qt_meta_stringdata_U2__LocalWorkflow__WevoteWorker 10016da8     moc_WevoteWorker.obj
 0002:00001e38       _qt_meta_data_U2__LocalWorkflow__WevoteWorker 10016e38     moc_WevoteWorker.obj
 0002:00001ea4       _GS_ExceptionPointers      10016ea4     MSVCRT:gs_report.obj
 0002:000030b8       __catchsym$?_Copy@?$basic_string@DU?$char_traits@D@std@@V?$allocator@D@2@@std@@QAEXII@Z$5 100180b8     PrepareWevoteTaxonomyDataTask.obj
 0002:000030c8       __catchsym$?_Copy@?$basic_string@DU?$char_traits@D@std@@V?$allocator@D@2@@std@@QAEXII@Z$4 100180c8     PrepareWevoteTaxonomyDataTask.obj
 0002:000030d8       __unwindtable$?_Copy@?$basic_string@DU?$char_traits@D@std@@V?$allocator@D@2@@std@@QAEXII@Z 100180d8     PrepareWevoteTaxonomyDataTask.obj
 0002:000030f8       __ehfuncinfo$?_Copy@?$basic_string@DU?$char_traits@D@std@@V?$allocator@D@2@@std@@QAEXII@Z 100180f8     PrepareWevoteTaxonomyDataTask.obj
 0002:0000311c       __tryblocktable$?_Copy@?$basic_string@DU?$char_traits@D@std@@V?$allocator@D@2@@std@@QAEXII@Z 1001811c     PrepareWevoteTaxonomyDataTask.obj
 0002:00003144       __unwindtable$??H@YA?BVQString@@ABV0@0@Z 10018144     PrepareWevoteTaxonomyDataTask.obj
 0002:0000314c       __ehfuncinfo$??H@YA?BVQString@@ABV0@0@Z 1001814c     PrepareWevoteTaxonomyDataTask.obj
 0002:00003170       __unwindtable$??H@YA?BVQString@@ABV0@PBD@Z 10018170     PrepareWevoteTaxonomyDataTask.obj
 0002:00003180       __ehfuncinfo$??H@YA?BVQString@@ABV0@PBD@Z 10018180     PrepareWevoteTaxonomyDataTask.obj
 0002:000031a4       __unwindtable$??__EalgoLog@U2@@YAXXZ 100181a4     PrepareWevoteTaxonomyDataTask.obj
 0002:000031ac       __ehfuncinfo$??__EalgoLog@U2@@YAXXZ 100181ac     PrepareWevoteTaxonomyDataTask.obj
 0002:000031d0       __unwindtable$??__EcmdLog@U2@@YAXXZ 100181d0     PrepareWevoteTaxonomyDataTask.obj
 0002:000031d8       __ehfuncinfo$??__EcmdLog@U2@@YAXXZ 100181d8     PrepareWevoteTaxonomyDataTask.obj
 0002:000031fc       __unwindtable$??__EcoreLog@U2@@YAXXZ 100181fc     PrepareWevoteTaxonomyDataTask.obj
 0002:00003204       __ehfuncinfo$??__EcoreLog@U2@@YAXXZ 10018204     PrepareWevoteTaxonomyDataTask.obj
 0002:00003228       __unwindtable$??__EioLog@U2@@YAXXZ 10018228     PrepareWevoteTaxonomyDataTask.obj
 0002:00003230       __ehfuncinfo$??__EioLog@U2@@YAXXZ 10018230     PrepareWevoteTaxonomyDataTask.obj
 0002:00003254       __unwindtable$??__EperfLog@U2@@YAXXZ 10018254     PrepareWevoteTaxonomyDataTask.obj
 0002:0000325c       __ehfuncinfo$??__EperfLog@U2@@YAXXZ 1001825c     PrepareWevoteTaxonomyDataTask.obj
 0002:00003280       __unwindtable$??__EscriptLog@U2@@YAXXZ 10018280     PrepareWevoteTaxonomyDataTask.obj
 0002:00003288       __ehfuncinfo$??__EscriptLog@U2@@YAXXZ 10018288     PrepareWevoteTaxonomyDataTask.obj
 0002:000032ac       __unwindtable$??__EtaskLog@U2@@YAXXZ 100182ac     PrepareWevoteTaxonomyDataTask.obj
 0002:000032b4       __ehfuncinfo$??__EtaskLog@U2@@YAXXZ 100182b4     PrepareWevoteTaxonomyDataTask.obj
 0002:000032d8       __unwindtable$??__EuiLog@U2@@YAXXZ 100182d8     PrepareWevoteTaxonomyDataTask.obj
 0002:000032e0       __ehfuncinfo$??__EuiLog@U2@@YAXXZ 100182e0     PrepareWevoteTaxonomyDataTask.obj
 0002:00003304       __unwindtable$??__EuserActLog@U2@@YAXXZ 10018304     PrepareWevoteTaxonomyDataTask.obj
 0002:0000330c       __ehfuncinfo$??__EuserActLog@U2@@YAXXZ 1001830c     PrepareWevoteTaxonomyDataTask.obj
 0002:00003330       __ehfuncinfo$??0PrepareWevoteTaxonomyDataTask@U2@@QAE@AAVWorkflowProcess@FileStorage@1@@Z 10018330     PrepareWevoteTaxonomyDataTask.obj
 0002:00003354       __unwindtable$??0PrepareWevoteTaxonomyDataTask@U2@@QAE@AAVWorkflowProcess@FileStorage@1@@Z 10018354     PrepareWevoteTaxonomyDataTask.obj
 0002:000033f4       __unwindtable$?run@PrepareWevoteTaxonomyDataTask@U2@@EAEXXZ 100183f4     PrepareWevoteTaxonomyDataTask.obj
 0002:00003404       __ehfuncinfo$?run@PrepareWevoteTaxonomyDataTask@U2@@EAEXXZ 10018404     PrepareWevoteTaxonomyDataTask.obj
 0002:00003428       __ehfuncinfo$?report@PrepareWevoteTaxonomyDataTask@U2@@EAE?AW4ReportResult@Task@2@XZ 10018428     PrepareWevoteTaxonomyDataTask.obj
 0002:0000344c       __unwindtable$?report@PrepareWevoteTaxonomyDataTask@U2@@EAE?AW4ReportResult@Task@2@XZ 1001844c     PrepareWevoteTaxonomyDataTask.obj
 0002:0000347c       __unwindtable$?isActual@PrepareWevoteTaxonomyDataTask@U2@@ABE_NXZ 1001847c     PrepareWevoteTaxonomyDataTask.obj
 0002:00003484       __ehfuncinfo$?isActual@PrepareWevoteTaxonomyDataTask@U2@@ABE_NXZ 10018484     PrepareWevoteTaxonomyDataTask.obj
 0002:000034a8       __ehfuncinfo$?prepareNamesFile@PrepareWevoteTaxonomyDataTask@U2@@AAEXXZ 100184a8     PrepareWevoteTaxonomyDataTask.obj
 0002:000034cc       __unwindtable$?prepareNamesFile@PrepareWevoteTaxonomyDataTask@U2@@AAEXXZ 100184cc     PrepareWevoteTaxonomyDataTask.obj
 0002:0000357c       __ehfuncinfo$?prepareNodesFile@PrepareWevoteTaxonomyDataTask@U2@@AAEXXZ 1001857c     PrepareWevoteTaxonomyDataTask.obj
 0002:000035a0       __unwindtable$?prepareNodesFile@PrepareWevoteTaxonomyDataTask@U2@@AAEXXZ 100185a0     PrepareWevoteTaxonomyDataTask.obj
 0002:00003640       __unwindtable$??1PrepareWevoteTaxonomyDataTask@U2@@UAE@XZ 10018640     PrepareWevoteTaxonomyDataTask.obj
 0002:00003658       __ehfuncinfo$??1PrepareWevoteTaxonomyDataTask@U2@@UAE@XZ 10018658     PrepareWevoteTaxonomyDataTask.obj
 0002:0000367c       __unwindtable$??_GPrepareWevoteTaxonomyDataTask@U2@@UAEPAXI@Z 1001867c     PrepareWevoteTaxonomyDataTask.obj
 0002:00003694       __ehfuncinfo$??_GPrepareWevoteTaxonomyDataTask@U2@@UAEPAXI@Z 10018694     PrepareWevoteTaxonomyDataTask.obj
 0002:000036b8       __unwindtable$??__EalgoLog@U2@@YAXXZ 100186b8     WevotePrompter.obj
 0002:000036c0       __ehfuncinfo$??__EalgoLog@U2@@YAXXZ 100186c0     WevotePrompter.obj
 0002:000036e4       __unwindtable$??__EcmdLog@U2@@YAXXZ 100186e4     WevotePrompter.obj
 0002:000036ec       __ehfuncinfo$??__EcmdLog@U2@@YAXXZ 100186ec     WevotePrompter.obj
 0002:00003710       __unwindtable$??__EcoreLog@U2@@YAXXZ 10018710     WevotePrompter.obj
 0002:00003718       __ehfuncinfo$??__EcoreLog@U2@@YAXXZ 10018718     WevotePrompter.obj
 0002:0000373c       __unwindtable$??__EioLog@U2@@YAXXZ 1001873c     WevotePrompter.obj
 0002:00003744       __ehfuncinfo$??__EioLog@U2@@YAXXZ 10018744     WevotePrompter.obj
 0002:00003768       __unwindtable$??__EperfLog@U2@@YAXXZ 10018768     WevotePrompter.obj
 0002:00003770       __ehfuncinfo$??__EperfLog@U2@@YAXXZ 10018770     WevotePrompter.obj
 0002:00003794       __unwindtable$??__EscriptLog@U2@@YAXXZ 10018794     WevotePrompter.obj
 0002:0000379c       __ehfuncinfo$??__EscriptLog@U2@@YAXXZ 1001879c     WevotePrompter.obj
 0002:000037c0       __unwindtable$??__EtaskLog@U2@@YAXXZ 100187c0     WevotePrompter.obj
 0002:000037c8       __ehfuncinfo$??__EtaskLog@U2@@YAXXZ 100187c8     WevotePrompter.obj
 0002:000037ec       __unwindtable$??__EuiLog@U2@@YAXXZ 100187ec     WevotePrompter.obj
 0002:000037f4       __ehfuncinfo$??__EuiLog@U2@@YAXXZ 100187f4     WevotePrompter.obj
 0002:00003818       __unwindtable$??__EuserActLog@U2@@YAXXZ 10018818     WevotePrompter.obj
 0002:00003820       __ehfuncinfo$??__EuserActLog@U2@@YAXXZ 10018820     WevotePrompter.obj
 0002:00003844       __ehfuncinfo$?createDescription@?$PrompterBase@VWevotePrompter@LocalWorkflow@U2@@@U2@@UAEPAVActorDocument@Workflow@2@PAVActor@42@@Z 10018844     WevotePrompter.obj
 0002:00003868       __unwindtable$?createDescription@?$PrompterBase@VWevotePrompter@LocalWorkflow@U2@@@U2@@UAEPAVActorDocument@Workflow@2@PAVActor@42@@Z 10018868     WevotePrompter.obj
 0002:000038a0       __catchsym$??0?$QList@PAVPort@Workflow@U2@@@@QAE@ABV0@@Z$2 100188a0     WevotePrompter.obj
 0002:000038b0       __unwindtable$??0?$QList@PAVPort@Workflow@U2@@@@QAE@ABV0@@Z 100188b0     WevotePrompter.obj
 0002:000038c0       __tryblocktable$??0?$QList@PAVPort@Workflow@U2@@@@QAE@ABV0@@Z 100188c0     WevotePrompter.obj
 0002:000038d4       __ehfuncinfo$??0?$QList@PAVPort@Workflow@U2@@@@QAE@ABV0@@Z 100188d4     WevotePrompter.obj
 0002:000038f8       __unwindtable$??0WevoteSupport@U2@@QAE@XZ 100188f8     WevoteSupport.obj
 0002:00003910       __ehfuncinfo$??0WevoteSupport@U2@@QAE@XZ 10018910     WevoteSupport.obj
 0002:00003934       __unwindtable$??0WevoteSupportPlugin@U2@@QAE@XZ 10018934     WevoteSupportPlugin.obj
 0002:00003944       __ehfuncinfo$??0WevoteSupportPlugin@U2@@QAE@XZ 10018944     WevoteSupportPlugin.obj
 0002:00003968       __unwindtable$??1WevoteSupportPlugin@U2@@UAE@XZ 10018968     WevoteSupportPlugin.obj
 0002:00003970       __ehfuncinfo$??1WevoteSupportPlugin@U2@@UAE@XZ 10018970     WevoteSupportPlugin.obj
 0002:00003994       __unwindtable$??_GWevoteSupportPlugin@U2@@UAEPAXI@Z 10018994     WevoteSupportPlugin.obj
 0002:0000399c       __ehfuncinfo$??_GWevoteSupportPlugin@U2@@UAEPAXI@Z 1001899c     WevoteSupportPlugin.obj
 0002:000039c0       __unwindtable$??__EalgoLog@U2@@YAXXZ 100189c0     WevoteSupportPlugin.obj
 0002:000039c8       __ehfuncinfo$??__EalgoLog@U2@@YAXXZ 100189c8     WevoteSupportPlugin.obj
 0002:000039ec       __unwindtable$??__EcmdLog@U2@@YAXXZ 100189ec     WevoteSupportPlugin.obj
 0002:000039f4       __ehfuncinfo$??__EcmdLog@U2@@YAXXZ 100189f4     WevoteSupportPlugin.obj
 0002:00003a18       __unwindtable$??__EcoreLog@U2@@YAXXZ 10018a18     WevoteSupportPlugin.obj
 0002:00003a20       __ehfuncinfo$??__EcoreLog@U2@@YAXXZ 10018a20     WevoteSupportPlugin.obj
 0002:00003a44       __unwindtable$??__EioLog@U2@@YAXXZ 10018a44     WevoteSupportPlugin.obj
 0002:00003a4c       __ehfuncinfo$??__EioLog@U2@@YAXXZ 10018a4c     WevoteSupportPlugin.obj
 0002:00003a70       __unwindtable$??__EperfLog@U2@@YAXXZ 10018a70     WevoteSupportPlugin.obj
 0002:00003a78       __ehfuncinfo$??__EperfLog@U2@@YAXXZ 10018a78     WevoteSupportPlugin.obj
 0002:00003a9c       __unwindtable$??__EscriptLog@U2@@YAXXZ 10018a9c     WevoteSupportPlugin.obj
 0002:00003aa4       __ehfuncinfo$??__EscriptLog@U2@@YAXXZ 10018aa4     WevoteSupportPlugin.obj
 0002:00003ac8       __unwindtable$??__EtaskLog@U2@@YAXXZ 10018ac8     WevoteSupportPlugin.obj
 0002:00003ad0       __ehfuncinfo$??__EtaskLog@U2@@YAXXZ 10018ad0     WevoteSupportPlugin.obj
 0002:00003af4       __unwindtable$??__EuiLog@U2@@YAXXZ 10018af4     WevoteSupportPlugin.obj
 0002:00003afc       __ehfuncinfo$??__EuiLog@U2@@YAXXZ 10018afc     WevoteSupportPlugin.obj
 0002:00003b20       __unwindtable$??__EuserActLog@U2@@YAXXZ 10018b20     WevoteSupportPlugin.obj
 0002:00003b28       __ehfuncinfo$??__EuserActLog@U2@@YAXXZ 10018b28     WevoteSupportPlugin.obj
 0002:00003b4c       __catchsym$??0?$QList@VQString@@@@QAE@ABV0@@Z$2 10018b4c     WevoteTask.obj
 0002:00003b5c       __unwindtable$??0?$QList@VQString@@@@QAE@ABV0@@Z 10018b5c     WevoteTask.obj
 0002:00003b6c       __tryblocktable$??0?$QList@VQString@@@@QAE@ABV0@@Z 10018b6c     WevoteTask.obj
 0002:00003b80       __ehfuncinfo$??0?$QList@VQString@@@@QAE@ABV0@@Z 10018b80     WevoteTask.obj
 0002:00003ba4       __catchsym$?append@?$QList@VQString@@@@QAEXABVQString@@@Z$13 10018ba4     WevoteTask.obj
 0002:00003bb4       __catchsym$?append@?$QList@VQString@@@@QAEXABVQString@@@Z$12 10018bb4     WevoteTask.obj
 0002:00003bc4       __ehfuncinfo$?append@?$QList@VQString@@@@QAEXABVQString@@@Z 10018bc4     WevoteTask.obj
 0002:00003be8       __tryblocktable$?append@?$QList@VQString@@@@QAEXABVQString@@@Z 10018be8     WevoteTask.obj
 0002:00003c10       __unwindtable$?append@?$QList@VQString@@@@QAEXABVQString@@@Z 10018c10     WevoteTask.obj
 0002:00003c70       __catchsym$?detach_helper_grow@?$QList@VQString@@@@AAEPAUNode@1@HH@Z$5 10018c70     WevoteTask.obj
 0002:00003c80       __catchsym$?detach_helper_grow@?$QList@VQString@@@@AAEPAUNode@1@HH@Z$4 10018c80     WevoteTask.obj
 0002:00003c90       __unwindtable$?detach_helper_grow@?$QList@VQString@@@@AAEPAUNode@1@HH@Z 10018c90     WevoteTask.obj
 0002:00003cb0       __ehfuncinfo$?detach_helper_grow@?$QList@VQString@@@@AAEPAUNode@1@HH@Z 10018cb0     WevoteTask.obj
 0002:00003cd4       __tryblocktable$?detach_helper_grow@?$QList@VQString@@@@AAEPAUNode@1@HH@Z 10018cd4     WevoteTask.obj
 0002:00003cfc       __unwindtable$?node_construct@?$QList@VQString@@@@AAEXPAUNode@1@ABVQString@@@Z 10018cfc     WevoteTask.obj
 0002:00003d0c       __ehfuncinfo$?node_construct@?$QList@VQString@@@@AAEXPAUNode@1@ABVQString@@@Z 10018d0c     WevoteTask.obj
 0002:00003d30       __catchsym$?node_copy@?$QList@VQString@@@@AAEXPAUNode@1@00@Z$6 10018d30     WevoteTask.obj
 0002:00003d40       __tryblocktable$?node_copy@?$QList@VQString@@@@AAEXPAUNode@1@00@Z 10018d40     WevoteTask.obj
 0002:00003d54       __ehfuncinfo$?node_copy@?$QList@VQString@@@@AAEXPAUNode@1@00@Z 10018d54     WevoteTask.obj
 0002:00003d78       __unwindtable$?node_copy@?$QList@VQString@@@@AAEXPAUNode@1@00@Z 10018d78     WevoteTask.obj
 0002:00003da8       __unwindtable$??__EalgoLog@U2@@YAXXZ 10018da8     WevoteTask.obj
 0002:00003db0       __ehfuncinfo$??__EalgoLog@U2@@YAXXZ 10018db0     WevoteTask.obj
 0002:00003dd4       __unwindtable$??__EcmdLog@U2@@YAXXZ 10018dd4     WevoteTask.obj
 0002:00003ddc       __ehfuncinfo$??__EcmdLog@U2@@YAXXZ 10018ddc     WevoteTask.obj
 0002:00003e00       __unwindtable$??__EcoreLog@U2@@YAXXZ 10018e00     WevoteTask.obj
 0002:00003e08       __ehfuncinfo$??__EcoreLog@U2@@YAXXZ 10018e08     WevoteTask.obj
 0002:00003e2c       __unwindtable$??__EioLog@U2@@YAXXZ 10018e2c     WevoteTask.obj
 0002:00003e34       __ehfuncinfo$??__EioLog@U2@@YAXXZ 10018e34     WevoteTask.obj
 0002:00003e58       __unwindtable$??__EperfLog@U2@@YAXXZ 10018e58     WevoteTask.obj
 0002:00003e60       __ehfuncinfo$??__EperfLog@U2@@YAXXZ 10018e60     WevoteTask.obj
 0002:00003e84       __unwindtable$??__EscriptLog@U2@@YAXXZ 10018e84     WevoteTask.obj
 0002:00003e8c       __ehfuncinfo$??__EscriptLog@U2@@YAXXZ 10018e8c     WevoteTask.obj
 0002:00003eb0       __unwindtable$??__EtaskLog@U2@@YAXXZ 10018eb0     WevoteTask.obj
 0002:00003eb8       __ehfuncinfo$??__EtaskLog@U2@@YAXXZ 10018eb8     WevoteTask.obj
 0002:00003edc       __unwindtable$??__EuiLog@U2@@YAXXZ 10018edc     WevoteTask.obj
 0002:00003ee4       __ehfuncinfo$??__EuiLog@U2@@YAXXZ 10018ee4     WevoteTask.obj
 0002:00003f08       __unwindtable$??__EuserActLog@U2@@YAXXZ 10018f08     WevoteTask.obj
 0002:00003f10       __ehfuncinfo$??__EuserActLog@U2@@YAXXZ 10018f10     WevoteTask.obj
 0002:00003f34       __catchsym$?append@?$QList@PAVTask@U2@@@@QAEXABQAVTask@U2@@@Z$6 10018f34     WevoteTask.obj
 0002:00003f44       __tryblocktable$?append@?$QList@PAVTask@U2@@@@QAEXABQAVTask@U2@@@Z 10018f44     WevoteTask.obj
 0002:00003f58       __ehfuncinfo$?append@?$QList@PAVTask@U2@@@@QAEXABQAVTask@U2@@@Z 10018f58     WevoteTask.obj
 0002:00003f7c       __unwindtable$?append@?$QList@PAVTask@U2@@@@QAEXABQAVTask@U2@@@Z 10018f7c     WevoteTask.obj
 0002:00003fac       __catchsym$?detach_helper_grow@?$QList@PAVTask@U2@@@@AAEPAUNode@1@HH@Z$5 10018fac     WevoteTask.obj
 0002:00003fbc       __catchsym$?detach_helper_grow@?$QList@PAVTask@U2@@@@AAEPAUNode@1@HH@Z$4 10018fbc     WevoteTask.obj
 0002:00003fcc       __unwindtable$?detach_helper_grow@?$QList@PAVTask@U2@@@@AAEPAUNode@1@HH@Z 10018fcc     WevoteTask.obj
 0002:00003fec       __ehfuncinfo$?detach_helper_grow@?$QList@PAVTask@U2@@@@AAEPAUNode@1@HH@Z 10018fec     WevoteTask.obj
 0002:00004010       __tryblocktable$?detach_helper_grow@?$QList@PAVTask@U2@@@@AAEPAUNode@1@HH@Z 10019010     WevoteTask.obj
 0002:00004038       __unwindtable$??0WevoteTaskSettings@U2@@QAE@XZ 10019038     WevoteTask.obj
 0002:00004048       __ehfuncinfo$??0WevoteTaskSettings@U2@@QAE@XZ 10019048     WevoteTask.obj
 0002:0000406c       __unwindtable$??1WevoteTaskSettings@U2@@QAE@XZ 1001906c     WevoteTask.obj
 0002:0000407c       __ehfuncinfo$??1WevoteTaskSettings@U2@@QAE@XZ 1001907c     WevoteTask.obj
 0002:000040a0       __unwindtable$??0WevoteTaskSettings@U2@@QAE@ABU01@@Z 100190a0     WevoteTask.obj
 0002:000040b0       __ehfuncinfo$??0WevoteTaskSettings@U2@@QAE@ABU01@@Z 100190b0     WevoteTask.obj
 0002:000040d4       __ehfuncinfo$??0WevoteTask@U2@@QAE@ABUWevoteTaskSettings@1@AAVWorkflowProcess@FileStorage@1@@Z 100190d4     WevoteTask.obj
 0002:000040f8       __unwindtable$??0WevoteTask@U2@@QAE@ABUWevoteTaskSettings@1@AAVWorkflowProcess@FileStorage@1@@Z 100190f8     WevoteTask.obj
 0002:00004168       __unwindtable$?prepare@WevoteTask@U2@@EAEXXZ 10019168     WevoteTask.obj
 0002:00004170       __ehfuncinfo$?prepare@WevoteTask@U2@@EAEXXZ 10019170     WevoteTask.obj
 0002:00004194       __ehfuncinfo$?onSubTaskFinished@WevoteTask@U2@@EAE?AV?$QList@PAVTask@U2@@@@PAVTask@2@@Z 10019194     WevoteTask.obj
 0002:000041b8       __unwindtable$?onSubTaskFinished@WevoteTask@U2@@EAE?AV?$QList@PAVTask@U2@@@@PAVTask@2@@Z 100191b8     WevoteTask.obj
 0002:00004210       __unwindtable$?run@WevoteTask@U2@@EAEXXZ 10019210     WevoteTask.obj
 0002:00004228       __ehfuncinfo$?run@WevoteTask@U2@@EAEXXZ 10019228     WevoteTask.obj
 0002:0000424c       __ehfuncinfo$?checkSettings@WevoteTask@U2@@AAEXXZ 1001924c     WevoteTask.obj
 0002:00004270       __unwindtable$?checkSettings@WevoteTask@U2@@AAEXXZ 10019270     WevoteTask.obj
 0002:000042a0       __ehfuncinfo$?getArguments@WevoteTask@U2@@AAE?AVQStringList@@XZ 100192a0     WevoteTask.obj
 0002:000042c4       __unwindtable$?getArguments@WevoteTask@U2@@AAE?AVQStringList@@XZ 100192c4     WevoteTask.obj
 0002:0000434c       __unwindtable$?moveFile@WevoteTask@U2@@AAEXXZ 1001934c     WevoteTask.obj
 0002:0000436c       __ehfuncinfo$?moveFile@WevoteTask@U2@@AAEXXZ 1001936c     WevoteTask.obj
 0002:00004390       __ehfuncinfo$?parseClassification@WevoteTask@U2@@AAEXXZ 10019390     WevoteTask.obj
 0002:000043b4       __unwindtable$?parseClassification@WevoteTask@U2@@AAEXXZ 100193b4     WevoteTask.obj
 0002:000043f4       __ehfuncinfo$??1WevoteTask@U2@@UAE@XZ 100193f4     WevoteTask.obj
 0002:00004418       __unwindtable$??1WevoteTask@U2@@UAE@XZ 10019418     WevoteTask.obj
 0002:00004440       __catchsym$?createNode@?$QMapData@VQString@@I@@QAEPAU?$QMapNode@VQString@@I@@ABVQString@@ABIPAU2@_N@Z$5 10019440     WevoteTask.obj
 0002:00004450       __tryblocktable$?createNode@?$QMapData@VQString@@I@@QAEPAU?$QMapNode@VQString@@I@@ABVQString@@ABIPAU2@_N@Z 10019450     WevoteTask.obj
 0002:00004464       __ehfuncinfo$?createNode@?$QMapData@VQString@@I@@QAEPAU?$QMapNode@VQString@@I@@ABVQString@@ABIPAU2@_N@Z 10019464     WevoteTask.obj
 0002:00004488       __unwindtable$?createNode@?$QMapData@VQString@@I@@QAEPAU?$QMapNode@VQString@@I@@ABVQString@@ABIPAU2@_N@Z 10019488     WevoteTask.obj
 0002:000044b0       __unwindtable$??__EalgoLog@U2@@YAXXZ 100194b0     WevoteValidator.obj
 0002:000044b8       __ehfuncinfo$??__EalgoLog@U2@@YAXXZ 100194b8     WevoteValidator.obj
 0002:000044dc       __unwindtable$??__EcmdLog@U2@@YAXXZ 100194dc     WevoteValidator.obj
 0002:000044e4       __ehfuncinfo$??__EcmdLog@U2@@YAXXZ 100194e4     WevoteValidator.obj
 0002:00004508       __unwindtable$??__EcoreLog@U2@@YAXXZ 10019508     WevoteValidator.obj
 0002:00004510       __ehfuncinfo$??__EcoreLog@U2@@YAXXZ 10019510     WevoteValidator.obj
 0002:00004534       __unwindtable$??__EioLog@U2@@YAXXZ 10019534     WevoteValidator.obj
 0002:0000453c       __ehfuncinfo$??__EioLog@U2@@YAXXZ 1001953c     WevoteValidator.obj
 0002:00004560       __unwindtable$??__EperfLog@U2@@YAXXZ 10019560     WevoteValidator.obj
 0002:00004568       __ehfuncinfo$??__EperfLog@U2@@YAXXZ 10019568     WevoteValidator.obj
 0002:0000458c       __unwindtable$??__EscriptLog@U2@@YAXXZ 1001958c     WevoteValidator.obj
 0002:00004594       __ehfuncinfo$??__EscriptLog@U2@@YAXXZ 10019594     WevoteValidator.obj
 0002:000045b8       __unwindtable$??__EtaskLog@U2@@YAXXZ 100195b8     WevoteValidator.obj
 0002:000045c0       __ehfuncinfo$??__EtaskLog@U2@@YAXXZ 100195c0     WevoteValidator.obj
 0002:000045e4       __unwindtable$??__EuiLog@U2@@YAXXZ 100195e4     WevoteValidator.obj
 0002:000045ec       __ehfuncinfo$??__EuiLog@U2@@YAXXZ 100195ec     WevoteValidator.obj
 0002:00004610       __unwindtable$??__EuserActLog@U2@@YAXXZ 10019610     WevoteValidator.obj
 0002:00004618       __ehfuncinfo$??__EuserActLog@U2@@YAXXZ 10019618     WevoteValidator.obj
 0002:0000463c       __ehfuncinfo$?validateTaxonomy@WevoteValidator@Workflow@U2@@ABE_NPBVActor@23@AAV?$QList@VWorkflowNotification@U2@@@@@Z 1001963c     WevoteValidator.obj
 0002:00004660       __unwindtable$?validateTaxonomy@WevoteValidator@Workflow@U2@@ABE_NPBVActor@23@AAV?$QList@VWorkflowNotification@U2@@@@@Z 10019660     WevoteValidator.obj
 0002:000046c8       __catchsym$?append@?$QList@VWorkflowNotification@U2@@@@QAEXABVWorkflowNotification@U2@@@Z$11 100196c8     WevoteValidator.obj
 0002:000046d8       __catchsym$?append@?$QList@VWorkflowNotification@U2@@@@QAEXABVWorkflowNotification@U2@@@Z$10 100196d8     WevoteValidator.obj
 0002:000046e8       __ehfuncinfo$?append@?$QList@VWorkflowNotification@U2@@@@QAEXABVWorkflowNotification@U2@@@Z 100196e8     WevoteValidator.obj
 0002:0000470c       __tryblocktable$?append@?$QList@VWorkflowNotification@U2@@@@QAEXABVWorkflowNotification@U2@@@Z 1001970c     WevoteValidator.obj
 0002:00004734       __unwindtable$?append@?$QList@VWorkflowNotification@U2@@@@QAEXABVWorkflowNotification@U2@@@Z 10019734     WevoteValidator.obj
 0002:00004784       __catchsym$?detach_helper_grow@?$QList@VWorkflowNotification@U2@@@@AAEPAUNode@1@HH@Z$5 10019784     WevoteValidator.obj
 0002:00004794       __catchsym$?detach_helper_grow@?$QList@VWorkflowNotification@U2@@@@AAEPAUNode@1@HH@Z$4 10019794     WevoteValidator.obj
 0002:000047a4       __unwindtable$?detach_helper_grow@?$QList@VWorkflowNotification@U2@@@@AAEPAUNode@1@HH@Z 100197a4     WevoteValidator.obj
 0002:000047c4       __ehfuncinfo$?detach_helper_grow@?$QList@VWorkflowNotification@U2@@@@AAEPAUNode@1@HH@Z 100197c4     WevoteValidator.obj
 0002:000047e8       __tryblocktable$?detach_helper_grow@?$QList@VWorkflowNotification@U2@@@@AAEPAUNode@1@HH@Z 100197e8     WevoteValidator.obj
 0002:00004810       __unwindtable$?node_construct@?$QList@VWorkflowNotification@U2@@@@AAEXPAUNode@1@ABVWorkflowNotification@U2@@@Z 10019810     WevoteValidator.obj
 0002:00004820       __ehfuncinfo$?node_construct@?$QList@VWorkflowNotification@U2@@@@AAEXPAUNode@1@ABVWorkflowNotification@U2@@@Z 10019820     WevoteValidator.obj
 0002:00004844       __catchsym$?node_copy@?$QList@VWorkflowNotification@U2@@@@AAEXPAUNode@1@00@Z$6 10019844     WevoteValidator.obj
 0002:00004854       __tryblocktable$?node_copy@?$QList@VWorkflowNotification@U2@@@@AAEXPAUNode@1@00@Z 10019854     WevoteValidator.obj
 0002:00004868       __ehfuncinfo$?node_copy@?$QList@VWorkflowNotification@U2@@@@AAEXPAUNode@1@00@Z 10019868     WevoteValidator.obj
 0002:0000488c       __unwindtable$?node_copy@?$QList@VWorkflowNotification@U2@@@@AAEXPAUNode@1@00@Z 1001988c     WevoteValidator.obj
 0002:000048bc       __unwindtable$?qt_metatype_id@?$QMetaTypeId@VQAssociativeIterableImpl@QtMetaTypePrivate@@@@SAHXZ 100198bc     WevoteWorker.obj
 0002:000048c4       __ehfuncinfo$?qt_metatype_id@?$QMetaTypeId@VQAssociativeIterableImpl@QtMetaTypePrivate@@@@SAHXZ 100198c4     WevoteWorker.obj
 0002:000048e8       __unwindtable$??$qRegisterMetaType@VQAssociativeIterableImpl@QtMetaTypePrivate@@@@YAHPBDPAVQAssociativeIterableImpl@QtMetaTypePrivate@@W4DefinedType@?$MetaTypeDefinedHelper@VQAssociativeIterableImpl@QtMetaTypePrivate@@$00@QtPrivate@@@Z 100198e8     WevoteWorker.obj
 0002:000048f0       __ehfuncinfo$??$qRegisterMetaType@VQAssociativeIterableImpl@QtMetaTypePrivate@@@@YAHPBDPAVQAssociativeIterableImpl@QtMetaTypePrivate@@W4DefinedType@?$MetaTypeDefinedHelper@VQAssociativeIterableImpl@QtMetaTypePrivate@@$00@QtPrivate@@@Z 100198f0     WevoteWorker.obj
 0002:00004914       __unwindtable$??A?$QMap@VQString@@VQVariant@@@@QAEAAVQVariant@@ABVQString@@@Z 10019914     WevoteWorker.obj
 0002:0000491c       __ehfuncinfo$??A?$QMap@VQString@@VQVariant@@@@QAEAAVQVariant@@ABVQString@@@Z 1001991c     WevoteWorker.obj
 0002:00004940       __unwindtable$??__EalgoLog@U2@@YAXXZ 10019940     WevoteWorker.obj
 0002:00004948       __ehfuncinfo$??__EalgoLog@U2@@YAXXZ 10019948     WevoteWorker.obj
 0002:0000496c       __unwindtable$??__EcmdLog@U2@@YAXXZ 1001996c     WevoteWorker.obj
 0002:00004974       __ehfuncinfo$??__EcmdLog@U2@@YAXXZ 10019974     WevoteWorker.obj
 0002:00004998       __unwindtable$??__EcoreLog@U2@@YAXXZ 10019998     WevoteWorker.obj
 0002:000049a0       __ehfuncinfo$??__EcoreLog@U2@@YAXXZ 100199a0     WevoteWorker.obj
 0002:000049c4       __unwindtable$??__EioLog@U2@@YAXXZ 100199c4     WevoteWorker.obj
 0002:000049cc       __ehfuncinfo$??__EioLog@U2@@YAXXZ 100199cc     WevoteWorker.obj
 0002:000049f0       __unwindtable$??__EperfLog@U2@@YAXXZ 100199f0     WevoteWorker.obj
 0002:000049f8       __ehfuncinfo$??__EperfLog@U2@@YAXXZ 100199f8     WevoteWorker.obj
 0002:00004a1c       __unwindtable$??__EscriptLog@U2@@YAXXZ 10019a1c     WevoteWorker.obj
 0002:00004a24       __ehfuncinfo$??__EscriptLog@U2@@YAXXZ 10019a24     WevoteWorker.obj
 0002:00004a48       __unwindtable$??__EtaskLog@U2@@YAXXZ 10019a48     WevoteWorker.obj
 0002:00004a50       __ehfuncinfo$??__EtaskLog@U2@@YAXXZ 10019a50     WevoteWorker.obj
 0002:00004a74       __unwindtable$??__EuiLog@U2@@YAXXZ 10019a74     WevoteWorker.obj
 0002:00004a7c       __ehfuncinfo$??__EuiLog@U2@@YAXXZ 10019a7c     WevoteWorker.obj
 0002:00004aa0       __unwindtable$??__EuserActLog@U2@@YAXXZ 10019aa0     WevoteWorker.obj
 0002:00004aa8       __ehfuncinfo$??__EuserActLog@U2@@YAXXZ 10019aa8     WevoteWorker.obj
 0002:00004acc       __catchsym$??0?$QList@VDescriptor@U2@@@@QAE@ABV0@@Z$2 10019acc     WevoteWorker.obj
 0002:00004adc       __unwindtable$??0?$QList@VDescriptor@U2@@@@QAE@ABV0@@Z 10019adc     WevoteWorker.obj
 0002:00004aec       __tryblocktable$??0?$QList@VDescriptor@U2@@@@QAE@ABV0@@Z 10019aec     WevoteWorker.obj
 0002:00004b00       __ehfuncinfo$??0?$QList@VDescriptor@U2@@@@QAE@ABV0@@Z 10019b00     WevoteWorker.obj
 0002:00004b24       __catchsym$?append@?$QList@VDescriptor@U2@@@@QAEXABVDescriptor@U2@@@Z$9 10019b24     WevoteWorker.obj
 0002:00004b34       __catchsym$?append@?$QList@VDescriptor@U2@@@@QAEXABVDescriptor@U2@@@Z$8 10019b34     WevoteWorker.obj
 0002:00004b44       __ehfuncinfo$?append@?$QList@VDescriptor@U2@@@@QAEXABVDescriptor@U2@@@Z 10019b44     WevoteWorker.obj
 0002:00004b68       __tryblocktable$?append@?$QList@VDescriptor@U2@@@@QAEXABVDescriptor@U2@@@Z 10019b68     WevoteWorker.obj
 0002:00004b90       __unwindtable$?append@?$QList@VDescriptor@U2@@@@QAEXABVDescriptor@U2@@@Z 10019b90     WevoteWorker.obj
 0002:00004bd0       __catchsym$?detach_helper_grow@?$QList@VDescriptor@U2@@@@AAEPAUNode@1@HH@Z$5 10019bd0     WevoteWorker.obj
 0002:00004be0       __catchsym$?detach_helper_grow@?$QList@VDescriptor@U2@@@@AAEPAUNode@1@HH@Z$4 10019be0     WevoteWorker.obj
 0002:00004bf0       __unwindtable$?detach_helper_grow@?$QList@VDescriptor@U2@@@@AAEPAUNode@1@HH@Z 10019bf0     WevoteWorker.obj
 0002:00004c10       __ehfuncinfo$?detach_helper_grow@?$QList@VDescriptor@U2@@@@AAEPAUNode@1@HH@Z 10019c10     WevoteWorker.obj
 0002:00004c34       __tryblocktable$?detach_helper_grow@?$QList@VDescriptor@U2@@@@AAEPAUNode@1@HH@Z 10019c34     WevoteWorker.obj
 0002:00004c5c       __catchsym$?detach_helper@?$QList@VDescriptor@U2@@@@AAEXH@Z$2 10019c5c     WevoteWorker.obj
 0002:00004c6c       __unwindtable$?detach_helper@?$QList@VDescriptor@U2@@@@AAEXH@Z 10019c6c     WevoteWorker.obj
 0002:00004c7c       __tryblocktable$?detach_helper@?$QList@VDescriptor@U2@@@@AAEXH@Z 10019c7c     WevoteWorker.obj
 0002:00004c90       __ehfuncinfo$?detach_helper@?$QList@VDescriptor@U2@@@@AAEXH@Z 10019c90     WevoteWorker.obj
 0002:00004cb4       __unwindtable$?node_construct@?$QList@VDescriptor@U2@@@@AAEXPAUNode@1@ABVDescriptor@U2@@@Z 10019cb4     WevoteWorker.obj
 0002:00004cc4       __ehfuncinfo$?node_construct@?$QList@VDescriptor@U2@@@@AAEXPAUNode@1@ABVDescriptor@U2@@@Z 10019cc4     WevoteWorker.obj
 0002:00004ce8       __catchsym$?node_copy@?$QList@VDescriptor@U2@@@@AAEXPAUNode@1@00@Z$6 10019ce8     WevoteWorker.obj
 0002:00004cf8       __tryblocktable$?node_copy@?$QList@VDescriptor@U2@@@@AAEXPAUNode@1@00@Z 10019cf8     WevoteWorker.obj
 0002:00004d0c       __ehfuncinfo$?node_copy@?$QList@VDescriptor@U2@@@@AAEXPAUNode@1@00@Z 10019d0c     WevoteWorker.obj
 0002:00004d30       __unwindtable$?node_copy@?$QList@VDescriptor@U2@@@@AAEXPAUNode@1@00@Z 10019d30     WevoteWorker.obj
 0002:00004d60       __unwindtable$??A?$QMap@VQString@@VQScriptValue@@@@QAEAAVQScriptValue@@ABVQString@@@Z 10019d60     WevoteWorker.obj
 0002:00004d68       __ehfuncinfo$??A?$QMap@VQString@@VQScriptValue@@@@QAEAAVQScriptValue@@ABVQString@@@Z 10019d68     WevoteWorker.obj
 0002:00004d8c       __unwindtable$?uniqueKeys@?$QMap@VDescriptor@U2@@VQVariant@@@@QBE?AV?$QList@VDescriptor@U2@@@@XZ 10019d8c     WevoteWorker.obj
 0002:00004d94       __ehfuncinfo$?uniqueKeys@?$QMap@VDescriptor@U2@@VQVariant@@@@QBE?AV?$QList@VDescriptor@U2@@@@XZ 10019d94     WevoteWorker.obj
 0002:00004db8       __ehfuncinfo$??$getAttributeValue@VQString@@@Attribute@U2@@QBE?AVQString@@PAVWorkflowContext@Workflow@1@@Z 10019db8     WevoteWorker.obj
 0002:00004ddc       __unwindtable$??$getAttributeValue@VQString@@@Attribute@U2@@QBE?AVQString@@PAVWorkflowContext@Workflow@1@@Z 10019ddc     WevoteWorker.obj
 0002:00004e4c       __ehfuncinfo$??$getAttributeValue@H@Attribute@U2@@QBEHPAVWorkflowContext@Workflow@1@@Z 10019e4c     WevoteWorker.obj
 0002:00004e70       __unwindtable$??$getAttributeValue@H@Attribute@U2@@QBEHPAVWorkflowContext@Workflow@1@@Z 10019e70     WevoteWorker.obj
 0002:00004ed8       __unwindtable$?qt_metatype_id@?$QMetaTypeId@V?$QMap@VQString@@I@@@@SAHXZ 10019ed8     WevoteWorker.obj
 0002:00004ee0       __ehfuncinfo$?qt_metatype_id@?$QMetaTypeId@V?$QMap@VQString@@I@@@@SAHXZ 10019ee0     WevoteWorker.obj
 0002:00004f04       __unwindtable$??$qRegisterMetaType@V?$QMap@VQString@@I@@@@YAHPBDPAV?$QMap@VQString@@I@@W4DefinedType@?$MetaTypeDefinedHelper@V?$QMap@VQString@@I@@$00@QtPrivate@@@Z 10019f04     WevoteWorker.obj
 0002:00004f0c       __ehfuncinfo$??$qRegisterMetaType@V?$QMap@VQString@@I@@@@YAHPBDPAV?$QMap@VQString@@I@@W4DefinedType@?$MetaTypeDefinedHelper@V?$QMap@VQString@@I@@$00@QtPrivate@@@Z 10019f0c     WevoteWorker.obj
 0002:00004f30       __unwindtable$??$getValue@VQString@@@BaseWorker@LocalWorkflow@U2@@IBE?AVQString@@ABV3@@Z 10019f30     WevoteWorker.obj
 0002:00004f40       __ehfuncinfo$??$getValue@VQString@@@BaseWorker@LocalWorkflow@U2@@IBE?AVQString@@ABV3@@Z 10019f40     WevoteWorker.obj
 0002:00004f64       __ehfuncinfo$?init@WevoteWorker@LocalWorkflow@U2@@UAEXXZ 10019f64     WevoteWorker.obj
 0002:00004f88       __unwindtable$?init@WevoteWorker@LocalWorkflow@U2@@UAEXXZ 10019f88     WevoteWorker.obj
 0002:00004ff8       __ehfuncinfo$?tick@WevoteWorker@LocalWorkflow@U2@@UAEPAVTask@3@XZ 10019ff8     WevoteWorker.obj
 0002:0000501c       __unwindtable$?tick@WevoteWorker@LocalWorkflow@U2@@UAEPAVTask@3@XZ 1001a01c     WevoteWorker.obj
 0002:0000506c       __ehfuncinfo$?sl_taskFinished@WevoteWorker@LocalWorkflow@U2@@AAEXPAVTask@3@@Z 1001a06c     WevoteWorker.obj
 0002:00005090       __unwindtable$?sl_taskFinished@WevoteWorker@LocalWorkflow@U2@@AAEXPAVTask@3@@Z 1001a090     WevoteWorker.obj
 0002:000050f8       __ehfuncinfo$?getSettings@WevoteWorker@LocalWorkflow@U2@@AAE?AUWevoteTaskSettings@3@AAVU2OpStatus@3@@Z 1001a0f8     WevoteWorker.obj
 0002:0000511c       __unwindtable$?getSettings@WevoteWorker@LocalWorkflow@U2@@AAE?AUWevoteTaskSettings@3@AAVU2OpStatus@3@@Z 1001a11c     WevoteWorker.obj
 0002:00005214       __catchsym$?createNode@?$QMapData@VQString@@VQVariant@@@@QAEPAU?$QMapNode@VQString@@VQVariant@@@@ABVQString@@ABVQVariant@@PAU2@_N@Z$7 1001a214     WevoteWorker.obj
 0002:00005224       __catchsym$?createNode@?$QMapData@VQString@@VQVariant@@@@QAEPAU?$QMapNode@VQString@@VQVariant@@@@ABVQString@@ABVQVariant@@PAU2@_N@Z$6 1001a224     WevoteWorker.obj
 0002:00005234       __ehfuncinfo$?createNode@?$QMapData@VQString@@VQVariant@@@@QAEPAU?$QMapNode@VQString@@VQVariant@@@@ABVQString@@ABVQVariant@@PAU2@_N@Z 1001a234     WevoteWorker.obj
 0002:00005258       __tryblocktable$?createNode@?$QMapData@VQString@@VQVariant@@@@QAEPAU?$QMapNode@VQString@@VQVariant@@@@ABVQString@@ABVQVariant@@PAU2@_N@Z 1001a258     WevoteWorker.obj
 0002:00005280       __unwindtable$?createNode@?$QMapData@VQString@@VQVariant@@@@QAEPAU?$QMapNode@VQString@@VQVariant@@@@ABVQString@@ABVQVariant@@PAU2@_N@Z 1001a280     WevoteWorker.obj
 0002:000052b0       __catchsym$?createNode@?$QMapData@VQString@@VQScriptValue@@@@QAEPAU?$QMapNode@VQString@@VQScriptValue@@@@ABVQString@@ABVQScriptValue@@PAU2@_N@Z$7 1001a2b0     WevoteWorker.obj
 0002:000052c0       __catchsym$?createNode@?$QMapData@VQString@@VQScriptValue@@@@QAEPAU?$QMapNode@VQString@@VQScriptValue@@@@ABVQString@@ABVQScriptValue@@PAU2@_N@Z$6 1001a2c0     WevoteWorker.obj
 0002:000052d0       __ehfuncinfo$?createNode@?$QMapData@VQString@@VQScriptValue@@@@QAEPAU?$QMapNode@VQString@@VQScriptValue@@@@ABVQString@@ABVQScriptValue@@PAU2@_N@Z 1001a2d0     WevoteWorker.obj
 0002:000052f4       __tryblocktable$?createNode@?$QMapData@VQString@@VQScriptValue@@@@QAEPAU?$QMapNode@VQString@@VQScriptValue@@@@ABVQString@@ABVQScriptValue@@PAU2@_N@Z 1001a2f4     WevoteWorker.obj
 0002:0000531c       __unwindtable$?createNode@?$QMapData@VQString@@VQScriptValue@@@@QAEPAU?$QMapNode@VQString@@VQScriptValue@@@@ABVQString@@ABVQScriptValue@@PAU2@_N@Z 1001a31c     WevoteWorker.obj
 0002:0000534c       __unwindtable$?metaType@?$QVariantValueHelper@VQString@@@QtPrivate@@SA?AVQString@@ABVQVariant@@@Z 1001a34c     WevoteWorker.obj
 0002:0000535c       __ehfuncinfo$?metaType@?$QVariantValueHelper@VQString@@@QtPrivate@@SA?AVQString@@ABVQVariant@@@Z 1001a35c     WevoteWorker.obj
 0002:00005380       __unwindtable$?Create@?$QMetaTypeFunctionHelper@V?$QMap@VQString@@I@@$00@QtMetaTypePrivate@@SAPAXPBX@Z 1001a380     WevoteWorker.obj
 0002:00005388       __ehfuncinfo$?Create@?$QMetaTypeFunctionHelper@V?$QMap@VQString@@I@@$00@QtMetaTypePrivate@@SAPAXPBX@Z 1001a388     WevoteWorker.obj
 0002:000053ac       __unwindtable$?Construct@?$QMetaTypeFunctionHelper@V?$QMap@VQString@@I@@$00@QtMetaTypePrivate@@SAPAXPAXPBX@Z 1001a3ac     WevoteWorker.obj
 0002:000053b4       __ehfuncinfo$?Construct@?$QMetaTypeFunctionHelper@V?$QMap@VQString@@I@@$00@QtMetaTypePrivate@@SAPAXPAXPBX@Z 1001a3b4     WevoteWorker.obj
 0002:000053d8       __unwindtable$??0QStringList@@QAE@ABVQString@@@Z 1001a3d8     WevoteWorkerFactory.obj
 0002:000053e0       __ehfuncinfo$??0QStringList@@QAE@ABVQString@@@Z 1001a3e0     WevoteWorkerFactory.obj
 0002:00005404       __unwindtable$??__EalgoLog@U2@@YAXXZ 1001a404     WevoteWorkerFactory.obj
 0002:0000540c       __ehfuncinfo$??__EalgoLog@U2@@YAXXZ 1001a40c     WevoteWorkerFactory.obj
 0002:00005430       __unwindtable$??__EcmdLog@U2@@YAXXZ 1001a430     WevoteWorkerFactory.obj
 0002:00005438       __ehfuncinfo$??__EcmdLog@U2@@YAXXZ 1001a438     WevoteWorkerFactory.obj
 0002:0000545c       __unwindtable$??__EcoreLog@U2@@YAXXZ 1001a45c     WevoteWorkerFactory.obj
 0002:00005464       __ehfuncinfo$??__EcoreLog@U2@@YAXXZ 1001a464     WevoteWorkerFactory.obj
 0002:00005488       __unwindtable$??__EioLog@U2@@YAXXZ 1001a488     WevoteWorkerFactory.obj
 0002:00005490       __ehfuncinfo$??__EioLog@U2@@YAXXZ 1001a490     WevoteWorkerFactory.obj
 0002:000054b4       __unwindtable$??__EperfLog@U2@@YAXXZ 1001a4b4     WevoteWorkerFactory.obj
 0002:000054bc       __ehfuncinfo$??__EperfLog@U2@@YAXXZ 1001a4bc     WevoteWorkerFactory.obj
 0002:000054e0       __unwindtable$??__EscriptLog@U2@@YAXXZ 1001a4e0     WevoteWorkerFactory.obj
 0002:000054e8       __ehfuncinfo$??__EscriptLog@U2@@YAXXZ 1001a4e8     WevoteWorkerFactory.obj
 0002:0000550c       __unwindtable$??__EtaskLog@U2@@YAXXZ 1001a50c     WevoteWorkerFactory.obj
 0002:00005514       __ehfuncinfo$??__EtaskLog@U2@@YAXXZ 1001a514     WevoteWorkerFactory.obj
 0002:00005538       __unwindtable$??__EuiLog@U2@@YAXXZ 1001a538     WevoteWorkerFactory.obj
 0002:00005540       __ehfuncinfo$??__EuiLog@U2@@YAXXZ 1001a540     WevoteWorkerFactory.obj
 0002:00005564       __unwindtable$??__EuserActLog@U2@@YAXXZ 1001a564     WevoteWorkerFactory.obj
 0002:0000556c       __ehfuncinfo$??__EuserActLog@U2@@YAXXZ 1001a56c     WevoteWorkerFactory.obj
 0002:00005590       __unwindtable$??A?$QMap@VDescriptor@U2@@V?$QExplicitlySharedDataPointer@VDataType@U2@@@@@@QAEAAV?$QExplicitlySharedDataPointer@VDataType@U2@@@@ABVDescriptor@U2@@@Z 1001a590     WevoteWorkerFactory.obj
 0002:00005598       __ehfuncinfo$??A?$QMap@VDescriptor@U2@@V?$QExplicitlySharedDataPointer@VDataType@U2@@@@@@QAEAAV?$QExplicitlySharedDataPointer@VDataType@U2@@@@ABVDescriptor@U2@@@Z 1001a598     WevoteWorkerFactory.obj
 0002:000055bc       __catchsym$?append@?$QList@PAVAttribute@U2@@@@QAEXABQAVAttribute@U2@@@Z$6 1001a5bc     WevoteWorkerFactory.obj
 0002:000055cc       __tryblocktable$?append@?$QList@PAVAttribute@U2@@@@QAEXABQAVAttribute@U2@@@Z 1001a5cc     WevoteWorkerFactory.obj
 0002:000055e0       __ehfuncinfo$?append@?$QList@PAVAttribute@U2@@@@QAEXABQAVAttribute@U2@@@Z 1001a5e0     WevoteWorkerFactory.obj
 0002:00005604       __unwindtable$?append@?$QList@PAVAttribute@U2@@@@QAEXABQAVAttribute@U2@@@Z 1001a604     WevoteWorkerFactory.obj
 0002:00005634       __catchsym$?detach_helper_grow@?$QList@PAVAttribute@U2@@@@AAEPAUNode@1@HH@Z$5 1001a634     WevoteWorkerFactory.obj
 0002:00005644       __catchsym$?detach_helper_grow@?$QList@PAVAttribute@U2@@@@AAEPAUNode@1@HH@Z$4 1001a644     WevoteWorkerFactory.obj
 0002:00005654       __unwindtable$?detach_helper_grow@?$QList@PAVAttribute@U2@@@@AAEPAUNode@1@HH@Z 1001a654     WevoteWorkerFactory.obj
 0002:00005674       __ehfuncinfo$?detach_helper_grow@?$QList@PAVAttribute@U2@@@@AAEPAUNode@1@HH@Z 1001a674     WevoteWorkerFactory.obj
 0002:00005698       __tryblocktable$?detach_helper_grow@?$QList@PAVAttribute@U2@@@@AAEPAUNode@1@HH@Z 1001a698     WevoteWorkerFactory.obj
 0002:000056c0       __catchsym$?append@?$QList@PAVPortDescriptor@Workflow@U2@@@@QAEXABQAVPortDescriptor@Workflow@U2@@@Z$6 1001a6c0     WevoteWorkerFactory.obj
 0002:000056d0       __tryblocktable$?append@?$QList@PAVPortDescriptor@Workflow@U2@@@@QAEXABQAVPortDescriptor@Workflow@U2@@@Z 1001a6d0     WevoteWorkerFactory.obj
 0002:000056e4       __ehfuncinfo$?append@?$QList@PAVPortDescriptor@Workflow@U2@@@@QAEXABQAVPortDescriptor@Workflow@U2@@@Z 1001a6e4     WevoteWorkerFactory.obj
 0002:00005708       __unwindtable$?append@?$QList@PAVPortDescriptor@Workflow@U2@@@@QAEXABQAVPortDescriptor@Workflow@U2@@@Z 1001a708     WevoteWorkerFactory.obj
 0002:00005738       __catchsym$?detach_helper_grow@?$QList@PAVPortDescriptor@Workflow@U2@@@@AAEPAUNode@1@HH@Z$5 1001a738     WevoteWorkerFactory.obj
 0002:00005748       __catchsym$?detach_helper_grow@?$QList@PAVPortDescriptor@Workflow@U2@@@@AAEPAUNode@1@HH@Z$4 1001a748     WevoteWorkerFactory.obj
 0002:00005758       __unwindtable$?detach_helper_grow@?$QList@PAVPortDescriptor@Workflow@U2@@@@AAEPAUNode@1@HH@Z 1001a758     WevoteWorkerFactory.obj
 0002:00005778       __ehfuncinfo$?detach_helper_grow@?$QList@PAVPortDescriptor@Workflow@U2@@@@AAEPAUNode@1@HH@Z 1001a778     WevoteWorkerFactory.obj
 0002:0000579c       __tryblocktable$?detach_helper_grow@?$QList@PAVPortDescriptor@Workflow@U2@@@@AAEPAUNode@1@HH@Z 1001a79c     WevoteWorkerFactory.obj
 0002:000057c4       __unwindtable$?createWorker@WevoteWorkerFactory@LocalWorkflow@U2@@UAEPAVWorker@Workflow@3@PAVActor@53@@Z 1001a7c4     WevoteWorkerFactory.obj
 0002:000057cc       __ehfuncinfo$?createWorker@WevoteWorkerFactory@LocalWorkflow@U2@@UAEPAVWorker@Workflow@3@PAVActor@53@@Z 1001a7cc     WevoteWorkerFactory.obj
 0002:000057f0       __ehfuncinfo$?init@WevoteWorkerFactory@LocalWorkflow@U2@@SAXXZ 1001a7f0     WevoteWorkerFactory.obj
 0002:00005814       __unwindtable$?init@WevoteWorkerFactory@LocalWorkflow@U2@@SAXXZ 1001a814     WevoteWorkerFactory.obj
 0002:00005c4c       __catchsym$?createNode@?$QMapData@VDescriptor@U2@@V?$QExplicitlySharedDataPointer@VDataType@U2@@@@@@QAEPAU?$QMapNode@VDescriptor@U2@@V?$QExplicitlySharedDataPointer@VDataType@U2@@@@@@ABVDescriptor@U2@@ABV?$QExplicitlySharedDataPointer@VDataType@U2@@@@PAU2@_N@Z$6 1001ac4c     WevoteWorkerFactory.obj
 0002:00005c5c       __tryblocktable$?createNode@?$QMapData@VDescriptor@U2@@V?$QExplicitlySharedDataPointer@VDataType@U2@@@@@@QAEPAU?$QMapNode@VDescriptor@U2@@V?$QExplicitlySharedDataPointer@VDataType@U2@@@@@@ABVDescriptor@U2@@ABV?$QExplicitlySharedDataPointer@VDataType@U2@@@@PAU2@_N@Z 1001ac5c     WevoteWorkerFactory.obj
 0002:00005c70       __ehfuncinfo$?createNode@?$QMapData@VDescriptor@U2@@V?$QExplicitlySharedDataPointer@VDataType@U2@@@@@@QAEPAU?$QMapNode@VDescriptor@U2@@V?$QExplicitlySharedDataPointer@VDataType@U2@@@@@@ABVDescriptor@U2@@ABV?$QExplicitlySharedDataPointer@VDataType@U2@@@@PAU2@_N@Z 1001ac70     WevoteWorkerFactory.obj
 0002:00005c94       __unwindtable$?createNode@?$QMapData@VDescriptor@U2@@V?$QExplicitlySharedDataPointer@VDataType@U2@@@@@@QAEPAU?$QMapNode@VDescriptor@U2@@V?$QExplicitlySharedDataPointer@VDataType@U2@@@@@@ABVDescriptor@U2@@ABV?$QExplicitlySharedDataPointer@VDataType@U2@@@@PAU2@_N@Z 1001ac94     WevoteWorkerFactory.obj
 0002:00005cbc       __catchsym$?createNode@?$QMapData@VQString@@PAVPropertyDelegate@U2@@@@QAEPAU?$QMapNode@VQString@@PAVPropertyDelegate@U2@@@@ABVQString@@ABQAVPropertyDelegate@U2@@PAU2@_N@Z$5 1001acbc     WevoteWorkerFactory.obj
 0002:00005ccc       __tryblocktable$?createNode@?$QMapData@VQString@@PAVPropertyDelegate@U2@@@@QAEPAU?$QMapNode@VQString@@PAVPropertyDelegate@U2@@@@ABVQString@@ABQAVPropertyDelegate@U2@@PAU2@_N@Z 1001accc     WevoteWorkerFactory.obj
 0002:00005ce0       __ehfuncinfo$?createNode@?$QMapData@VQString@@PAVPropertyDelegate@U2@@@@QAEPAU?$QMapNode@VQString@@PAVPropertyDelegate@U2@@@@ABVQString@@ABQAVPropertyDelegate@U2@@PAU2@_N@Z 1001ace0     WevoteWorkerFactory.obj
 0002:00005d04       __unwindtable$?createNode@?$QMapData@VQString@@PAVPropertyDelegate@U2@@@@QAEPAU?$QMapNode@VQString@@PAVPropertyDelegate@U2@@@@ABVQString@@ABQAVPropertyDelegate@U2@@PAU2@_N@Z 1001ad04     WevoteWorkerFactory.obj
 0002:00005d2c       __unwindtable$??__EalgoLog@U2@@YAXXZ 1001ad2c     moc_WevotePrompter.obj
 0002:00005d34       __ehfuncinfo$??__EalgoLog@U2@@YAXXZ 1001ad34     moc_WevotePrompter.obj
 0002:00005d58       __unwindtable$??__EcmdLog@U2@@YAXXZ 1001ad58     moc_WevotePrompter.obj
 0002:00005d60       __ehfuncinfo$??__EcmdLog@U2@@YAXXZ 1001ad60     moc_WevotePrompter.obj
 0002:00005d84       __unwindtable$??__EcoreLog@U2@@YAXXZ 1001ad84     moc_WevotePrompter.obj
 0002:00005d8c       __ehfuncinfo$??__EcoreLog@U2@@YAXXZ 1001ad8c     moc_WevotePrompter.obj
 0002:00005db0       __unwindtable$??__EioLog@U2@@YAXXZ 1001adb0     moc_WevotePrompter.obj
 0002:00005db8       __ehfuncinfo$??__EioLog@U2@@YAXXZ 1001adb8     moc_WevotePrompter.obj
 0002:00005ddc       __unwindtable$??__EperfLog@U2@@YAXXZ 1001addc     moc_WevotePrompter.obj
 0002:00005de4       __ehfuncinfo$??__EperfLog@U2@@YAXXZ 1001ade4     moc_WevotePrompter.obj
 0002:00005e08       __unwindtable$??__EscriptLog@U2@@YAXXZ 1001ae08     moc_WevotePrompter.obj
 0002:00005e10       __ehfuncinfo$??__EscriptLog@U2@@YAXXZ 1001ae10     moc_WevotePrompter.obj
 0002:00005e34       __unwindtable$??__EtaskLog@U2@@YAXXZ 1001ae34     moc_WevotePrompter.obj
 0002:00005e3c       __ehfuncinfo$??__EtaskLog@U2@@YAXXZ 1001ae3c     moc_WevotePrompter.obj
 0002:00005e60       __unwindtable$??__EuiLog@U2@@YAXXZ 1001ae60     moc_WevotePrompter.obj
 0002:00005e68       __ehfuncinfo$??__EuiLog@U2@@YAXXZ 1001ae68     moc_WevotePrompter.obj
 0002:00005e8c       __unwindtable$??__EuserActLog@U2@@YAXXZ 1001ae8c     moc_WevotePrompter.obj
 0002:00005e94       __ehfuncinfo$??__EuserActLog@U2@@YAXXZ 1001ae94     moc_WevotePrompter.obj
 0002:00005eb8       __unwindtable$??__EalgoLog@U2@@YAXXZ 1001aeb8     moc_WevoteTask.obj
 0002:00005ec0       __ehfuncinfo$??__EalgoLog@U2@@YAXXZ 1001aec0     moc_WevoteTask.obj
 0002:00005ee4       __unwindtable$??__EcmdLog@U2@@YAXXZ 1001aee4     moc_WevoteTask.obj
 0002:00005eec       __ehfuncinfo$??__EcmdLog@U2@@YAXXZ 1001aeec     moc_WevoteTask.obj
 0002:00005f10       __unwindtable$??__EcoreLog@U2@@YAXXZ 1001af10     moc_WevoteTask.obj
 0002:00005f18       __ehfuncinfo$??__EcoreLog@U2@@YAXXZ 1001af18     moc_WevoteTask.obj
 0002:00005f3c       __unwindtable$??__EioLog@U2@@YAXXZ 1001af3c     moc_WevoteTask.obj
 0002:00005f44       __ehfuncinfo$??__EioLog@U2@@YAXXZ 1001af44     moc_WevoteTask.obj
 0002:00005f68       __unwindtable$??__EperfLog@U2@@YAXXZ 1001af68     moc_WevoteTask.obj
 0002:00005f70       __ehfuncinfo$??__EperfLog@U2@@YAXXZ 1001af70     moc_WevoteTask.obj
 0002:00005f94       __unwindtable$??__EscriptLog@U2@@YAXXZ 1001af94     moc_WevoteTask.obj
 0002:00005f9c       __ehfuncinfo$??__EscriptLog@U2@@YAXXZ 1001af9c     moc_WevoteTask.obj
 0002:00005fc0       __unwindtable$??__EtaskLog@U2@@YAXXZ 1001afc0     moc_WevoteTask.obj
 0002:00005fc8       __ehfuncinfo$??__EtaskLog@U2@@YAXXZ 1001afc8     moc_WevoteTask.obj
 0002:00005fec       __unwindtable$??__EuiLog@U2@@YAXXZ 1001afec     moc_WevoteTask.obj
 0002:00005ff4       __ehfuncinfo$??__EuiLog@U2@@YAXXZ 1001aff4     moc_WevoteTask.obj
 0002:00006018       __unwindtable$??__EuserActLog@U2@@YAXXZ 1001b018     moc_WevoteTask.obj
 0002:00006020       __ehfuncinfo$??__EuserActLog@U2@@YAXXZ 1001b020     moc_WevoteTask.obj
 0002:00006044       __unwindtable$??__EalgoLog@U2@@YAXXZ 1001b044     moc_WevoteWorker.obj
 0002:0000604c       __ehfuncinfo$??__EalgoLog@U2@@YAXXZ 1001b04c     moc_WevoteWorker.obj
 0002:00006070       __unwindtable$??__EcmdLog@U2@@YAXXZ 1001b070     moc_WevoteWorker.obj
 0002:00006078       __ehfuncinfo$??__EcmdLog@U2@@YAXXZ 1001b078     moc_WevoteWorker.obj
 0002:0000609c       __unwindtable$??__EcoreLog@U2@@YAXXZ 1001b09c     moc_WevoteWorker.obj
 0002:000060a4       __ehfuncinfo$??__EcoreLog@U2@@YAXXZ 1001b0a4     moc_WevoteWorker.obj
 0002:000060c8       __unwindtable$??__EioLog@U2@@YAXXZ 1001b0c8     moc_WevoteWorker.obj
 0002:000060d0       __ehfuncinfo$??__EioLog@U2@@YAXXZ 1001b0d0     moc_WevoteWorker.obj
 0002:000060f4       __unwindtable$??__EperfLog@U2@@YAXXZ 1001b0f4     moc_WevoteWorker.obj
 0002:000060fc       __ehfuncinfo$??__EperfLog@U2@@YAXXZ 1001b0fc     moc_WevoteWorker.obj
 0002:00006120       __unwindtable$??__EscriptLog@U2@@YAXXZ 1001b120     moc_WevoteWorker.obj
 0002:00006128       __ehfuncinfo$??__EscriptLog@U2@@YAXXZ 1001b128     moc_WevoteWorker.obj
 0002:0000614c       __unwindtable$??__EtaskLog@U2@@YAXXZ 1001b14c     moc_WevoteWorker.obj
 0002:00006154       __ehfuncinfo$??__EtaskLog@U2@@YAXXZ 1001b154     moc_WevoteWorker.obj
 0002:00006178       __unwindtable$??__EuiLog@U2@@YAXXZ 1001b178     moc_WevoteWorker.obj
 0002:00006180       __ehfuncinfo$??__EuiLog@U2@@YAXXZ 1001b180     moc_WevoteWorker.obj
 0002:000061a4       __unwindtable$??__EuserActLog@U2@@YAXXZ 1001b1a4     moc_WevoteWorker.obj
 0002:000061ac       __ehfuncinfo$??__EuserActLog@U2@@YAXXZ 1001b1ac     moc_WevoteWorker.obj
 0002:000061d0       __unwindtable$?qt_metatype_id@?$QMetaTypeIdQObject@PAVTask@U2@@$00@@SAHXZ 1001b1d0     moc_WevoteWorker.obj
 0002:000061d8       __ehfuncinfo$?qt_metatype_id@?$QMetaTypeIdQObject@PAVTask@U2@@$00@@SAHXZ 1001b1d8     moc_WevoteWorker.obj
 0002:00006200       __sehtable$__onexit        1001b200     MSVCRT:atonexit.obj
 0002:00006220       __sehtable$___DllMainCRTStartup 1001b220     MSVCRT:crtdll.obj
 0002:00006248       __sehtable$??_M@YGXPAXIHP6EX0@Z@Z 1001b248     MSVCRT:ehvecdtr.obj
 0002:00006268       __sehtable$?__ArrayUnwind@@YGXPAXIHP6EX0@Z@Z 1001b268     MSVCRT:ehvecdtr.obj
 0002:00006288       __sehtable$__IsNonwritableInCurrentImage 1001b288     MSVCRT:pesect.obj
 0002:000062b0       .edata                     1001b2b0     wevote_support.exp
 0002:000062d8       rgpv                       1001b2d8     wevote_support.exp
 0002:000062dc       rgszName                   1001b2dc     wevote_support.exp
 0002:000062e0       rgwOrd                     1001b2e0     wevote_support.exp
 0002:000062e2       szName                     1001b2e2     wevote_support.exp
 0002:000062f5       $N00001                    1001b2f5     wevote_support.exp
 0002:00006e24       .idata$6                   1001be24     ngs_reads_classification:ngs_reads_classification.dll
 0002:000085ce       .idata$6                   1001d5ce     U2Core:U2Core.dll
 0002:000086b8       .idata$6                   1001d6b8     U2Formats:U2Formats.dll
 0002:0000871c       .idata$6                   1001d71c     U2Gui:U2Gui.dll
 0002:0000a62a       .idata$6                   1001f62a     U2Lang:U2Lang.dll
 0002:0000af4c       .idata$6                   1001ff4c     U2Designer:U2Designer.dll
 0002:0000b39c       .idata$6                   1002039c     Qt5Widgets:Qt5Widgets.dll
 0002:0000b44e       .idata$6                   1002044e     Qt5Gui:Qt5Gui.dll
 0002:0000b5c0       .idata$6                   100205c0     Qt5Script:Qt5Script.dll
 0002:0000c4d0       .idata$6                   100214d0     Qt5Core:Qt5Core.dll
 0002:0000c576       .idata$6                   10021576     msvcprt:MSVCP120.dll
 0002:0000c5fa       .idata$6                   100215fa     MSVCRT:MSVCR120.dll
 0002:0000c80e       .idata$6                   1002180e     kernel32:KERNEL32.dll
 0003:000007f8       __Tuple_alloc              100227f8     PrepareWevoteTaxonomyDataTask.obj
 0003:000007f9       _ignore                    100227f9     PrepareWevoteTaxonomyDataTask.obj
 0003:000007fa       _allocator_arg             100227fa     PrepareWevoteTaxonomyDataTask.obj
 0003:000007fb       _piecewise_construct       100227fb     PrepareWevoteTaxonomyDataTask.obj
 0003:000007fc       _taskLog                   100227fc     PrepareWevoteTaxonomyDataTask.obj
 0003:00000804       _algoLog                   10022804     PrepareWevoteTaxonomyDataTask.obj
 0003:00000810       _userActLog                10022810     PrepareWevoteTaxonomyDataTask.obj
 0003:00000818       _ioLog                     10022818     PrepareWevoteTaxonomyDataTask.obj
 0003:00000828       _coreLog                   10022828     PrepareWevoteTaxonomyDataTask.obj
 0003:00000834       _uiLog                     10022834     PrepareWevoteTaxonomyDataTask.obj
 0003:0000083c       _scriptLog                 1002283c     PrepareWevoteTaxonomyDataTask.obj
 0003:00000844       _perfLog                   10022844     PrepareWevoteTaxonomyDataTask.obj
 0003:0000084c       _cmdLog                    1002284c     PrepareWevoteTaxonomyDataTask.obj
 0003:0000085c       __Tuple_alloc              1002285c     WevotePrompter.obj
 0003:0000085d       _ignore                    1002285d     WevotePrompter.obj
 0003:0000085e       _allocator_arg             1002285e     WevotePrompter.obj
 0003:0000085f       _piecewise_construct       1002285f     WevotePrompter.obj
 0003:00000860       _taskLog                   10022860     WevotePrompter.obj
 0003:00000868       _algoLog                   10022868     WevotePrompter.obj
 0003:00000870       _userActLog                10022870     WevotePrompter.obj
 0003:00000878       _ioLog                     10022878     WevotePrompter.obj
 0003:00000880       _coreLog                   10022880     WevotePrompter.obj
 0003:00000888       _uiLog                     10022888     WevotePrompter.obj
 0003:00000890       _scriptLog                 10022890     WevotePrompter.obj
 0003:00000898       _perfLog                   10022898     WevotePrompter.obj
 0003:000008a0       _cmdLog                    100228a0     WevotePrompter.obj
 0003:000008a8       __Tuple_alloc              100228a8     WevoteSupport.obj
 0003:000008a9       _ignore                    100228a9     WevoteSupport.obj
 0003:000008aa       _allocator_arg             100228aa     WevoteSupport.obj
 0003:000008ab       _piecewise_construct       100228ab     WevoteSupport.obj
 0003:000008b0       __Tuple_alloc              100228b0     WevoteSupportPlugin.obj
 0003:000008b1       _ignore                    100228b1     WevoteSupportPlugin.obj
 0003:000008b2       _allocator_arg             100228b2     WevoteSupportPlugin.obj
 0003:000008b3       _piecewise_construct       100228b3     WevoteSupportPlugin.obj
 0003:000008b4       _taskLog                   100228b4     WevoteSupportPlugin.obj
 0003:000008bc       _algoLog                   100228bc     WevoteSupportPlugin.obj
 0003:000008cc       _userActLog                100228cc     WevoteSupportPlugin.obj
 0003:000008d4       _ioLog                     100228d4     WevoteSupportPlugin.obj
 0003:000008dc       _coreLog                   100228dc     WevoteSupportPlugin.obj
 0003:000008e4       _uiLog                     100228e4     WevoteSupportPlugin.obj
 0003:000008ec       _scriptLog                 100228ec     WevoteSupportPlugin.obj
 0003:000008f4       _perfLog                   100228f4     WevoteSupportPlugin.obj
 0003:000008fc       _cmdLog                    100228fc     WevoteSupportPlugin.obj
 0003:00000904       __Tuple_alloc              10022904     WevoteTask.obj
 0003:00000905       _ignore                    10022905     WevoteTask.obj
 0003:00000906       _allocator_arg             10022906     WevoteTask.obj
 0003:00000907       _piecewise_construct       10022907     WevoteTask.obj
 0003:00000908       _taskLog                   10022908     WevoteTask.obj
 0003:00000910       _algoLog                   10022910     WevoteTask.obj
 0003:00000918       _userActLog                10022918     WevoteTask.obj
 0003:00000920       _ioLog                     10022920     WevoteTask.obj
 0003:00000928       _coreLog                   10022928     WevoteTask.obj
 0003:00000930       _uiLog                     10022930     WevoteTask.obj
 0003:00000938       _scriptLog                 10022938     WevoteTask.obj
 0003:00000940       _perfLog                   10022940     WevoteTask.obj
 0003:00000948       _cmdLog                    10022948     WevoteTask.obj
 0003:00000954       __Tuple_alloc              10022954     WevoteValidator.obj
 0003:00000955       _ignore                    10022955     WevoteValidator.obj
 0003:00000956       _allocator_arg             10022956     WevoteValidator.obj
 0003:00000957       _piecewise_construct       10022957     WevoteValidator.obj
 0003:00000958       _taskLog                   10022958     WevoteValidator.obj
 0003:00000960       _algoLog                   10022960     WevoteValidator.obj
 0003:00000968       _userActLog                10022968     WevoteValidator.obj
 0003:00000970       _ioLog                     10022970     WevoteValidator.obj
 0003:00000978       _coreLog                   10022978     WevoteValidator.obj
 0003:00000980       _uiLog                     10022980     WevoteValidator.obj
 0003:00000988       _scriptLog                 10022988     WevoteValidator.obj
 0003:00000990       _perfLog                   10022990     WevoteValidator.obj
 0003:00000998       _cmdLog                    10022998     WevoteValidator.obj
 0003:000009a0       __Tuple_alloc              100229a0     WevoteWorker.obj
 0003:000009a1       _ignore                    100229a1     WevoteWorker.obj
 0003:000009a2       _allocator_arg             100229a2     WevoteWorker.obj
 0003:000009a3       _piecewise_construct       100229a3     WevoteWorker.obj
 0003:000009a4       _taskLog                   100229a4     WevoteWorker.obj
 0003:000009ac       _algoLog                   100229ac     WevoteWorker.obj
 0003:000009b4       _userActLog                100229b4     WevoteWorker.obj
 0003:000009bc       _ioLog                     100229bc     WevoteWorker.obj
 0003:000009c4       _coreLog                   100229c4     WevoteWorker.obj
 0003:000009d0       _uiLog                     100229d0     WevoteWorker.obj
 0003:000009d8       _scriptLog                 100229d8     WevoteWorker.obj
 0003:000009e0       _perfLog                   100229e0     WevoteWorker.obj
 0003:000009e8       _cmdLog                    100229e8     WevoteWorker.obj
 0003:00000a04       __Tuple_alloc              10022a04     WevoteWorkerFactory.obj
 0003:00000a05       _ignore                    10022a05     WevoteWorkerFactory.obj
 0003:00000a06       _allocator_arg             10022a06     WevoteWorkerFactory.obj
 0003:00000a07       _piecewise_construct       10022a07     WevoteWorkerFactory.obj
 0003:00000a10       _taskLog                   10022a10     WevoteWorkerFactory.obj
 0003:00000a18       _algoLog                   10022a18     WevoteWorkerFactory.obj
 0003:00000a20       _userActLog                10022a20     WevoteWorkerFactory.obj
 0003:00000a28       _ioLog                     10022a28     WevoteWorkerFactory.obj
 0003:00000a30       _coreLog                   10022a30     WevoteWorkerFactory.obj
 0003:00000a40       _uiLog                     10022a40     WevoteWorkerFactory.obj
 0003:00000a48       _scriptLog                 10022a48     WevoteWorkerFactory.obj
 0003:00000a54       _perfLog                   10022a54     WevoteWorkerFactory.obj
 0003:00000a5c       _cmdLog                    10022a5c     WevoteWorkerFactory.obj
 0003:00000a74       __Tuple_alloc              10022a74     moc_WevotePrompter.obj
 0003:00000a75       _ignore                    10022a75     moc_WevotePrompter.obj
 0003:00000a76       _allocator_arg             10022a76     moc_WevotePrompter.obj
 0003:00000a77       _piecewise_construct       10022a77     moc_WevotePrompter.obj
 0003:00000a78       _taskLog                   10022a78     moc_WevotePrompter.obj
 0003:00000a80       _algoLog                   10022a80     moc_WevotePrompter.obj
 0003:00000a88       _userActLog                10022a88     moc_WevotePrompter.obj
 0003:00000a90       _ioLog                     10022a90     moc_WevotePrompter.obj
 0003:00000a98       _coreLog                   10022a98     moc_WevotePrompter.obj
 0003:00000aa0       _uiLog                     10022aa0     moc_WevotePrompter.obj
 0003:00000aa8       _scriptLog                 10022aa8     moc_WevotePrompter.obj
 0003:00000ab0       _perfLog                   10022ab0     moc_WevotePrompter.obj
 0003:00000ab8       _cmdLog                    10022ab8     moc_WevotePrompter.obj
 0003:00000ac0       __Tuple_alloc              10022ac0     moc_WevoteSupportPlugin.obj
 0003:00000ac1       _ignore                    10022ac1     moc_WevoteSupportPlugin.obj
 0003:00000ac2       _allocator_arg             10022ac2     moc_WevoteSupportPlugin.obj
 0003:00000ac3       _piecewise_construct       10022ac3     moc_WevoteSupportPlugin.obj
 0003:00000ac4       __Tuple_alloc              10022ac4     moc_WevoteTask.obj
 0003:00000ac5       _ignore                    10022ac5     moc_WevoteTask.obj
 0003:00000ac6       _allocator_arg             10022ac6     moc_WevoteTask.obj
 0003:00000ac7       _piecewise_construct       10022ac7     moc_WevoteTask.obj
 0003:00000ac8       _taskLog                   10022ac8     moc_WevoteTask.obj
 0003:00000ad0       _algoLog                   10022ad0     moc_WevoteTask.obj
 0003:00000ad8       _userActLog                10022ad8     moc_WevoteTask.obj
 0003:00000ae0       _ioLog                     10022ae0     moc_WevoteTask.obj
 0003:00000ae8       _coreLog                   10022ae8     moc_WevoteTask.obj
 0003:00000af0       _uiLog                     10022af0     moc_WevoteTask.obj
 0003:00000af8       _scriptLog                 10022af8     moc_WevoteTask.obj
 0003:00000b00       _perfLog                   10022b00     moc_WevoteTask.obj
 0003:00000b08       _cmdLog                    10022b08     moc_WevoteTask.obj
 0003:00000b10       __Tuple_alloc              10022b10     moc_WevoteWorker.obj
 0003:00000b11       _ignore                    10022b11     moc_WevoteWorker.obj
 0003:00000b12       _allocator_arg             10022b12     moc_WevoteWorker.obj
 0003:00000b13       _piecewise_construct       10022b13     moc_WevoteWorker.obj
 0003:00000b14       _taskLog                   10022b14     moc_WevoteWorker.obj
 0003:00000b1c       _algoLog                   10022b1c     moc_WevoteWorker.obj
 0003:00000b24       _userActLog                10022b24     moc_WevoteWorker.obj
 0003:00000b2c       _ioLog                     10022b2c     moc_WevoteWorker.obj
 0003:00000b34       _coreLog                   10022b34     moc_WevoteWorker.obj
 0003:00000b3c       _uiLog                     10022b3c     moc_WevoteWorker.obj
 0003:00000b44       _scriptLog                 10022b44     moc_WevoteWorker.obj
 0003:00000b4c       _perfLog                   10022b4c     moc_WevoteWorker.obj
 0003:00000b54       _cmdLog                    10022b54     moc_WevoteWorker.obj
 0003:00000b60       ___proc_attached           10022b60     MSVCRT:crtdll.obj
 0003:00000b68       _GS_ExceptionRecord        10022b68     MSVCRT:gs_report.obj
 0003:00000bb8       _GS_ContextRecord          10022bb8     MSVCRT:gs_report.obj
 0003:00000e84       _DebuggerWasPresent        10022e84     MSVCRT:gs_report.obj
 0004:00000060       $R000000                   10023060     * linker generated manifest res *

 Exports

  ordinal    name

        1    _ugene_plugin_init
               exported name: ugene_plugin_init
